 ProcList

 Timestamp is 5f5c3d78 (Sat Sep 12 04:16:08 2020)

 Preferred load address is 10000000

 Start         Length     Name                   Class
 0001:00000000 00000004H .CRT$XCA                CODE
 0001:00000004 0000000cH .CRT$XCC                CODE
 0001:00000010 00000008H .CRT$XCL                CODE
 0001:00000018 0000000cH .CRT$XCU                CODE
 0001:00000024 00000004H .CRT$XCZ                CODE
 0001:00000028 00000004H .CRT$XIA                CODE
 0001:0000002c 00000018H .CRT$XIC                CODE
 0001:00000044 00000004H .CRT$XIZ                CODE
 0001:00000048 00000004H .CRT$XPA                CODE
 0001:0000004c 00000008H .CRT$XPX                CODE
 0001:00000054 00000004H .CRT$XPXA               CODE
 0001:00000058 00000004H .CRT$XPZ                CODE
 0001:0000005c 00000004H .CRT$XTA                CODE
 0001:00000060 00000010H .CRT$XTZ                CODE
 0001:00000064 00000000H .gfids$y                CODE
 0001:00000070 0000da64H .rdata                  CODE
 0001:0000dad4 0000047cH .rdata$r                CODE
 0001:0000df50 00000130H .rdata$sxdata           CODE
 0001:0000e080 000002fcH .rdata$zzzdbg           CODE
 0001:0000e37c 00000004H .rtc$IAA                CODE
 0001:0000e380 00000004H .rtc$IZZ                CODE
 0001:0000e384 00000004H .rtc$TAA                CODE
 0001:0000e388 00000008H .rtc$TZZ                CODE
 0001:0000e390 00000080H .text$di                CODE
 0001:0000e410 00037a90H .text$mn                CODE
 0001:00045ea0 00001060H .text$x                 CODE
 0001:00046f00 00000170H .text$yd                CODE
 0001:00047070 00001bc0H .xdata$x                CODE
 0001:00048c30 00000192H .edata                  CODE
 0002:00000000 000009e0H .data                   DATA
 0002:000009e0 00000320H .data$r                 DATA
 0002:00000d00 00001be4H .bss                    DATA
 0003:00000000 00000240H .idata$5                DATA
 0003:00000240 00000004H .00cfg                  DATA
 0003:00000244 000000a0H .idata$2                DATA
 0003:000002e4 00000014H .idata$3                DATA
 0003:000002f8 00000240H .idata$4                DATA
 0003:00000538 00000a0eH .idata$6                DATA
 0004:00000000 00000060H .rsrc$01                DATA
 0004:00000060 00000378H .rsrc$02                DATA

  Address         Publics by Value              Rva+Base       Lib:Object

 0000:00000000       __except_list              00000000     <absolute>
 0000:00000000       ___dynamic_value_reloc_table 00000000     <absolute>
 0000:00000000       ___guard_iat_count         00000000     <absolute>
 0000:00000000       ___guard_fids_count        00000000     <absolute>
 0000:00000000       ___guard_longjmp_table     00000000     <absolute>
 0000:00000000       ___hybrid_code_map_count   00000000     <absolute>
 0000:00000000       ___hybrid_auxiliary_iat    00000000     <absolute>
 0000:00000000       ___guard_longjmp_count     00000000     <absolute>
 0000:00000000       ___guard_fids_table        00000000     <absolute>
 0000:00000000       ___volatile_metadata       00000000     <absolute>
 0000:00000000       ___guard_iat_table         00000000     <absolute>
 0000:00000000       ___AbsoluteZero            00000000     <absolute>
 0000:00000000       ___enclave_config          00000000     <absolute>
 0000:00000000       ___hybrid_code_map         00000000     <absolute>
 0000:0000004c       ___safe_se_handler_count   0000004c     <absolute>
 0000:00000100       ___guard_flags             00000100     <absolute>
 0000:00000000       ___ImageBase               10000000     <linker-defined>
 0001:00000000       ___xc_a                    10001000     LIBCMT:initializers.obj
 0001:00000024       ___xc_z                    10001024     LIBCMT:initializers.obj
 0001:00000028       ___xi_a                    10001028     LIBCMT:initializers.obj
 0001:00000034       ___acrt_stdio_initializer  10001034     libucrt:stdio_initializer.obj
 0001:00000038       ___acrt_tran_sse2_initializer 10001038     libucrt:sse2_initializer.obj
 0001:0000003c       ___acrt_timeset_initializer 1000103c     libucrt:timeset_initializer.obj
 0001:00000040       ___acrt_multibyte_initializer 10001040     libucrt:multibyte_initializer.obj
 0001:00000044       ___xi_z                    10001044     LIBCMT:initializers.obj
 0001:00000048       ___xp_a                    10001048     LIBCMT:initializers.obj
 0001:0000004c       ___acrt_locale_terminator  1000104c     libucrt:locale_initializer.obj
 0001:00000050       ___dcrt_console_output_terminator 10001050     libucrt:console_output_initializer.obj
 0001:00000054       ___acrt_stdio_terminator   10001054     libucrt:stdio_initializer.obj
 0001:00000058       ___xp_z                    10001058     LIBCMT:initializers.obj
 0001:0000005c       ___xt_a                    1000105c     LIBCMT:initializers.obj
 0001:00000060       ___xt_z                    10001060     LIBCMT:initializers.obj
 0001:00000070       ?powers_of_10_64@?$basic_data@X@detail@v6@fmt@@2QB_KB 10001070     format.obj
 0001:00000110       ?zero_or_powers_of_10_32@?$basic_data@X@detail@v6@fmt@@2QBIB 10001110     format.obj
 0001:00000138       ?zero_or_powers_of_10_64@?$basic_data@X@detail@v6@fmt@@2QB_KB 10001138     format.obj
 0001:000001d8       ?pow10_significands@?$basic_data@X@detail@v6@fmt@@2QB_KB 100011d8     format.obj
 0001:00000490       ?pow10_exponents@?$basic_data@X@detail@v6@fmt@@2QBFB 10001490     format.obj
 0001:00000540       ?digits@?$basic_data@X@detail@v6@fmt@@2QAY01$$CBDA 10001540     format.obj
 0001:00000608       ?hex_digits@?$basic_data@X@detail@v6@fmt@@2QBDB 10001608     format.obj
 0001:0000061c       ?signs@?$basic_data@X@detail@v6@fmt@@2QBDB 1000161c     format.obj
 0001:00000620       ?left_padding_shifts@?$basic_data@X@detail@v6@fmt@@2QBDB 10001620     format.obj
 0001:00000628       ?right_padding_shifts@?$basic_data@X@detail@v6@fmt@@2QBDB 10001628     format.obj
 0001:00000630       ??_C@_0BC@EOODALEL@Unknown?5exception@ 10001630     format.obj
 0001:00000644       ??_C@_0BF@KINCDENJ@bad?5array?5new?5length@ 10001644     format.obj
 0001:00000659       ??_C@_00CNPNBAHC@@         10001659     format.obj
 0001:0000065c       ??_C@_0BA@ELKIONDK@bad?5locale?5name@ 1000165c     format.obj
 0001:0000066c       ??_C@_05LAPONLG@false@     1000166c     format.obj
 0001:00000674       ??_C@_04LOAJBDKD@true@     10001674     format.obj
 0001:0000067c       ??_7format_error@v6@fmt@@6B@ 1000167c     format.obj
 0001:00000684       ??_7?$basic_memory_buffer@_W$0BPE@V?$allocator@_W@std@@@v6@fmt@@6B@ 10001684     format.obj
 0001:0000068c       ??_7?$basic_memory_buffer@D$0BPE@V?$allocator@D@std@@@v6@fmt@@6B@ 1000168c     format.obj
 0001:00000694       ??_7?$basic_memory_buffer@I$0CA@V?$allocator@I@std@@@v6@fmt@@6B@ 10001694     format.obj
 0001:0000069c       ??_C@_0BD@DBEDGLNA@argument?5not?5found@ 1000169c     format.obj
 0001:000006b0       ??_C@_0BA@JFNIOLAK@string?5too?5long@ 100016b0     format.obj
 0001:000006c0       ??_C@_0BP@NMGMJOEM@unmatched?5?8?$HN?8?5in?5format?5string@ 100016c0     format.obj
 0001:000006e0       ??_C@_0BG@PEJKJNLA@invalid?5format?5string@ 100016e0     format.obj
 0001:000006f8       ??_C@_0BJ@JNDNOEDN@unknown?5format?5specifier@ 100016f8     format.obj
 0001:00000714       ??_C@_0BN@JNLAGDD@missing?5?8?$HN?8?5in?5format?5string@ 10001714     format.obj
 0001:00000734       ??_C@_0DJ@LMIJFHJI@cannot?5switch?5from?5automatic?5to@ 10001734     format.obj
 0001:00000770       ??_C@_0BL@KNEDAEPA@invalid?5fill?5character?5?8?$HL?8@ 10001770     format.obj
 0001:0000078c       ??_C@_0CL@CFEEEDMP@format?5specifier?5requires?5numer@ 1000178c     format.obj
 0001:000007b8       ??_C@_0BC@MDEIBHGE@number?5is?5too?5big@ 100017b8     format.obj
 0001:000007cc       ??_C@_0BH@CIKPCHEG@invalid?5type?5specifier@ 100017cc     format.obj
 0001:000007e4       ??_C@_0CK@IBNNAPH@format?5specifier?5requires?5signe@ 100017e4     format.obj
 0001:00000810       ??_C@_0N@EFEDKJEI@invalid?5fill@ 10001810     format.obj
 0001:00000820       ??_C@_0DJ@GHJONFIH@cannot?5switch?5from?5manual?5to?5au@ 10001820     format.obj
 0001:0000085c       ??_C@_0CC@ELFJMMCC@invalid?5format?5specifier?5for?5ch@ 1000185c     format.obj
 0001:00000880       ??_C@_0BM@IEKLBNBK@missing?5precision?5specifier@ 10001880     format.obj
 0001:0000089c       ??_C@_0BH@IEEDMHI@string?5pointer?5is?5null@ 1000189c     format.obj
 0001:000008b4       ??_C@_0CN@KMEDLGAJ@precision?5not?5allowed?5for?5this?5@ 100018b4     format.obj
 0001:000008e4       ??_C@_03OEIAHPBN@INF@      100018e4     format.obj
 0001:000008e8       ??_C@_03OJHLLCGB@inf@      100018e8     format.obj
 0001:000008ec       ??_C@_03LKNCIKJB@NAN@      100018ec     format.obj
 0001:000008f0       ??_C@_03LHCJEHON@nan@      100018f0     format.obj
 0001:000008f4       ??_C@_0BB@JGGOGLEG@0123456789ABCDEF@ 100018f4     format.obj
 0001:00000908       ??_C@_0BD@PKKFPMLC@negative?5precision@ 10001908     format.obj
 0001:0000091c       ??_C@_0P@DAPDPGEO@negative?5width@ 1000191c     format.obj
 0001:0000092c       ??_C@_0BJ@KKLAKOOL@precision?5is?5not?5integer@ 1000192c     format.obj
 0001:00000948       ??_C@_0BF@KEAPHPPE@width?5is?5not?5integer@ 10001948     format.obj
 0001:00000974       ??_C@_11LOCGONAA@@         10001974     handles.obj
 0001:00000978       ??_C@_1BA@NMDNJJOO@?$AAP?$AAr?$AAo?$AAc?$AAe?$AAs?$AAs@ 10001978     handles.obj
 0001:00000988       ??_C@_1O@CDOGJPJJ@?$AAT?$AAh?$AAr?$AAe?$AAa?$AAd@ 10001988     handles.obj
 0001:00000998       ??_C@_17KACEIPNC@?$AAK?$AAe?$AAy@ 10001998     handles.obj
 0001:000009a0       ??_C@_19DDLLJDOO@?$AAF?$AAi?$AAl?$AAe@ 100019a0     handles.obj
 0001:000009ac       ??_C@_1O@ECECHNAE@?$AA?$DM?$AAp?$AAi?$AAp?$AAe?$AA?$DO@ 100019ac     handles.obj
 0001:000009bc       ??_C@_1BE@FGECLHKD@?$AA?$HL?$AA0?$AA?$HN?$AA?5?$AA?$CI?$AA?$HL?$AA1?$AA?$HN?$AA?$CJ@ 100019bc     handles.obj
 0001:000009d0       ??_C@_1BC@HBCEGEJN@?$AAT?$AAI?$AAD?$AA?3?$AA?5?$AA?$HL?$AA0?$AA?$HN@ 100019d0     handles.obj
 0001:000009e4       ??_C@_1BE@ELICABCK@?$AA?$DM?$AAu?$AAn?$AAk?$AAn?$AAo?$AAw?$AAn?$AA?$DO@ 100019e4     handles.obj
 0001:000009f8       ??_C@_1BG@OKCBELMP@?$AA?2?$AAR?$AAE?$AAG?$AAI?$AAS?$AAT?$AAR?$AAY?$AA?2@ 100019f8     handles.obj
 0001:00000a10       ??_C@_19KGHAHCFG@?$AAU?$AAS?$AAE?$AAR@ 10001a10     handles.obj
 0001:00000a1c       ??_C@_1DC@OIDKFHBF@?$AAM?$AAA?$AAC?$AAH?$AAI?$AAN?$AAE?$AA?2?$AAS?$AAO?$AAF?$AAT?$AAW?$AAA?$AAR@ 10001a1c     handles.obj
 0001:00000a50       ??_C@_1BA@INBMCOAP@?$AAM?$AAA?$AAC?$AAH?$AAI?$AAN?$AAE@ 10001a50     handles.obj
 0001:00000a60       ??_C@_1BC@DCCOJFBE@?$AA_?$AAC?$AAL?$AAA?$AAS?$AAS?$AAE?$AAS@ 10001a60     handles.obj
 0001:00000a74       ??_C@_13FPGAJAPJ@?$AA?2@   10001a74     handles.obj
 0001:00000a78       ??_C@_19DIHHCHDI@?$AAH?$AAK?$AAU?$AA?2@ 10001a78     handles.obj
 0001:00000a84       ??_C@_19JAPAIJDE@?$AAH?$AAK?$AAC?$AAU@ 10001a84     handles.obj
 0001:00000a90       ??_C@_1BK@OEABCBLA@?$AAH?$AAK?$AAC?$AAU?$AA?2?$AAC?$AAl?$AAa?$AAs?$AAs?$AAe?$AAs@ 10001a90     handles.obj
 0001:00000aac       ??_C@_17PJOJPMPB@?$AAH?$AAK?$AAU@ 10001aac     handles.obj
 0001:00000ab4       ??_C@_19NCHLBIN@?$AAH?$AAK?$AAC?$AAR@ 10001ab4     handles.obj
 0001:00000ac0       ??_C@_19PEALEEJB@?$AAH?$AAK?$AAL?$AAM@ 10001ac0     handles.obj
 0001:00000acc       ??_C@_1DK@KBLGALJE@?$AA?6?$AA?$HL?$AA0?$AA?$HN?$AA?6?$AA?$HL?$AA1?$AA?3?$AA6?$AA?$HN?$AA?5?$AA?$HL?$AA2?$AA?3?$AA8@ 10001acc     handles.obj
 0001:00000b08       ??_C@_1DG@HOLPNCNP@?$AA?$HL?$AA0?$AA?3?$AA6?$AAX?$AA?$HN?$AA?5?$AA?$HL?$AA1?$AA?3?$AA0?$AA8?$AAX?$AA?$HN?$AA?5@ 10001b08     handles.obj
 0001:00000b40       ??_C@_0BN@OFDOGPDL@invalid?5string_view?5position@ 10001b40     handles.obj
 0001:00000b60       ??_7PluginCheckBoxBinding@@6B@ 10001b60     Pcfg.obj
 0001:00000b68       ??_C@_1O@BJPKKLLM@?$AAC?$AAo?$AAn?$AAf?$AAi?$AAg@ 10001b68     Pcfg.obj
 0001:00000b78       ??_C@_1BO@NGDOFANC@?$AAA?$AAd?$AAd?$AAT?$AAo?$AAD?$AAi?$AAs?$AAk?$AAs?$AAM?$AAe?$AAn?$AAu@ 10001b78     Pcfg.obj
 0001:00000b98       ??_C@_1CC@PNNAOHJC@?$AAA?$AAd?$AAd?$AAT?$AAo?$AAP?$AAl?$AAu?$AAg?$AAi?$AAn?$AAs?$AAM?$AAe?$AAn@ 10001b98     Pcfg.obj
 0001:00000bbc       ??_C@_1CE@JIPJNDMD@?$AAE?$AAx?$AAp?$AAo?$AAr?$AAt?$AAE?$AAn?$AAv?$AAi?$AAr?$AAo?$AAn?$AAm?$AAe@ 10001bbc     Pcfg.obj
 0001:00000be0       ??_C@_1CC@OABICAMP@?$AAE?$AAx?$AAp?$AAo?$AAr?$AAt?$AAM?$AAo?$AAd?$AAu?$AAl?$AAe?$AAI?$AAn?$AAf@ 10001be0     Pcfg.obj
 0001:00000c04       ??_C@_1CI@OFLGHPDG@?$AAE?$AAx?$AAp?$AAo?$AAr?$AAt?$AAM?$AAo?$AAd?$AAu?$AAl?$AAe?$AAV?$AAe?$AAr@ 10001c04     Pcfg.obj
 0001:00000c2c       ??_C@_1CE@GNMOKOAL@?$AAE?$AAx?$AAp?$AAo?$AAr?$AAt?$AAP?$AAe?$AAr?$AAf?$AAo?$AAr?$AAm?$AAa?$AAn@ 10001c2c     Pcfg.obj
 0001:00000c50       ??_C@_1BM@KMCHODLM@?$AAE?$AAx?$AAp?$AAo?$AAr?$AAt?$AAH?$AAa?$AAn?$AAd?$AAl?$AAe?$AAs@ 10001c50     Pcfg.obj
 0001:00000c6c       ??_C@_1CK@CLFOOHFA@?$AAE?$AAx?$AAp?$AAo?$AAr?$AAt?$AAH?$AAa?$AAn?$AAd?$AAl?$AAe?$AAs?$AAU?$AAn@ 10001c6c     Pcfg.obj
 0001:00000c98       ??_C@_1BE@PKILIDFH@?$AAE?$AAn?$AAa?$AAb?$AAl?$AAe?$AAW?$AAM?$AAI@ 10001c98     Pcfg.obj
 0001:00000cac       ??_7PluginEditFieldBinding@@6B@ 10001cac     Pclass.obj
 0001:00000cb4       ??_C@_1BK@GMMKGKID@?$AA?$HL?$AA0?$AA?$HN?$AA?4?$AA?$HL?$AA1?$AA?3?$AA0?$AA?$HL?$AA2?$AA?$HN?$AA?$HN@ 10001cb4     Pclass.obj
 0001:00000cd0       ??_C@_1BA@BHJJFMCM@?$AAB?$AAK?$AAM?$AAG?$AAT?$AAP?$AAE@ 10001cd0     Pclass.obj
 0001:00000ce0       ??_C@_1BC@HGOMHBK@?$AA?$HL?$AA0?$AA?3?$AA?$DM?$AA2?$AA1?$AA?$HN?$AA?5@ 10001ce0     Pclass.obj
 0001:00000cf4       ??_C@_1BC@IALIJCAM@?$AAS?$AAo?$AAr?$AAt?$AAM?$AAo?$AAd?$AAe@ 10001cf4     Pclass.obj
 0001:00000d08       ??_C@_1BO@OMKAPLPJ@?$AAS?$AAt?$AAa?$AAr?$AAt?$AAP?$AAa?$AAn?$AAe?$AAl?$AAM?$AAo?$AAd?$AAe@ 10001d08     Pclass.obj
 0001:00000d48       ??_C@_1BA@JOLGFBLP@?$AAM?$AAo?$AAd?$AAe?$AA?$HL?$AA0?$AA?$HN@ 10001d48     Pclass.obj
 0001:00000d58       ??_C@_1CM@KGJLHHPG@?$AAN?$AA?0?$AAX?$AA1?$AA5?$AAF?$AA?0?$AAX?$AA1?$AA6?$AAF?$AA?0?$AAX?$AA1?$AA7@ 10001d58     Pclass.obj
 0001:00000d84       ??_C@_1BG@MNPGDOEP@?$AA1?$AA2?$AA?0?$AA0?$AA?0?$AA0?$AA?0?$AA0?$AA?0?$AA4@ 10001d84     Pclass.obj
 0001:00000d9c       ??_C@_1CG@OHFJBKLN@?$AAN?$AA?0?$AAX?$AAI?$AA?0?$AAX?$AAB?$AA?0?$AAX?$AAP?$AA?0?$AAX?$AA0?$AAS?$AA?0@ 10001d9c     Pclass.obj
 0001:00000dc4       ??_C@_1BI@EFANNANC@?$AA0?$AA?0?$AA6?$AA?0?$AA2?$AA?0?$AA2?$AA?0?$AA3?$AA?0?$AA9@ 10001dc4     Pclass.obj
 0001:00000ddc       ??_C@_17KNGPBKAK@?$AAN?$AA?0?$AAN@ 10001ddc     Pclass.obj
 0001:00000de4       ??_C@_17JPFFEOAH@?$AA0?$AA?0?$AA0@ 10001de4     Pclass.obj
 0001:00000dec       ??_C@_1BO@JAFIOFIL@?$AAN?$AA?0?$AAX?$AAI?$AA?0?$AAX?$AAB?$AA?0?$AAX?$AAC?$AA?0?$AAD?$AA?0?$AAT@ 10001dec     Pclass.obj
 0001:00000e0c       ??_C@_1BI@LFIMKDME@?$AA0?$AA?0?$AA6?$AA?0?$AA2?$AA?0?$AA6?$AA?0?$AA0?$AA?0?$AA0@ 10001e0c     Pclass.obj
 0001:00000e24       ??_C@_1BK@IEHCCPMO@?$AAN?$AA?0?$AAX?$AAI?$AA?0?$AAX?$AA4?$AAF?$AA?0?$AAX?$AA6?$AAF@ 10001e24     Pclass.obj
 0001:00000e40       ??_C@_1BA@MMHHFCDG@?$AA0?$AA?0?$AA6?$AA?0?$AA9?$AA?0?$AA9@ 10001e40     Pclass.obj
 0001:00000e50       ??_C@_1EA@CMHCGANC@?$AAN?$AA?0?$AAX?$AAI?$AA?0?$AAX?$AA4?$AAF?$AA?0?$AAX?$AA6?$AAF?$AA?0?$AAX?$AA1@ 10001e50     Pclass.obj
 0001:00000e90       ??_C@_1CE@LPFIEDMN@?$AA0?$AA?0?$AA6?$AA?0?$AA9?$AA?0?$AA9?$AA?0?$AA9?$AA?0?$AA9?$AA?0?$AA8?$AA?0?$AA8@ 10001e90     Pclass.obj
 0001:00000eb4       ??_C@_19ILLMDDHI@?$AAN?$AA?0?$AAZ?$AAD@ 10001eb4     Pclass.obj
 0001:00000ec0       ??_C@_19NMOJBHGD@?$AA1?$AA2?$AA?0?$AA0@ 10001ec0     Pclass.obj
 0001:00000ed0       ??_C@_1EC@OFLHMCFD@?$AAN?$AA?0?$AAX?$AAP?$AA?0?$AAX?$AA0?$AAS?$AA?0?$AAX?$AA1?$AAS?$AA?0?$AAX?$AA2@ 10001ed0     Pclass.obj
 0001:00000f14       ??_C@_1CA@MGMNHCLL@?$AA0?$AA?0?$AA2?$AA?0?$AA3?$AA?0?$AA2?$AA?0?$AA2?$AA?0?$AA3?$AA?0?$AA4?$AA?0?$AA3@ 10001f14     Pclass.obj
 0001:00000f34       ??_C@_1O@JGFFCAGM@?$AAN?$AA?0?$AAX?$AAI?$AA?0?$AAO@ 10001f34     Pclass.obj
 0001:00000f44       ??_C@_1O@FLEOANAI@?$AA0?$AA?0?$AA6?$AA?0?$AA1?$AA5@ 10001f44     Pclass.obj
 0001:00000f54       ??_C@_1CC@FANCGEGE@?$AAN?$AA?0?$AAX?$AAI?$AA?0?$AAX?$AAT?$AA?0?$AAX?$AA3?$AA?0?$AAX?$AAG?$AA?0?$AAX@ 10001f54     Pclass.obj
 0001:00000f78       ??_C@_1BI@PMPHDFGH@?$AA0?$AA?0?$AA6?$AA?0?$AA3?$AA?0?$AA4?$AA?0?$AA4?$AA?0?$AA4@ 10001f78     Pclass.obj
 0001:00000f90       ??_C@_1BG@COBJEPBB@?$AAN?$AA?0?$AAX?$AAI?$AA?0?$AAX?$AAT?$AA?0?$AAX?$AA3@ 10001f90     Pclass.obj
 0001:00000fa8       ??_C@_1BA@KPNNJGCD@?$AA0?$AA?0?$AA6?$AA?0?$AA3?$AA?0?$AA4@ 10001fa8     Pclass.obj
 0001:00000fb8       ??_C@_1CA@HLBJOHGN@?$AAF?$AAu?$AAl?$AAl?$AAS?$AAc?$AAr?$AAe?$AAe?$AAn?$AAL?$AAo?$AAc?$AAa?$AAl@ 10001fb8     Pclass.obj
 0001:00000fd8       ??_C@_1CC@EBBNDNOD@?$AAF?$AAu?$AAl?$AAl?$AAS?$AAc?$AAr?$AAe?$AAe?$AAn?$AAR?$AAe?$AAm?$AAo?$AAt@ 10001fd8     Pclass.obj
 0001:00000ffc       ??_C@_1BK@HMOODHKK@?$AAC?$AAo?$AAl?$AAu?$AAm?$AAn?$AAs?$AAL?$AAo?$AAc?$AAa?$AAl@ 10001ffc     Pclass.obj
 0001:00001018       ??_C@_1BM@EDHFKJEJ@?$AAC?$AAo?$AAl?$AAu?$AAm?$AAn?$AAs?$AAR?$AAe?$AAm?$AAo?$AAt?$AAe@ 10002018     Pclass.obj
 0001:00001034       ??_C@_1BI@FOOHDOCI@?$AAW?$AAi?$AAd?$AAt?$AAh?$AAs?$AAL?$AAo?$AAc?$AAa?$AAl@ 10002034     Pclass.obj
 0001:0000104c       ??_C@_1BK@DDBMMJCN@?$AAW?$AAi?$AAd?$AAt?$AAh?$AAs?$AAR?$AAe?$AAm?$AAo?$AAt?$AAe@ 1000204c     Pclass.obj
 0001:00001068       ??_C@_13DEFPDAGF@?$AA?0@   10002068     Pclass.obj
 0001:0000106c       ??_C@_15LNKNCLHH@?$AAS?$AAs@ 1000206c     Pclass.obj
 0001:00001074       ??_C@_1M@PBHOFL@?$AA?5?$AA?$HL?$AA0?$AA?$HN?$AA?5@ 10002074     Pclass.obj
 0001:00001080       ??_C@_1BE@JJMDGICA@?$AA?$HL?$AA0?$AA?$HN?$AA?3?$AA?5?$AA?$HL?$AA1?$AA?$HN?$AA?5@ 10002080     Pclass.obj
 0001:00001094       ??_C@_15JOGBDECP@?$AA?0?$AA?5@ 10002094     Pclass.obj
 0001:0000109c       ??_C@_15DNHPCDHG@?$AAT?$AAt@ 1000209c     Pclass.obj
 0001:000010a4       ??_C@_15IJHBBPPC@?$AAF?$AAf@ 100020a4     Pclass.obj
 0001:000010ac       ??_C@_1BC@OMEIHGFC@?$AAW?$AAS?$AA_?$AAP?$AAO?$AAP?$AAU?$AAP@ 100020ac     Pclass.obj
 0001:000010c0       ??_C@_1BC@ONEEOLLM@?$AAW?$AAS?$AA_?$AAC?$AAH?$AAI?$AAL?$AAD@ 100020c0     Pclass.obj
 0001:000010d4       ??_C@_1BI@GHDIGAD@?$AAW?$AAS?$AA_?$AAM?$AAI?$AAN?$AAI?$AAM?$AAI?$AAZ?$AAE@ 100020d4     Pclass.obj
 0001:000010ec       ??_C@_1BG@KLPFHNBP@?$AAW?$AAS?$AA_?$AAV?$AAI?$AAS?$AAI?$AAB?$AAL?$AAE@ 100020ec     Pclass.obj
 0001:00001104       ??_C@_1BI@NKODCGOF@?$AAW?$AAS?$AA_?$AAD?$AAI?$AAS?$AAA?$AAB?$AAL?$AAE?$AAD@ 10002104     Pclass.obj
 0001:0000111c       ??_C@_1CA@PCFJBBHH@?$AAW?$AAS?$AA_?$AAC?$AAL?$AAI?$AAP?$AAS?$AAI?$AAB?$AAL?$AAI?$AAN?$AAG?$AAS@ 1000211c     Pclass.obj
 0001:0000113c       ??_C@_1CA@MPLGGIO@?$AAW?$AAS?$AA_?$AAC?$AAL?$AAI?$AAP?$AAC?$AAH?$AAI?$AAL?$AAD?$AAR?$AAE?$AAN@ 1000213c     Pclass.obj
 0001:0000115c       ??_C@_1BI@OLBAGOJG@?$AAW?$AAS?$AA_?$AAM?$AAA?$AAX?$AAI?$AAM?$AAI?$AAZ?$AAE@ 1000215c     Pclass.obj
 0001:00001174       ??_C@_1BE@DAMMEKNP@?$AAW?$AAS?$AA_?$AAB?$AAO?$AAR?$AAD?$AAE?$AAR@ 10002174     Pclass.obj
 0001:00001188       ??_C@_1BI@EDHINADK@?$AAW?$AAS?$AA_?$AAD?$AAL?$AAG?$AAF?$AAR?$AAA?$AAM?$AAE@ 10002188     Pclass.obj
 0001:000011a0       ??_C@_1BG@CKCLFGFA@?$AAW?$AAS?$AA_?$AAV?$AAS?$AAC?$AAR?$AAO?$AAL?$AAL@ 100021a0     Pclass.obj
 0001:000011b8       ??_C@_1BG@OMIOJOGF@?$AAW?$AAS?$AA_?$AAH?$AAS?$AAC?$AAR?$AAO?$AAL?$AAL@ 100021b8     Pclass.obj
 0001:000011d0       ??_C@_1BG@KJOBMDJC@?$AAW?$AAS?$AA_?$AAS?$AAY?$AAS?$AAM?$AAE?$AAN?$AAU@ 100021d0     Pclass.obj
 0001:000011e8       ??_C@_1BM@GPNNOPCH@?$AAW?$AAS?$AA_?$AAT?$AAH?$AAI?$AAC?$AAK?$AAF?$AAR?$AAA?$AAM?$AAE@ 100021e8     Pclass.obj
 0001:00001204       ??_C@_1BO@FODKBODI@?$AAW?$AAS?$AA_?$AAM?$AAI?$AAN?$AAI?$AAM?$AAI?$AAZ?$AAE?$AAB?$AAO?$AAX@ 10002204     Pclass.obj
 0001:00001224       ??_C@_1BO@IDJMAOMI@?$AAW?$AAS?$AA_?$AAM?$AAA?$AAX?$AAI?$AAM?$AAI?$AAZ?$AAE?$AAB?$AAO?$AAX@ 10002224     Pclass.obj
 0001:00001244       ??_C@_1CI@PKBCIOPN@?$AAW?$AAS?$AA_?$AAE?$AAX?$AA_?$AAD?$AAL?$AAG?$AAM?$AAO?$AAD?$AAA?$AAL?$AAF@ 10002244     Pclass.obj
 0001:0000126c       ??_C@_1CK@KJECLHMG@?$AAW?$AAS?$AA_?$AAE?$AAX?$AA_?$AAN?$AAO?$AAP?$AAA?$AAR?$AAE?$AAN?$AAT?$AAN@ 1000226c     Pclass.obj
 0001:00001298       ??_C@_1BM@OCBKBALE@?$AAW?$AAS?$AA_?$AAE?$AAX?$AA_?$AAT?$AAO?$AAP?$AAM?$AAO?$AAS?$AAT@ 10002298     Pclass.obj
 0001:000012b4       ??_C@_1CE@JIDMMICL@?$AAW?$AAS?$AA_?$AAE?$AAX?$AA_?$AAA?$AAC?$AAC?$AAE?$AAP?$AAT?$AAF?$AAI?$AAL@ 100022b4     Pclass.obj
 0001:000012d8       ??_C@_1CE@PFFPBMCF@?$AAW?$AAS?$AA_?$AAE?$AAX?$AA_?$AAT?$AAR?$AAA?$AAN?$AAS?$AAP?$AAA?$AAR?$AAE@ 100022d8     Pclass.obj
 0001:000012fc       ??_C@_1BO@MEOEJPLO@?$AAW?$AAS?$AA_?$AAE?$AAX?$AA_?$AAM?$AAD?$AAI?$AAC?$AAH?$AAI?$AAL?$AAD@ 100022fc     Pclass.obj
 0001:0000131c       ??_C@_1CC@IEIGGJGG@?$AAW?$AAS?$AA_?$AAE?$AAX?$AA_?$AAT?$AAO?$AAO?$AAL?$AAW?$AAI?$AAN?$AAD?$AAO@ 1000231c     Pclass.obj
 0001:00001340       ??_C@_1CC@PLPNIKGL@?$AAW?$AAS?$AA_?$AAE?$AAX?$AA_?$AAW?$AAI?$AAN?$AAD?$AAO?$AAW?$AAE?$AAD?$AAG@ 10002340     Pclass.obj
 0001:00001364       ??_C@_1CC@IAPGCLEG@?$AAW?$AAS?$AA_?$AAE?$AAX?$AA_?$AAC?$AAL?$AAI?$AAE?$AAN?$AAT?$AAE?$AAD?$AAG@ 10002364     Pclass.obj
 0001:00001388       ??_C@_1CE@EANKNCIF@?$AAW?$AAS?$AA_?$AAE?$AAX?$AA_?$AAC?$AAO?$AAN?$AAT?$AAE?$AAX?$AAT?$AAH?$AAE@ 10002388     Pclass.obj
 0001:000013ac       ??_C@_1BI@GFIADCMK@?$AAW?$AAS?$AA_?$AAE?$AAX?$AA_?$AAR?$AAI?$AAG?$AAH?$AAT@ 100023ac     Pclass.obj
 0001:000013c4       ??_C@_1CC@JOFCJJPB@?$AAW?$AAS?$AA_?$AAE?$AAX?$AA_?$AAR?$AAT?$AAL?$AAR?$AAE?$AAA?$AAD?$AAI?$AAN@ 100023c4     Pclass.obj
 0001:000013e8       ??_C@_1CI@EFLDECAB@?$AAW?$AAS?$AA_?$AAE?$AAX?$AA_?$AAL?$AAE?$AAF?$AAT?$AAS?$AAC?$AAR?$AAO?$AAL@ 100023e8     Pclass.obj
 0001:00001410       ??_C@_1CI@CIFGFFJB@?$AAW?$AAS?$AA_?$AAE?$AAX?$AA_?$AAC?$AAO?$AAN?$AAT?$AAR?$AAO?$AAL?$AAP?$AAA@ 10002410     Pclass.obj
 0001:00001438       ??_C@_1CC@BGEPLDCA@?$AAW?$AAS?$AA_?$AAE?$AAX?$AA_?$AAS?$AAT?$AAA?$AAT?$AAI?$AAC?$AAE?$AAD?$AAG@ 10002438     Pclass.obj
 0001:0000145c       ??_C@_1CA@DOAIHHLO@?$AAW?$AAS?$AA_?$AAE?$AAX?$AA_?$AAA?$AAP?$AAP?$AAW?$AAI?$AAN?$AAD?$AAO?$AAW@ 1000245c     Pclass.obj
 0001:0000147c       ??_C@_1BM@FAODAMGD@?$AAW?$AAS?$AA_?$AAE?$AAX?$AA_?$AAL?$AAA?$AAY?$AAE?$AAR?$AAE?$AAD@ 1000247c     Pclass.obj
 0001:00001498       ??_C@_1CM@DJKNBOGD@?$AAW?$AAS?$AA_?$AAE?$AAX?$AA_?$AAN?$AAO?$AAI?$AAN?$AAH?$AAE?$AAR?$AAI?$AAT@ 10002498     Pclass.obj
 0001:000014c4       ??_C@_1CA@KMHLBMFI@?$AAW?$AAS?$AA_?$AAE?$AAX?$AA_?$AAL?$AAA?$AAY?$AAO?$AAU?$AAT?$AAR?$AAT?$AAL@ 100024c4     Pclass.obj
 0001:000014e4       ??_C@_1CC@LOFMDOPL@?$AAW?$AAS?$AA_?$AAE?$AAX?$AA_?$AAN?$AAO?$AAA?$AAC?$AAT?$AAI?$AAV?$AAA?$AAT@ 100024e4     Pclass.obj
 0001:00001508       ??_C@_1BA@PCPLEJNM@?$AA?$HL?$AA0?$AA?3?$AA2?$AA0?$AA?$HN?$AA?6@ 10002508     Pclass.obj
 0001:00001518       ??_C@_1CA@PGPHFLML@?$AA?$HL?$AA0?$AA?3?$AA?$DO?$AA2?$AA0?$AA?$HN?$AA?5?$AA?$HL?$AA1?$AA?3?$AA7?$AA?$HN?$AA?$CF?$AA?6@ 10002518     Pclass.obj
 0001:00001538       ??_C@_1CE@BCAPNIMO@?$AA?$HL?$AA0?$AA?3?$AA2?$AA0?$AA?$HN?$AA?5?$AA?5?$AA?$HL?$AA1?$AA?3?$AA7?$AA?$HN?$AA?$HL?$AA2@ 10002538     Pclass.obj
 0001:00001574       ??_C@_1CA@CGMHBFCH@?$AA?$HL?$AA0?$AA?$HN?$AA?$HL?$AA1?$AA?$HN?$AA?0?$AA?5?$AA?$HL?$AA2?$AA?$HN?$AA?$HL?$AA3?$AA?$HN?$AA?6@ 10002574     Pclass.obj
 0001:00001594       ??_C@_1BA@BIAFDLFH@?$AA?$HL?$AA0?$AA?$HN?$AA?$HL?$AA1?$AA?$HN?$AA?6@ 10002594     Pclass.obj
 0001:000015a4       ??_C@_1BI@DHFBAHCI@?$AA?$HL?$AA0?$AA?$HN?$AA?5?$AA?5?$AA?$CI?$AA?$HL?$AA1?$AA?$HN?$AA?$CJ?$AA?6@ 100025a4     Pclass.obj
 0001:000015bc       ??_C@_19EPBAEEOA@?$AA?$HL?$AA0?$AA?$HN?$AA?6@ 100025bc     Pclass.obj
 0001:000015c8       ??_C@_1BK@FKNCLDML@?$AA?6?$AA?$HL?$AA0?$AA?$HN?$AA?$HL?$AA1?$AA?$HN?$AA?5?$AA?$HL?$AA2?$AA?$HN?$AA?6@ 100025c8     Pclass.obj
 0001:000015e4       ??_C@_1BC@IBCAHKMA@?$AA?6?$AA?$HL?$AA0?$AA?$HN?$AA?$HL?$AA1?$AA?$HN?$AA?6@ 100025e4     Pclass.obj
 0001:000015f8       ??_C@_1BE@EKPFJOAB@?$AA?6?$AA?$HL?$AA0?$AA?$HN?$AA?6?$AA?$HL?$AA1?$AA?$HN?$AA?6@ 100025f8     Pclass.obj
 0001:0000160c       ??_C@_1CA@MEPGLLIO@?$AA?$HL?$AA0?$AA?$HN?$AA?$HL?$AA1?$AA?3?$AA0?$AA8?$AAX?$AA?$HN?$AA?5?$AA?$HL?$AA2?$AA?$HN?$AA?6@ 1000260c     Pclass.obj
 0001:0000162c       ??_C@_1DE@IMIBLDFN@?$AA?6?$AA?$HL?$AA0?$AA?$HN?$AA?6?$AA?$HL?$AA1?$AA?3?$AA?$DM?$AA?$HL?$AA2?$AA?$HN?$AA?$HN?$AA?5?$AA?$HL@ 1000262c     Pclass.obj
 0001:00001660       ??_C@_19GGNHIDOH@?$AA?4?$AAt?$AAx?$AAt@ 10002660     Pclass.obj
 0001:0000166c       ??_C@_19OPNPIOHE@?$AAH?$AAW?$AAN?$AAD@ 1000266c     Pclass.obj
 0001:00001678       ??_C@_15GKIJICBO@?$AAZ?$AAC@ 10002678     Pclass.obj
 0001:00001680       ??_C@_17JJIMNMHK@?$AA?5?$AA?$CG?$AA?$FO@ 10002680     Pclass.obj
 0001:00001688       ??_C@_13HOIJIPNN@?$AA?5@   10002688     Pclass.obj
 0001:0000168c       ??_C@_15LEKKCGMK@?$AA?2?$AA?2@ 1000268c     Pclass.obj
 0001:000016a8       ??_C@_1M@CHPAGEIC@?$AA?$CF?$AA?5?$AA?$HL?$AA0?$AA?$HN@ 100026a8     Pclass.obj
 0001:000016b4       ??_C@_1O@DLMEBHDD@?$AA?$HL?$AA0?$AA?$HN?$AA?$HL?$AA1?$AA?$HN@ 100026b4     Pclass.obj
 0001:000016c4       ??_C@_15DDHGOCBH@?$AA?4?$AA?4@ 100026c4     Pclass.obj
 0001:000016cc       ??_C@_17FJPEEFCB@?$AAp?$AAr?$AAc@ 100026cc     Pclass.obj
 0001:000016d4       ??_C@_1BC@ENICKDH@?$AAC?$AAo?$AAn?$AAt?$AAe?$AAn?$AAt?$AAs@ 100026d4     Pclass.obj
 0001:000016e8       ??_C@_1CK@DGKCELDD@?$AAP?$AAr?$AAo?$AAc?$AAe?$AAs?$AAs?$AAL?$AAi?$AAs?$AAt?$AA?4?$AAC?$AAo?$AAm@ 100026e8     Pclass.obj
 0001:00001714       ??_C@_1CK@ECJCGOEK@?$AAP?$AAr?$AAo?$AAc?$AAe?$AAs?$AAs?$AAL?$AAi?$AAs?$AAt?$AA?4?$AAU?$AAs?$AAe@ 10002714     Pclass.obj
 0001:00001740       ??_C@_1EA@IELLPLEF@?$AA?$HL?$AA0?$AA?$HN?$AA?5?$AA?$HL?$AA1?$AA?3?$AA0?$AA2?$AA?$HN?$AA?3?$AA?$HL?$AA2?$AA?3?$AA0@ 10002740     Pclass.obj
 0001:00001780       ??_C@_1DI@BCOMPFMM@?$AA?$HL?$AA0?$AA?3?$AA0?$AA2?$AA?$HN?$AA?3?$AA?$HL?$AA1?$AA?3?$AA0?$AA2?$AA?$HN?$AA?3?$AA?$HL@ 10002780     Pclass.obj
 0001:000017b8       ??_C@_1EA@HECKBAAG@?$AA?2?$AAS?$AAt?$AAr?$AAi?$AAn?$AAg?$AAF?$AAi?$AAl?$AAe?$AAI?$AAn?$AAf?$AAo@ 100027b8     Pclass.obj
 0001:000017f8       ??_C@_19JHEHLFPM@?$AA?2?$AA?$DP?$AA?$DP?$AA?2@ 100027f8     Pclass.obj
 0001:00001804       ??_C@_1DC@HCLBMGIA@?$AA?2?$AAV?$AAa?$AAr?$AAF?$AAi?$AAl?$AAe?$AAI?$AAn?$AAf?$AAo?$AA?2?$AAT?$AAr@ 10002804     Pclass.obj
 0001:00001838       ??_C@_1BI@HCCAONKE@?$AAF?$AAi?$AAl?$AAe?$AAV?$AAe?$AAr?$AAs?$AAi?$AAo?$AAn@ 10002838     Pclass.obj
 0001:00001850       ??_C@_1CA@JGBAIPOO@?$AAF?$AAi?$AAl?$AAe?$AAD?$AAe?$AAs?$AAc?$AAr?$AAi?$AAp?$AAt?$AAi?$AAo?$AAn@ 10002850     Pclass.obj
 0001:00001870       ??_C@_19KBHGBEJO@?$AA?$HL?$AA0?$AA?$HN?$AA?2@ 10002870     Pclass.obj
 0001:0000187c       ??_C@_1O@BMPPIAFP@?$AA?5?$AA?$CI?$AA?$HL?$AA0?$AA?$HN?$AA?$CJ@ 1000287c     Pclass.obj
 0001:0000188c       ??_C@_1BC@OMEIBLAI@?$AAw?$AAb?$AAe?$AAm?$AAc?$AAo?$AAm?$AAn@ 1000288c     Pclass.obj
 0001:000018a0       ??_C@_0BI@CFPLBAOH@invalid?5string?5position@ 100028a0     Pclass.obj
 0001:000018b8       ??_C@_15LGINNLBP@?$AA?$HL?$AA?$HN@ 100028b8     Pclass.obj
 0001:000018c0       ??_C@_0BA@FOIKENOD@vector?5too?5long@ 100028c0     Pclass.obj
 0001:000018d0       ??_C@_0BL@GOIGLPKN@unordered_map?1set?5too?5long@ 100028d0     Pclass.obj
 0001:000018ec       ??_C@_0BK@OGNNAFAB@invalid?5hash?5bucket?5count@ 100028ec     Pclass.obj
 0001:00001908       __real@4024000000000000    10002908     Pclass.obj
 0001:00001910       __real@41f0000000000000    10002910     Pclass.obj
 0001:00001918       __real@43e0000000000000    10002918     Pclass.obj
 0001:00001920       __real@4f800000            10002920     Pclass.obj
 0001:00001928       ?Counters@@3QBUcounters@@B 10002928     perfthread.obj
 0001:00001a30       ??_C@_1CC@DNHMJIKH@?$AA?$CF?$AA?5?$AAP?$AAr?$AAo?$AAc?$AAe?$AAs?$AAs?$AAo?$AAr?$AA?5?$AAT?$AAi?$AAm@ 10002a30     perfthread.obj
 0001:00001a54       ??_C@_1CE@FNEMIHOD@?$AA?$CF?$AA?5?$AAP?$AAr?$AAi?$AAv?$AAi?$AAl?$AAe?$AAg?$AAe?$AAd?$AA?5?$AAT?$AAi@ 10002a54     perfthread.obj
 0001:00001a78       ??_C@_1BI@IIOPEKIO@?$AA?$CF?$AA?5?$AAU?$AAs?$AAe?$AAr?$AA?5?$AAT?$AAi?$AAm?$AAe@ 10002a78     perfthread.obj
 0001:00001a90       ??_C@_1BK@FAAJNJIB@?$AAH?$AAa?$AAn?$AAd?$AAl?$AAe?$AA?5?$AAC?$AAo?$AAu?$AAn?$AAt@ 10002a90     perfthread.obj
 0001:00001aac       ??_C@_1CA@KJMNGIDJ@?$AAP?$AAa?$AAg?$AAe?$AA?5?$AAF?$AAi?$AAl?$AAe?$AA?5?$AAB?$AAy?$AAt?$AAe?$AAs@ 10002aac     perfthread.obj
 0001:00001acc       ??_C@_1CK@FGGMBBIH@?$AAP?$AAa?$AAg?$AAe?$AA?5?$AAF?$AAi?$AAl?$AAe?$AA?5?$AAB?$AAy?$AAt?$AAe?$AAs@ 10002acc     perfthread.obj
 0001:00001af8       ??_C@_1BI@GCOMDKEO@?$AAW?$AAo?$AAr?$AAk?$AAi?$AAn?$AAg?$AA?5?$AAS?$AAe?$AAt@ 10002af8     perfthread.obj
 0001:00001b10       ??_C@_1CC@OFJLEPCP@?$AAW?$AAo?$AAr?$AAk?$AAi?$AAn?$AAg?$AA?5?$AAS?$AAe?$AAt?$AA?5?$AAP?$AAe?$AAa@ 10002b10     perfthread.obj
 0001:00001b34       ??_C@_1CI@LLKMGPEG@?$AAP?$AAo?$AAo?$AAl?$AA?5?$AAN?$AAo?$AAn?$AAp?$AAa?$AAg?$AAe?$AAd?$AA?5?$AAB@ 10002b34     perfthread.obj
 0001:00001b5c       ??_C@_1CC@IMBAECJF@?$AAP?$AAo?$AAo?$AAl?$AA?5?$AAP?$AAa?$AAg?$AAe?$AAd?$AA?5?$AAB?$AAy?$AAt?$AAe@ 10002b5c     perfthread.obj
 0001:00001b80       ??_C@_1BM@DGDPAMAA@?$AAP?$AAr?$AAi?$AAv?$AAa?$AAt?$AAe?$AA?5?$AAB?$AAy?$AAt?$AAe?$AAs@ 10002b80     perfthread.obj
 0001:00001b9c       ??_C@_1CA@GADAGCME@?$AAP?$AAa?$AAg?$AAe?$AA?5?$AAF?$AAa?$AAu?$AAl?$AAt?$AAs?$AA?1?$AAs?$AAe?$AAc@ 10002b9c     perfthread.obj
 0001:00001bbc       ??_C@_1BM@FMIOMJAE@?$AAV?$AAi?$AAr?$AAt?$AAu?$AAa?$AAl?$AA?5?$AAB?$AAy?$AAt?$AAe?$AAs@ 10002bbc     perfthread.obj
 0001:00001bd8       ??_C@_1CG@KJOKFONA@?$AAV?$AAi?$AAr?$AAt?$AAu?$AAa?$AAl?$AA?5?$AAB?$AAy?$AAt?$AAe?$AAs?$AA?5?$AAP@ 10002bd8     perfthread.obj
 0001:00001c00       ??_C@_1CE@DFDFLLAO@?$AAI?$AAO?$AA?5?$AAD?$AAa?$AAt?$AAa?$AA?5?$AAB?$AAy?$AAt?$AAe?$AAs?$AA?1?$AAs@ 10002c00     perfthread.obj
 0001:00001c24       ??_C@_1CE@EFLEKJAB@?$AAI?$AAO?$AA?5?$AAR?$AAe?$AAa?$AAd?$AA?5?$AAB?$AAy?$AAt?$AAe?$AAs?$AA?1?$AAs@ 10002c24     perfthread.obj
 0001:00001c48       ??_C@_1CG@MEJHKKKF@?$AAI?$AAO?$AA?5?$AAW?$AAr?$AAi?$AAt?$AAe?$AA?5?$AAB?$AAy?$AAt?$AAe?$AAs?$AA?1@ 10002c48     perfthread.obj
 0001:00001c70       ??_C@_1CG@LBBBPCJA@?$AAI?$AAO?$AA?5?$AAO?$AAt?$AAh?$AAe?$AAr?$AA?5?$AAB?$AAy?$AAt?$AAe?$AAs?$AA?1@ 10002c70     perfthread.obj
 0001:00001c98       ??_C@_1CO@LIEOHDCC@?$AAI?$AAO?$AA?5?$AAD?$AAa?$AAt?$AAa?$AA?5?$AAO?$AAp?$AAe?$AAr?$AAa?$AAt?$AAi@ 10002c98     perfthread.obj
 0001:00001cc8       ??_C@_1CO@LIIKBHDH@?$AAI?$AAO?$AA?5?$AAR?$AAe?$AAa?$AAd?$AA?5?$AAO?$AAp?$AAe?$AAr?$AAa?$AAt?$AAi@ 10002cc8     perfthread.obj
 0001:00001cf8       ??_C@_1DA@HICMAFKK@?$AAI?$AAO?$AA?5?$AAW?$AAr?$AAi?$AAt?$AAe?$AA?5?$AAO?$AAp?$AAe?$AAr?$AAa?$AAt@ 10002cf8     perfthread.obj
 0001:00001d28       ??_C@_1DA@BEHINMGJ@?$AAI?$AAO?$AA?5?$AAO?$AAt?$AAh?$AAe?$AAr?$AA?5?$AAO?$AAp?$AAe?$AAr?$AAa?$AAt@ 10002d28     perfthread.obj
 0001:00001d58       ??_C@_1HK@MEBPBHGJ@?$AAS?$AAo?$AAf?$AAt?$AAw?$AAa?$AAr?$AAe?$AA?2?$AAM?$AAi?$AAc?$AAr?$AAo?$AAs@ 10002d58     perfthread.obj
 0001:00001dd4       ??_C@_1BC@IICCDNLG@?$AAC?$AAo?$AAu?$AAn?$AAt?$AAe?$AAr?$AAs@ 10002dd4     perfthread.obj
 0001:00001de8       ??_C@_1BG@NKNJPBCD@?$AAI?$AAD?$AA?5?$AAP?$AAr?$AAo?$AAc?$AAe?$AAs?$AAs@ 10002de8     perfthread.obj
 0001:00001e00       ??_C@_1BM@KCAKLHJN@?$AAP?$AAr?$AAi?$AAo?$AAr?$AAi?$AAt?$AAy?$AA?5?$AAB?$AAa?$AAs?$AAe@ 10002e00     perfthread.obj
 0001:00001e1c       ??_C@_1BK@KCHPPKHP@?$AAT?$AAh?$AAr?$AAe?$AAa?$AAd?$AA?5?$AAC?$AAo?$AAu?$AAn?$AAt@ 10002e1c     perfthread.obj
 0001:00001e38       ??_C@_1CI@FNIEMNAI@?$AAC?$AAr?$AAe?$AAa?$AAt?$AAi?$AAn?$AAg?$AA?5?$AAP?$AAr?$AAo?$AAc?$AAe?$AAs@ 10002e38     perfthread.obj
 0001:00001e60       ??_C@_1BK@IKAFHKBD@?$AAE?$AAl?$AAa?$AAp?$AAs?$AAe?$AAd?$AA?5?$AAT?$AAi?$AAm?$AAe@ 10002e60     perfthread.obj
 0001:00001e7c       ??_C@_19DLCFHDFF@?$AAP?$AAE?$AAR?$AAF@ 10002e7c     perfthread.obj
 0001:00001e88       ??_C@_19DOGDICKI@?$AA?4?$AAe?$AAx?$AAe@ 10002e88     perfthread.obj
 0001:00001e94       ??_C@_1O@NKAIMMPD@?$AA_?$AAT?$AAo?$AAt?$AAa?$AAl@ 10002e94     Plist.obj
 0001:00001ea4       ??_C@_1CC@DMDJMJLM@?$AAS?$AAe?$AAD?$AAe?$AAb?$AAu?$AAg?$AAP?$AAr?$AAi?$AAv?$AAi?$AAl?$AAe?$AAg@ 10002ea4     Plist.obj
 0001:00001ec8       ??_C@_1BC@HFCOGKPP@?$AA?$HL?$AA0?$AA?$HN?$AA?6?$AA?$HL?$AA1?$AA?$HN?$AA?6@ 10002ec8     Plist.obj
 0001:00001edc       ??_C@_1M@DNHIACJI@?$AA?6?$AA?$HL?$AA0?$AA?$HN?$AA?6@ 10002edc     Plist.obj
 0001:00001ee8       ??_C@_1BG@JBKHLPML@?$AA?$HL?$AA0?$AA?$HN?$AA?5?$AA?$HL?$AA1?$AA?3?$AA8?$AAX?$AA?$HN@ 10002ee8     Plist.obj
 0001:00001f00       ??_C@_19DPDNGGHD@?$AA?5?$AA?$HL?$AA0?$AA?$HN@ 10002f00     Plist.obj
 0001:00001f0c       ??_C@_1BE@EMDGEBAH@?$AA?$HL?$AA0?$AA?3?$AA0?$AA?$HL?$AA1?$AA?$HN?$AAX?$AA?$HN@ 10002f0c     Plist.obj
 0001:00001f20       ??_C@_1BC@INJAHLHL@?$AA?$HL?$AA0?$AA?3?$AA0?$AA1?$AA6?$AAX?$AA?$HN@ 10002f20     Plist.obj
 0001:00001f4c       ??_7?$_Func_impl_no_alloc@V<lambda_ca95615ebb3c7b16132ff39b7c245039>@@_NPA_WI@std@@6B@ 10002f4c     Plist.obj
 0001:00001f64       ??_7?$_Func_impl_no_alloc@V<lambda_7407d5cd5d4425cb98b7ee1223d84907>@@_NPA_WI@std@@6B@ 10002f64     Plist.obj
 0001:00001f7c       ??_C@_1CA@CCAFOKCB@?$AAE?$AAr?$AAr?$AAo?$AAr?$AA?5?$AA0?$AAx?$AA?$HL?$AA0?$AA?3?$AA0?$AA8?$AAX?$AA?$HN@ 10002f7c     Pmix.obj
 0001:00001f9c       ??_C@_15JNBOKNOG@?$AA?$AN?$AA?6@ 10002f9c     Pmix.obj
 0001:00001fa4       _IID_IWbemLocator          10002fa4     WMI.obj
 0001:00001fb4       _CLSID_WbemLocator         10002fb4     WMI.obj
 0001:00001fc4       ??_C@_1DC@LAIEFOLO@?$AAW?$AAi?$AAn?$AA3?$AA2?$AA_?$AAP?$AAr?$AAo?$AAc?$AAe?$AAs?$AAs?$AA?4?$AAH@ 10002fc4     WMI.obj
 0001:00001ff8       ??_C@_1BO@CLCOBGDE@?$AAE?$AAx?$AAe?$AAc?$AAu?$AAt?$AAa?$AAb?$AAl?$AAe?$AAP?$AAa?$AAt?$AAh@ 10002ff8     WMI.obj
 0001:00002018       ??_C@_1BI@LPJNJKGA@?$AAC?$AAo?$AAm?$AAm?$AAa?$AAn?$AAd?$AAL?$AAi?$AAn?$AAe@ 10003018     WMI.obj
 0001:00002030       ??_C@_1BC@JHNNEHFE@?$AAP?$AAr?$AAi?$AAo?$AAr?$AAi?$AAt?$AAy@ 10003030     WMI.obj
 0001:00002044       ??_C@_1BC@HJJANEGO@?$AAG?$AAe?$AAt?$AAO?$AAw?$AAn?$AAe?$AAr@ 10003044     WMI.obj
 0001:00002058       ??_C@_19PIJILKAI@?$AAU?$AAs?$AAe?$AAr@ 10003058     WMI.obj
 0001:00002064       ??_C@_1O@OAMNPMOM@?$AAD?$AAo?$AAm?$AAa?$AAi?$AAn@ 10003064     WMI.obj
 0001:00002074       ??_C@_1BI@OIPNMPCL@?$AAG?$AAe?$AAt?$AAO?$AAw?$AAn?$AAe?$AAr?$AAS?$AAi?$AAd@ 10003074     WMI.obj
 0001:0000208c       ??_C@_17NKMLOKHF@?$AAS?$AAi?$AAd@ 1000308c     WMI.obj
 0001:00002094       ??_C@_1BE@CFEJJKFE@?$AAS?$AAe?$AAs?$AAs?$AAi?$AAo?$AAn?$AAI?$AAd@ 10003094     WMI.obj
 0001:000020a8       ??_C@_1BM@MLGLIGHJ@?$AAW?$AAi?$AAn?$AA3?$AA2?$AA_?$AAP?$AAr?$AAo?$AAc?$AAe?$AAs?$AAs@ 100030a8     WMI.obj
 0001:000020c4       ??_C@_1BI@FLOHINJE@?$AAR?$AAe?$AAt?$AAu?$AAr?$AAn?$AAV?$AAa?$AAl?$AAu?$AAe@ 100030c4     WMI.obj
 0001:000020dc       ??_C@_1BI@NKNJJIDM@?$AAS?$AAe?$AAt?$AAP?$AAr?$AAi?$AAo?$AAr?$AAi?$AAt?$AAy@ 100030dc     WMI.obj
 0001:000020f4       ??_C@_1O@GGHBFGJC@?$AAR?$AAe?$AAa?$AAs?$AAo?$AAn@ 100030f4     WMI.obj
 0001:00002104       ??_C@_1BE@PBPGMODO@?$AAT?$AAe?$AAr?$AAm?$AAi?$AAn?$AAa?$AAt?$AAe@ 10003104     WMI.obj
 0001:00002118       ??_C@_1CC@OGNCBAIB@?$AA?2?$AA?2?$AA?$HL?$AA0?$AA?$HN?$AA?2?$AAr?$AAo?$AAo?$AAt?$AA?2?$AAc?$AAi?$AAm?$AAv@ 10003118     WMI.obj
 0001:0000213c       ??_C@_13JOFGPIOO@?$AA?4@   1000313c     WMI.obj
 0001:00002170       _MainGuid                  10003170     Proclist.obj
 0001:00002180       _MenuGuid                  10003180     Proclist.obj
 0001:00002190       _ConfigDialogGuid          10003190     Proclist.obj
 0001:000021a0       ??_C@_1M@OAIMIKLP@?$AAn?$AAt?$AAd?$AAl?$AAl@ 100031a0     Proclist.obj
 0001:000021ac       ??_C@_0BK@EGDDIFMK@NtQueryInformationProcess@ 100031ac     Proclist.obj
 0001:000021c8       ??_C@_0BJ@HKKELGGC@NtQueryInformationThread@ 100031c8     Proclist.obj
 0001:000021e4       ??_C@_0O@IFMDHOMC@NtQueryObject@ 100031e4     Proclist.obj
 0001:000021f4       ??_C@_0BJ@NDLOPGCH@NtQuerySystemInformation@ 100031f4     Proclist.obj
 0001:00002210       ??_C@_0BH@DLPGICA@NtQueryInformationFile@ 10003210     Proclist.obj
 0001:00002228       ??_C@_0CB@GDPHBMJN@NtWow64QueryInformationProcess6@ 10003228     Proclist.obj
 0001:0000224c       ??_C@_0BL@NJDHCDMK@NtWow64ReadVirtualMemory64@ 1000324c     Proclist.obj
 0001:00002268       ??_C@_1BC@GDMECMAK@?$AAk?$AAe?$AAr?$AAn?$AAe?$AAl?$AA3?$AA2@ 10003268     Proclist.obj
 0001:0000227c       ??_C@_0P@LKABJJMO@IsWow64Process@ 1000327c     Proclist.obj
 0001:0000228c       ??_C@_1BC@DNHGCMLG@?$AAa?$AAd?$AAv?$AAa?$AAp?$AAi?$AA3?$AA2@ 1000328c     Proclist.obj
 0001:000022a0       ??_C@_0L@KJHKJIPF@IsValidSid@ 100032a0     Proclist.obj
 0001:000022ac       ??_C@_0BK@FIHGNING@GetSidIdentifierAuthority@ 100032ac     Proclist.obj
 0001:000022c8       ??_C@_0BI@LPFJALDI@GetSidSubAuthorityCount@ 100032c8     Proclist.obj
 0001:000022e0       ??_C@_0BD@LMGFHOAE@GetSidSubAuthority@ 100032e0     Proclist.obj
 0001:000022f4       ??_C@_1O@BCCLBEOE@?$AAu?$AAs?$AAe?$AAr?$AA3?$AA2@ 100032f4     Proclist.obj
 0001:00002304       ??_C@_0BA@FKGDNIJG@GetGuiResources@ 10003304     Proclist.obj
 0001:00002314       ??_C@_1M@FFPAMFOB@?$AAo?$AAl?$AAe?$AA3?$AA2@ 10003314     Proclist.obj
 0001:00002320       ??_C@_0BC@IOEGILCE@CoSetProxyBlanket@ 10003320     Proclist.obj
 0001:00002334       ??_C@_1M@OMFDJDJC@?$AAp?$AAs?$AAa?$AAp?$AAi@ 10003334     Proclist.obj
 0001:00002340       ??_C@_0BF@LEEEDPDK@EnumProcessModulesEx@ 10003340     Proclist.obj
 0001:00002358       ??_C@_1BC@PDEABLIN@?$AAP?$AAr?$AAo?$AAc?$AAL?$AAi?$AAs?$AAt@ 10003358     Proclist.obj
 0001:0000236c       ??_C@_1DK@DCAMPEPJ@?$AAP?$AAr?$AAo?$AAc?$AAe?$AAs?$AAs?$AA?5?$AAL?$AAi?$AAs?$AAt?$AA?5?$AAf?$AAo@ 1000336c     Proclist.obj
 0001:000023a8       ??_C@_1DE@BGKMIKPD@?$AAE?$AAu?$AAg?$AAe?$AAn?$AAe?$AA?5?$AAR?$AAo?$AAs?$AAh?$AAa?$AAl?$AA?5?$AA?$CG@ 100033a8     Proclist.obj
 0001:000023dc       ??_C@_1M@MNPEKPKO@?$AAp?$AAl?$AAi?$AAs?$AAt@ 100033dc     Proclist.obj
 0001:000023f0       __imp__EncodePointer@4     100033f0     vc_crt_fix.obj
 0001:000023f4       __imp__DecodePointer@4     100033f4     vc_crt_fix.obj
 0001:000023f8       __imp__GetModuleHandleExW@12 100033f8     vc_crt_fix.obj
 0001:000023fc       __imp__InitializeSListHead@4 100033fc     vc_crt_fix.obj
 0001:00002400       __imp__InterlockedFlushSList@4 10003400     vc_crt_fix.obj
 0001:00002404       __imp__InterlockedPopEntrySList@4 10003404     vc_crt_fix.obj
 0001:00002408       __imp__InterlockedPushEntrySList@8 10003408     vc_crt_fix.obj
 0001:0000240c       __imp__InterlockedPushListSListEx@16 1000340c     vc_crt_fix.obj
 0001:00002410       __imp__RtlFirstEntrySList@4 10003410     vc_crt_fix.obj
 0001:00002414       __imp__QueryDepthSList@4   10003414     vc_crt_fix.obj
 0001:00002418       __imp__GetNumaHighestNodeNumber@4 10003418     vc_crt_fix.obj
 0001:0000241c       __imp__GetLogicalProcessorInformation@8 1000341c     vc_crt_fix.obj
 0001:00002420       __imp__SetThreadStackGuarantee@4 10003420     vc_crt_fix.obj
 0001:00002444       ??_C@_0O@NLDKAIKN@EncodePointer@ 10003444     vc_crt_fix_impl.obj
 0001:00002454       ??_C@_0O@KBPMFGHI@DecodePointer@ 10003454     vc_crt_fix_impl.obj
 0001:00002464       ??_C@_0BD@GIGEJCNH@GetModuleHandleExW@ 10003464     vc_crt_fix_impl.obj
 0001:00002478       ??_C@_0BE@NBEJPEJA@InitializeSListHead@ 10003478     vc_crt_fix_impl.obj
 0001:0000248c       ??_C@_0BG@PLLPFLHB@InterlockedFlushSList@ 1000348c     vc_crt_fix_impl.obj
 0001:000024a4       ??_C@_0BJ@PNEEKDOK@InterlockedPopEntrySList@ 100034a4     vc_crt_fix_impl.obj
 0001:000024c0       ??_C@_0BK@JFGGAIOA@InterlockedPushEntrySList@ 100034c0     vc_crt_fix_impl.obj
 0001:000024dc       ??_C@_0BL@FOECAEGO@InterlockedPushListSListEx@ 100034dc     vc_crt_fix_impl.obj
 0001:000024f8       ??_C@_0BD@FHMMIGCI@RtlFirstEntrySList@ 100034f8     vc_crt_fix_impl.obj
 0001:0000250c       ??_C@_0BA@FGPHPMJB@QueryDepthSList@ 1000350c     vc_crt_fix_impl.obj
 0001:0000251c       ??_C@_0BJ@NLNFLAMA@GetNumaHighestNodeNumber@ 1000351c     vc_crt_fix_impl.obj
 0001:00002538       ??_C@_0BP@KHGALBC@GetLogicalProcessorInformation@ 10003538     vc_crt_fix_impl.obj
 0001:00002558       ??_C@_0BI@BKLFFAPO@SetThreadStackGuarantee@ 10003558     vc_crt_fix_impl.obj
 0001:00002574       ??_7exception@std@@6B@     10003574     libcpmt:xthrow.obj
 0001:00002580       ??_7bad_alloc@std@@6B@     10003580     libcpmt:xthrow.obj
 0001:00002588       ??_C@_0P@GHFPNOJB@bad?5allocation@ 10003588     libcpmt:xthrow.obj
 0001:0000259c       ??_7logic_error@std@@6B@   1000359c     libcpmt:xthrow.obj
 0001:000025a8       ??_7length_error@std@@6B@  100035a8     libcpmt:xthrow.obj
 0001:000025b4       ??_7out_of_range@std@@6B@  100035b4     libcpmt:xthrow.obj
 0001:000025c0       ??_7runtime_error@std@@6B@ 100035c0     libcpmt:xthrow.obj
 0001:000025cc       ??_7bad_function_call@std@@6B@ 100035cc     libcpmt:xthrow.obj
 0001:000025d4       ??_C@_0BC@DPJNKNAF@bad?5function?5call@ 100035d4     libcpmt:xthrow.obj
 0001:000025ec       ??_7_Facet_base@std@@6B@   100035ec     libcpmt:locale0.obj
 0001:000025fc       ??_7_Locimp@locale@std@@6B@ 100035fc     libcpmt:locale0.obj
 0001:00002608       ??_C@_01NBENCBCI@?$CK@     10003608     libcpmt:locale0.obj
 0001:0000260c       ??_C@_01GFHCPBMG@C@        1000360c     libcpmt:locale0.obj
 0001:00002614       ??_7bad_array_new_length@std@@6B@ 10003614     libcpmt:locale.obj
 0001:0000261c       ??_C@_1BK@MGMFAEKH@?$AAk?$AAe?$AAr?$AAn?$AAe?$AAl?$AA3?$AA2?$AA?4?$AAd?$AAl?$AAl@ 1000361c     libcpmt:winapisupp.obj
 0001:00002638       ??_C@_08KNHFBNJ@FlsAlloc@  10003638     libcpmt:winapisupp.obj
 0001:00002644       ??_C@_07PEJMOBNF@FlsFree@  10003644     libcpmt:winapisupp.obj
 0001:0000264c       ??_C@_0M@GDNOONDI@FlsGetValue@ 1000364c     libcpmt:winapisupp.obj
 0001:00002658       ??_C@_0M@JCPCPOEF@FlsSetValue@ 10003658     libcpmt:winapisupp.obj
 0001:00002664       ??_C@_0BM@HCFOFFN@InitializeCriticalSectionEx@ 10003664     libcpmt:winapisupp.obj
 0001:00002680       ??_C@_0BE@GPLMMCMH@InitOnceExecuteOnce@ 10003680     libcpmt:winapisupp.obj
 0001:00002694       ??_C@_0P@DLHPPCNH@CreateEventExW@ 10003694     libcpmt:winapisupp.obj
 0001:000026a4       ??_C@_0BB@MEFPJLHN@CreateSemaphoreW@ 100036a4     libcpmt:winapisupp.obj
 0001:000026b8       ??_C@_0BD@KIEEOEEH@CreateSemaphoreExW@ 100036b8     libcpmt:winapisupp.obj
 0001:000026cc       ??_C@_0BG@OGFAJCKC@CreateThreadpoolTimer@ 100036cc     libcpmt:winapisupp.obj
 0001:000026e4       ??_C@_0BD@LPLEMMDI@SetThreadpoolTimer@ 100036e4     libcpmt:winapisupp.obj
 0001:000026f8       ??_C@_0CA@FMNJENH@WaitForThreadpoolTimerCallbacks@ 100036f8     libcpmt:winapisupp.obj
 0001:00002718       ??_C@_0BF@DCFCCNOC@CloseThreadpoolTimer@ 10003718     libcpmt:winapisupp.obj
 0001:00002730       ??_C@_0BF@FLABGKKM@CreateThreadpoolWait@ 10003730     libcpmt:winapisupp.obj
 0001:00002748       ??_C@_0BC@MGCOHNA@SetThreadpoolWait@ 10003748     libcpmt:winapisupp.obj
 0001:0000275c       ??_C@_0BE@OCIOMIMP@CloseThreadpoolWait@ 1000375c     libcpmt:winapisupp.obj
 0001:00002770       ??_C@_0BJ@LKGHFHBO@FlushProcessWriteBuffers@ 10003770     libcpmt:winapisupp.obj
 0001:0000278c       ??_C@_0BP@KALKKPMO@FreeLibraryWhenCallbackReturns@ 1000378c     libcpmt:winapisupp.obj
 0001:000027ac       ??_C@_0BK@DFNBACLA@GetCurrentProcessorNumber@ 100037ac     libcpmt:winapisupp.obj
 0001:000027c8       ??_C@_0BE@FKKLLFLM@CreateSymbolicLinkW@ 100037c8     libcpmt:winapisupp.obj
 0001:000027dc       ??_C@_0BE@JOGNEJCI@GetCurrentPackageId@ 100037dc     libcpmt:winapisupp.obj
 0001:000027f0       ??_C@_0P@CDHHOHKP@GetTickCount64@ 100037f0     libcpmt:winapisupp.obj
 0001:00002800       ??_C@_0BN@NEEHBBPO@GetFileInformationByHandleEx@ 10003800     libcpmt:winapisupp.obj
 0001:00002820       ??_C@_0BL@KBBHGKCM@SetFileInformationByHandle@ 10003820     libcpmt:winapisupp.obj
 0001:0000283c       ??_C@_0BP@FPNJPEJC@GetSystemTimePreciseAsFileTime@ 1000383c     libcpmt:winapisupp.obj
 0001:0000285c       ??_C@_0BM@HLJJNPAH@InitializeConditionVariable@ 1000385c     libcpmt:winapisupp.obj
 0001:00002878       ??_C@_0BG@BFNILBLN@WakeConditionVariable@ 10003878     libcpmt:winapisupp.obj
 0001:00002890       ??_C@_0BJ@PGPPEPCC@WakeAllConditionVariable@ 10003890     libcpmt:winapisupp.obj
 0001:000028ac       ??_C@_0BJ@JEBJOJFJ@SleepConditionVariableCS@ 100038ac     libcpmt:winapisupp.obj
 0001:000028c8       ??_C@_0BC@MMLHEBPB@InitializeSRWLock@ 100038c8     libcpmt:winapisupp.obj
 0001:000028dc       ??_C@_0BI@OMNLIJDB@AcquireSRWLockExclusive@ 100038dc     libcpmt:winapisupp.obj
 0001:000028f4       ??_C@_0BL@OGHFEMNA@TryAcquireSRWLockExclusive@ 100038f4     libcpmt:winapisupp.obj
 0001:00002910       ??_C@_0BI@HMIEPCNJ@ReleaseSRWLockExclusive@ 10003910     libcpmt:winapisupp.obj
 0001:00002928       ??_C@_0BK@LGACAGIC@SleepConditionVariableSRW@ 10003928     libcpmt:winapisupp.obj
 0001:00002944       ??_C@_0BF@GGPHFPJA@CreateThreadpoolWork@ 10003944     libcpmt:winapisupp.obj
 0001:0000295c       ??_C@_0BF@NHDAIMMO@SubmitThreadpoolWork@ 1000395c     libcpmt:winapisupp.obj
 0001:00002974       ??_C@_0BE@NPHIPNPD@CloseThreadpoolWork@ 10003974     libcpmt:winapisupp.obj
 0001:00002988       ??_C@_0BA@IHGNDAEB@CompareStringEx@ 10003988     libcpmt:winapisupp.obj
 0001:00002998       ??_C@_0BA@ONOKGCMP@GetLocaleInfoEx@ 10003998     libcpmt:winapisupp.obj
 0001:000029a8       ??_C@_0O@KKBNKAPF@LCMapStringEx@ 100039a8     libcpmt:winapisupp.obj
 0001:000029bc       ??_7?$numpunct@_W@std@@6B@ 100039bc     libcpmt:wlocale.obj
 0001:000029dc       ??_C@_13IMODFHAA@?$AA?9@   100039dc     libcpmt:wlocale.obj
 0001:000029e0       ??_C@_01JOAMLHOP@?9@       100039e0     libcpmt:wlocale.obj
 0001:000038c8       ??_C@_15EMKDOKLE@?$AAa?$AAr@ 100048c8     libcpmt:winapinls.obj
 0001:000038d0       ??_C@_15KNPADPLH@?$AAb?$AAg@ 100048d0     libcpmt:winapinls.obj
 0001:000038d8       ??_C@_15EDMHLDMO@?$AAc?$AAa@ 100048d8     libcpmt:winapinls.obj
 0001:000038e0       ??_C@_1O@BPEAJADD@?$AAz?$AAh?$AA?9?$AAC?$AAH?$AAS@ 100048e0     libcpmt:winapinls.obj
 0001:000038f0       ??_C@_15LJNHCMNK@?$AAc?$AAs@ 100048f0     libcpmt:winapinls.obj
 0001:000038f8       ??_C@_15FOMCIDHG@?$AAd?$AAa@ 100048f8     libcpmt:winapinls.obj
 0001:00003900       ??_C@_15NBKABECB@?$AAd?$AAe@ 10004900     libcpmt:winapinls.obj
 0001:00003908       ??_C@_15GHPEIIAO@?$AAe?$AAl@ 10004908     libcpmt:winapinls.obj
 0001:00003910       ??_C@_15MNPNEAIF@?$AAe?$AAn@ 10004910     libcpmt:winapinls.obj
 0001:00003918       ??_C@_15GPIOMPMH@?$AAe?$AAs@ 10004918     libcpmt:winapinls.obj
 0001:00003920       ??_C@_15NGLOAKJC@?$AAf?$AAi@ 10004920     libcpmt:winapinls.obj
 0001:00003928       ??_C@_15FBKGNKAM@?$AAf?$AAr@ 10004928     libcpmt:winapinls.obj
 0001:00003930       ??_C@_15KGGCNEFK@?$AAh?$AAe@ 10004930     libcpmt:winapinls.obj
 0001:00003938       ??_C@_15PGHLIDMF@?$AAh?$AAu@ 10004938     libcpmt:winapinls.obj
 0001:00003940       ??_C@_15BIEMAPLM@?$AAi?$AAs@ 10004940     libcpmt:winapinls.obj
 0001:00003948       ??_C@_15IFJLDHAF@?$AAi?$AAt@ 10004948     libcpmt:winapinls.obj
 0001:00003950       ??_C@_15GEMIOCAG@?$AAj?$AAa@ 10004950     libcpmt:winapinls.obj
 0001:00003958       ??_C@_15EPELEGJA@?$AAk?$AAo@ 10004958     libcpmt:winapinls.obj
 0001:00003960       ??_C@_15NDDHIMN@?$AAn?$AAl@ 10004960     libcpmt:winapinls.obj
 0001:00003968       ??_C@_15BPIGNHCD@?$AAn?$AAo@ 10004968     libcpmt:winapinls.obj
 0001:00003970       ??_C@_15DEOPBLCG@?$AAp?$AAl@ 10004970     libcpmt:winapinls.obj
 0001:00003978       ??_C@_15KBECGEFG@?$AAp?$AAt@ 10004978     libcpmt:winapinls.obj
 0001:00003980       ??_C@_15GLJCBFMD@?$AAr?$AAo@ 10004980     libcpmt:winapinls.obj
 0001:00003988       ??_C@_15FEDGKCDI@?$AAr?$AAu@ 10004988     libcpmt:winapinls.obj
 0001:00003990       ??_C@_15GLKMLLHM@?$AAh?$AAr@ 10004990     libcpmt:winapinls.obj
 0001:00003998       ??_C@_15CPKMFBDB@?$AAs?$AAk@ 10004998     libcpmt:winapinls.obj
 0001:000039a0       ??_C@_15BAAIOGMK@?$AAs?$AAq@ 100049a0     libcpmt:winapinls.obj
 0001:000039a8       ??_C@_15INNPNOHD@?$AAs?$AAv@ 100049a8     libcpmt:winapinls.obj
 0001:000039b0       ??_C@_15CABMMOGH@?$AAt?$AAh@ 100049b0     libcpmt:winapinls.obj
 0001:000039b8       ??_C@_15BPLIHJJM@?$AAt?$AAr@ 100049b8     libcpmt:winapinls.obj
 0001:000039c0       ??_C@_15NEOEKKDJ@?$AAu?$AAr@ 100049c0     libcpmt:winapinls.obj
 0001:000039c8       ??_C@_15NFICGAJK@?$AAi?$AAd@ 100049c8     libcpmt:winapinls.obj
 0001:000039d0       ??_C@_15PJPFLCCM@?$AAu?$AAk@ 100049d0     libcpmt:winapinls.obj
 0001:000039d8       ??_C@_15HPJPHDM@?$AAb?$AAe@ 100049d8     libcpmt:winapinls.obj
 0001:000039e0       ??_C@_15LCHLGJII@?$AAs?$AAl@ 100049e0     libcpmt:winapinls.obj
 0001:000039e8       ??_C@_15PCFJPHHO@?$AAe?$AAt@ 100049e8     libcpmt:winapinls.obj
 0001:000039f0       ??_C@_15HPFPGODN@?$AAl?$AAv@ 100049f0     libcpmt:winapinls.obj
 0001:000039f8       ??_C@_15NFFGKGLG@?$AAl?$AAt@ 100049f8     libcpmt:winapinls.obj
 0001:00003a00       ??_C@_15BDAKCCHN@?$AAf?$AAa@ 10004a00     libcpmt:winapinls.obj
 0001:00003a08       ??_C@_15NFGIAIAJ@?$AAv?$AAi@ 10004a08     libcpmt:winapinls.obj
 0001:00003a10       ??_C@_15LMKNDMHN@?$AAh?$AAy@ 10004a10     libcpmt:winapinls.obj
 0001:00003a18       ??_C@_15IJBHMCFL@?$AAa?$AAz@ 10004a18     libcpmt:winapinls.obj
 0001:00003a20       ??_C@_15EKOFJABL@?$AAe?$AAu@ 10004a20     libcpmt:winapinls.obj
 0001:00003a28       ??_C@_15BGHADCNK@?$AAm?$AAk@ 10004a28     libcpmt:winapinls.obj
 0001:00003a30       ??_C@_15JDNICKHM@?$AAa?$AAf@ 10004a30     libcpmt:winapinls.obj
 0001:00003a38       ??_C@_15KPJEDBKD@?$AAk?$AAa@ 10004a38     libcpmt:winapinls.obj
 0001:00003a40       ??_C@_15PDNFFFEO@?$AAf?$AAo@ 10004a40     libcpmt:winapinls.obj
 0001:00003a48       ??_C@_15OMLEGLOC@?$AAh?$AAi@ 10004a48     libcpmt:winapinls.obj
 0001:00003a50       ??_C@_15IDNNENKK@?$AAm?$AAs@ 10004a50     libcpmt:winapinls.obj
 0001:00003a58       ??_C@_15MACJNBMH@?$AAk?$AAk@ 10004a58     libcpmt:winapinls.obj
 0001:00003a60       ??_C@_15DKDJEOND@?$AAk?$AAy@ 10004a60     libcpmt:winapinls.obj
 0001:00003a68       ??_C@_15DFGDLJBG@?$AAs?$AAw@ 10004a68     libcpmt:winapinls.obj
 0001:00003a70       ??_C@_15BBFAICNG@?$AAu?$AAz@ 10004a70     libcpmt:winapinls.obj
 0001:00003a78       ??_C@_15DKNDCGEA@?$AAt?$AAt@ 10004a78     libcpmt:winapinls.obj
 0001:00003a80       ??_C@_15MGIFMDPL@?$AAp?$AAa@ 10004a80     libcpmt:winapinls.obj
 0001:00003a88       ??_C@_15HCNDBBA@?$AAg?$AAu@ 10004a88     libcpmt:winapinls.obj
 0001:00003a90       ??_C@_15FNBEIBON@?$AAt?$AAa@ 10004a90     libcpmt:winapinls.obj
 0001:00003a98       ??_C@_15NCHGBGLK@?$AAt?$AAe@ 10004a98     libcpmt:winapinls.obj
 0001:00003aa0       ??_C@_15PHPHCBPF@?$AAk?$AAn@ 10004aa0     libcpmt:winapinls.obj
 0001:00003aa8       ??_C@_15DLGBCKMP@?$AAm?$AAr@ 10004aa8     libcpmt:winapinls.obj
 0001:00003ab0       ??_C@_15EABBLBFF@?$AAs?$AAa@ 10004ab0     libcpmt:winapinls.obj
 0001:00003ab8       ??_C@_15CBKOMCOI@?$AAm?$AAn@ 10004ab8     libcpmt:winapinls.obj
 0001:00003ac0       ??_C@_15CKDMCJAF@?$AAg?$AAl@ 10004ac0     libcpmt:winapinls.obj
 0001:00003ac8       ??_C@_17CNJFBPG@?$AAk?$AAo?$AAk@ 10004ac8     libcpmt:winapinls.obj
 0001:00003ad0       ??_C@_17FFBJICPL@?$AAs?$AAy?$AAr@ 10004ad0     libcpmt:winapinls.obj
 0001:00003ad8       ??_C@_17KPNDCPAF@?$AAd?$AAi?$AAv@ 10004ad8     libcpmt:winapinls.obj
 0001:00003ae0       ??_C@_1M@OKAHONE@?$AAa?$AAr?$AA?9?$AAS?$AAA@ 10004ae0     libcpmt:winapinls.obj
 0001:00003aec       ??_C@_1M@FFFIGIGK@?$AAb?$AAg?$AA?9?$AAB?$AAG@ 10004aec     libcpmt:winapinls.obj
 0001:00003af8       ??_C@_1M@BJNKEDC@?$AAc?$AAa?$AA?9?$AAE?$AAS@ 10004af8     libcpmt:winapinls.obj
 0001:00003b04       ??_C@_1M@CLNBBOPM@?$AAz?$AAh?$AA?9?$AAT?$AAW@ 10004b04     libcpmt:winapinls.obj
 0001:00003b10       ??_C@_1M@IJJHFJHA@?$AAc?$AAs?$AA?9?$AAC?$AAZ@ 10004b10     libcpmt:winapinls.obj
 0001:00003b1c       ??_C@_1M@CLPEOBGI@?$AAd?$AAa?$AA?9?$AAD?$AAK@ 10004b1c     libcpmt:winapinls.obj
 0001:00003b28       ??_C@_1M@MCMADGCB@?$AAd?$AAe?$AA?9?$AAD?$AAE@ 10004b28     libcpmt:winapinls.obj
 0001:00003b34       ??_C@_1M@OOCKEMAM@?$AAe?$AAl?$AA?9?$AAG?$AAR@ 10004b34     libcpmt:winapinls.obj
 0001:00003b40       ??_C@_1M@BMHNFIME@?$AAe?$AAn?$AA?9?$AAU?$AAS@ 10004b40     libcpmt:winapinls.obj
 0001:00003b4c       ??_C@_1M@DDNJFGID@?$AAf?$AAi?$AA?9?$AAF?$AAI@ 10004b4c     libcpmt:winapinls.obj
 0001:00003b58       ??_C@_1M@GLIPPMAC@?$AAf?$AAr?$AA?9?$AAF?$AAR@ 10004b58     libcpmt:winapinls.obj
 0001:00003b64       ??_C@_1M@GFMCHPE@?$AAh?$AAe?$AA?9?$AAI?$AAL@ 10004b64     libcpmt:winapinls.obj
 0001:00003b70       ??_C@_1M@MHLPGNKM@?$AAh?$AAu?$AA?9?$AAH?$AAU@ 10004b70     libcpmt:winapinls.obj
 0001:00003b7c       ??_C@_1M@LPDDNNPN@?$AAi?$AAs?$AA?9?$AAI?$AAS@ 10004b7c     libcpmt:winapinls.obj
 0001:00003b88       ??_C@_1M@MADIPODN@?$AAi?$AAt?$AA?9?$AAI?$AAT@ 10004b88     libcpmt:winapinls.obj
 0001:00003b94       ??_C@_1M@HPNHIDJI@?$AAj?$AAa?$AA?9?$AAJ?$AAP@ 10004b94     libcpmt:winapinls.obj
 0001:00003ba0       ??_C@_1M@JLOOOEGK@?$AAk?$AAo?$AA?9?$AAK?$AAR@ 10004ba0     libcpmt:winapinls.obj
 0001:00003bac       ??_C@_1M@IHBJJGG@?$AAn?$AAl?$AA?9?$AAN?$AAL@ 10004bac     libcpmt:winapinls.obj
 0001:00003bb8       ??_C@_1M@EANAGDL@?$AAn?$AAb?$AA?9?$AAN?$AAO@ 10004bb8     libcpmt:winapinls.obj
 0001:00003bc4       ??_C@_1M@NEIEMEGP@?$AAp?$AAl?$AA?9?$AAP?$AAL@ 10004bc4     libcpmt:winapinls.obj
 0001:00003bd0       ??_C@_1M@BOCFIGEP@?$AAp?$AAt?$AA?9?$AAB?$AAR@ 10004bd0     libcpmt:winapinls.obj
 0001:00003bdc       ??_C@_1M@IMPFOPBG@?$AAr?$AAo?$AA?9?$AAR?$AAO@ 10004bdc     libcpmt:winapinls.obj
 0001:00003be8       ??_C@_1M@IDNNEJMM@?$AAr?$AAu?$AA?9?$AAR?$AAU@ 10004be8     libcpmt:winapinls.obj
 0001:00003bf4       ??_C@_1M@LILEEOGM@?$AAh?$AAr?$AA?9?$AAH?$AAR@ 10004bf4     libcpmt:winapinls.obj
 0001:00003c00       ??_C@_1M@FKIFEHPB@?$AAs?$AAk?$AA?9?$AAS?$AAK@ 10004c00     libcpmt:winapinls.obj
 0001:00003c0c       ??_C@_1M@LJMAMNPJ@?$AAs?$AAq?$AA?9?$AAA?$AAL@ 10004c0c     libcpmt:winapinls.obj
 0001:00003c18       ??_C@_1M@GIAKDKJK@?$AAs?$AAv?$AA?9?$AAS?$AAE@ 10004c18     libcpmt:winapinls.obj
 0001:00003c24       ??_C@_1M@MKJKIKCL@?$AAt?$AAh?$AA?9?$AAT?$AAH@ 10004c24     libcpmt:winapinls.obj
 0001:00003c30       ??_C@_1M@MFLCCMPB@?$AAt?$AAr?$AA?9?$AAT?$AAR@ 10004c30     libcpmt:winapinls.obj
 0001:00003c3c       ??_C@_1M@OIJHDKJN@?$AAu?$AAr?$AA?9?$AAP?$AAK@ 10004c3c     libcpmt:winapinls.obj
 0001:00003c48       ??_C@_1M@LHIPCIEK@?$AAi?$AAd?$AA?9?$AAI?$AAD@ 10004c48     libcpmt:winapinls.obj
 0001:00003c54       ??_C@_1M@MFMOBGI@?$AAu?$AAk?$AA?9?$AAU?$AAA@ 10004c54     libcpmt:winapinls.obj
 0001:00003c60       ??_C@_1M@OBGLJIPL@?$AAb?$AAe?$AA?9?$AAB?$AAY@ 10004c60     libcpmt:winapinls.obj
 0001:00003c6c       ??_C@_1M@BCFAJEAD@?$AAs?$AAl?$AA?9?$AAS?$AAI@ 10004c6c     libcpmt:winapinls.obj
 0001:00003c78       ??_C@_1M@FKFFEDDN@?$AAe?$AAt?$AA?9?$AAE?$AAE@ 10004c78     libcpmt:winapinls.obj
 0001:00003c84       ??_C@_1M@KGKKAACI@?$AAl?$AAv?$AA?9?$AAL?$AAV@ 10004c84     libcpmt:winapinls.obj
 0001:00003c90       ??_C@_1M@IFGBIJO@?$AAl?$AAt?$AA?9?$AAL?$AAT@ 10004c90     libcpmt:winapinls.obj
 0001:00003c9c       ??_C@_1M@FGEAHEDM@?$AAf?$AAa?$AA?9?$AAI?$AAR@ 10004c9c     libcpmt:winapinls.obj
 0001:00003ca8       ??_C@_1M@KBMAIBFN@?$AAv?$AAi?$AA?9?$AAV?$AAN@ 10004ca8     libcpmt:winapinls.obj
 0001:00003cb4       ??_C@_1M@GPCBKDJK@?$AAh?$AAy?$AA?9?$AAA?$AAM@ 10004cb4     libcpmt:winapinls.obj
 0001:00003cc0       ??_C@_1BG@BECMDDJB@?$AAa?$AAz?$AA?9?$AAA?$AAZ?$AA?9?$AAL?$AAa?$AAt?$AAn@ 10004cc0     libcpmt:winapinls.obj
 0001:00003cd8       ??_C@_1M@MAOFCAEA@?$AAe?$AAu?$AA?9?$AAE?$AAS@ 10004cd8     libcpmt:winapinls.obj
 0001:00003ce4       ??_C@_1M@IGHABKPI@?$AAm?$AAk?$AA?9?$AAM?$AAK@ 10004ce4     libcpmt:winapinls.obj
 0001:00003cf0       ??_C@_1M@IAIGNEJG@?$AAt?$AAn?$AA?9?$AAZ?$AAA@ 10004cf0     libcpmt:winapinls.obj
 0001:00003cfc       ??_C@_1M@IIJCOJFA@?$AAx?$AAh?$AA?9?$AAZ?$AAA@ 10004cfc     libcpmt:winapinls.obj
 0001:00003d08       ??_C@_1M@LGPJHNJH@?$AAz?$AAu?$AA?9?$AAZ?$AAA@ 10004d08     libcpmt:winapinls.obj
 0001:00003d14       ??_C@_1M@HOKAOIO@?$AAa?$AAf?$AA?9?$AAZ?$AAA@ 10004d14     libcpmt:winapinls.obj
 0001:00003d20       ??_C@_1M@DPCLHLIE@?$AAk?$AAa?$AA?9?$AAG?$AAE@ 10004d20     libcpmt:winapinls.obj
 0001:00003d2c       ??_C@_1M@BLKMHJBI@?$AAf?$AAo?$AA?9?$AAF?$AAO@ 10004d2c     libcpmt:winapinls.obj
 0001:00003d38       ??_C@_1M@LGGJAPPB@?$AAh?$AAi?$AA?9?$AAI?$AAN@ 10004d38     libcpmt:winapinls.obj
 0001:00003d44       ??_C@_1M@FIKPIHFE@?$AAm?$AAt?$AA?9?$AAM?$AAT@ 10004d44     libcpmt:winapinls.obj
 0001:00003d50       ??_C@_1M@HEGGPBFA@?$AAs?$AAe?$AA?9?$AAN?$AAO@ 10004d50     libcpmt:winapinls.obj
 0001:00003d5c       ??_C@_1M@EIBJEEPA@?$AAm?$AAs?$AA?9?$AAM?$AAY@ 10004d5c     libcpmt:winapinls.obj
 0001:00003d68       ??_C@_1M@FHLBGMPP@?$AAk?$AAk?$AA?9?$AAK?$AAZ@ 10004d68     libcpmt:winapinls.obj
 0001:00003d74       ??_C@_1M@NGJJLCGI@?$AAk?$AAy?$AA?9?$AAK?$AAG@ 10004d74     libcpmt:winapinls.obj
 0001:00003d80       ??_C@_1M@GIENNBFC@?$AAs?$AAw?$AA?9?$AAK?$AAE@ 10004d80     libcpmt:winapinls.obj
 0001:00003d8c       ??_C@_1BG@NDGMJIMJ@?$AAu?$AAz?$AA?9?$AAU?$AAZ?$AA?9?$AAL?$AAa?$AAt?$AAn@ 10004d8c     libcpmt:winapinls.obj
 0001:00003da4       ??_C@_1M@IDCCIHBC@?$AAt?$AAt?$AA?9?$AAR?$AAU@ 10004da4     libcpmt:winapinls.obj
 0001:00003db0       ??_C@_1M@LOICPMOJ@?$AAb?$AAn?$AA?9?$AAI?$AAN@ 10004db0     libcpmt:winapinls.obj
 0001:00003dbc       ??_C@_1M@KPKKNEAH@?$AAp?$AAa?$AA?9?$AAI?$AAN@ 10004dbc     libcpmt:winapinls.obj
 0001:00003dc8       ??_C@_1M@PJGPPBOG@?$AAg?$AAu?$AA?9?$AAI?$AAN@ 10004dc8     libcpmt:winapinls.obj
 0001:00003dd4       ??_C@_1M@KMKMOPHI@?$AAt?$AAa?$AA?9?$AAI?$AAN@ 10004dd4     libcpmt:winapinls.obj
 0001:00003de0       ??_C@_1M@KFEHEPAC@?$AAt?$AAe?$AA?9?$AAI?$AAN@ 10004de0     libcpmt:winapinls.obj
 0001:00003dec       ??_C@_1M@CDCLMGHI@?$AAk?$AAn?$AA?9?$AAI?$AAN@ 10004dec     libcpmt:winapinls.obj
 0001:00003df8       ??_C@_1M@MIODLDKF@?$AAm?$AAl?$AA?9?$AAI?$AAN@ 10004df8     libcpmt:winapinls.obj
 0001:00003e04       ??_C@_1M@PBIEACPO@?$AAm?$AAr?$AA?9?$AAI?$AAN@ 10004e04     libcpmt:winapinls.obj
 0001:00003e10       ??_C@_1M@NIDEAGPH@?$AAs?$AAa?$AA?9?$AAI?$AAN@ 10004e10     libcpmt:winapinls.obj
 0001:00003e1c       ??_C@_1M@FHIHCBIO@?$AAm?$AAn?$AA?9?$AAM?$AAN@ 10004e1c     libcpmt:winapinls.obj
 0001:00003e28       ??_C@_1M@JAIJPENP@?$AAc?$AAy?$AA?9?$AAG?$AAB@ 10004e28     libcpmt:winapinls.obj
 0001:00003e34       ??_C@_1M@PHGFBEPN@?$AAg?$AAl?$AA?9?$AAE?$AAS@ 10004e34     libcpmt:winapinls.obj
 0001:00003e40       ??_C@_1O@KPIPDNCP@?$AAk?$AAo?$AAk?$AA?9?$AAI?$AAN@ 10004e40     libcpmt:winapinls.obj
 0001:00003e50       ??_C@_1O@KNHJLDJA@?$AAs?$AAy?$AAr?$AA?9?$AAS?$AAY@ 10004e50     libcpmt:winapinls.obj
 0001:00003e60       ??_C@_1O@MKEKBLAH@?$AAd?$AAi?$AAv?$AA?9?$AAM?$AAV@ 10004e60     libcpmt:winapinls.obj
 0001:00003e70       ??_C@_1O@OHDCKDDF@?$AAq?$AAu?$AAz?$AA?9?$AAB?$AAO@ 10004e70     libcpmt:winapinls.obj
 0001:00003e80       ??_C@_1M@LEPJNLFD@?$AAn?$AAs?$AA?9?$AAZ?$AAA@ 10004e80     libcpmt:winapinls.obj
 0001:00003e8c       ??_C@_1M@OMLEIIJB@?$AAm?$AAi?$AA?9?$AAN?$AAZ@ 10004e8c     libcpmt:winapinls.obj
 0001:00003e98       ??_C@_1M@PMPEAILG@?$AAa?$AAr?$AA?9?$AAI?$AAQ@ 10004e98     libcpmt:winapinls.obj
 0001:00003ea4       ??_C@_1M@BIBDDEMK@?$AAz?$AAh?$AA?9?$AAC?$AAN@ 10004ea4     libcpmt:winapinls.obj
 0001:00003eb0       ??_C@_1M@CNKPNOEE@?$AAd?$AAe?$AA?9?$AAC?$AAH@ 10004eb0     libcpmt:winapinls.obj
 0001:00003ebc       ??_C@_1M@LKMGMLKO@?$AAe?$AAn?$AA?9?$AAG?$AAB@ 10004ebc     libcpmt:winapinls.obj
 0001:00003ec8       ??_C@_1M@PGKJFFGL@?$AAe?$AAs?$AA?9?$AAM?$AAX@ 10004ec8     libcpmt:winapinls.obj
 0001:00003ed4       ??_C@_1M@DNNANBDC@?$AAf?$AAr?$AA?9?$AAB?$AAE@ 10004ed4     libcpmt:winapinls.obj
 0001:00003ee0       ??_C@_1M@HLGMDFHM@?$AAi?$AAt?$AA?9?$AAC?$AAH@ 10004ee0     libcpmt:winapinls.obj
 0001:00003eec       ??_C@_1M@CLLBGJH@?$AAn?$AAl?$AA?9?$AAB?$AAE@ 10004eec     libcpmt:winapinls.obj
 0001:00003ef8       ??_C@_1M@BODBOGLF@?$AAn?$AAn?$AA?9?$AAN?$AAO@ 10004ef8     libcpmt:winapinls.obj
 0001:00003f04       ??_C@_1M@HFFAHKAD@?$AAp?$AAt?$AA?9?$AAP?$AAT@ 10004f04     libcpmt:winapinls.obj
 0001:00003f10       ??_C@_1BG@LNOAKHIE@?$AAs?$AAr?$AA?9?$AAS?$AAP?$AA?9?$AAL?$AAa?$AAt?$AAn@ 10004f10     libcpmt:winapinls.obj
 0001:00003f28       ??_C@_1M@HBMHBGAK@?$AAs?$AAv?$AA?9?$AAF?$AAI@ 10004f28     libcpmt:winapinls.obj
 0001:00003f34       ??_C@_1BG@DGCJGJBE@?$AAa?$AAz?$AA?9?$AAA?$AAZ?$AA?9?$AAC?$AAy?$AAr?$AAl@ 10004f34     libcpmt:winapinls.obj
 0001:00003f4c       ??_C@_1M@KEJDAAHB@?$AAs?$AAe?$AA?9?$AAS?$AAE@ 10004f4c     libcpmt:winapinls.obj
 0001:00003f58       ??_C@_1M@HEIBJJAD@?$AAm?$AAs?$AA?9?$AAB?$AAN@ 10004f58     libcpmt:winapinls.obj
 0001:00003f64       ??_C@_1BG@PBGJMCEM@?$AAu?$AAz?$AA?9?$AAU?$AAZ?$AA?9?$AAC?$AAy?$AAr?$AAl@ 10004f64     libcpmt:winapinls.obj
 0001:00003f7c       ??_C@_1O@LAOBCMDF@?$AAq?$AAu?$AAz?$AA?9?$AAE?$AAC@ 10004f7c     libcpmt:winapinls.obj
 0001:00003f8c       ??_C@_1M@POEEMAIO@?$AAa?$AAr?$AA?9?$AAE?$AAG@ 10004f8c     libcpmt:winapinls.obj
 0001:00003f98       ??_C@_1M@EFAKDEDL@?$AAz?$AAh?$AA?9?$AAH?$AAK@ 10004f98     libcpmt:winapinls.obj
 0001:00003fa4       ??_C@_1M@HKKIJHGI@?$AAd?$AAe?$AA?9?$AAA?$AAT@ 10004fa4     libcpmt:winapinls.obj
 0001:00003fb0       ??_C@_1M@KBFBEHJF@?$AAe?$AAn?$AA?9?$AAA?$AAU@ 10004fb0     libcpmt:winapinls.obj
 0001:00003fbc       ??_C@_1M@MNPLFAAH@?$AAe?$AAs?$AA?9?$AAE?$AAS@ 10004fbc     libcpmt:winapinls.obj
 0001:00003fc8       ??_C@_1M@HJOOJFMA@?$AAf?$AAr?$AA?9?$AAC?$AAA@ 10004fc8     libcpmt:winapinls.obj
 0001:00003fd4       ??_C@_1BG@JPOFPNAB@?$AAs?$AAr?$AA?9?$AAS?$AAP?$AA?9?$AAC?$AAy?$AAr?$AAl@ 10004fd4     libcpmt:winapinls.obj
 0001:00003fec       ??_C@_1M@LNFOCMOB@?$AAs?$AAe?$AA?9?$AAF?$AAI@ 10004fec     libcpmt:winapinls.obj
 0001:00003ff8       ??_C@_1O@MGJBOAMB@?$AAq?$AAu?$AAz?$AA?9?$AAP?$AAE@ 10004ff8     libcpmt:winapinls.obj
 0001:00004008       ??_C@_1M@GJINLBOK@?$AAa?$AAr?$AA?9?$AAL?$AAY@ 10005008     libcpmt:winapinls.obj
 0001:00004014       ??_C@_1M@GGMNHJNL@?$AAz?$AAh?$AA?9?$AAS?$AAG@ 10005014     libcpmt:winapinls.obj
 0001:00004020       ??_C@_1M@HOIKODND@?$AAd?$AAe?$AA?9?$AAL?$AAU@ 10005020     libcpmt:winapinls.obj
 0001:0000402c       ??_C@_1M@DDOCCGFG@?$AAe?$AAn?$AA?9?$AAC?$AAA@ 1000502c     libcpmt:winapinls.obj
 0001:00004038       ??_C@_1M@BNOEMJLF@?$AAe?$AAs?$AA?9?$AAG?$AAT@ 10005038     libcpmt:winapinls.obj
 0001:00004044       ??_C@_1M@EOGNKEK@?$AAf?$AAr?$AA?9?$AAC?$AAH@ 10005044     libcpmt:winapinls.obj
 0001:00004050       ??_C@_1M@FLIDJFHL@?$AAh?$AAr?$AA?9?$AAB?$AAA@ 10005050     libcpmt:winapinls.obj
 0001:0000405c       ??_C@_1O@FMCELNAJ@?$AAs?$AAm?$AAj?$AA?9?$AAN?$AAO@ 1000505c     libcpmt:winapinls.obj
 0001:0000406c       ??_C@_1M@JHGLJMGJ@?$AAa?$AAr?$AA?9?$AAD?$AAZ@ 1000506c     libcpmt:winapinls.obj
 0001:00004078       ??_C@_1M@JKKFDCNP@?$AAz?$AAh?$AA?9?$AAM?$AAO@ 10005078     libcpmt:winapinls.obj
 0001:00004084       ??_C@_1M@GEEFALPE@?$AAd?$AAe?$AA?9?$AAL?$AAI@ 10005084     libcpmt:winapinls.obj
 0001:00004090       ??_C@_1M@IGEOFBG@?$AAe?$AAn?$AA?9?$AAN?$AAZ@ 10005090     libcpmt:winapinls.obj
 0001:0000409c       ??_C@_1M@KDBONEHP@?$AAe?$AAs?$AA?9?$AAC?$AAR@ 1000509c     libcpmt:winapinls.obj
 0001:000040a8       ??_C@_1M@FHMDOHNN@?$AAf?$AAr?$AA?9?$AAL?$AAU@ 100050a8     libcpmt:winapinls.obj
 0001:000040b4       ??_C@_1BG@NFKKMAFG@?$AAb?$AAs?$AA?9?$AAB?$AAA?$AA?9?$AAL?$AAa?$AAt?$AAn@ 100050b4     libcpmt:winapinls.obj
 0001:000040cc       ??_C@_1O@IMNBEMCI@?$AAs?$AAm?$AAj?$AA?9?$AAS?$AAE@ 100050cc     libcpmt:winapinls.obj
 0001:000040dc       ??_C@_1M@DHHMBNDP@?$AAa?$AAr?$AA?9?$AAM?$AAA@ 100050dc     libcpmt:winapinls.obj
 0001:000040e8       ??_C@_1M@BNBLJCGH@?$AAe?$AAn?$AA?9?$AAI?$AAE@ 100050e8     libcpmt:winapinls.obj
 0001:000040f4       ??_C@_1M@GEPAFMDL@?$AAe?$AAs?$AA?9?$AAP?$AAA@ 100050f4     libcpmt:winapinls.obj
 0001:00004100       ??_C@_1M@OJONDMDL@?$AAf?$AAr?$AA?9?$AAM?$AAC@ 10005100     libcpmt:winapinls.obj
 0001:0000410c       ??_C@_1BG@OBCNFJB@?$AAs?$AAr?$AA?9?$AAB?$AAA?$AA?9?$AAL?$AAa?$AAt?$AAn@ 1000510c     libcpmt:winapinls.obj
 0001:00004124       ??_C@_1O@KEMEEGPO@?$AAs?$AAm?$AAa?$AA?9?$AAN?$AAO@ 10005124     libcpmt:winapinls.obj
 0001:00004134       ??_C@_1M@ELMGFODK@?$AAa?$AAr?$AA?9?$AAT?$AAN@ 10005134     libcpmt:winapinls.obj
 0001:00004140       ??_C@_1M@BHDLHFAF@?$AAe?$AAn?$AA?9?$AAZ?$AAA@ 10005140     libcpmt:winapinls.obj
 0001:0000414c       ??_C@_1M@BMGIGLIF@?$AAe?$AAs?$AA?9?$AAD?$AAO@ 1000514c     libcpmt:winapinls.obj
 0001:00004158       ??_C@_1BG@CMBHIPBE@?$AAs?$AAr?$AA?9?$AAB?$AAA?$AA?9?$AAC?$AAy?$AAr?$AAl@ 10005158     libcpmt:winapinls.obj
 0001:00004170       ??_C@_1O@HEDBLHNP@?$AAs?$AAm?$AAa?$AA?9?$AAS?$AAE@ 10005170     libcpmt:winapinls.obj
 0001:00004180       ??_C@_1M@DAGCADIM@?$AAa?$AAr?$AA?9?$AAO?$AAM@ 10005180     libcpmt:winapinls.obj
 0001:0000418c       ??_C@_1M@FODLMICG@?$AAe?$AAn?$AA?9?$AAJ?$AAM@ 1000518c     libcpmt:winapinls.obj
 0001:00004198       ??_C@_1M@DNMLCIHB@?$AAe?$AAs?$AA?9?$AAV?$AAE@ 10005198     libcpmt:winapinls.obj
 0001:000041a4       ??_C@_1O@EOKHMKJK@?$AAs?$AAm?$AAs?$AA?9?$AAF?$AAI@ 100051a4     libcpmt:winapinls.obj
 0001:000041b4       ??_C@_1M@CAFJMKOF@?$AAa?$AAr?$AA?9?$AAY?$AAE@ 100051b4     libcpmt:winapinls.obj
 0001:000041c0       ??_C@_1M@CBFHIJLI@?$AAe?$AAn?$AA?9?$AAC?$AAB@ 100051c0     libcpmt:winapinls.obj
 0001:000041cc       ??_C@_1M@BGNFLDN@?$AAe?$AAs?$AA?9?$AAC?$AAO@ 100051cc     libcpmt:winapinls.obj
 0001:000041d8       ??_C@_1O@JMPHMAMC@?$AAs?$AAm?$AAn?$AA?9?$AAF?$AAI@ 100051d8     libcpmt:winapinls.obj
 0001:000041e8       ??_C@_1M@JLANABKE@?$AAa?$AAr?$AA?9?$AAS?$AAY@ 100051e8     libcpmt:winapinls.obj
 0001:000041f4       ??_C@_1M@HPKGCFGN@?$AAe?$AAn?$AA?9?$AAB?$AAZ@ 100051f4     libcpmt:winapinls.obj
 0001:00004200       ??_C@_1M@OLJCMLGM@?$AAe?$AAs?$AA?9?$AAP?$AAE@ 10005200     libcpmt:winapinls.obj
 0001:0000420c       ??_C@_1M@MKKGFKLE@?$AAa?$AAr?$AA?9?$AAJ?$AAO@ 1000520c     libcpmt:winapinls.obj
 0001:00004218       ??_C@_1M@EKPGLDNI@?$AAe?$AAn?$AA?9?$AAT?$AAT@ 10005218     libcpmt:winapinls.obj
 0001:00004224       ??_C@_1M@OONGHFHE@?$AAe?$AAs?$AA?9?$AAA?$AAR@ 10005224     libcpmt:winapinls.obj
 0001:00004230       ??_C@_1M@OOJFGBHE@?$AAa?$AAr?$AA?9?$AAL?$AAB@ 10005230     libcpmt:winapinls.obj
 0001:0000423c       ??_C@_1M@GCEJHNEG@?$AAe?$AAn?$AA?9?$AAZ?$AAW@ 1000523c     libcpmt:winapinls.obj
 0001:00004248       ??_C@_1M@JNOCAHJI@?$AAe?$AAs?$AA?9?$AAE?$AAC@ 10005248     libcpmt:winapinls.obj
 0001:00004254       ??_C@_1M@JEFHPGGB@?$AAa?$AAr?$AA?9?$AAK?$AAW@ 10005254     libcpmt:winapinls.obj
 0001:00004260       ??_C@_1M@MLKIBJOJ@?$AAe?$AAn?$AA?9?$AAP?$AAH@ 10005260     libcpmt:winapinls.obj
 0001:0000426c       ??_C@_1M@BDNIPEND@?$AAe?$AAs?$AA?9?$AAC?$AAL@ 1000526c     libcpmt:winapinls.obj
 0001:00004278       ??_C@_1M@MPNMEKBD@?$AAa?$AAr?$AA?9?$AAA?$AAE@ 10005278     libcpmt:winapinls.obj
 0001:00004284       ??_C@_1M@KBJALCPI@?$AAe?$AAs?$AA?9?$AAU?$AAY@ 10005284     libcpmt:winapinls.obj
 0001:00004290       ??_C@_1M@LLCCOAGA@?$AAa?$AAr?$AA?9?$AAB?$AAH@ 10005290     libcpmt:winapinls.obj
 0001:0000429c       ??_C@_1M@PBFNCDEL@?$AAe?$AAs?$AA?9?$AAP?$AAY@ 1000529c     libcpmt:winapinls.obj
 0001:000042a8       ??_C@_1M@EDGINPNP@?$AAa?$AAr?$AA?9?$AAQ?$AAA@ 100052a8     libcpmt:winapinls.obj
 0001:000042b4       ??_C@_1M@MKDBIIJI@?$AAe?$AAs?$AA?9?$AAB?$AAO@ 100052b4     libcpmt:winapinls.obj
 0001:000042c0       ??_C@_1M@CPKKEBLD@?$AAe?$AAs?$AA?9?$AAS?$AAV@ 100052c0     libcpmt:winapinls.obj
 0001:000042cc       ??_C@_1M@NDBGMMJL@?$AAe?$AAs?$AA?9?$AAH?$AAN@ 100052cc     libcpmt:winapinls.obj
 0001:000042d8       ??_C@_1M@JIJIBHDP@?$AAe?$AAs?$AA?9?$AAN?$AAI@ 100052d8     libcpmt:winapinls.obj
 0001:000042e4       ??_C@_1M@CGFMKEEK@?$AAe?$AAs?$AA?9?$AAP?$AAR@ 100052e4     libcpmt:winapinls.obj
 0001:000042f0       ??_C@_1O@ICJHKIIK@?$AAz?$AAh?$AA?9?$AAC?$AAH?$AAT@ 100052f0     libcpmt:winapinls.obj
 0001:00004300       ??_C@_15CLNEJCE@?$AAs?$AAr@ 10005300     libcpmt:winapinls.obj
 0001:00004308       ??_C@_1M@KAHEKEIG@?$AAa?$AAf?$AA?9?$AAz?$AAa@ 10005308     libcpmt:winapinls.obj
 0001:00004314       ??_C@_1M@GIECOABL@?$AAa?$AAr?$AA?9?$AAa?$AAe@ 10005314     libcpmt:winapinls.obj
 0001:00004320       ??_C@_1M@BMLMEKGI@?$AAa?$AAr?$AA?9?$AAb?$AAh@ 10005320     libcpmt:winapinls.obj
 0001:0000432c       ??_C@_1M@DAPFDGGB@?$AAa?$AAr?$AA?9?$AAd?$AAz@ 1000532c     libcpmt:winapinls.obj
 0001:00004338       ??_C@_1M@FJNKGKIG@?$AAa?$AAr?$AA?9?$AAe?$AAg@ 10005338     libcpmt:winapinls.obj
 0001:00004344       ??_C@_1M@FLGKKCLO@?$AAa?$AAr?$AA?9?$AAi?$AAq@ 10005344     libcpmt:winapinls.obj
 0001:00004350       ??_C@_1M@GNDIPALM@?$AAa?$AAr?$AA?9?$AAj?$AAo@ 10005350     libcpmt:winapinls.obj
 0001:0000435c       ??_C@_1M@DDMJFMGJ@?$AAa?$AAr?$AA?9?$AAk?$AAw@ 1000535c     libcpmt:winapinls.obj
 0001:00004368       ??_C@_1M@EJALMLHM@?$AAa?$AAr?$AA?9?$AAl?$AAb@ 10005368     libcpmt:winapinls.obj
 0001:00004374       ??_C@_1M@MOBDBLOC@?$AAa?$AAr?$AA?9?$AAl?$AAy@ 10005374     libcpmt:winapinls.obj
 0001:00004380       ??_C@_1M@JAOCLHDH@?$AAa?$AAr?$AA?9?$AAm?$AAa@ 10005380     libcpmt:winapinls.obj
 0001:0000438c       ??_C@_1M@JHPMKJIE@?$AAa?$AAr?$AA?9?$AAo?$AAm@ 1000538c     libcpmt:winapinls.obj
 0001:00004398       ??_C@_1M@OEPGHFNH@?$AAa?$AAr?$AA?9?$AAq?$AAa@ 10005398     libcpmt:winapinls.obj
 0001:000043a4       ??_C@_1M@KJDONENM@?$AAa?$AAr?$AA?9?$AAs?$AAa@ 100053a4     libcpmt:winapinls.obj
 0001:000043b0       ??_C@_1M@DMJDKLKM@?$AAa?$AAr?$AA?9?$AAs?$AAy@ 100053b0     libcpmt:winapinls.obj
 0001:000043bc       ??_C@_1M@OMFIPEDC@?$AAa?$AAr?$AA?9?$AAt?$AAn@ 100053bc     libcpmt:winapinls.obj
 0001:000043c8       ??_C@_1M@IHMHGAON@?$AAa?$AAr?$AA?9?$AAy?$AAe@ 100053c8     libcpmt:winapinls.obj
 0001:000043d4       ??_C@_1BG@KDCPGJGB@?$AAa?$AAz?$AA?9?$AAa?$AAz?$AA?9?$AAc?$AAy?$AAr?$AAl@ 100053d4     libcpmt:winapinls.obj
 0001:000043ec       ??_C@_1BG@IBCKDDOE@?$AAa?$AAz?$AA?9?$AAa?$AAz?$AA?9?$AAl?$AAa?$AAt?$AAn@ 100053ec     libcpmt:winapinls.obj
 0001:00004404       ??_C@_1M@EGPFDCPD@?$AAb?$AAe?$AA?9?$AAb?$AAy@ 10005404     libcpmt:winapinls.obj
 0001:00004410       ??_C@_1M@PCMGMCGC@?$AAb?$AAg?$AA?9?$AAb?$AAg@ 10005410     libcpmt:winapinls.obj
 0001:0000441c       ??_C@_1M@BJBMFGOB@?$AAb?$AAn?$AA?9?$AAi?$AAn@ 1000541c     libcpmt:winapinls.obj
 0001:00004428       ??_C@_1BG@EAKMMACD@?$AAb?$AAs?$AA?9?$AAb?$AAa?$AA?9?$AAl?$AAa?$AAt?$AAn@ 10005428     libcpmt:winapinls.obj
 0001:00004440       ??_C@_1M@KGADAODK@?$AAc?$AAa?$AA?9?$AAe?$AAs@ 10005440     libcpmt:winapinls.obj
 0001:0000444c       ??_C@_1M@COAJPDHI@?$AAc?$AAs?$AA?9?$AAc?$AAz@ 1000544c     libcpmt:winapinls.obj
 0001:00004458       ??_C@_1M@DHBHFONH@?$AAc?$AAy?$AA?9?$AAg?$AAb@ 10005458     libcpmt:winapinls.obj
 0001:00004464       ??_C@_1M@IMGKELGA@?$AAd?$AAa?$AA?9?$AAd?$AAk@ 10005464     libcpmt:winapinls.obj
 0001:00004470       ??_C@_1M@NNDGDNGA@?$AAd?$AAe?$AA?9?$AAa?$AAt@ 10005470     libcpmt:winapinls.obj
 0001:0000447c       ??_C@_1M@IKDBHEEM@?$AAd?$AAe?$AA?9?$AAc?$AAh@ 1000547c     libcpmt:winapinls.obj
 0001:00004488       ??_C@_1M@GFFOJMCJ@?$AAd?$AAe?$AA?9?$AAd?$AAe@ 10005488     libcpmt:winapinls.obj
 0001:00004494       ??_C@_1M@MDNLKBPM@?$AAd?$AAe?$AA?9?$AAl?$AAi@ 10005494     libcpmt:winapinls.obj
 0001:000044a0       ??_C@_1M@NJBEEJNL@?$AAd?$AAe?$AA?9?$AAl?$AAu@ 100054a0     libcpmt:winapinls.obj
 0001:000044ac       ??_C@_1O@GNNELBAP@?$AAd?$AAi?$AAv?$AA?9?$AAm?$AAv@ 100054ac     libcpmt:winapinls.obj
 0001:000044bc       ??_C@_1M@EJLEOGAE@?$AAe?$AAl?$AA?9?$AAg?$AAr@ 100054bc     libcpmt:winapinls.obj
 0001:000044c8       ??_C@_1M@GMPONJN@?$AAe?$AAn?$AA?9?$AAa?$AAu@ 100054c8     libcpmt:winapinls.obj
 0001:000044d4       ??_C@_1M@NIDIIPGF@?$AAe?$AAn?$AA?9?$AAb?$AAz@ 100054d4     libcpmt:winapinls.obj
 0001:000044e0       ??_C@_1M@JEHMIMFO@?$AAe?$AAn?$AA?9?$AAc?$AAa@ 100054e0     libcpmt:winapinls.obj
 0001:000044ec       ??_C@_1M@IGMJCDLA@?$AAe?$AAn?$AA?9?$AAc?$AAb@ 100054ec     libcpmt:winapinls.obj
 0001:000044f8       ??_C@_1M@BNFIGBKG@?$AAe?$AAn?$AA?9?$AAg?$AAb@ 100054f8     libcpmt:winapinls.obj
 0001:00004504       ??_C@_1M@LKIFDIGP@?$AAe?$AAn?$AA?9?$AAi?$AAe@ 10005504     libcpmt:winapinls.obj
 0001:00004510       ??_C@_1M@PJKFGCCO@?$AAe?$AAn?$AA?9?$AAj?$AAm@ 10005510     libcpmt:winapinls.obj
 0001:0000451c       ??_C@_1M@KPPKEPBO@?$AAe?$AAn?$AA?9?$AAn?$AAz@ 1000551c     libcpmt:winapinls.obj
 0001:00004528       ??_C@_1M@GMDGLDOB@?$AAe?$AAn?$AA?9?$AAp?$AAh@ 10005528     libcpmt:winapinls.obj
 0001:00004534       ??_C@_1M@ONGIBJNA@?$AAe?$AAn?$AA?9?$AAt?$AAt@ 10005534     libcpmt:winapinls.obj
 0001:00004540       ??_C@_1M@LLODPCMM@?$AAe?$AAn?$AA?9?$AAu?$AAs@ 10005540     libcpmt:winapinls.obj
 0001:0000454c       ??_C@_1M@LAKFNPAN@?$AAe?$AAn?$AA?9?$AAz?$AAa@ 1000554c     libcpmt:winapinls.obj
 0001:00004558       ??_C@_1M@MFNHNHEO@?$AAe?$AAn?$AA?9?$AAz?$AAw@ 10005558     libcpmt:winapinls.obj
 0001:00004564       ??_C@_1M@EJEINPHM@?$AAe?$AAs?$AA?9?$AAa?$AAr@ 10005564     libcpmt:winapinls.obj
 0001:00004570       ??_C@_1M@GNKPCCJA@?$AAe?$AAs?$AA?9?$AAb?$AAo@ 10005570     libcpmt:winapinls.obj
 0001:0000457c       ??_C@_1M@LEEGFONL@?$AAe?$AAs?$AA?9?$AAc?$AAl@ 1000557c     libcpmt:winapinls.obj
 0001:00004588       ??_C@_1M@KGPDPBDF@?$AAe?$AAs?$AA?9?$AAc?$AAo@ 10005588     libcpmt:winapinls.obj
 0001:00004594       ??_C@_1M@EIAHOHH@?$AAe?$AAs?$AA?9?$AAc?$AAr@ 10005594     libcpmt:winapinls.obj
 0001:000045a0       ??_C@_1M@LLPGMBIN@?$AAe?$AAs?$AA?9?$AAd?$AAo@ 100055a0     libcpmt:winapinls.obj
 0001:000045ac       ??_C@_1M@DKHMKNJA@?$AAe?$AAs?$AA?9?$AAe?$AAc@ 100055ac     libcpmt:winapinls.obj
 0001:000045b8       ??_C@_1M@GKGFPKAP@?$AAe?$AAs?$AA?9?$AAe?$AAs@ 100055b8     libcpmt:winapinls.obj
 0001:000045c4       ??_C@_1M@LKHKGDLN@?$AAe?$AAs?$AA?9?$AAg?$AAt@ 100055c4     libcpmt:winapinls.obj
 0001:000045d0       ??_C@_1M@HEIIGGJD@?$AAe?$AAs?$AA?9?$AAh?$AAn@ 100055d0     libcpmt:winapinls.obj
 0001:000045dc       ??_C@_1M@FBDHPPGD@?$AAe?$AAs?$AA?9?$AAm?$AAx@ 100055dc     libcpmt:winapinls.obj
 0001:000045e8       ??_C@_1M@DPAGLNDH@?$AAe?$AAs?$AA?9?$AAn?$AAi@ 100055e8     libcpmt:winapinls.obj
 0001:000045f4       ??_C@_1M@MDGOPGDD@?$AAe?$AAs?$AA?9?$AAp?$AAa@ 100055f4     libcpmt:winapinls.obj
 0001:00004600       ??_C@_1M@EMAMGBGE@?$AAe?$AAs?$AA?9?$AAp?$AAe@ 10005600     libcpmt:winapinls.obj
 0001:0000460c       ??_C@_1M@IBMCAOEC@?$AAe?$AAs?$AA?9?$AAp?$AAr@ 1000560c     libcpmt:winapinls.obj
 0001:00004618       ??_C@_1M@FGMDIJED@?$AAe?$AAs?$AA?9?$AAp?$AAy@ 10005618     libcpmt:winapinls.obj
 0001:00004624       ??_C@_1M@IIDEOLLL@?$AAe?$AAs?$AA?9?$AAs?$AAv@ 10005624     libcpmt:winapinls.obj
 0001:00004630       ??_C@_1M@GAOBIPA@?$AAe?$AAs?$AA?9?$AAu?$AAy@ 10005630     libcpmt:winapinls.obj
 0001:0000463c       ??_C@_1M@JKFFICHJ@?$AAe?$AAs?$AA?9?$AAv?$AAe@ 1000563c     libcpmt:winapinls.obj
 0001:00004648       ??_C@_1M@PNMLOJDF@?$AAe?$AAt?$AA?9?$AAe?$AAe@ 10005648     libcpmt:winapinls.obj
 0001:00004654       ??_C@_1M@GHHLIKEI@?$AAe?$AAu?$AA?9?$AAe?$AAs@ 10005654     libcpmt:winapinls.obj
 0001:00004660       ??_C@_1M@PBNONODE@?$AAf?$AAa?$AA?9?$AAi?$AAr@ 10005660     libcpmt:winapinls.obj
 0001:0000466c       ??_C@_1M@JEEHPMIL@?$AAf?$AAi?$AA?9?$AAf?$AAi@ 1000566c     libcpmt:winapinls.obj
 0001:00004678       ??_C@_1M@LMDCNDBA@?$AAf?$AAo?$AA?9?$AAf?$AAo@ 10005678     libcpmt:winapinls.obj
 0001:00004684       ??_C@_1M@JKEOHLDK@?$AAf?$AAr?$AA?9?$AAb?$AAe@ 10005684     libcpmt:winapinls.obj
 0001:00004690       ??_C@_1M@NOHADPMI@?$AAf?$AAr?$AA?9?$AAc?$AAa@ 10005690     libcpmt:winapinls.obj
 0001:0000469c       ??_C@_1M@KDHIHAEC@?$AAf?$AAr?$AA?9?$AAc?$AAh@ 1000569c     libcpmt:winapinls.obj
 0001:000046a8       ??_C@_1M@MMBBFGAK@?$AAf?$AAr?$AA?9?$AAf?$AAr@ 100056a8     libcpmt:winapinls.obj
 0001:000046b4       ??_C@_1M@PAFNENNF@?$AAf?$AAr?$AA?9?$AAl?$AAu@ 100056b4     libcpmt:winapinls.obj
 0001:000046c0       ??_C@_1M@EOHDJGDD@?$AAf?$AAr?$AA?9?$AAm?$AAc@ 100056c0     libcpmt:winapinls.obj
 0001:000046cc       ??_C@_1M@FAPLLOPF@?$AAg?$AAl?$AA?9?$AAe?$AAs@ 100056cc     libcpmt:winapinls.obj
 0001:000046d8       ??_C@_1M@FOPBFLOO@?$AAg?$AAu?$AA?9?$AAi?$AAn@ 100056d8     libcpmt:winapinls.obj
 0001:000046e4       ??_C@_1M@KBMCINPM@?$AAh?$AAe?$AA?9?$AAi?$AAl@ 100056e4     libcpmt:winapinls.obj
 0001:000046f0       ??_C@_1M@BBPHKFPJ@?$AAh?$AAi?$AA?9?$AAi?$AAn@ 100056f0     libcpmt:winapinls.obj
 0001:000046fc       ??_C@_1M@PMBNDPHD@?$AAh?$AAr?$AA?9?$AAb?$AAa@ 100056fc     libcpmt:winapinls.obj
 0001:00004708       ??_C@_1M@BPCKOEGE@?$AAh?$AAr?$AA?9?$AAh?$AAr@ 10005708     libcpmt:winapinls.obj
 0001:00004714       ??_C@_1M@GACBMHKE@?$AAh?$AAu?$AA?9?$AAh?$AAu@ 10005714     libcpmt:winapinls.obj
 0001:00004720       ??_C@_1M@MILPAJJC@?$AAh?$AAy?$AA?9?$AAa?$AAm@ 10005720     libcpmt:winapinls.obj
 0001:0000472c       ??_C@_1M@BABBICEC@?$AAi?$AAd?$AA?9?$AAi?$AAd@ 1000572c     libcpmt:winapinls.obj
 0001:00004738       ??_C@_1M@BIKNHHPF@?$AAi?$AAs?$AA?9?$AAi?$AAs@ 10005738     libcpmt:winapinls.obj
 0001:00004744       ??_C@_1M@NMPCJPHE@?$AAi?$AAt?$AA?9?$AAc?$AAh@ 10005744     libcpmt:winapinls.obj
 0001:00004750       ??_C@_1M@GHKGFEDF@?$AAi?$AAt?$AA?9?$AAi?$AAt@ 10005750     libcpmt:winapinls.obj
 0001:0000475c       ??_C@_1M@NIEJCJJA@?$AAj?$AAa?$AA?9?$AAj?$AAp@ 1000575c     libcpmt:winapinls.obj
 0001:00004768       ??_C@_1M@JILFNBIM@?$AAk?$AAa?$AA?9?$AAg?$AAe@ 10005768     libcpmt:winapinls.obj
 0001:00004774       ??_C@_1M@PACPMGPH@?$AAk?$AAk?$AA?9?$AAk?$AAz@ 10005774     libcpmt:winapinls.obj
 0001:00004780       ??_C@_1M@IELFGMHA@?$AAk?$AAn?$AA?9?$AAi?$AAn@ 10005780     libcpmt:winapinls.obj
 0001:0000478c       ??_C@_1M@DMHAEOGC@?$AAk?$AAo?$AA?9?$AAk?$AAr@ 1000578c     libcpmt:winapinls.obj
 0001:00004798       ??_C@_1O@IBBJHCH@?$AAk?$AAo?$AAk?$AA?9?$AAi?$AAn@ 10005798     libcpmt:winapinls.obj
 0001:000047a8       ??_C@_1M@HBAHBIGA@?$AAk?$AAy?$AA?9?$AAk?$AAg@ 100057a8     libcpmt:winapinls.obj
 0001:000047b4       ??_C@_1M@KPMILCJG@?$AAl?$AAt?$AA?9?$AAl?$AAt@ 100057b4     libcpmt:winapinls.obj
 0001:000047c0       ??_C@_1M@BDEKKCA@?$AAl?$AAv?$AA?9?$AAl?$AAv@ 100057c0     libcpmt:winapinls.obj
 0001:000047cc       ??_C@_1M@ELCKCCJJ@?$AAm?$AAi?$AA?9?$AAn?$AAz@ 100057cc     libcpmt:winapinls.obj
 0001:000047d8       ??_C@_1M@CBOOLAPA@?$AAm?$AAk?$AA?9?$AAm?$AAk@ 100057d8     libcpmt:winapinls.obj
 0001:000047e4       ??_C@_1M@GPHNBJKN@?$AAm?$AAl?$AA?9?$AAi?$AAn@ 100057e4     libcpmt:winapinls.obj
 0001:000047f0       ??_C@_1M@PABJILIG@?$AAm?$AAn?$AA?9?$AAm?$AAn@ 100057f0     libcpmt:winapinls.obj
 0001:000047fc       ??_C@_1M@FGBKKIPG@?$AAm?$AAr?$AA?9?$AAi?$AAn@ 100057fc     libcpmt:winapinls.obj
 0001:00004808       ??_C@_1M@NDBPDDAL@?$AAm?$AAs?$AA?9?$AAb?$AAn@ 10005808     libcpmt:winapinls.obj
 0001:00004814       ??_C@_1M@OPIHOOPI@?$AAm?$AAs?$AA?9?$AAm?$AAy@ 10005814     libcpmt:winapinls.obj
 0001:00004820       ??_C@_1M@PPDBCNFM@?$AAm?$AAt?$AA?9?$AAm?$AAt@ 10005820     libcpmt:winapinls.obj
 0001:0000482c       ??_C@_1M@KDJDKMDD@?$AAn?$AAb?$AA?9?$AAn?$AAo@ 1000582c     libcpmt:winapinls.obj
 0001:00004838       ??_C@_1M@KFCFLMJP@?$AAn?$AAl?$AA?9?$AAb?$AAe@ 10005838     libcpmt:winapinls.obj
 0001:00004844       ??_C@_1M@KPOPDDGO@?$AAn?$AAl?$AA?9?$AAn?$AAl@ 10005844     libcpmt:winapinls.obj
 0001:00004850       ??_C@_1M@LJKPEMLN@?$AAn?$AAn?$AA?9?$AAn?$AAo@ 10005850     libcpmt:winapinls.obj
 0001:0000485c       ??_C@_1M@BDGHHBFL@?$AAn?$AAs?$AA?9?$AAz?$AAa@ 1000585c     libcpmt:winapinls.obj
 0001:00004868       ??_C@_1M@IDEHOAP@?$AAp?$AAa?$AA?9?$AAi?$AAn@ 10005868     libcpmt:winapinls.obj
 0001:00004874       ??_C@_1M@HDBKGOGH@?$AAp?$AAl?$AA?9?$AAp?$AAl@ 10005874     libcpmt:winapinls.obj
 0001:00004880       ??_C@_1M@LJLLCMEH@?$AAp?$AAt?$AA?9?$AAb?$AAr@ 10005880     libcpmt:winapinls.obj
 0001:0000488c       ??_C@_1M@NCMONAAL@?$AAp?$AAt?$AA?9?$AAp?$AAt@ 1000588c     libcpmt:winapinls.obj
 0001:00004898       ??_C@_1O@EAKMAJDN@?$AAq?$AAu?$AAz?$AA?9?$AAb?$AAo@ 10005898     libcpmt:winapinls.obj
 0001:000048a8       ??_C@_1O@BHHPIGDN@?$AAq?$AAu?$AAz?$AA?9?$AAe?$AAc@ 100058a8     libcpmt:winapinls.obj
 0001:000048b8       ??_C@_1O@GBAPEKMJ@?$AAq?$AAu?$AAz?$AA?9?$AAp?$AAe@ 100058b8     libcpmt:winapinls.obj
 0001:000048c8       ??_C@_1M@CLGLEFBO@?$AAr?$AAo?$AA?9?$AAr?$AAo@ 100058c8     libcpmt:winapinls.obj
 0001:000048d4       ??_C@_1M@CEEDODME@?$AAr?$AAu?$AA?9?$AAr?$AAu@ 100058d4     libcpmt:winapinls.obj
 0001:000048e0       ??_C@_1M@HPKKKMPP@?$AAs?$AAa?$AA?9?$AAi?$AAn@ 100058e0     libcpmt:winapinls.obj
 0001:000048ec       ??_C@_1M@BKMAIGOJ@?$AAs?$AAe?$AA?9?$AAf?$AAi@ 100058ec     libcpmt:winapinls.obj
 0001:000048f8       ??_C@_1M@NDPIFLFI@?$AAs?$AAe?$AA?9?$AAn?$AAo@ 100058f8     libcpmt:winapinls.obj
 0001:00004904       ??_C@_1M@DANKKHJ@?$AAs?$AAe?$AA?9?$AAs?$AAe@ 10005904     libcpmt:winapinls.obj
 0001:00004910       ??_C@_1M@PNBLONPJ@?$AAs?$AAk?$AA?9?$AAs?$AAk@ 10005910     libcpmt:winapinls.obj
 0001:0000491c       ??_C@_1M@LFMODOAL@?$AAs?$AAl?$AA?9?$AAs?$AAi@ 1000591c     libcpmt:winapinls.obj
 0001:00004928       ??_C@_1O@DFKOMPG@?$AAs?$AAm?$AAa?$AA?9?$AAn?$AAo@ 10005928     libcpmt:winapinls.obj
 0001:00004938       ??_C@_1O@NDKPBNNH@?$AAs?$AAm?$AAa?$AA?9?$AAs?$AAe@ 10005938     libcpmt:winapinls.obj
 0001:00004948       ??_C@_1O@PLLKBHAB@?$AAs?$AAm?$AAj?$AA?9?$AAn?$AAo@ 10005948     libcpmt:winapinls.obj
 0001:00004958       ??_C@_1O@CLEPOGCA@?$AAs?$AAm?$AAj?$AA?9?$AAs?$AAe@ 10005958     libcpmt:winapinls.obj
 0001:00004968       ??_C@_1O@DLGJGKMK@?$AAs?$AAm?$AAn?$AA?9?$AAf?$AAi@ 10005968     libcpmt:winapinls.obj
 0001:00004978       ??_C@_1O@OJDJGAJC@?$AAs?$AAm?$AAs?$AA?9?$AAf?$AAi@ 10005978     libcpmt:winapinls.obj
 0001:00004988       ??_C@_1M@BOFOGHPB@?$AAs?$AAq?$AA?9?$AAa?$AAl@ 10005988     libcpmt:winapinls.obj
 0001:00004994       ??_C@_1BG@LJBBIPGB@?$AAs?$AAr?$AA?9?$AAb?$AAa?$AA?9?$AAc?$AAy?$AAr?$AAl@ 10005994     libcpmt:winapinls.obj
 0001:000049ac       ??_C@_1BG@JLBENFOE@?$AAs?$AAr?$AA?9?$AAb?$AAa?$AA?9?$AAl?$AAa?$AAt?$AAn@ 100059ac     libcpmt:winapinls.obj
 0001:000049c4       ??_C@_1BG@KODPNHE@?$AAs?$AAr?$AA?9?$AAs?$AAp?$AA?9?$AAc?$AAy?$AAr?$AAl@ 100059c4     libcpmt:winapinls.obj
 0001:000049dc       ??_C@_1BG@CIOGKHPB@?$AAs?$AAr?$AA?9?$AAs?$AAp?$AA?9?$AAl?$AAa?$AAt?$AAn@ 100059dc     libcpmt:winapinls.obj
 0001:000049f4       ??_C@_1M@NGFJLMAC@?$AAs?$AAv?$AA?9?$AAf?$AAi@ 100059f4     libcpmt:winapinls.obj
 0001:00004a00       ??_C@_1M@MPJEJAJC@?$AAs?$AAv?$AA?9?$AAs?$AAe@ 10005a00     libcpmt:winapinls.obj
 0001:00004a0c       ??_C@_1M@MPNDHLFK@?$AAs?$AAw?$AA?9?$AAk?$AAe@ 10005a0c     libcpmt:winapinls.obj
 0001:00004a18       ??_C@_1O@KOHBJJI@?$AAs?$AAy?$AAr?$AA?9?$AAs?$AAy@ 10005a18     libcpmt:winapinls.obj
 0001:00004a28       ??_C@_1M@LDCEFHA@?$AAt?$AAa?$AA?9?$AAi?$AAn@ 10005a28     libcpmt:winapinls.obj
 0001:00004a34       ??_C@_1M@CNJOFAK@?$AAt?$AAe?$AA?9?$AAi?$AAn@ 10005a34     libcpmt:winapinls.obj
 0001:00004a40       ??_C@_1M@GNAECACD@?$AAt?$AAh?$AA?9?$AAt?$AAh@ 10005a40     libcpmt:winapinls.obj
 0001:00004a4c       ??_C@_1M@CHBIHOJO@?$AAt?$AAn?$AA?9?$AAz?$AAa@ 10005a4c     libcpmt:winapinls.obj
 0001:00004a58       ??_C@_1M@GCCMIGPJ@?$AAt?$AAr?$AA?9?$AAt?$AAr@ 10005a58     libcpmt:winapinls.obj
 0001:00004a64       ??_C@_1M@CELMCNBK@?$AAt?$AAt?$AA?9?$AAr?$AAu@ 10005a64     libcpmt:winapinls.obj
 0001:00004a70       ??_C@_1M@KLMCELGA@?$AAu?$AAk?$AA?9?$AAu?$AAa@ 10005a70     libcpmt:winapinls.obj
 0001:00004a7c       ??_C@_1M@EPAJJAJF@?$AAu?$AAr?$AA?9?$AAp?$AAk@ 10005a7c     libcpmt:winapinls.obj
 0001:00004a88       ??_C@_1BG@GEGPMCDJ@?$AAu?$AAz?$AA?9?$AAu?$AAz?$AA?9?$AAc?$AAy?$AAr?$AAl@ 10005a88     libcpmt:winapinls.obj
 0001:00004aa0       ??_C@_1BG@EGGKJILM@?$AAu?$AAz?$AA?9?$AAu?$AAz?$AA?9?$AAl?$AAa?$AAt?$AAn@ 10005aa0     libcpmt:winapinls.obj
 0001:00004ab8       ??_C@_1M@GFOCLFF@?$AAv?$AAi?$AA?9?$AAv?$AAn@ 10005ab8     libcpmt:winapinls.obj
 0001:00004ac4       ??_C@_1M@CPAMEDFI@?$AAx?$AAh?$AA?9?$AAz?$AAa@ 10005ac4     libcpmt:winapinls.obj
 0001:00004ad0       ??_C@_1O@EBKIFIGN@?$AAz?$AAh?$AA?9?$AAc?$AAh?$AAs@ 10005ad0     libcpmt:winapinls.obj
 0001:00004ae0       ??_C@_1O@NMHPGANE@?$AAz?$AAh?$AA?9?$AAc?$AAh?$AAt@ 10005ae0     libcpmt:winapinls.obj
 0001:00004af0       ??_C@_1M@LPINJOMC@?$AAz?$AAh?$AA?9?$AAc?$AAn@ 10005af0     libcpmt:winapinls.obj
 0001:00004afc       ??_C@_1M@OCJEJODD@?$AAz?$AAh?$AA?9?$AAh?$AAk@ 10005afc     libcpmt:winapinls.obj
 0001:00004b08       ??_C@_1M@DNDLJINH@?$AAz?$AAh?$AA?9?$AAm?$AAo@ 10005b08     libcpmt:winapinls.obj
 0001:00004b14       ??_C@_1M@MBFDNDND@?$AAz?$AAh?$AA?9?$AAs?$AAg@ 10005b14     libcpmt:winapinls.obj
 0001:00004b20       ??_C@_1M@IMEPLEPE@?$AAz?$AAh?$AA?9?$AAt?$AAw@ 10005b20     libcpmt:winapinls.obj
 0001:00004b2c       ??_C@_1M@BBGHNHJP@?$AAz?$AAu?$AA?9?$AAz?$AAa@ 10005b2c     libcpmt:winapinls.obj
 0001:00004b3c       ??_7type_info@@6B@         10005b3c     LIBCMT:std_type_info_static.obj
 0001:00004b4c       __pDefaultRawDllMain       10005b4c     LIBCMT:dll_dllmain.obj
 0001:00004b4c       __pRawDllMain              10005b4c     LIBCMT:dll_dllmain.obj
 0001:00004b58       __pDestructExceptionObject 10005b58     libvcruntime:ehhelpers.obj
 0001:00004b60       ??_7bad_exception@std@@6B@ 10005b60     libvcruntime:frame.obj
 0001:00004b68       ??_C@_0O@DPKOEFFH@bad?5exception@ 10005b68     libvcruntime:frame.obj
 0001:00004ef8       ??_C@_08EHJDFFNH@__based?$CI@ 10005ef8     libvcruntime:undname.obj
 0001:00004f04       ??_C@_07KOLFKCDI@__cdecl@  10005f04     libvcruntime:undname.obj
 0001:00004f0c       ??_C@_08GHMPAG@__pascal@   10005f0c     libvcruntime:undname.obj
 0001:00004f18       ??_C@_09IFJBGAPI@__stdcall@ 10005f18     libvcruntime:undname.obj
 0001:00004f24       ??_C@_0L@NPHFGOKO@__thiscall@ 10005f24     libvcruntime:undname.obj
 0001:00004f30       ??_C@_0L@JMKHOMEK@__fastcall@ 10005f30     libvcruntime:undname.obj
 0001:00004f3c       ??_C@_0N@BCKKPABJ@__vectorcall@ 10005f3c     libvcruntime:undname.obj
 0001:00004f4c       ??_C@_09HIJEGCPM@__clrcall@ 10005f4c     libvcruntime:undname.obj
 0001:00004f58       ??_C@_06GHPCKEAG@__eabi@   10005f58     libvcruntime:undname.obj
 0001:00004f60       ??_C@_09IOPIDJLG@__swift_1@ 10005f60     libvcruntime:undname.obj
 0001:00004f6c       ??_C@_09KFNFGKHF@__swift_2@ 10005f6c     libvcruntime:undname.obj
 0001:00004f78       ??_C@_07JOMMBBKO@__ptr64@  10005f78     libvcruntime:undname.obj
 0001:00004f80       ??_C@_0L@PILCLIHE@__restrict@ 10005f80     libvcruntime:undname.obj
 0001:00004f8c       ??_C@_0M@GFIIJFMG@__unaligned@ 10005f8c     libvcruntime:undname.obj
 0001:00004f98       ??_C@_09DHDLOLLB@restrict?$CI@ 10005f98     libvcruntime:undname.obj
 0001:00004fa4       ??_C@_04NIHEBCM@?5new@     10005fa4     libvcruntime:undname.obj
 0001:00004fac       ??_C@_07FPCDHGMM@?5delete@ 10005fac     libvcruntime:undname.obj
 0001:00004fb4       ??_C@_01NEMOKFLO@?$DN@     10005fb4     libvcruntime:undname.obj
 0001:00004fb8       ??_C@_02GPIOPFAK@?$DO?$DO@ 10005fb8     libvcruntime:undname.obj
 0001:00004fbc       ??_C@_02FODMEDOG@?$DM?$DM@ 10005fbc     libvcruntime:undname.obj
 0001:00004fc0       ??_C@_01DCLJPIOD@?$CB@     10005fc0     libvcruntime:undname.obj
 0001:00004fc4       ??_C@_02EGOFBIJA@?$DN?$DN@ 10005fc4     libvcruntime:undname.obj
 0001:00004fc8       ??_C@_02FDNJECIE@?$CB?$DN@ 10005fc8     libvcruntime:undname.obj
 0001:00004fcc       ??_C@_02GPECMEKF@?$FL?$FN@ 10005fcc     libvcruntime:undname.obj
 0001:00004fd0       ??_C@_08LHJFAFGD@operator@ 10005fd0     libvcruntime:undname.obj
 0001:00004fdc       ??_C@_02HBOOOICD@?9?$DO@   10005fdc     libvcruntime:undname.obj
 0001:00004fe0       ??_C@_02ECNGHCIF@?$CL?$CL@ 10005fe0     libvcruntime:undname.obj
 0001:00004fe4       ??_C@_02BAABKJLB@?9?9@     10005fe4     libvcruntime:undname.obj
 0001:00004fe8       ??_C@_01MIFGBAGJ@?$CL@     10005fe8     libvcruntime:undname.obj
 0001:00004fec       ??_C@_01HNPIGOCE@?$CG@     10005fec     libvcruntime:undname.obj
 0001:00004ff0       ??_C@_03MNHNFDLC@?9?$DO?$CK@ 10005ff0     libvcruntime:undname.obj
 0001:00004ff4       ??_C@_01KMDKNFGN@?1@       10005ff4     libvcruntime:undname.obj
 0001:00004ff8       ??_C@_01FGNFDNOH@?$CF@     10005ff8     libvcruntime:undname.obj
 0001:00004ffc       ??_C@_01MNNFJEPP@?$DM@     10005ffc     libvcruntime:undname.obj
 0001:00005000       ??_C@_02EHCHHCKH@?$DM?$DN@ 10006000     libvcruntime:undname.obj
 0001:00005004       ??_C@_01PPODPGHN@?$DO@     10006004     libvcruntime:undname.obj
 0001:00005008       ??_C@_02EEKDKGMJ@?$DO?$DN@ 10006008     libvcruntime:undname.obj
 0001:0000500c       ??_C@_01IHBHIGKO@?0@       1000600c     libvcruntime:undname.obj
 0001:00005010       ??_C@_02HCKGKOFO@?$CI?$CJ@ 10006010     libvcruntime:undname.obj
 0001:00005014       ??_C@_01PJKLJHI@?$HO@      10006014     libvcruntime:undname.obj
 0001:00005018       ??_C@_01JKBOJNNK@?$FO@     10006018     libvcruntime:undname.obj
 0001:0000501c       ??_C@_01DNKMNLPK@?$HM@     1000601c     libvcruntime:undname.obj
 0001:00005020       ??_C@_02PPKAJPJL@?$CG?$CG@ 10006020     libvcruntime:undname.obj
 0001:00005024       ??_C@_02NONPIBCD@?$HM?$HM@ 10006024     libvcruntime:undname.obj
 0001:00005028       ??_C@_02FPIMKNGF@?$CK?$DN@ 10006028     libvcruntime:undname.obj
 0001:0000502c       ??_C@_02FOEOMHFC@?$CL?$DN@ 1000602c     libvcruntime:undname.obj
 0001:00005030       ??_C@_02FKMDLLOA@?9?$DN@   10006030     libvcruntime:undname.obj
 0001:00005034       ??_C@_02FJEHGPIO@?1?$DN@   10006034     libvcruntime:undname.obj
 0001:00005038       ??_C@_02FENAOKFI@?$CF?$DN@ 10006038     libvcruntime:undname.obj
 0001:0000503c       ??_C@_03IKFCCPFF@?$DO?$DO?$DN@ 1000603c     libvcruntime:undname.obj
 0001:00005040       ??_C@_03CDNPDDLA@?$DM?$DM?$DN@ 10006040     libvcruntime:undname.obj
 0001:00005044       ??_C@_02FGJGFEAB@?$CG?$DN@ 10006044     libvcruntime:undname.obj
 0001:00005048       ??_C@_02DHLNPPGH@?$HM?$DN@ 10006048     libvcruntime:undname.obj
 0001:0000504c       ??_C@_02MHEGNOJ@?$FO?$DN@  1000604c     libvcruntime:undname.obj
 0001:00005050       ??_C@_09IFPLHPGF@?$GAvftable?8@ 10006050     libvcruntime:undname.obj
 0001:0000505c       ??_C@_09BLBHBJP@?$GAvbtable?8@ 1000605c     libvcruntime:undname.obj
 0001:00005068       ??_C@_07FEEIOKP@?$GAvcall?8@ 10006068     libvcruntime:undname.obj
 0001:00005070       ??_C@_08LLFFHHDJ@?$GAtypeof?8@ 10006070     libvcruntime:undname.obj
 0001:0000507c       ??_C@_0BF@KDPPACIK@?$GAlocal?5static?5guard?8@ 1000607c     libvcruntime:undname.obj
 0001:00005094       ??_C@_08OBABFOLI@?$GAstring?8@ 10006094     libvcruntime:undname.obj
 0001:000050a0       ??_C@_0BD@JDLKDPAB@?$GAvbase?5destructor?8@ 100060a0     libvcruntime:undname.obj
 0001:000050b4       ??_C@_0BN@DEGPLNFK@?$GAvector?5deleting?5destructor?8@ 100060b4     libvcruntime:undname.obj
 0001:000050d4       ??_C@_0BO@OBMKPJIG@?$GAdefault?5constructor?5closure?8@ 100060d4     libvcruntime:undname.obj
 0001:000050f4       ??_C@_0BN@IMDCHIKM@?$GAscalar?5deleting?5destructor?8@ 100060f4     libvcruntime:undname.obj
 0001:00005114       ??_C@_0BO@PFGOCPJJ@?$GAvector?5constructor?5iterator?8@ 10006114     libvcruntime:undname.obj
 0001:00005134       ??_C@_0BN@LFPFMEDL@?$GAvector?5destructor?5iterator?8@ 10006134     libvcruntime:undname.obj
 0001:00005154       ??_C@_0CE@IKBNEHA@?$GAvector?5vbase?5constructor?5itera@ 10006154     libvcruntime:undname.obj
 0001:00005178       ??_C@_0BL@NILFHHPC@?$GAvirtual?5displacement?5map?8@ 10006178     libvcruntime:undname.obj
 0001:00005194       ??_C@_0CB@JONCMFFK@?$GAeh?5vector?5constructor?5iterator@ 10006194     libvcruntime:undname.obj
 0001:000051b8       ??_C@_0CA@GCEOPDGL@?$GAeh?5vector?5destructor?5iterator?8@ 100061b8     libvcruntime:undname.obj
 0001:000051d8       ??_C@_0CH@OOJPLCPH@?$GAeh?5vector?5vbase?5constructor?5it@ 100061d8     libvcruntime:undname.obj
 0001:00005200       ??_C@_0BL@LLKPOHJI@?$GAcopy?5constructor?5closure?8@ 10006200     libvcruntime:undname.obj
 0001:0000521c       ??_C@_0BA@KBCDOMBN@?$GAudt?5returning?8@ 1000621c     libvcruntime:undname.obj
 0001:0000522c       ??_C@_03KLGMFNMG@?$GAEH@   1000622c     libvcruntime:undname.obj
 0001:00005230       ??_C@_05KHLCHHI@?$GARTTI@  10006230     libvcruntime:undname.obj
 0001:00005238       ??_C@_0BA@KKLDJDLB@?$GAlocal?5vftable?8@ 10006238     libvcruntime:undname.obj
 0001:00005248       ??_C@_0CE@IIHCMGGL@?$GAlocal?5vftable?5constructor?5clos@ 10006248     libvcruntime:undname.obj
 0001:0000526c       ??_C@_06FHBGPFGH@?5new?$FL?$FN@ 1000626c     libvcruntime:undname.obj
 0001:00005274       ??_C@_09LBNFPBCA@?5delete?$FL?$FN@ 10006274     libvcruntime:undname.obj
 0001:00005280       ??_C@_0P@HJKNJFNN@?$GAomni?5callsig?8@ 10006280     libvcruntime:undname.obj
 0001:00005290       ??_C@_0BL@CNOONJFP@?$GAplacement?5delete?5closure?8@ 10006290     libvcruntime:undname.obj
 0001:000052ac       ??_C@_0BN@CKNJLHMB@?$GAplacement?5delete?$FL?$FN?5closure?8@ 100062ac     libvcruntime:undname.obj
 0001:000052cc       ??_C@_0CG@CFDHKGGD@?$GAmanaged?5vector?5constructor?5ite@ 100062cc     libvcruntime:undname.obj
 0001:000052f4       ??_C@_0CF@IMGKMJNO@?$GAmanaged?5vector?5destructor?5iter@ 100062f4     libvcruntime:undname.obj
 0001:0000531c       ??_C@_0CG@HLDDJMAG@?$GAeh?5vector?5copy?5constructor?5ite@ 1000631c     libvcruntime:undname.obj
 0001:00005344       ??_C@_0CM@FCBBDIGB@?$GAeh?5vector?5vbase?5copy?5construct@ 10006344     libvcruntime:undname.obj
 0001:00005370       ??_C@_0BL@CLIPGLGB@?$GAdynamic?5initializer?5for?5?8@ 10006370     libvcruntime:undname.obj
 0001:0000538c       ??_C@_0CB@PDBIFEP@?$GAdynamic?5atexit?5destructor?5for?5@ 1000638c     libvcruntime:undname.obj
 0001:000053b0       ??_C@_0CD@CGAJBKEJ@?$GAvector?5copy?5constructor?5iterat@ 100063b0     libvcruntime:undname.obj
 0001:000053d4       ??_C@_0CJ@GJELGAMM@?$GAvector?5vbase?5copy?5constructor?5@ 100063d4     libvcruntime:undname.obj
 0001:00005400       ??_C@_0CL@FGIJHLCE@?$GAmanaged?5vector?5copy?5constructo@ 10006400     libvcruntime:undname.obj
 0001:0000542c       ??_C@_0BM@PMGGMLDN@?$GAlocal?5static?5thread?5guard?8@ 1000642c     libvcruntime:undname.obj
 0001:00005448       ??_C@_0N@BDNMDMOL@operator?5?$CC?$CC?5@ 10006448     libvcruntime:undname.obj
 0001:00005458       ??_C@_0BC@GGEBGALA@operator?5co_await@ 10006458     libvcruntime:undname.obj
 0001:0000546c       ??_C@_0M@GAAIMMOH@operator?$DM?$DN?$DO@ 1000646c     libvcruntime:undname.obj
 0001:00005478       ??_C@_0BC@DAFEJGAK@?5Type?5Descriptor?8@ 10006478     libvcruntime:undname.obj
 0001:0000548c       ??_C@_0BM@LDKODKLH@?5Base?5Class?5Descriptor?5at?5?$CI@ 1000648c     libvcruntime:undname.obj
 0001:000054a8       ??_C@_0BD@LGICGFMM@?5Base?5Class?5Array?8@ 100064a8     libvcruntime:undname.obj
 0001:000054bc       ??_C@_0BN@MECKDCOJ@?5Class?5Hierarchy?5Descriptor?8@ 100064bc     libvcruntime:undname.obj
 0001:000054dc       ??_C@_0BK@CFCOFLF@?5Complete?5Object?5Locator?8@ 100064dc     libvcruntime:undname.obj
 0001:000054f8       ??_C@_0BG@JNJLAMPM@?$GAanonymous?5namespace?8@ 100064f8     libvcruntime:undname.obj
 0001:0000551c       ??_C@_1DM@KHCHBNEB@?$AAa?$AAp?$AAi?$AA?9?$AAm?$AAs?$AA?9?$AAw?$AAi?$AAn?$AA?9?$AAc?$AAo?$AAr?$AAe@ 1000651c     libvcruntime:winapi_downlevel.obj
 0001:00005558       ??_C@_1DK@LPPGFMPP@?$AAa?$AAp?$AAi?$AA?9?$AAm?$AAs?$AA?9?$AAw?$AAi?$AAn?$AA?9?$AAc?$AAo?$AAr?$AAe@ 10006558     libvcruntime:winapi_downlevel.obj
 0001:00005594       ??_C@_1BA@PFFKHIOG@?$AAa?$AAp?$AAi?$AA?9?$AAm?$AAs?$AA?9@ 10006594     libvcruntime:winapi_downlevel.obj
 0001:00005738       _format_validation_lookup_table 10006738     libucrt:output.obj
 0001:00005794       ??_C@_1O@CEDCILHN@?$AA?$CI?$AAn?$AAu?$AAl?$AAl?$AA?$CJ@ 10006794     libucrt:output.obj
 0001:000057a4       ??_C@_06OJHGLDPL@?$CInull?$CJ@ 100067a4     libucrt:output.obj
 0001:000057b0       __real@3e54ae0bf85ddf44    100067b0     libucrt:log2d.obj
 0001:000057b8       __real@3e5526e50e32a6ab    100067b8     libucrt:log2d.obj
 0001:000057c0       __real@3e7427de7fbcc47c    100067c0     libucrt:log2d.obj
 0001:000057c8       __real@3e7f7d1cf79abc9e    100067c8     libucrt:log2d.obj
 0001:000057d0       __real@3fc2f8d8bf29def7    100067d0     libucrt:log2d.obj
 0001:000057d8       __real@3fc3991accfeb3f4    100067d8     libucrt:log2d.obj
 0001:000057e0       __real@3fc7466fd968cb62    100067e0     libucrt:log2d.obj
 0001:000057e8       __real@3fcc71c4da12c9c6    100067e8     libucrt:log2d.obj
 0001:000057f0       __real@3fd24924948ae94a    100067f0     libucrt:log2d.obj
 0001:000057f8       __real@3fd3441300000000    100067f8     libucrt:log2d.obj
 0001:00005800       __real@3fd9999999975ff7    10006800     libucrt:log2d.obj
 0001:00005808       __real@3fdbcb7b00000000    10006808     libucrt:log2d.obj
 0001:00005810       __real@3fdbcb7b1526e50e    10006810     libucrt:log2d.obj
 0001:00005818       __real@3fe55555555555bc    10006818     libucrt:log2d.obj
 0001:00005820       __real@3fe62e42c0000000    10006820     libucrt:log2d.obj
 0001:00005828       __real@3fe6a09e667f3bcd    10006828     libucrt:log2d.obj
 0001:00005830       __real@3ff0000000000000    10006830     libucrt:log2d.obj
 0001:00005838       __real@3ff7154760000000    10006838     libucrt:log2d.obj
 0001:00005840       __real@3ff71547652b82fe    10006840     libucrt:log2d.obj
 0001:000058a4       __half                     100068a4     libucrt:pow_impl.obj
 0001:000058f8       ___newctype                100068f8     libucrt:ctype.obj
 0001:00005bf8       ___newclmap                10006bf8     libucrt:ctype.obj
 0001:00005d78       ___newcumap                10006d78     libucrt:ctype.obj
 0001:00005ef8       __wctype                   10006ef8     libucrt:ctype.obj
 0001:00006100       ?large_power_data@?1??multiply_by_power_of_ten@__crt_strtox@@YA_NAAUbig_integer@2@I@Z@4QBIB 10007100     libucrt:strtod.obj
 0001:00006a08       ?small_powers_of_ten@?1??multiply_by_power_of_ten@__crt_strtox@@YA_NAAUbig_integer@2@I@Z@4QBIB 10007a08     libucrt:strtod.obj
 0001:00006a30       ___acrt_exception_action_table 10007a30     libucrt:exception_filter.obj
 0001:00006ac0       ___acrt_signal_action_table_count 10007ac0     libucrt:exception_filter.obj
 0001:00006ac4       ___acrt_signal_action_first_fpe_index 10007ac4     libucrt:exception_filter.obj
 0001:00006ac8       ___acrt_signal_action_fpe_count 10007ac8     libucrt:exception_filter.obj
 0001:00006acc       ??_C@_1BI@BGOHAHKC@?$AAm?$AAs?$AAc?$AAo?$AAr?$AAe?$AAe?$AA?4?$AAd?$AAl?$AAl@ 10007acc     libucrt:exit.obj
 0001:00006ae4       ??_C@_0P@MIGLKIOC@CorExitProcess@ 10007ae4     libucrt:exit.obj
 0001:00006ba8       __Inf_C                    10007ba8     libucrt:_values.obj
 0001:00006bb0       __Nan_C                    10007bb0     libucrt:_values.obj
 0001:00006c08       ??_C@_1EA@JGEFHKEI@?$AAa?$AAp?$AAi?$AA?9?$AAm?$AAs?$AA?9?$AAw?$AAi?$AAn?$AA?9?$AAc?$AAo?$AAr?$AAe@ 10007c08     libucrt:winapi_thunks.obj
 0001:00006c48       ??_C@_1DI@IJCEHOCB@?$AAa?$AAp?$AAi?$AA?9?$AAm?$AAs?$AA?9?$AAw?$AAi?$AAn?$AA?9?$AAc?$AAo?$AAr?$AAe@ 10007c48     libucrt:winapi_thunks.obj
 0001:00006c80       ??_C@_1EI@MPIAOHOC@?$AAa?$AAp?$AAi?$AA?9?$AAm?$AAs?$AA?9?$AAw?$AAi?$AAn?$AA?9?$AAc?$AAo?$AAr?$AAe@ 10007c80     libucrt:winapi_thunks.obj
 0001:00006cc8       ??_C@_1FK@FPHCKFIE@?$AAa?$AAp?$AAi?$AA?9?$AAm?$AAs?$AA?9?$AAw?$AAi?$AAn?$AA?9?$AAc?$AAo?$AAr?$AAe@ 10007cc8     libucrt:winapi_thunks.obj
 0001:00006d28       ??_C@_1EM@DILCGIIO@?$AAa?$AAp?$AAi?$AA?9?$AAm?$AAs?$AA?9?$AAw?$AAi?$AAn?$AA?9?$AAc?$AAo?$AAr?$AAe@ 10007d28     libucrt:winapi_thunks.obj
 0001:00006d74       ??_C@_1DM@LNCGDDPN@?$AAa?$AAp?$AAi?$AA?9?$AAm?$AAs?$AA?9?$AAw?$AAi?$AAn?$AA?9?$AAc?$AAo?$AAr?$AAe@ 10007d74     libucrt:winapi_thunks.obj
 0001:00006db0       ??_C@_1DO@FPAPJEMD@?$AAa?$AAp?$AAi?$AA?9?$AAm?$AAs?$AA?9?$AAw?$AAi?$AAn?$AA?9?$AAc?$AAo?$AAr?$AAe@ 10007db0     libucrt:winapi_thunks.obj
 0001:00006df0       ??_C@_1DK@NDHNAHIO@?$AAa?$AAp?$AAi?$AA?9?$AAm?$AAs?$AA?9?$AAw?$AAi?$AAn?$AA?9?$AAc?$AAo?$AAr?$AAe@ 10007df0     libucrt:winapi_thunks.obj
 0001:00006e2c       ??_C@_1DM@KGHDGBCM@?$AAa?$AAp?$AAi?$AA?9?$AAm?$AAs?$AA?9?$AAw?$AAi?$AAn?$AA?9?$AAc?$AAo?$AAr?$AAe@ 10007e2c     libucrt:winapi_thunks.obj
 0001:00006e68       ??_C@_1EO@IJIOEFOH@?$AAa?$AAp?$AAi?$AA?9?$AAm?$AAs?$AA?9?$AAw?$AAi?$AAn?$AA?9?$AAr?$AAt?$AAc?$AAo@ 10007e68     libucrt:winapi_thunks.obj
 0001:00006eb8       ??_C@_1FG@HHGEKANL@?$AAa?$AAp?$AAi?$AA?9?$AAm?$AAs?$AA?9?$AAw?$AAi?$AAn?$AA?9?$AAs?$AAe?$AAc?$AAu@ 10007eb8     libucrt:winapi_thunks.obj
 0001:00006f10       ??_C@_1EG@DBIOJECG@?$AAe?$AAx?$AAt?$AA?9?$AAm?$AAs?$AA?9?$AAw?$AAi?$AAn?$AA?9?$AAn?$AAt?$AAu?$AAs@ 10007f10     libucrt:winapi_thunks.obj
 0001:00006f58       ??_C@_1EO@FIHMJCLF@?$AAe?$AAx?$AAt?$AA?9?$AAm?$AAs?$AA?9?$AAw?$AAi?$AAn?$AA?9?$AAn?$AAt?$AAu?$AAs@ 10007f58     libucrt:winapi_thunks.obj
 0001:00006fa8       ??_C@_1EG@DPGNFKGC@?$AAa?$AAp?$AAi?$AA?9?$AAm?$AAs?$AA?9?$AAw?$AAi?$AAn?$AA?9?$AAa?$AAp?$AAp?$AAm@ 10007fa8     libucrt:winapi_thunks.obj
 0001:00006ff0       ??_C@_1BA@IAIFMGEF@?$AAe?$AAx?$AAt?$AA?9?$AAm?$AAs?$AA?9@ 10007ff0     libucrt:winapi_thunks.obj
 0001:00007004       ??_C@_0BA@FHFNEAED@AreFileApisANSI@ 10008004     libucrt:winapi_thunks.obj
 0001:00007024       ??_C@_0BE@LJANKFHF@EnumSystemLocalesEx@ 10008024     libucrt:winapi_thunks.obj
 0001:00007060       ??_C@_0BA@EPCJIIPD@GetDateFormatEx@ 10008060     libucrt:winapi_thunks.obj
 0001:00007080       ??_C@_0BA@CIJJKCJJ@GetTimeFormatEx@ 10008080     libucrt:winapi_thunks.obj
 0001:00007098       ??_C@_0BJ@PBCCBIPI@GetUserDefaultLocaleName@ 10008098     libucrt:winapi_thunks.obj
 0001:000070c4       ??_C@_0BC@CELBKLLA@IsValidLocaleName@ 100080c4     libucrt:winapi_thunks.obj
 0001:000070e8       ??_C@_0BB@CDHDDLLP@LCIDToLocaleName@ 100080e8     libucrt:winapi_thunks.obj
 0001:00007104       ??_C@_0BB@HBDEELFH@LocaleNameToLCID@ 10008104     libucrt:winapi_thunks.obj
 0001:0000711c       ??_C@_0CF@OJOFEIGO@AppPolicyGetProcessTerminationM@ 1000811c     libucrt:winapi_thunks.obj
 0001:00007188       ??_C@_09OFJJIMPC@NAN?$CISNAN?$CJ@ 10008188     libucrt:cvt.obj
 0001:00007194       ??_C@_09IPFBKMDL@nan?$CIsnan?$CJ@ 10008194     libucrt:cvt.obj
 0001:000071a0       ??_C@_08IKHNHAJ@NAN?$CIIND?$CJ@ 100081a0     libucrt:cvt.obj
 0001:000071ac       ??_C@_08OFCDMILK@nan?$CIind?$CJ@ 100081ac     libucrt:cvt.obj
 0001:000071b8       ??_C@_05KLBDPFGC@e?$CL000@ 100081b8     libucrt:cvt.obj
 0001:00007240       ___lc_category             10008240     libucrt:wsetlocale.obj
 0001:00007288       ??_C@_1O@GIFLHMA@?$AAL?$AAC?$AA_?$AAA?$AAL?$AAL@ 10008288     libucrt:wsetlocale.obj
 0001:00007298       ??_C@_1BG@PPOMIBNJ@?$AAL?$AAC?$AA_?$AAC?$AAO?$AAL?$AAL?$AAA?$AAT?$AAE@ 10008298     libucrt:wsetlocale.obj
 0001:000072b0       ??_C@_1BC@FFJGAPJM@?$AAL?$AAC?$AA_?$AAC?$AAT?$AAY?$AAP?$AAE@ 100082b0     libucrt:wsetlocale.obj
 0001:000072c4       ??_C@_1BI@PCKFNJFB@?$AAL?$AAC?$AA_?$AAM?$AAO?$AAN?$AAE?$AAT?$AAA?$AAR?$AAY@ 100082c4     libucrt:wsetlocale.obj
 0001:000072dc       ??_C@_1BG@ENIEDKID@?$AAL?$AAC?$AA_?$AAN?$AAU?$AAM?$AAE?$AAR?$AAI?$AAC@ 100082dc     libucrt:wsetlocale.obj
 0001:000072f4       ??_C@_1BA@HAAOMIIG@?$AAL?$AAC?$AA_?$AAT?$AAI?$AAM?$AAE@ 100082f4     libucrt:wsetlocale.obj
 0001:00007304       ??_C@_15NBPDDFIP@?$AA?$DN?$AA?$DL@ 10008304     libucrt:wsetlocale.obj
 0001:0000730c       ??_C@_13PJJBFPED@?$AA?$DL@ 1000830c     libucrt:wsetlocale.obj
 0001:00007310       ??_C@_13NMPKAAJP@?$AA?$DN@ 10008310     libucrt:wsetlocale.obj
 0001:00007314       ??_C@_17EFJLDFDO@?$AA?9?$AA_?$AA?4@ 10008314     libucrt:wsetlocale.obj
 0001:0000731c       ??_C@_13FHBKNHDA@?$AAC@    1000831c     libucrt:wsetlocale.obj
 0001:00007320       ??_C@_17MBJJLFDM@?$AA_?$AA?4?$AA?0@ 10008320     libucrt:wsetlocale.obj
 0001:00007328       ??_C@_13ENNFDPBH@?$AA_@    10008328     libucrt:wsetlocale.obj
 0001:00007330       ___lc_time_c               10008330     libucrt:nlsdata.obj
 0001:00007494       ??_C@_03KOEHGMDN@Sun@      10008494     libucrt:nlsdata.obj
 0001:00007498       ??_C@_03PDAGKDH@Mon@       10008498     libucrt:nlsdata.obj
 0001:0000749c       ??_C@_03NAGEINEP@Tue@      1000849c     libucrt:nlsdata.obj
 0001:000074a0       ??_C@_03MHOMLAJA@Wed@      100084a0     libucrt:nlsdata.obj
 0001:000074a4       ??_C@_03IOFIKPDN@Thu@      100084a4     libucrt:nlsdata.obj
 0001:000074a8       ??_C@_03IDIOELNC@Fri@      100084a8     libucrt:nlsdata.obj
 0001:000074ac       ??_C@_03FEFJNEK@Sat@       100084ac     libucrt:nlsdata.obj
 0001:000074b0       ??_C@_06OOPIFAJ@Sunday@    100084b0     libucrt:nlsdata.obj
 0001:000074b8       ??_C@_06JLEDEDGH@Monday@   100084b8     libucrt:nlsdata.obj
 0001:000074c0       ??_C@_07BAAGCFCM@Tuesday@  100084c0     libucrt:nlsdata.obj
 0001:000074c8       ??_C@_09DLIGFAKA@Wednesday@ 100084c8     libucrt:nlsdata.obj
 0001:000074d4       ??_C@_08HACCIKIA@Thursday@ 100084d4     libucrt:nlsdata.obj
 0001:000074e0       ??_C@_06JECMNKMI@Friday@   100084e0     libucrt:nlsdata.obj
 0001:000074e8       ??_C@_08INBOOONO@Saturday@ 100084e8     libucrt:nlsdata.obj
 0001:000074f4       ??_C@_03JIHJHPIE@Jan@      100084f4     libucrt:nlsdata.obj
 0001:000074f8       ??_C@_03HJBDCHOM@Feb@      100084f8     libucrt:nlsdata.obj
 0001:000074fc       ??_C@_03ODNJBKGA@Mar@      100084fc     libucrt:nlsdata.obj
 0001:00007500       ??_C@_03LEOLGMJP@Apr@      10008500     libucrt:nlsdata.obj
 0001:00007504       ??_C@_03CNMDKL@May@        10008504     libucrt:nlsdata.obj
 0001:00007508       ??_C@_03IDFGHECI@Jun@      10008508     libucrt:nlsdata.obj
 0001:0000750c       ??_C@_03LBGABGKK@Jul@      1000850c     libucrt:nlsdata.obj
 0001:00007510       ??_C@_03IFJFEIGA@Aug@      10008510     libucrt:nlsdata.obj
 0001:00007514       ??_C@_03GGCAPAJC@Sep@      10008514     libucrt:nlsdata.obj
 0001:00007518       ??_C@_03BMAOKBAD@Oct@      10008518     libucrt:nlsdata.obj
 0001:0000751c       ??_C@_03JPJOFNIA@Nov@      1000851c     libucrt:nlsdata.obj
 0001:00007520       ??_C@_03MKABNOCG@Dec@      10008520     libucrt:nlsdata.obj
 0001:00007524       ??_C@_07CGJPFGJA@January@  10008524     libucrt:nlsdata.obj
 0001:0000752c       ??_C@_08GNJGEPFN@February@ 1000852c     libucrt:nlsdata.obj
 0001:00007538       ??_C@_05HPCKOFNC@March@    10008538     libucrt:nlsdata.obj
 0001:00007540       ??_C@_05DMJDNLEJ@April@    10008540     libucrt:nlsdata.obj
 0001:00007548       ??_C@_04CNLMGBGM@June@     10008548     libucrt:nlsdata.obj
 0001:00007550       ??_C@_04MIEPOIFP@July@     10008550     libucrt:nlsdata.obj
 0001:00007558       ??_C@_06LBBHFDDG@August@   10008558     libucrt:nlsdata.obj
 0001:00007560       ??_C@_09BHHEALKD@September@ 10008560     libucrt:nlsdata.obj
 0001:0000756c       ??_C@_07JJNFCEND@October@  1000856c     libucrt:nlsdata.obj
 0001:00007574       ??_C@_08HCHEGEOA@November@ 10008574     libucrt:nlsdata.obj
 0001:00007580       ??_C@_08EDHMEBNP@December@ 10008580     libucrt:nlsdata.obj
 0001:0000758c       ??_C@_02DEDBPAFC@AM@       1000858c     libucrt:nlsdata.obj
 0001:00007590       ??_C@_02CJNFDJBF@PM@       10008590     libucrt:nlsdata.obj
 0001:00007594       ??_C@_08BPBNCDIB@MM?1dd?1yy@ 10008594     libucrt:nlsdata.obj
 0001:000075a0       ??_C@_0BE@CKGJFCPC@dddd?0?5MMMM?5dd?0?5yyyy@ 100085a0     libucrt:nlsdata.obj
 0001:000075b4       ??_C@_08JCCMCCIL@HH?3mm?3ss@ 100085b4     libucrt:nlsdata.obj
 0001:000075c0       ??_C@_17MBGCMIPB@?$AAS?$AAu?$AAn@ 100085c0     libucrt:nlsdata.obj
 0001:000075c8       ??_C@_17KBOMKBF@?$AAM?$AAo?$AAn@ 100085c8     libucrt:nlsdata.obj
 0001:000075d0       ??_C@_17BMKGEGOJ@?$AAT?$AAu?$AAe@ 100085d0     libucrt:nlsdata.obj
 0001:000075d8       ??_C@_17CJEDCEPE@?$AAW?$AAe?$AAd@ 100085d8     libucrt:nlsdata.obj
 0001:000075e0       ??_C@_17PDPHAADD@?$AAT?$AAh?$AAu@ 100085e0     libucrt:nlsdata.obj
 0001:000075e8       ??_C@_17HFOLPPLP@?$AAF?$AAr?$AAi@ 100085e8     libucrt:nlsdata.obj
 0001:000075f0       ??_C@_17GGIBDPIH@?$AAS?$AAa?$AAt@ 100085f0     libucrt:nlsdata.obj
 0001:000075f8       ??_C@_1O@IHNHDHPB@?$AAS?$AAu?$AAn?$AAd?$AAa?$AAy@ 100085f8     libucrt:nlsdata.obj
 0001:00007608       ??_C@_1O@MMNBFLIA@?$AAM?$AAo?$AAn?$AAd?$AAa?$AAy@ 10008608     libucrt:nlsdata.obj
 0001:00007618       ??_C@_1BA@ENFBFFEK@?$AAT?$AAu?$AAe?$AAs?$AAd?$AAa?$AAy@ 10008618     libucrt:nlsdata.obj
 0001:00007628       ??_C@_1BE@EBOGMDOH@?$AAW?$AAe?$AAd?$AAn?$AAe?$AAs?$AAd?$AAa?$AAy@ 10008628     libucrt:nlsdata.obj
 0001:0000763c       ??_C@_1BC@HHMNLIHE@?$AAT?$AAh?$AAu?$AAr?$AAs?$AAd?$AAa?$AAy@ 1000863c     libucrt:nlsdata.obj
 0001:00007650       ??_C@_1O@PDICJHAG@?$AAF?$AAr?$AAi?$AAd?$AAa?$AAy@ 10008650     libucrt:nlsdata.obj
 0001:00007660       ??_C@_1BC@ENMNNPAJ@?$AAS?$AAa?$AAt?$AAu?$AAr?$AAd?$AAa?$AAy@ 10008660     libucrt:nlsdata.obj
 0001:00007674       ??_C@_17DKNBKCHM@?$AAJ?$AAa?$AAn@ 10008674     libucrt:nlsdata.obj
 0001:0000767c       ??_C@_17LMDJEKJN@?$AAF?$AAe?$AAb@ 1000867c     libucrt:nlsdata.obj
 0001:00007684       ??_C@_17CKNLEDEC@?$AAM?$AAa?$AAr@ 10008684     libucrt:nlsdata.obj
 0001:0000768c       ??_C@_17LFPOIHDD@?$AAA?$AAp?$AAr@ 1000868c     libucrt:nlsdata.obj
 0001:00007694       ??_C@_17PNNKMEED@?$AAM?$AAa?$AAy@ 10008694     libucrt:nlsdata.obj
 0001:0000769c       ??_C@_17KCJGOCPB@?$AAJ?$AAu?$AAn@ 1000869c     libucrt:nlsdata.obj
 0001:000076a4       ??_C@_17IJPCKHK@?$AAJ?$AAu?$AAl@ 100086a4     libucrt:nlsdata.obj
 0001:000076ac       ??_C@_17ICPELBCN@?$AAA?$AAu?$AAg@ 100086ac     libucrt:nlsdata.obj
 0001:000076b4       ??_C@_17HCHCOKMG@?$AAS?$AAe?$AAp@ 100086b4     libucrt:nlsdata.obj
 0001:000076bc       ??_C@_17FNLKOI@?$AAO?$AAc?$AAt@ 100086bc     libucrt:nlsdata.obj
 0001:000076c4       ??_C@_17BBDMLCIG@?$AAN?$AAo?$AAv@ 100086c4     libucrt:nlsdata.obj
 0001:000076cc       ??_C@_17EGKACKIF@?$AAD?$AAe?$AAc@ 100086cc     libucrt:nlsdata.obj
 0001:000076d4       ??_C@_1BA@EFMEIEBA@?$AAJ?$AAa?$AAn?$AAu?$AAa?$AAr?$AAy@ 100086d4     libucrt:nlsdata.obj
 0001:000076e4       ??_C@_1BC@JGDDFFAM@?$AAF?$AAe?$AAb?$AAr?$AAu?$AAa?$AAr?$AAy@ 100086e4     libucrt:nlsdata.obj
 0001:000076f8       ??_C@_1M@IKEENEDF@?$AAM?$AAa?$AAr?$AAc?$AAh@ 100086f8     libucrt:nlsdata.obj
 0001:00007704       ??_C@_1M@GJNLMHFD@?$AAA?$AAp?$AAr?$AAi?$AAl@ 10008704     libucrt:nlsdata.obj
 0001:00007710       ??_C@_19EPFLPGAP@?$AAJ?$AAu?$AAn?$AAe@ 10008710     libucrt:nlsdata.obj
 0001:0000771c       ??_C@_19BIFMLPCD@?$AAJ?$AAu?$AAl?$AAy@ 1000871c     libucrt:nlsdata.obj
 0001:00007728       ??_C@_1O@PAHLKOAC@?$AAA?$AAu?$AAg?$AAu?$AAs?$AAt@ 10008728     libucrt:nlsdata.obj
 0001:00007738       ??_C@_1BE@DKAAMBJL@?$AAS?$AAe?$AAp?$AAt?$AAe?$AAm?$AAb?$AAe?$AAr@ 10008738     libucrt:nlsdata.obj
 0001:0000774c       ??_C@_1BA@EPANDLNG@?$AAO?$AAc?$AAt?$AAo?$AAb?$AAe?$AAr@ 1000874c     libucrt:nlsdata.obj
 0001:0000775c       ??_C@_1BC@BGLIFPF@?$AAN?$AAo?$AAv?$AAe?$AAm?$AAb?$AAe?$AAr@ 1000875c     libucrt:nlsdata.obj
 0001:00007770       ??_C@_1BC@FEMKIFH@?$AAD?$AAe?$AAc?$AAe?$AAm?$AAb?$AAe?$AAr@ 10008770     libucrt:nlsdata.obj
 0001:00007784       ??_C@_15ODEHAHHF@?$AAA?$AAM@ 10008784     libucrt:nlsdata.obj
 0001:0000778c       ??_C@_15CLMNNGEL@?$AAP?$AAM@ 1000878c     libucrt:nlsdata.obj
 0001:00007794       ??_C@_1BC@IEBCMHCM@?$AAM?$AAM?$AA?1?$AAd?$AAd?$AA?1?$AAy?$AAy@ 10008794     libucrt:nlsdata.obj
 0001:000077a8       ??_C@_1CI@KNAKOEBC@?$AAd?$AAd?$AAd?$AAd?$AA?0?$AA?5?$AAM?$AAM?$AAM?$AAM?$AA?5?$AAd?$AAd?$AA?0?$AA?5@ 100087a8     libucrt:nlsdata.obj
 0001:000077d0       ??_C@_1BC@GDGBMEMK@?$AAH?$AAH?$AA?3?$AAm?$AAm?$AA?3?$AAs?$AAs@ 100087d0     libucrt:nlsdata.obj
 0001:000077e4       ??_C@_03MGHMBJCF@log@      100087e4     libucrt:libm_error.obj
 0001:000077e8       ??_C@_05HGHHAHAP@log10@    100087e8     libucrt:libm_error.obj
 0001:000077f0       ??_C@_03KHJOGHMM@exp@      100087f0     libucrt:libm_error.obj
 0001:000077f4       ??_C@_03JGHBODFD@pow@      100087f4     libucrt:libm_error.obj
 0001:000077f8       ??_C@_04FIHNOPOL@asin@     100087f8     libucrt:libm_error.obj
 0001:00007800       ??_C@_04PDIFKINK@acos@     10008800     libucrt:libm_error.obj
 0001:00007808       ??_C@_04EIAKFFMI@sqrt@     10008808     libucrt:libm_error.obj
 0001:00007910       __infinity                 10008910     libucrt:87tran.obj
 0001:0000791a       __minfinity                1000891a     libucrt:87tran.obj
 0001:00007924       __logemax                  10008924     libucrt:87tran.obj
 0001:0000794a       __OP_EXPjmptab             1000894a     libucrt:87tran.obj
 0001:00007970       __indefinite               10008970     libucrt:87disp.obj
 0001:0000797a       __piby2                    1000897a     libucrt:87disp.obj
 0001:00007984       __piby4                    10008984     libucrt:87disp.obj
 0001:000079b8       __DEFAULT_CW_in_mem        100089b8     libucrt:common.obj
 0001:000079ba       __pi_by_2_to_61            100089ba     libucrt:common.obj
 0001:00007ac0       __real@3fe0000000000000    10008ac0     libucrt:powhlp.obj
 0001:00007bb0       ??_C@_04COOMCNPB@sinh@     10008bb0     libucrt:fpexcept.obj
 0001:00007bb8       ??_C@_04HPJJNFIM@cosh@     10008bb8     libucrt:fpexcept.obj
 0001:00007bc0       ??_C@_04FJHINJAO@tanh@     10008bc0     libucrt:fpexcept.obj
 0001:00007bc8       ??_C@_04MLLJIGOK@atan@     10008bc8     libucrt:fpexcept.obj
 0001:00007bd0       ??_C@_05KNGEOGJB@atan2@    10008bd0     libucrt:fpexcept.obj
 0001:00007bd8       ??_C@_03BLEJJJBH@sin@      10008bd8     libucrt:fpexcept.obj
 0001:00007bdc       ??_C@_03LALBNOCG@cos@      10008bdc     libucrt:fpexcept.obj
 0001:00007be0       ??_C@_03IIINPABG@tan@      10008be0     libucrt:fpexcept.obj
 0001:00007be4       ??_C@_04GFPJNGEK@ceil@     10008be4     libucrt:fpexcept.obj
 0001:00007bec       ??_C@_05PBJFFIGL@floor@    10008bec     libucrt:fpexcept.obj
 0001:00007bf4       ??_C@_04ODHECPBC@fabs@     10008bf4     libucrt:fpexcept.obj
 0001:00007bfc       ??_C@_04EHEDPDJG@modf@     10008bfc     libucrt:fpexcept.obj
 0001:00007c04       ??_C@_05CEJMAHNP@ldexp@    10008c04     libucrt:fpexcept.obj
 0001:00007c0c       ??_C@_05KBKMEMPO@_cabs@    10008c0c     libucrt:fpexcept.obj
 0001:00007c14       ??_C@_06MEIMCGCF@_hypot@   10008c14     libucrt:fpexcept.obj
 0001:00007c1c       ??_C@_04KEPJIHGP@fmod@     10008c1c     libucrt:fpexcept.obj
 0001:00007c24       ??_C@_05GKKHEGJL@frexp@    10008c24     libucrt:fpexcept.obj
 0001:00007c2c       ??_C@_03MJLDFKDL@_y0@      10008c2c     libucrt:fpexcept.obj
 0001:00007c30       ??_C@_03NAKIGLHK@_y1@      10008c30     libucrt:fpexcept.obj
 0001:00007c34       ??_C@_03ONILCKOB@_yn@      10008c34     libucrt:fpexcept.obj
 0001:00007c38       ??_C@_05JGDBENOH@_logb@    10008c38     libucrt:fpexcept.obj
 0001:00007c40       ??_C@_0L@KDOEJCKC@_nextafter@ 10008c40     libucrt:fpexcept.obj
 0001:00007c50       __d_inf                    10008c50     libucrt:util.obj
 0001:00007c58       __d_ind                    10008c58     libucrt:util.obj
 0001:00007c60       __d_max                    10008c60     libucrt:util.obj
 0001:00007c68       __d_mzero                  10008c68     libucrt:util.obj
 0001:00008b70       ??_C@_01GBGANLPD@0@        10009b70     libucrt:cfout.obj
 0001:00008b74       ??_C@_05DNEBIAHO@1?$CDINF@ 10009b74     libucrt:cfout.obj
 0001:00008b7c       ??_C@_06IMKFLFPG@1?$CDQNAN@ 10009b7c     libucrt:cfout.obj
 0001:00008b84       ??_C@_06PGGFOGJG@1?$CDSNAN@ 10009b84     libucrt:cfout.obj
 0001:00008b8c       ??_C@_05PHHOCPM@1?$CDIND@  10009b8c     libucrt:cfout.obj
 0001:00008b98       ___acrt_rg_language        10009b98     libucrt:get_qualified_locale.obj
 0001:00008ea4       ___acrt_rg_language_count  10009ea4     libucrt:get_qualified_locale.obj
 0001:00008ea8       ___acrt_rg_country         10009ea8     libucrt:get_qualified_locale.obj
 0001:00008fbc       ___acrt_rg_country_count   10009fbc     libucrt:get_qualified_locale.obj
 0001:00008fc0       ??_C@_1BC@LLOKLNP@?$AAa?$AAm?$AAe?$AAr?$AAi?$AAc?$AAa?$AAn@ 10009fc0     libucrt:get_qualified_locale.obj
 0001:00008fd4       ??_C@_1CC@HEIGCDGG@?$AAa?$AAm?$AAe?$AAr?$AAi?$AAc?$AAa?$AAn?$AA?5?$AAe?$AAn?$AAg?$AAl?$AAi?$AAs@ 10009fd4     libucrt:get_qualified_locale.obj
 0001:00008ff8       ??_C@_1CC@IHCNOMIN@?$AAa?$AAm?$AAe?$AAr?$AAi?$AAc?$AAa?$AAn?$AA?9?$AAe?$AAn?$AAg?$AAl?$AAi?$AAs@ 10009ff8     libucrt:get_qualified_locale.obj
 0001:0000901c       ??_C@_1BG@GKAGPCGG@?$AAa?$AAu?$AAs?$AAt?$AAr?$AAa?$AAl?$AAi?$AAa?$AAn@ 1000a01c     libucrt:get_qualified_locale.obj
 0001:00009034       ??_C@_1BA@GMENCENF@?$AAb?$AAe?$AAl?$AAg?$AAi?$AAa?$AAn@ 1000a034     libucrt:get_qualified_locale.obj
 0001:00009044       ??_C@_1BC@PJMIIAAN@?$AAc?$AAa?$AAn?$AAa?$AAd?$AAi?$AAa?$AAn@ 1000a044     libucrt:get_qualified_locale.obj
 0001:00009058       ??_C@_17NOIMNFBF@?$AAc?$AAh?$AAh@ 1000a058     libucrt:get_qualified_locale.obj
 0001:00009060       ??_C@_17GGDALCHA@?$AAc?$AAh?$AAi@ 1000a060     libucrt:get_qualified_locale.obj
 0001:00009068       ??_C@_1BA@NPNJKIBL@?$AAc?$AAh?$AAi?$AAn?$AAe?$AAs?$AAe@ 1000a068     libucrt:get_qualified_locale.obj
 0001:00009078       ??_C@_1CC@DINBAMMJ@?$AAc?$AAh?$AAi?$AAn?$AAe?$AAs?$AAe?$AA?9?$AAh?$AAo?$AAn?$AAg?$AAk?$AAo?$AAn@ 1000a078     libucrt:get_qualified_locale.obj
 0001:0000909c       ??_C@_1CG@IOBJPACO@?$AAc?$AAh?$AAi?$AAn?$AAe?$AAs?$AAe?$AA?9?$AAs?$AAi?$AAm?$AAp?$AAl?$AAi?$AAf@ 1000a09c     libucrt:get_qualified_locale.obj
 0001:000090c4       ??_C@_1CE@GAJNDCKG@?$AAc?$AAh?$AAi?$AAn?$AAe?$AAs?$AAe?$AA?9?$AAs?$AAi?$AAn?$AAg?$AAa?$AAp?$AAo@ 1000a0c4     libucrt:get_qualified_locale.obj
 0001:000090e8       ??_C@_1CI@PAJPIOOD@?$AAc?$AAh?$AAi?$AAn?$AAe?$AAs?$AAe?$AA?9?$AAt?$AAr?$AAa?$AAd?$AAi?$AAt?$AAi@ 1000a0e8     libucrt:get_qualified_locale.obj
 0001:00009110       ??_C@_1BM@NILJBMMD@?$AAd?$AAu?$AAt?$AAc?$AAh?$AA?9?$AAb?$AAe?$AAl?$AAg?$AAi?$AAa?$AAn@ 1000a110     libucrt:get_qualified_locale.obj
 0001:0000912c       ??_C@_1CC@OOJPJNEJ@?$AAe?$AAn?$AAg?$AAl?$AAi?$AAs?$AAh?$AA?9?$AAa?$AAm?$AAe?$AAr?$AAi?$AAc?$AAa@ 1000a12c     libucrt:get_qualified_locale.obj
 0001:00009150       ??_C@_1BI@IOLFEEM@?$AAe?$AAn?$AAg?$AAl?$AAi?$AAs?$AAh?$AA?9?$AAa?$AAu?$AAs@ 1000a150     libucrt:get_qualified_locale.obj
 0001:00009168       ??_C@_1BO@HFFNLENJ@?$AAe?$AAn?$AAg?$AAl?$AAi?$AAs?$AAh?$AA?9?$AAb?$AAe?$AAl?$AAi?$AAz?$AAe@ 1000a168     libucrt:get_qualified_locale.obj
 0001:00009188       ??_C@_1BI@HAPKJMPO@?$AAe?$AAn?$AAg?$AAl?$AAi?$AAs?$AAh?$AA?9?$AAc?$AAa?$AAn@ 1000a188     libucrt:get_qualified_locale.obj
 0001:000091a0       ??_C@_1CE@HLNDMIOJ@?$AAe?$AAn?$AAg?$AAl?$AAi?$AAs?$AAh?$AA?9?$AAc?$AAa?$AAr?$AAi?$AAb?$AAb?$AAe@ 1000a1a0     libucrt:get_qualified_locale.obj
 0001:000091c4       ??_C@_1BI@LDHJHHAC@?$AAe?$AAn?$AAg?$AAl?$AAi?$AAs?$AAh?$AA?9?$AAi?$AAr?$AAe@ 1000a1c4     libucrt:get_qualified_locale.obj
 0001:000091dc       ??_C@_1CA@NJMMCFOC@?$AAe?$AAn?$AAg?$AAl?$AAi?$AAs?$AAh?$AA?9?$AAj?$AAa?$AAm?$AAa?$AAi?$AAc?$AAa@ 1000a1dc     libucrt:get_qualified_locale.obj
 0001:000091fc       ??_C@_1BG@BHJEBBGG@?$AAe?$AAn?$AAg?$AAl?$AAi?$AAs?$AAh?$AA?9?$AAn?$AAz@ 1000a1fc     libucrt:get_qualified_locale.obj
 0001:00009214       ??_C@_1CK@FGOEJJCO@?$AAe?$AAn?$AAg?$AAl?$AAi?$AAs?$AAh?$AA?9?$AAs?$AAo?$AAu?$AAt?$AAh?$AA?5?$AAa@ 1000a214     libucrt:get_qualified_locale.obj
 0001:00009240       ??_C@_1DE@PDBJPCJ@?$AAe?$AAn?$AAg?$AAl?$AAi?$AAs?$AAh?$AA?9?$AAt?$AAr?$AAi?$AAn?$AAi?$AAd?$AAa@ 1000a240     libucrt:get_qualified_locale.obj
 0001:00009274       ??_C@_1BG@JGCANDME@?$AAe?$AAn?$AAg?$AAl?$AAi?$AAs?$AAh?$AA?9?$AAu?$AAk@ 1000a274     libucrt:get_qualified_locale.obj
 0001:0000928c       ??_C@_1BG@DINKMLE@?$AAe?$AAn?$AAg?$AAl?$AAi?$AAs?$AAh?$AA?9?$AAu?$AAs@ 1000a28c     libucrt:get_qualified_locale.obj
 0001:000092a4       ??_C@_1BI@NMFDBHJE@?$AAe?$AAn?$AAg?$AAl?$AAi?$AAs?$AAh?$AA?9?$AAu?$AAs?$AAa@ 1000a2a4     libucrt:get_qualified_locale.obj
 0001:000092bc       ??_C@_1BO@OIHKJKII@?$AAf?$AAr?$AAe?$AAn?$AAc?$AAh?$AA?9?$AAb?$AAe?$AAl?$AAg?$AAi?$AAa?$AAn@ 1000a2bc     libucrt:get_qualified_locale.obj
 0001:000092dc       ??_C@_1CA@NKAELJKI@?$AAf?$AAr?$AAe?$AAn?$AAc?$AAh?$AA?9?$AAc?$AAa?$AAn?$AAa?$AAd?$AAi?$AAa?$AAn@ 1000a2dc     libucrt:get_qualified_locale.obj
 0001:000092fc       ??_C@_1CE@MGKCNLGN@?$AAf?$AAr?$AAe?$AAn?$AAc?$AAh?$AA?9?$AAl?$AAu?$AAx?$AAe?$AAm?$AAb?$AAo?$AAu@ 1000a2fc     libucrt:get_qualified_locale.obj
 0001:00009320       ??_C@_1BK@CEGEAILM@?$AAf?$AAr?$AAe?$AAn?$AAc?$AAh?$AA?9?$AAs?$AAw?$AAi?$AAs?$AAs@ 1000a320     libucrt:get_qualified_locale.obj
 0001:0000933c       ??_C@_1CA@PAFKEOCC@?$AAg?$AAe?$AAr?$AAm?$AAa?$AAn?$AA?9?$AAa?$AAu?$AAs?$AAt?$AAr?$AAi?$AAa?$AAn@ 1000a33c     libucrt:get_qualified_locale.obj
 0001:0000935c       ??_C@_1CI@HCFHGOFD@?$AAg?$AAe?$AAr?$AAm?$AAa?$AAn?$AA?9?$AAl?$AAi?$AAc?$AAh?$AAt?$AAe?$AAn?$AAs@ 1000a35c     libucrt:get_qualified_locale.obj
 0001:00009384       ??_C@_1CE@FEDDNPDG@?$AAg?$AAe?$AAr?$AAm?$AAa?$AAn?$AA?9?$AAl?$AAu?$AAx?$AAe?$AAm?$AAb?$AAo?$AAu@ 1000a384     libucrt:get_qualified_locale.obj
 0001:000093a8       ??_C@_1BK@LIMINNMN@?$AAg?$AAe?$AAr?$AAm?$AAa?$AAn?$AA?9?$AAs?$AAw?$AAi?$AAs?$AAs@ 1000a3a8     libucrt:get_qualified_locale.obj
 0001:000093c4       ??_C@_1BM@LGMDBEPD@?$AAi?$AAr?$AAi?$AAs?$AAh?$AA?9?$AAe?$AAn?$AAg?$AAl?$AAi?$AAs?$AAh@ 1000a3c4     libucrt:get_qualified_locale.obj
 0001:000093e0       ??_C@_1BM@NNCFBAEE@?$AAi?$AAt?$AAa?$AAl?$AAi?$AAa?$AAn?$AA?9?$AAs?$AAw?$AAi?$AAs?$AAs@ 1000a3e0     libucrt:get_qualified_locale.obj
 0001:000093fc       ??_C@_1BE@FEDJNPIB@?$AAn?$AAo?$AAr?$AAw?$AAe?$AAg?$AAi?$AAa?$AAn@ 1000a3fc     libucrt:get_qualified_locale.obj
 0001:00009410       ??_C@_1CC@CILKDEIE@?$AAn?$AAo?$AAr?$AAw?$AAe?$AAg?$AAi?$AAa?$AAn?$AA?9?$AAb?$AAo?$AAk?$AAm?$AAa@ 1000a410     libucrt:get_qualified_locale.obj
 0001:00009434       ??_C@_1CE@DHMMHEPL@?$AAn?$AAo?$AAr?$AAw?$AAe?$AAg?$AAi?$AAa?$AAn?$AA?9?$AAn?$AAy?$AAn?$AAo?$AAr@ 1000a434     libucrt:get_qualified_locale.obj
 0001:00009458       ??_C@_1CK@OPNMHECD@?$AAp?$AAo?$AAr?$AAt?$AAu?$AAg?$AAu?$AAe?$AAs?$AAe?$AA?9?$AAb?$AAr?$AAa?$AAz@ 1000a458     libucrt:get_qualified_locale.obj
 0001:00009484       ??_C@_1CE@KEEHCDB@?$AAs?$AAp?$AAa?$AAn?$AAi?$AAs?$AAh?$AA?9?$AAa?$AAr?$AAg?$AAe?$AAn?$AAt?$AAi@ 1000a484     libucrt:get_qualified_locale.obj
 0001:000094a8       ??_C@_1CA@GIAOLHJD@?$AAs?$AAp?$AAa?$AAn?$AAi?$AAs?$AAh?$AA?9?$AAb?$AAo?$AAl?$AAi?$AAv?$AAi?$AAa@ 1000a4a8     libucrt:get_qualified_locale.obj
 0001:000094c8       ??_C@_1BM@OJNDFNPD@?$AAs?$AAp?$AAa?$AAn?$AAi?$AAs?$AAh?$AA?9?$AAc?$AAh?$AAi?$AAl?$AAe@ 1000a4c8     libucrt:get_qualified_locale.obj
 0001:000094e4       ??_C@_1CC@OCOLPALL@?$AAs?$AAp?$AAa?$AAn?$AAi?$AAs?$AAh?$AA?9?$AAc?$AAo?$AAl?$AAo?$AAm?$AAb?$AAi@ 1000a4e4     libucrt:get_qualified_locale.obj
 0001:00009508       ??_C@_1CG@BPOFMKBB@?$AAs?$AAp?$AAa?$AAn?$AAi?$AAs?$AAh?$AA?9?$AAc?$AAo?$AAs?$AAt?$AAa?$AA?5?$AAr@ 1000a508     libucrt:get_qualified_locale.obj
 0001:00009530       ??_C@_1DG@IGOBAPBB@?$AAs?$AAp?$AAa?$AAn?$AAi?$AAs?$AAh?$AA?9?$AAd?$AAo?$AAm?$AAi?$AAn?$AAi?$AAc@ 1000a530     libucrt:get_qualified_locale.obj
 0001:00009568       ??_C@_1CA@JHAPGEGI@?$AAs?$AAp?$AAa?$AAn?$AAi?$AAs?$AAh?$AA?9?$AAe?$AAc?$AAu?$AAa?$AAd?$AAo?$AAr@ 1000a568     libucrt:get_qualified_locale.obj
 0001:00009588       ??_C@_1CI@LAPALJPP@?$AAs?$AAp?$AAa?$AAn?$AAi?$AAs?$AAh?$AA?9?$AAe?$AAl?$AA?5?$AAs?$AAa?$AAl?$AAv@ 1000a588     libucrt:get_qualified_locale.obj
 0001:000095b0       ??_C@_1CE@PDGBOFOM@?$AAs?$AAp?$AAa?$AAn?$AAi?$AAs?$AAh?$AA?9?$AAg?$AAu?$AAa?$AAt?$AAe?$AAm?$AAa@ 1000a5b0     libucrt:get_qualified_locale.obj
 0001:000095d4       ??_C@_1CC@NBEBAODI@?$AAs?$AAp?$AAa?$AAn?$AAi?$AAs?$AAh?$AA?9?$AAh?$AAo?$AAn?$AAd?$AAu?$AAr?$AAa@ 1000a5d4     libucrt:get_qualified_locale.obj
 0001:000095f8       ??_C@_1CA@LLKGHBMF@?$AAs?$AAp?$AAa?$AAn?$AAi?$AAs?$AAh?$AA?9?$AAm?$AAe?$AAx?$AAi?$AAc?$AAa?$AAn@ 1000a5f8     libucrt:get_qualified_locale.obj
 0001:00009618       ??_C@_1BO@LKNDOIGD@?$AAs?$AAp?$AAa?$AAn?$AAi?$AAs?$AAh?$AA?9?$AAm?$AAo?$AAd?$AAe?$AAr?$AAn@ 1000a618     libucrt:get_qualified_locale.obj
 0001:00009638       ??_C@_1CE@NMDMOEEB@?$AAs?$AAp?$AAa?$AAn?$AAi?$AAs?$AAh?$AA?9?$AAn?$AAi?$AAc?$AAa?$AAr?$AAa?$AAg@ 1000a638     libucrt:get_qualified_locale.obj
 0001:0000965c       ??_C@_1BO@LLCBEJGB@?$AAs?$AAp?$AAa?$AAn?$AAi?$AAs?$AAh?$AA?9?$AAp?$AAa?$AAn?$AAa?$AAm?$AAa@ 1000a65c     libucrt:get_qualified_locale.obj
 0001:0000967c       ??_C@_1CC@FKPGGIHO@?$AAs?$AAp?$AAa?$AAn?$AAi?$AAs?$AAh?$AA?9?$AAp?$AAa?$AAr?$AAa?$AAg?$AAu?$AAa@ 1000a67c     libucrt:get_qualified_locale.obj
 0001:000096a0       ??_C@_1BK@CDEIHOOP@?$AAs?$AAp?$AAa?$AAn?$AAi?$AAs?$AAh?$AA?9?$AAp?$AAe?$AAr?$AAu@ 1000a6a0     libucrt:get_qualified_locale.obj
 0001:000096bc       ??_C@_1CI@GAHAKKGP@?$AAs?$AAp?$AAa?$AAn?$AAi?$AAs?$AAh?$AA?9?$AAp?$AAu?$AAe?$AAr?$AAt?$AAo?$AA?5@ 1000a6bc     libucrt:get_qualified_locale.obj
 0001:000096e4       ??_C@_1CA@NKJBCAGP@?$AAs?$AAp?$AAa?$AAn?$AAi?$AAs?$AAh?$AA?9?$AAu?$AAr?$AAu?$AAg?$AAu?$AAa?$AAy@ 1000a6e4     libucrt:get_qualified_locale.obj
 0001:00009704       ??_C@_1CE@ODILCONM@?$AAs?$AAp?$AAa?$AAn?$AAi?$AAs?$AAh?$AA?9?$AAv?$AAe?$AAn?$AAe?$AAz?$AAu?$AAe@ 1000a704     libucrt:get_qualified_locale.obj
 0001:00009728       ??_C@_1CA@OBNMCGFO@?$AAs?$AAw?$AAe?$AAd?$AAi?$AAs?$AAh?$AA?9?$AAf?$AAi?$AAn?$AAl?$AAa?$AAn?$AAd@ 1000a728     libucrt:get_qualified_locale.obj
 0001:00009748       ??_C@_1M@PIPDDPPI@?$AAs?$AAw?$AAi?$AAs?$AAs@ 1000a748     libucrt:get_qualified_locale.obj
 0001:00009754       ??_C@_15GMFIMNFM@?$AAu?$AAs@ 1000a754     libucrt:get_qualified_locale.obj
 0001:0000975c       ??_C@_17HAEBFAGL@?$AAu?$AAs?$AAa@ 1000a75c     libucrt:get_qualified_locale.obj
 0001:00009764       ??_C@_1BA@DPFJEPHB@?$AAa?$AAm?$AAe?$AAr?$AAi?$AAc?$AAa@ 1000a764     libucrt:get_qualified_locale.obj
 0001:00009774       ??_C@_1BA@ELOGGFK@?$AAb?$AAr?$AAi?$AAt?$AAa?$AAi?$AAn@ 1000a774     libucrt:get_qualified_locale.obj
 0001:00009784       ??_C@_1M@GHBGIGDA@?$AAc?$AAh?$AAi?$AAn?$AAa@ 1000a784     libucrt:get_qualified_locale.obj
 0001:00009790       ??_C@_1M@NCHEJOPO@?$AAc?$AAz?$AAe?$AAc?$AAh@ 1000a790     libucrt:get_qualified_locale.obj
 0001:0000979c       ??_C@_1BA@BKPAPBLA@?$AAe?$AAn?$AAg?$AAl?$AAa?$AAn?$AAd@ 1000a79c     libucrt:get_qualified_locale.obj
 0001:000097ac       ??_C@_1BM@HKBCKIPC@?$AAg?$AAr?$AAe?$AAa?$AAt?$AA?5?$AAb?$AAr?$AAi?$AAt?$AAa?$AAi?$AAn@ 1000a7ac     libucrt:get_qualified_locale.obj
 0001:000097c8       ??_C@_1BA@PPCHPGJB@?$AAh?$AAo?$AAl?$AAl?$AAa?$AAn?$AAd@ 1000a7c8     libucrt:get_qualified_locale.obj
 0001:000097d8       ??_C@_1BE@JBMPEGDG@?$AAh?$AAo?$AAn?$AAg?$AA?9?$AAk?$AAo?$AAn?$AAg@ 1000a7d8     libucrt:get_qualified_locale.obj
 0001:000097ec       ??_C@_1BI@KOELBBPJ@?$AAn?$AAe?$AAw?$AA?9?$AAz?$AAe?$AAa?$AAl?$AAa?$AAn?$AAd@ 1000a7ec     libucrt:get_qualified_locale.obj
 0001:00009804       ??_C@_15HIEBHAIO@?$AAn?$AAz@ 1000a804     libucrt:get_qualified_locale.obj
 0001:0000980c       ??_C@_1BC@CHBCPFPI@?$AAp?$AAr?$AA?5?$AAc?$AAh?$AAi?$AAn?$AAa@ 1000a80c     libucrt:get_qualified_locale.obj
 0001:00009820       ??_C@_1BC@JAOIIFKD@?$AAp?$AAr?$AA?9?$AAc?$AAh?$AAi?$AAn?$AAa@ 1000a820     libucrt:get_qualified_locale.obj
 0001:00009834       ??_C@_1BI@BEHPPHKC@?$AAp?$AAu?$AAe?$AAr?$AAt?$AAo?$AA?9?$AAr?$AAi?$AAc?$AAo@ 1000a834     libucrt:get_qualified_locale.obj
 0001:0000984c       ??_C@_1O@PAEOFKDI@?$AAs?$AAl?$AAo?$AAv?$AAa?$AAk@ 1000a84c     libucrt:get_qualified_locale.obj
 0001:0000985c       ??_C@_1BK@FIHMCKAM@?$AAs?$AAo?$AAu?$AAt?$AAh?$AA?5?$AAa?$AAf?$AAr?$AAi?$AAc?$AAa@ 1000a85c     libucrt:get_qualified_locale.obj
 0001:00009878       ??_C@_1BI@NAEOODKB@?$AAs?$AAo?$AAu?$AAt?$AAh?$AA?5?$AAk?$AAo?$AAr?$AAe?$AAa@ 1000a878     libucrt:get_qualified_locale.obj
 0001:00009890       ??_C@_1BK@FBDGGIFF@?$AAs?$AAo?$AAu?$AAt?$AAh?$AA?9?$AAa?$AAf?$AAr?$AAi?$AAc?$AAa@ 1000a890     libucrt:get_qualified_locale.obj
 0001:000098ac       ??_C@_1BI@GHLEJDPK@?$AAs?$AAo?$AAu?$AAt?$AAh?$AA?9?$AAk?$AAo?$AAr?$AAe?$AAa@ 1000a8ac     libucrt:get_qualified_locale.obj
 0001:000098c4       ??_C@_1CE@PLHLOMJF@?$AAt?$AAr?$AAi?$AAn?$AAi?$AAd?$AAa?$AAd?$AA?5?$AA?$CG?$AA?5?$AAt?$AAo?$AAb?$AAa@ 1000a8c4     libucrt:get_qualified_locale.obj
 0001:000098e8       ??_C@_1BO@MODIMHHI@?$AAu?$AAn?$AAi?$AAt?$AAe?$AAd?$AA?9?$AAk?$AAi?$AAn?$AAg?$AAd?$AAo?$AAm@ 1000a8e8     libucrt:get_qualified_locale.obj
 0001:00009908       ??_C@_1BM@FFHJONBJ@?$AAu?$AAn?$AAi?$AAt?$AAe?$AAd?$AA?9?$AAs?$AAt?$AAa?$AAt?$AAe?$AAs@ 1000a908     libucrt:get_qualified_locale.obj
 0001:00009924       ??_C@_19MPDNHKDG@?$AAu?$AAt?$AAf?$AA8@ 1000a924     libucrt:get_qualified_locale.obj
 0001:00009930       ??_C@_17DNCLJFIF@?$AAA?$AAC?$AAP@ 1000a930     libucrt:get_qualified_locale.obj
 0001:00009938       ??_C@_1M@FPEIIFAM@?$AAu?$AAt?$AAf?$AA?9?$AA8@ 1000a938     libucrt:get_qualified_locale.obj
 0001:00009944       ??_C@_17CIKBIHLH@?$AAO?$AAC?$AAP@ 1000a944     libucrt:get_qualified_locale.obj
 0001:0000994c       ___rglangidNotDefault      1000a94c     libucrt:getqloc_downlevel.obj
 0001:00009960       ___acrt_log10_table_t      1000a960     libucrt:log10_tables.obj
 0001:00009d70       ___acrt_log10_table_cb     1000ad70     libucrt:log10_tables.obj
 0001:0000a180       ___acrt_pow_rcp_t1         1000b180     libucrt:pow_tables.obj
 0001:0000a590       ___acrt_pow_log2_t1        1000b590     libucrt:pow_tables.obj
 0001:0000ada0       ___acrt_pow_rcp_t2         1000bda0     libucrt:pow_tables.obj
 0001:0000b1b0       ___acrt_pow_log2_t2        1000c1b0     libucrt:pow_tables.obj
 0001:0000b9c0       ___acrt_pow_rcp_t3         1000c9c0     libucrt:pow_tables.obj
 0001:0000c1d0       ___acrt_pow_log2_t3        1000d1d0     libucrt:pow_tables.obj
 0001:0000d1e0       ___acrt_pow_clv            1000e1e0     libucrt:pow_tables.obj
 0001:0000d200       ___acrt_pow_exp2_tbl       1000e200     libucrt:pow_tables.obj
 0001:0000da00       ??_C@_1BA@BALFACEM@?$AAC?$AAO?$AAN?$AAO?$AAU?$AAT?$AA$@ 1000ea00     libucrt:initcon.obj
 0001:0000da30       __load_config_used         1000ea30     LIBCMT:loadcfg.obj
 0001:0000dad4       ??_R4exception@std@@6B@    1000ead4     libcpmt:xthrow.obj
 0001:0000dae8       ??_R3exception@std@@8      1000eae8     libcpmt:xthrow.obj
 0001:0000daf8       ??_R2exception@std@@8      1000eaf8     libcpmt:xthrow.obj
 0001:0000db00       ??_R1A@?0A@EA@exception@std@@8 1000eb00     libcpmt:xthrow.obj
 0001:0000db1c       ??_R4bad_alloc@std@@6B@    1000eb1c     libcpmt:xthrow.obj
 0001:0000db30       ??_R3bad_alloc@std@@8      1000eb30     libcpmt:xthrow.obj
 0001:0000db40       ??_R2bad_alloc@std@@8      1000eb40     libcpmt:xthrow.obj
 0001:0000db4c       ??_R1A@?0A@EA@bad_alloc@std@@8 1000eb4c     libcpmt:xthrow.obj
 0001:0000db68       ??_R4logic_error@std@@6B@  1000eb68     libcpmt:xthrow.obj
 0001:0000db7c       ??_R3logic_error@std@@8    1000eb7c     libcpmt:xthrow.obj
 0001:0000db8c       ??_R2logic_error@std@@8    1000eb8c     libcpmt:xthrow.obj
 0001:0000db98       ??_R1A@?0A@EA@logic_error@std@@8 1000eb98     libcpmt:xthrow.obj
 0001:0000dbb4       ??_R4length_error@std@@6B@ 1000ebb4     libcpmt:xthrow.obj
 0001:0000dbc8       ??_R3length_error@std@@8   1000ebc8     libcpmt:xthrow.obj
 0001:0000dbd8       ??_R2length_error@std@@8   1000ebd8     libcpmt:xthrow.obj
 0001:0000dbe8       ??_R1A@?0A@EA@length_error@std@@8 1000ebe8     libcpmt:xthrow.obj
 0001:0000dc04       ??_R4out_of_range@std@@6B@ 1000ec04     libcpmt:xthrow.obj
 0001:0000dc18       ??_R3out_of_range@std@@8   1000ec18     libcpmt:xthrow.obj
 0001:0000dc28       ??_R2out_of_range@std@@8   1000ec28     libcpmt:xthrow.obj
 0001:0000dc38       ??_R1A@?0A@EA@out_of_range@std@@8 1000ec38     libcpmt:xthrow.obj
 0001:0000dc54       ??_R4runtime_error@std@@6B@ 1000ec54     libcpmt:xthrow.obj
 0001:0000dc68       ??_R3runtime_error@std@@8  1000ec68     libcpmt:xthrow.obj
 0001:0000dc78       ??_R2runtime_error@std@@8  1000ec78     libcpmt:xthrow.obj
 0001:0000dc84       ??_R1A@?0A@EA@runtime_error@std@@8 1000ec84     libcpmt:xthrow.obj
 0001:0000dca0       ??_R4bad_function_call@std@@6B@ 1000eca0     libcpmt:xthrow.obj
 0001:0000dcb4       ??_R3bad_function_call@std@@8 1000ecb4     libcpmt:xthrow.obj
 0001:0000dcc4       ??_R2bad_function_call@std@@8 1000ecc4     libcpmt:xthrow.obj
 0001:0000dcd0       ??_R1A@?0A@EA@bad_function_call@std@@8 1000ecd0     libcpmt:xthrow.obj
 0001:0000dcec       ??_R4_Facet_base@std@@6B@  1000ecec     libcpmt:locale0.obj
 0001:0000dd00       ??_R3_Facet_base@std@@8    1000ed00     libcpmt:locale0.obj
 0001:0000dd10       ??_R2_Facet_base@std@@8    1000ed10     libcpmt:locale0.obj
 0001:0000dd18       ??_R1A@?0A@EA@_Facet_base@std@@8 1000ed18     libcpmt:locale0.obj
 0001:0000dd34       ??_R4_Locimp@locale@std@@6B@ 1000ed34     libcpmt:locale0.obj
 0001:0000dd48       ??_R3_Locimp@locale@std@@8 1000ed48     libcpmt:locale0.obj
 0001:0000dd58       ??_R2_Locimp@locale@std@@8 1000ed58     libcpmt:locale0.obj
 0001:0000dd6c       ??_R1A@?0A@EA@_Locimp@locale@std@@8 1000ed6c     libcpmt:locale0.obj
 0001:0000dd88       ??_R1A@?0A@EA@facet@locale@std@@8 1000ed88     libcpmt:locale0.obj
 0001:0000dda4       ??_R3facet@locale@std@@8   1000eda4     libcpmt:locale0.obj
 0001:0000ddb4       ??_R2facet@locale@std@@8   1000edb4     libcpmt:locale0.obj
 0001:0000ddc4       ??_R13?0A@EA@_Crt_new_delete@std@@8 1000edc4     libcpmt:locale0.obj
 0001:0000dde0       ??_R3_Crt_new_delete@std@@8 1000ede0     libcpmt:locale0.obj
 0001:0000ddf0       ??_R2_Crt_new_delete@std@@8 1000edf0     libcpmt:locale0.obj
 0001:0000ddf8       ??_R1A@?0A@EA@_Crt_new_delete@std@@8 1000edf8     libcpmt:locale0.obj
 0001:0000de14       ??_R4bad_array_new_length@std@@6B@ 1000ee14     libcpmt:locale.obj
 0001:0000de28       ??_R3bad_array_new_length@std@@8 1000ee28     libcpmt:locale.obj
 0001:0000de38       ??_R2bad_array_new_length@std@@8 1000ee38     libcpmt:locale.obj
 0001:0000de48       ??_R1A@?0A@EA@bad_array_new_length@std@@8 1000ee48     libcpmt:locale.obj
 0001:0000de64       ??_R4?$numpunct@_W@std@@6B@ 1000ee64     libcpmt:wlocale.obj
 0001:0000de78       ??_R3?$numpunct@_W@std@@8  1000ee78     libcpmt:wlocale.obj
 0001:0000de88       ??_R2?$numpunct@_W@std@@8  1000ee88     libcpmt:wlocale.obj
 0001:0000de9c       ??_R1A@?0A@EA@?$numpunct@_W@std@@8 1000ee9c     libcpmt:wlocale.obj
 0001:0000deb8       ??_R4type_info@@6B@        1000eeb8     LIBCMT:std_type_info_static.obj
 0001:0000decc       ??_R3type_info@@8          1000eecc     LIBCMT:std_type_info_static.obj
 0001:0000dedc       ??_R2type_info@@8          1000eedc     LIBCMT:std_type_info_static.obj
 0001:0000dee4       ??_R1A@?0A@EA@type_info@@8 1000eee4     LIBCMT:std_type_info_static.obj
 0001:0000df00       ??_R4bad_exception@std@@6B@ 1000ef00     libvcruntime:frame.obj
 0001:0000df14       ??_R3bad_exception@std@@8  1000ef14     libvcruntime:frame.obj
 0001:0000df24       ??_R2bad_exception@std@@8  1000ef24     libvcruntime:frame.obj
 0001:0000df30       ??_R1A@?0A@EA@bad_exception@std@@8 1000ef30     libvcruntime:frame.obj
 0001:0000df50       ___safe_se_handler_table   1000ef50     <linker-defined>
 0001:0000e37c       ___rtc_iaa                 1000f37c     LIBCMT:initsect.obj
 0001:0000e380       ___rtc_izz                 1000f380     LIBCMT:initsect.obj
 0001:0000e384       ___rtc_taa                 1000f384     LIBCMT:initsect.obj
 0001:0000e388       ___rtc_tzz                 1000f388     LIBCMT:initsect.obj
 0001:0000e410       __alloca_probe             1000f410 f   chkstk.obj
 0001:0000e410       __chkstk                   1000f410 f   chkstk.obj
 0001:0000e440       ??1PerfLib@@QAE@XZ         1000f440 f i perfthread.obj
 0001:0000e440       ?_Tidy_deallocate@?$basic_string@_WU?$char_traits@_W@std@@V?$allocator@_W@2@@std@@AAEXXZ 1000f440 f i fileio.obj
 0001:0000e440       ??1?$basic_string@_WU?$char_traits@_W@std@@V?$allocator@_W@2@@std@@QAE@XZ 1000f440 f i fileio.obj
 0001:0000e4a0       ??1?$vector@Umode@@V?$allocator@Umode@@@std@@@std@@QAE@XZ 1000f4a0 f i fileio.obj
 0001:0000e530       ??1columns@@QAE@XZ         1000f530 f i fileio.obj
 0001:0000e620       ??1mode@@QAE@XZ            1000f620 f i fileio.obj
 0001:0000e640       ?WriteToFile@@YAIPAXABV?$basic_string_view@_WU?$char_traits@_W@std@@@std@@@Z 1000f640 f   fileio.obj
 0001:0000e670       ?WriteToFile@@YAIPAX_W@Z   1000f670 f   fileio.obj
 0001:0000e6a0       ?_Destroy@?$vector@Umode@@V?$allocator@Umode@@@std@@@std@@AAEXPAUmode@@0@Z 1000f6a0 f i fileio.obj
 0001:0000e6d0       ?deallocate@?$allocator@_W@std@@QAEXQA_WI@Z 1000f6d0 f i fileio.obj
 0001:0000e710       ??$format_float@N@detail@v6@fmt@@YAHNHUfloat_specs@012@AAV?$buffer@D@012@@Z 1000f710 f i format.obj
 0001:0000ed20       ??$?X_K@bigint@detail@v6@fmt@@QAEAAV0123@_K@Z 1000fd20 f i format.obj
 0001:0000ee00       ??$_Maklocstr@D@std@@YAPADPBDPADABU_Cvtvec@@@Z 1000fe00 f i format.obj
 0001:0000ee50       ??$_Maklocstr@_W@std@@YAPA_WPBDPA_WABU_Cvtvec@@@Z 1000fe50 f i format.obj
 0001:0000ef20       ??$assign@N$0A@@fp@detail@v6@fmt@@QAE_NN@Z 1000ff20 f i format.obj
 0001:0000ef20       ??$assign@O$0A@@fp@detail@v6@fmt@@QAE_NO@Z 1000ff20 f i format.obj
 0001:0000ef90       ??$decimal_point_impl@_W@detail@v6@fmt@@YA_WVlocale_ref@012@@Z 1000ff90 f i format.obj
 0001:0000f000       ??$do_throw@Vformat_error@v6@fmt@@@detail@v6@fmt@@YAXABVformat_error@12@@Z 10010000 f i format.obj
 0001:0000f030       ??$fallback_format@O@detail@v6@fmt@@YAXOAAV?$buffer@D@012@AAH@Z 10010030 f i format.obj
 0001:0000f030       ??$fallback_format@N@detail@v6@fmt@@YAXNAAV?$buffer@D@012@AAH@Z 10010030 f i format.obj
 0001:0000f790       ??$format_decimal@DI@detail@v6@fmt@@YA?AU?$format_decimal_result@PAD@012@PADIH@Z 10010790 f i format.obj
 0001:0000f7f0       ??$format_decimal@D_K@detail@v6@fmt@@YA?AU?$format_decimal_result@PAD@012@PAD_KH@Z 100107f0 f i format.obj
 0001:0000f910       ??$format_float@O@detail@v6@fmt@@YAHOHUfloat_specs@012@AAV?$buffer@D@012@@Z 10010910 f i format.obj
 0001:0000ff20       ??$get@Vlocale@std@@@locale_ref@detail@v6@fmt@@QBE?AVlocale@std@@XZ 10010f20 f i format.obj
 0001:0000ffe0       ??$grisu_gen_digits@Ufixed_handler@detail@v6@fmt@@@detail@v6@fmt@@YA?AW4result@digits@012@Vfp@012@_KAAHAAUfixed_handler@012@@Z 10010fe0 f i format.obj
 0001:00010460       ??$grisu_gen_digits@Ugrisu_shortest_handler@detail@v6@fmt@@@detail@v6@fmt@@YA?AW4result@digits@012@Vfp@012@_KAAHAAUgrisu_shortest_handler@012@@Z 10011460 f i format.obj
 0001:000106a0       ??$grouping_impl@_W@detail@v6@fmt@@YA?AV?$basic_string@DU?$char_traits@D@std@@V?$allocator@D@2@@std@@Vlocale_ref@012@@Z 100116a0 f i format.obj
 0001:00010710       ??$normalize@$00@detail@v6@fmt@@YA?AVfp@012@V3012@@Z 10011710 f i format.obj
 0001:00010770       ??$normalize@$0A@@detail@v6@fmt@@YA?AVfp@012@V3012@@Z 10011770 f i format.obj
 0001:000107d0       ??$snprintf_float@N@detail@v6@fmt@@YAHNHUfloat_specs@012@AAV?$buffer@D@012@@Z 100117d0 f i format.obj
 0001:000109f0       ??$snprintf_float@O@detail@v6@fmt@@YAHOHUfloat_specs@012@AAV?$buffer@D@012@@Z 100119f0 f i format.obj
 0001:00010c10       ??$thousands_sep_impl@_W@detail@v6@fmt@@YA_WVlocale_ref@012@@Z 10011c10 f i format.obj
 0001:00010c80       ??$use_facet@V?$numpunct@_W@std@@@std@@YAABV?$numpunct@_W@0@ABVlocale@0@@Z 10011c80 f i format.obj
 0001:00010ef0       ??0_Locinfo@std@@QAE@PBD@Z 10011ef0 f i format.obj
 0001:00010f90       ??0bad_alloc@std@@QAE@ABV01@@Z 10011f90 f i format.obj
 0001:00010fc0       ??0bad_array_new_length@std@@QAE@ABV01@@Z 10011fc0 f i format.obj
 0001:00010ff0       ??0bad_array_new_length@std@@QAE@XZ 10011ff0 f i format.obj
 0001:00011010       ??0exception@std@@QAE@ABV01@@Z 10012010 f i format.obj
 0001:00011040       ??0exception@std@@QAE@QBD@Z 10012040 f i format.obj
 0001:00011080       ??0format_error@v6@fmt@@QAE@ABV012@@Z 10012080 f i format.obj
 0001:000110b0       ??0format_error@v6@fmt@@QAE@PBD@Z 100120b0 f i format.obj
 0001:00011100       ??0runtime_error@std@@QAE@ABV01@@Z 10012100 f i format.obj
 0001:00011130       ??0runtime_error@std@@QAE@PBD@Z 10012130 f i format.obj
 0001:00011180       ??1?$_Tidy_guard@V?$numpunct@_W@std@@@std@@QAE@XZ 10012180 f i format.obj
 0001:000111b0       ??1?$_Yarn@D@std@@QAE@XZ   100121b0 f i format.obj
 0001:000111b0       ??1?$_Yarn@_W@std@@QAE@XZ  100121b0 f i format.obj
 0001:000111d0       ??1?$basic_memory_buffer@D$0BPE@V?$allocator@D@std@@@v6@fmt@@UAE@XZ 100121d0 f i format.obj
 0001:00011210       ??1bigint@detail@v6@fmt@@QAE@XZ 10012210 f i format.obj
 0001:00011210       ??1?$basic_memory_buffer@I$0CA@V?$allocator@I@std@@@v6@fmt@@UAE@XZ 10012210 f i format.obj
 0001:00011260       ??1?$basic_memory_buffer@_W$0BPE@V?$allocator@_W@std@@@v6@fmt@@UAE@XZ 10012260 f i format.obj
 0001:000112b0       ??1?$basic_string@DU?$char_traits@D@std@@V?$allocator@D@2@@std@@QAE@XZ 100122b0 f i format.obj
 0001:00011300       ??1?$unique_ptr@V_Facet_base@std@@U?$default_delete@V_Facet_base@std@@@2@@std@@QAE@XZ 10012300 f i format.obj
 0001:00011310       ??1_Locinfo@std@@QAE@XZ    10012310 f i format.obj
 0001:000113e0       ??1runtime_error@std@@UAE@XZ 100123e0 f i format.obj
 0001:000113e0       ??1length_error@std@@UAE@XZ 100123e0 f i libcpmt:xthrow.obj
 0001:000113e0       ??1format_error@v6@fmt@@UAE@XZ 100123e0 f i format.obj
 0001:000113e0       ??1bad_array_new_length@std@@UAE@XZ 100123e0 f i format.obj
 0001:000113e0       ??1bad_function_call@std@@UAE@XZ 100123e0 f i libcpmt:xthrow.obj
 0001:000113e0       ??1out_of_range@std@@UAE@XZ 100123e0 f i libcpmt:xthrow.obj
 0001:000113e0       ??1bad_alloc@std@@UAE@XZ   100123e0 f i format.obj
 0001:000113e0       ??1bad_exception@std@@UAE@XZ 100123e0 f i libvcruntime:frame.obj
 0001:00011400       ??1facet@locale@std@@MAE@XZ 10012400 f i format.obj
 0001:00011410       ??1locale@std@@QAE@XZ      10012410 f i format.obj
 0001:00011430       ??Ddetail@v6@fmt@@YA?AVfp@012@V3012@0@Z 10012430 f i format.obj
 0001:00011470       ??_3bigint@detail@v6@fmt@@QAEAAV0123@H@Z 10012470 f i format.obj
 0001:00011520       ??_E?$basic_memory_buffer@D$0BPE@V?$allocator@D@std@@@v6@fmt@@UAEPAXI@Z 10012520 f i format.obj
 0001:00011520       ??_G?$basic_memory_buffer@D$0BPE@V?$allocator@D@std@@@v6@fmt@@UAEPAXI@Z 10012520 f i format.obj
 0001:00011580       ??_G?$basic_memory_buffer@I$0CA@V?$allocator@I@std@@@v6@fmt@@UAEPAXI@Z 10012580 f i format.obj
 0001:00011580       ??_E?$basic_memory_buffer@I$0CA@V?$allocator@I@std@@@v6@fmt@@UAEPAXI@Z 10012580 f i format.obj
 0001:000115e0       ??_G?$basic_memory_buffer@_W$0BPE@V?$allocator@_W@std@@@v6@fmt@@UAEPAXI@Z 100125e0 f i format.obj
 0001:000115e0       ??_E?$basic_memory_buffer@_W$0BPE@V?$allocator@_W@std@@@v6@fmt@@UAEPAXI@Z 100125e0 f i format.obj
 0001:00011640       ??_E?$numpunct@_W@std@@MAEPAXI@Z 10012640 f i format.obj
 0001:00011640       ??_G?$numpunct@_W@std@@MAEPAXI@Z 10012640 f i format.obj
 0001:00011690       ??_E_Facet_base@std@@UAEPAXI@Z 10012690 f i format.obj
 0001:00011690       ??_G_Facet_base@std@@UAEPAXI@Z 10012690 f i format.obj
 0001:000116c0       ??_Gbad_alloc@std@@UAEPAXI@Z 100126c0 f i format.obj
 0001:000116c0       ??_Eexception@std@@UAEPAXI@Z 100126c0 f i format.obj
 0001:000116c0       ??_Ebad_alloc@std@@UAEPAXI@Z 100126c0 f i format.obj
 0001:000116c0       ??_Gexception@std@@UAEPAXI@Z 100126c0 f i format.obj
 0001:000116c0       ??_Gruntime_error@std@@UAEPAXI@Z 100126c0 f i format.obj
 0001:000116c0       ??_Eruntime_error@std@@UAEPAXI@Z 100126c0 f i format.obj
 0001:000116c0       ??_Eformat_error@v6@fmt@@UAEPAXI@Z 100126c0 f i format.obj
 0001:000116c0       ??_Gbad_array_new_length@std@@UAEPAXI@Z 100126c0 f i format.obj
 0001:000116c0       ??_Ebad_array_new_length@std@@UAEPAXI@Z 100126c0 f i format.obj
 0001:000116c0       ??_Gformat_error@v6@fmt@@UAEPAXI@Z 100126c0 f i format.obj
 0001:000116f0       ?_Decref@facet@locale@std@@UAEPAV_Facet_base@3@XZ 100126f0 f i format.obj
 0001:00011710       ?_Incref@facet@locale@std@@UAEXXZ 10012710 f i format.obj
 0001:00011720       ?_Throw_bad_array_new_length@std@@YAXXZ 10012720 f i format.obj
 0001:00011740       ?_Xlen@?$basic_string@DU?$char_traits@D@std@@V?$allocator@D@2@@std@@CAXXZ 10012740 f i format.obj
 0001:00011740       ?_Xlen@?$basic_string@_WU?$char_traits@_W@std@@V?$allocator@_W@2@@std@@CAXXZ 10012740 f i format.obj
 0001:00011750       ?add_compare@detail@v6@fmt@@YAHABVbigint@123@00@Z 10012750 f i format.obj
 0001:000118f0       ?allocate@?$allocator@E@std@@QAEPAEI@Z 100128f0 f i perfthread.obj
 0001:000118f0       ?allocate@?$allocator@D@std@@QAEPADI@Z 100128f0 f i format.obj
 0001:00011940       ?allocate@?$allocator@_W@std@@QAEPA_WI@Z 10012940 f i format.obj
 0001:000119a0       ?assign@?$basic_string@DU?$char_traits@D@std@@V?$allocator@D@2@@std@@QAEAAV12@QBDI@Z 100129a0 f i format.obj
 0001:00011a90       ?assign@?$basic_string@_WU?$char_traits@_W@std@@V?$allocator@_W@2@@std@@QAEAAV12@QB_WI@Z 10012a90 f i format.obj
 0001:00011b90       ?assign@bigint@detail@v6@fmt@@QAEX_K@Z 10012b90 f i format.obj
 0001:00011be0       ?assign_pow10@bigint@detail@v6@fmt@@QAEXH@Z 10012be0 f i format.obj
 0001:00011cc0       ?compare@detail@v6@fmt@@YAHABVbigint@123@0@Z 10012cc0 f i format.obj
 0001:00011d60       ?count_digits@detail@v6@fmt@@YAH_K@Z 10012d60 f i format.obj
 0001:00011dd0       ?divmod_assign@bigint@detail@v6@fmt@@QAEHABV1234@@Z 10012dd0 f i format.obj
 0001:00011f30       ?do_decimal_point@?$numpunct@_W@std@@MBE_WXZ 10012f30 f i format.obj
 0001:00011f40       ?do_falsename@?$numpunct@_W@std@@MBE?AV?$basic_string@_WU?$char_traits@_W@std@@V?$allocator@_W@2@@2@XZ 10012f40 f i format.obj
 0001:00011f80       ?do_grouping@?$numpunct@_W@std@@MBE?AV?$basic_string@DU?$char_traits@D@std@@V?$allocator@D@2@@2@XZ 10012f80 f i format.obj
 0001:00011fc0       ?do_thousands_sep@?$numpunct@_W@std@@MBE_WXZ 10012fc0 f i format.obj
 0001:00011fd0       ?do_truename@?$numpunct@_W@std@@MBE?AV?$basic_string@_WU?$char_traits@_W@std@@V?$allocator@_W@2@@2@XZ 10012fd0 f i format.obj
 0001:00012010       ?fmt_snprintf@detail@v6@fmt@@YAHPADIPBDZZ 10013010 f i format.obj
 0001:00012040       ?get_cached_power@detail@v6@fmt@@YA?AVfp@123@HAAH@Z 10013040 f i format.obj
 0001:000120a0       ?get_round_direction@detail@v6@fmt@@YA?AW4round_direction@123@_K00@Z 100130a0 f i format.obj
 0001:00012150       ?grisu_count_digits@detail@v6@fmt@@YAHI@Z 10013150 f i format.obj
 0001:000121d0       ?grow@?$basic_memory_buffer@D$0BPE@V?$allocator@D@std@@@v6@fmt@@MAEXI@Z 100131d0 f i format.obj
 0001:00012290       ?grow@?$basic_memory_buffer@I$0CA@V?$allocator@I@std@@@v6@fmt@@MAEXI@Z 10013290 f i format.obj
 0001:00012360       ?grow@?$basic_memory_buffer@_W$0BPE@V?$allocator@_W@std@@@v6@fmt@@MAEXI@Z 10013360 f i format.obj
 0001:00012430       ?multiply@detail@v6@fmt@@YA_K_K0@Z 10013430 f i format.obj
 0001:000124b0       ?on_digit@grisu_shortest_handler@detail@v6@fmt@@QAE?AW4result@digits@234@D_K00H_N@Z 100134b0 f i format.obj
 0001:000126a0       ?on_error@error_handler@detail@v6@fmt@@QAEXPBD@Z 100136a0 f   format.obj
 0001:00012740       ?push_back@?$buffer@D@detail@v6@fmt@@QAEXABD@Z 10013740 f i format.obj
 0001:00012770       ?resize@?$buffer@D@detail@v6@fmt@@QAEXI@Z 10013770 f i format.obj
 0001:00012790       ?square@bigint@detail@v6@fmt@@QAEXXZ 10013790 f i format.obj
 0001:00012a60       ?what@exception@std@@UBEPBDXZ 10013a60 f i format.obj
 0001:00012a70       ___local_stdio_printf_options 10013a70 f i format.obj
 0001:00012a80       ??$?0V?$basic_string_view@_WU?$char_traits@_W@std@@@std@@X@?$basic_string@_WU?$char_traits@_W@std@@V?$allocator@_W@2@@std@@QAE@ABV?$basic_string_view@_WU?$char_traits@_W@std@@@1@ABV?$allocator@_W@1@@Z 10013a80 f i handles.obj
 0001:00012ab0       ??$?0V?$value@V?$basic_format_context@V?$back_insert_iterator@V?$buffer@_W@detail@v6@fmt@@@std@@_W@v6@fmt@@@detail@v6@fmt@@V0123@V0123@V0123@V0123@@?$arg_data@V?$value@V?$basic_format_context@V?$back_insert_iterator@V?$buffer@_W@detail@v6@fmt@@@std@@_W@v6@fmt@@@detail@v6@fmt@@_W$04$0A@@detail@v6@fmt@@QAE@ABV?$value@V?$basic_format_context@V?$back_insert_iterator@V?$buffer@_W@detail@v6@fmt@@@std@@_W@v6@fmt@@@123@0000@Z 10013ab0 f i handles.obj
 0001:00012b10       ??$?RH$0A@@?$arg_formatter_base@V?$back_insert_iterator@V?$buffer@_W@detail@v6@fmt@@@std@@_WUerror_handler@detail@v6@fmt@@@detail@v6@fmt@@QAE?AV?$back_insert_iterator@V?$buffer@_W@detail@v6@fmt@@@std@@H@Z 10013b10 f i handles.obj
 0001:00012b60       ??$copy_str@_WPBDPA_W$0A@@detail@v6@fmt@@YAPA_WPBD0PA_W@Z 10013b60 f i handles.obj
 0001:00012b90       ??$copy_str@_WPBDVcounting_iterator@detail@v6@fmt@@$0A@@detail@v6@fmt@@YA?AVcounting_iterator@012@PBD0V3012@@Z 10013b90 f i handles.obj
 0001:00012bc0       ??$fill@PA_W_W@detail@v6@fmt@@YAPA_WPA_WIABU?$fill_t@_W@012@@Z 10013bc0 f i handles.obj
 0001:00012c30       ??$fill_n@PA_WH_W@std@@YAPA_WPA_WHAB_W@Z 10013c30 f i handles.obj
 0001:00012c60       ??$format_decimal@_WI@detail@v6@fmt@@YA?AU?$format_decimal_result@PA_W@012@PA_WIH@Z 10013c60 f i handles.obj
 0001:00012cf0       ??$format_decimal@_W_K@detail@v6@fmt@@YA?AU?$format_decimal_result@PA_W@012@PA_W_KH@Z 10013cf0 f i handles.obj
 0001:00012e20       ??$format_uint@$03_WI@detail@v6@fmt@@YAPA_WPA_WIH_N@Z 10013e20 f i handles.obj
 0001:00012e70       ??$get_dynamic_spec@Vprecision_checker@detail@v6@fmt@@V?$basic_format_arg@V?$basic_format_context@V?$back_insert_iterator@V?$buffer@_W@detail@v6@fmt@@@std@@_W@v6@fmt@@@34@Uerror_handler@234@@detail@v6@fmt@@YAHV?$basic_format_arg@V?$basic_format_context@V?$back_insert_iterator@V?$buffer@_W@detail@v6@fmt@@@std@@_W@v6@fmt@@@12@Uerror_handler@012@@Z 10013e70 f i handles.obj
 0001:00012f40       ??$get_dynamic_spec@Vwidth_checker@detail@v6@fmt@@V?$basic_format_arg@V?$basic_format_context@V?$back_insert_iterator@V?$buffer@_W@detail@v6@fmt@@@std@@_W@v6@fmt@@@34@Uerror_handler@234@@detail@v6@fmt@@YAHV?$basic_format_arg@V?$basic_format_context@V?$back_insert_iterator@V?$buffer@_W@detail@v6@fmt@@@std@@_W@v6@fmt@@@12@Uerror_handler@012@@Z 10013f40 f i handles.obj
 0001:00013010       ??$get_id@_W@?$basic_format_args@V?$basic_format_context@V?$back_insert_iterator@V?$buffer@_W@detail@v6@fmt@@@std@@_W@v6@fmt@@@v6@fmt@@QBEHV?$basic_string_view@_W@12@@Z 10014010 f i handles.obj
 0001:00013120       ??$handle_int_type_spec@AAU?$int_writer@V?$back_insert_iterator@V?$buffer@_W@detail@v6@fmt@@@std@@_WI@detail@v6@fmt@@@detail@v6@fmt@@YAXDAAU?$int_writer@V?$back_insert_iterator@V?$buffer@_W@detail@v6@fmt@@@std@@_WI@012@@Z 10014120 f i handles.obj
 0001:00013400       ??$handle_int_type_spec@AAU?$int_writer@V?$back_insert_iterator@V?$buffer@_W@detail@v6@fmt@@@std@@_W_K@detail@v6@fmt@@@detail@v6@fmt@@YAXDAAU?$int_writer@V?$back_insert_iterator@V?$buffer@_W@detail@v6@fmt@@@std@@_W_K@012@@Z 10014400 f i handles.obj
 0001:00013700       ??$is_name_start@_W@detail@v6@fmt@@YA_N_W@Z 10014700 f i handles.obj
 0001:00013740       ??$parse_arg_id@_WAAU?$id_adapter@AAU?$format_handler@V?$arg_formatter@V?$back_insert_iterator@V?$buffer@_W@detail@v6@fmt@@@std@@_W@detail@v6@fmt@@_WV?$basic_format_context@V?$back_insert_iterator@V?$buffer@_W@detail@v6@fmt@@@std@@_W@34@@detail@v6@fmt@@_W@detail@v6@fmt@@@detail@v6@fmt@@YAPB_WPB_W0AAU?$id_adapter@AAU?$format_handler@V?$arg_formatter@V?$back_insert_iterator@V?$buffer@_W@detail@v6@fmt@@@std@@_W@detail@v6@fmt@@_WV?$basic_format_context@V?$back_insert_iterator@V?$buffer@_W@detail@v6@fmt@@@std@@_W@34@@detail@v6@fmt@@_W@012@@Z 10014740 f i handles.obj
 0001:00013900       ??$parse_arg_id@_WU?$precision_adapter@AAV?$specs_checker@V?$specs_handler@V?$basic_format_parse_context@_WUerror_handler@detail@v6@fmt@@@v6@fmt@@V?$basic_format_context@V?$back_insert_iterator@V?$buffer@_W@detail@v6@fmt@@@std@@_W@23@@detail@v6@fmt@@@detail@v6@fmt@@_W@detail@v6@fmt@@@detail@v6@fmt@@YAPB_WPB_W0$$QAU?$precision_adapter@AAV?$specs_checker@V?$specs_handler@V?$basic_format_parse_context@_WUerror_handler@detail@v6@fmt@@@v6@fmt@@V?$basic_format_context@V?$back_insert_iterator@V?$buffer@_W@detail@v6@fmt@@@std@@_W@23@@detail@v6@fmt@@@detail@v6@fmt@@_W@012@@Z 10014900 f i handles.obj
 0001:00013b60       ??$parse_arg_id@_WU?$width_adapter@AAV?$specs_checker@V?$specs_handler@V?$basic_format_parse_context@_WUerror_handler@detail@v6@fmt@@@v6@fmt@@V?$basic_format_context@V?$back_insert_iterator@V?$buffer@_W@detail@v6@fmt@@@std@@_W@23@@detail@v6@fmt@@@detail@v6@fmt@@_W@detail@v6@fmt@@@detail@v6@fmt@@YAPB_WPB_W0$$QAU?$width_adapter@AAV?$specs_checker@V?$specs_handler@V?$basic_format_parse_context@_WUerror_handler@detail@v6@fmt@@@v6@fmt@@V?$basic_format_context@V?$back_insert_iterator@V?$buffer@_W@detail@v6@fmt@@@std@@_W@23@@detail@v6@fmt@@@detail@v6@fmt@@_W@012@@Z 10014b60 f i handles.obj
 0001:00013dc0       ??$parse_float_type_spec@Uerror_handler@detail@v6@fmt@@_W@detail@v6@fmt@@YA?AUfloat_specs@012@ABU?$basic_format_specs@_W@12@$$QAUerror_handler@012@@Z 10014dc0 f i handles.obj
 0001:00013f20       ??$parse_format_specs@_WAAV?$specs_checker@V?$specs_handler@V?$basic_format_parse_context@_WUerror_handler@detail@v6@fmt@@@v6@fmt@@V?$basic_format_context@V?$back_insert_iterator@V?$buffer@_W@detail@v6@fmt@@@std@@_W@23@@detail@v6@fmt@@@detail@v6@fmt@@@detail@v6@fmt@@YAPB_WPB_W0AAV?$specs_checker@V?$specs_handler@V?$basic_format_parse_context@_WUerror_handler@detail@v6@fmt@@@v6@fmt@@V?$basic_format_context@V?$back_insert_iterator@V?$buffer@_W@detail@v6@fmt@@@std@@_W@23@@detail@v6@fmt@@@012@@Z 10014f20 f i handles.obj
 0001:000142c0       ??$parse_format_string@$0A@_WAAU?$format_handler@V?$arg_formatter@V?$back_insert_iterator@V?$buffer@_W@detail@v6@fmt@@@std@@_W@detail@v6@fmt@@_WV?$basic_format_context@V?$back_insert_iterator@V?$buffer@_W@detail@v6@fmt@@@std@@_W@34@@detail@v6@fmt@@@detail@v6@fmt@@YAXV?$basic_string_view@_W@12@AAU?$format_handler@V?$arg_formatter@V?$back_insert_iterator@V?$buffer@_W@detail@v6@fmt@@@std@@_W@detail@v6@fmt@@_WV?$basic_format_context@V?$back_insert_iterator@V?$buffer@_W@detail@v6@fmt@@@std@@_W@34@@012@@Z 100152c0 f i handles.obj
 0001:00014540       ??$parse_nonnegative_int@_WAAV?$specs_checker@V?$specs_handler@V?$basic_format_parse_context@_WUerror_handler@detail@v6@fmt@@@v6@fmt@@V?$basic_format_context@V?$back_insert_iterator@V?$buffer@_W@detail@v6@fmt@@@std@@_W@23@@detail@v6@fmt@@@detail@v6@fmt@@@detail@v6@fmt@@YAHAAPB_WPB_WAAV?$specs_checker@V?$specs_handler@V?$basic_format_parse_context@_WUerror_handler@detail@v6@fmt@@@v6@fmt@@V?$basic_format_context@V?$back_insert_iterator@V?$buffer@_W@detail@v6@fmt@@@std@@_W@23@@detail@v6@fmt@@@012@@Z 10015540 f i handles.obj
 0001:000145b0       ??$parse_replacement_field@_WAAU?$format_handler@V?$arg_formatter@V?$back_insert_iterator@V?$buffer@_W@detail@v6@fmt@@@std@@_W@detail@v6@fmt@@_WV?$basic_format_context@V?$back_insert_iterator@V?$buffer@_W@detail@v6@fmt@@@std@@_W@34@@detail@v6@fmt@@@detail@v6@fmt@@YAPB_WPB_W0AAU?$format_handler@V?$arg_formatter@V?$back_insert_iterator@V?$buffer@_W@detail@v6@fmt@@@std@@_W@detail@v6@fmt@@_WV?$basic_format_context@V?$back_insert_iterator@V?$buffer@_W@detail@v6@fmt@@@std@@_W@34@@012@@Z 100155b0 f i handles.obj
 0001:000148b0       ??$prettify@PA_W@?$float_writer@_W@detail@v6@fmt@@ABEPA_WPA_W@Z 100158b0 f i handles.obj
 0001:00014bc0       ??$prettify@Vcounting_iterator@detail@v6@fmt@@@?$float_writer@_W@detail@v6@fmt@@ABE?AVcounting_iterator@123@V4123@@Z 10015bc0 f i handles.obj
 0001:00014d70       ??$reserve@V?$buffer@_W@detail@v6@fmt@@$0A@@detail@v6@fmt@@YAPA_WV?$back_insert_iterator@V?$buffer@_W@detail@v6@fmt@@@std@@I@Z 10015d70 f i handles.obj
 0001:00014da0       ??$vformat@_W$0A@@detail@v6@fmt@@YA?AV?$basic_string@_WU?$char_traits@_W@std@@V?$allocator@_W@2@@std@@V?$basic_string_view@_W@12@V?$basic_format_args@V?$basic_format_context@V?$back_insert_iterator@V?$buffer@_W@detail@v6@fmt@@@std@@_W@v6@fmt@@@12@@Z 10015da0 f i handles.obj
 0001:00014f50       ??$visit_format_arg@U?$default_arg_formatter@V?$back_insert_iterator@V?$buffer@_W@detail@v6@fmt@@@std@@_W@detail@v6@fmt@@V?$basic_format_context@V?$back_insert_iterator@V?$buffer@_W@detail@v6@fmt@@@std@@_W@34@@v6@fmt@@YA?AV?$back_insert_iterator@V?$buffer@_W@detail@v6@fmt@@@std@@$$QAU?$default_arg_formatter@V?$back_insert_iterator@V?$buffer@_W@detail@v6@fmt@@@std@@_W@detail@01@ABV?$basic_format_arg@V?$basic_format_context@V?$back_insert_iterator@V?$buffer@_W@detail@v6@fmt@@@std@@_W@v6@fmt@@@01@@Z 10015f50 f i handles.obj
 0001:00015360       ??$visit_format_arg@V?$arg_formatter@V?$back_insert_iterator@V?$buffer@_W@detail@v6@fmt@@@std@@_W@detail@v6@fmt@@V?$basic_format_context@V?$back_insert_iterator@V?$buffer@_W@detail@v6@fmt@@@std@@_W@34@@v6@fmt@@YA?AV?$back_insert_iterator@V?$buffer@_W@detail@v6@fmt@@@std@@$$QAV?$arg_formatter@V?$back_insert_iterator@V?$buffer@_W@detail@v6@fmt@@@std@@_W@detail@01@ABV?$basic_format_arg@V?$basic_format_context@V?$back_insert_iterator@V?$buffer@_W@detail@v6@fmt@@@std@@_W@v6@fmt@@@01@@Z 10016360 f i handles.obj
 0001:000159d0       ??$write@_WV?$back_insert_iterator@V?$buffer@_W@detail@v6@fmt@@@std@@@detail@v6@fmt@@YA?AV?$back_insert_iterator@V?$buffer@_W@detail@v6@fmt@@@std@@V34@_N@Z 100169d0 f i handles.obj
 0001:00015a50       ??$write@_WV?$back_insert_iterator@V?$buffer@_W@detail@v6@fmt@@@std@@H$0A@@detail@v6@fmt@@YA?AV?$back_insert_iterator@V?$buffer@_W@detail@v6@fmt@@@std@@V34@H@Z 10016a50 f i handles.obj
 0001:00015af0       ??$write@_WV?$back_insert_iterator@V?$buffer@_W@detail@v6@fmt@@@std@@I$0A@@detail@v6@fmt@@YA?AV?$back_insert_iterator@V?$buffer@_W@detail@v6@fmt@@@std@@V34@I@Z 10016af0 f i handles.obj
 0001:00015b70       ??$write@_WV?$back_insert_iterator@V?$buffer@_W@detail@v6@fmt@@@std@@M$0A@@detail@v6@fmt@@YA?AV?$back_insert_iterator@V?$buffer@_W@detail@v6@fmt@@@std@@V34@M@Z 10016b70 f i handles.obj
 0001:00015d80       ??$write@_WV?$back_insert_iterator@V?$buffer@_W@detail@v6@fmt@@@std@@M$0A@@detail@v6@fmt@@YA?AV?$back_insert_iterator@V?$buffer@_W@detail@v6@fmt@@@std@@V34@MU?$basic_format_specs@_W@12@Vlocale_ref@012@@Z 10016d80 f i handles.obj
 0001:00016110       ??$write@_WV?$back_insert_iterator@V?$buffer@_W@detail@v6@fmt@@@std@@N$0A@@detail@v6@fmt@@YA?AV?$back_insert_iterator@V?$buffer@_W@detail@v6@fmt@@@std@@V34@N@Z 10017110 f i handles.obj
 0001:00016320       ??$write@_WV?$back_insert_iterator@V?$buffer@_W@detail@v6@fmt@@@std@@N$0A@@detail@v6@fmt@@YA?AV?$back_insert_iterator@V?$buffer@_W@detail@v6@fmt@@@std@@V34@NU?$basic_format_specs@_W@12@Vlocale_ref@012@@Z 10017320 f i handles.obj
 0001:000166a0       ??$write@_WV?$back_insert_iterator@V?$buffer@_W@detail@v6@fmt@@@std@@O$0A@@detail@v6@fmt@@YA?AV?$back_insert_iterator@V?$buffer@_W@detail@v6@fmt@@@std@@V34@O@Z 100176a0 f i handles.obj
 0001:000168b0       ??$write@_WV?$back_insert_iterator@V?$buffer@_W@detail@v6@fmt@@@std@@O$0A@@detail@v6@fmt@@YA?AV?$back_insert_iterator@V?$buffer@_W@detail@v6@fmt@@@std@@V34@OU?$basic_format_specs@_W@12@Vlocale_ref@012@@Z 100178b0 f i handles.obj
 0001:00016c30       ??$write@_WV?$back_insert_iterator@V?$buffer@_W@detail@v6@fmt@@@std@@_J$0A@@detail@v6@fmt@@YA?AV?$back_insert_iterator@V?$buffer@_W@detail@v6@fmt@@@std@@V34@_J@Z 10017c30 f i handles.obj
 0001:00016cd0       ??$write@_WV?$back_insert_iterator@V?$buffer@_W@detail@v6@fmt@@@std@@_K$0A@@detail@v6@fmt@@YA?AV?$back_insert_iterator@V?$buffer@_W@detail@v6@fmt@@@std@@V34@_K@Z 10017cd0 f i handles.obj
 0001:00016d40       ??$write@_W_WV?$back_insert_iterator@V?$buffer@_W@detail@v6@fmt@@@std@@@detail@v6@fmt@@YA?AV?$back_insert_iterator@V?$buffer@_W@detail@v6@fmt@@@std@@V34@V?$basic_string_view@_W@12@ABU?$basic_format_specs@_W@12@@Z 10017d40 f i handles.obj
 0001:00016e20       ??$write_bytes@_WV?$back_insert_iterator@V?$buffer@_W@detail@v6@fmt@@@std@@@detail@v6@fmt@@YA?AV?$back_insert_iterator@V?$buffer@_W@detail@v6@fmt@@@std@@V34@V?$basic_string_view@D@12@ABU?$basic_format_specs@_W@12@@Z 10017e20 f i handles.obj
 0001:00016ef0       ??$write_int@H@?$arg_formatter_base@V?$back_insert_iterator@V?$buffer@_W@detail@v6@fmt@@@std@@_WUerror_handler@detail@v6@fmt@@@detail@v6@fmt@@AAEXHABU?$basic_format_specs@_W@23@@Z 10017ef0 f i handles.obj
 0001:00016f80       ??$write_int@V?$back_insert_iterator@V?$buffer@_W@detail@v6@fmt@@@std@@_WV<lambda_3cb9797f7e4785a78c67c53b4b64b0db>@@@detail@v6@fmt@@YA?AV?$back_insert_iterator@V?$buffer@_W@detail@v6@fmt@@@std@@V34@HV?$basic_string_view@D@12@ABU?$basic_format_specs@_W@12@V<lambda_3cb9797f7e4785a78c67c53b4b64b0db>@@@Z 10017f80 f i handles.obj
 0001:000170d0       ??$write_int@V?$back_insert_iterator@V?$buffer@_W@detail@v6@fmt@@@std@@_WV<lambda_63b26e08b5d772b586c0f4f48ae81e4a>@@@detail@v6@fmt@@YA?AV?$back_insert_iterator@V?$buffer@_W@detail@v6@fmt@@@std@@V34@HV?$basic_string_view@D@12@ABU?$basic_format_specs@_W@12@V<lambda_63b26e08b5d772b586c0f4f48ae81e4a>@@@Z 100180d0 f i handles.obj
 0001:00017220       ??$write_int@V?$back_insert_iterator@V?$buffer@_W@detail@v6@fmt@@@std@@_WV<lambda_652de128f75b23e4a41da5a1d17302a7>@@@detail@v6@fmt@@YA?AV?$back_insert_iterator@V?$buffer@_W@detail@v6@fmt@@@std@@V34@HV?$basic_string_view@D@12@ABU?$basic_format_specs@_W@12@V<lambda_652de128f75b23e4a41da5a1d17302a7>@@@Z 10018220 f i handles.obj
 0001:000173b0       ??$write_int@V?$back_insert_iterator@V?$buffer@_W@detail@v6@fmt@@@std@@_WV<lambda_6a38311184ff557693c326f9086ad568>@@@detail@v6@fmt@@YA?AV?$back_insert_iterator@V?$buffer@_W@detail@v6@fmt@@@std@@V34@HV?$basic_string_view@D@12@ABU?$basic_format_specs@_W@12@V<lambda_6a38311184ff557693c326f9086ad568>@@@Z 100183b0 f i handles.obj
 0001:00017510       ??$write_int@V?$back_insert_iterator@V?$buffer@_W@detail@v6@fmt@@@std@@_WV<lambda_7259ddfa3fd8cc4c1b6a3353d9d283f4>@@@detail@v6@fmt@@YA?AV?$back_insert_iterator@V?$buffer@_W@detail@v6@fmt@@@std@@V34@HV?$basic_string_view@D@12@ABU?$basic_format_specs@_W@12@V<lambda_7259ddfa3fd8cc4c1b6a3353d9d283f4>@@@Z 10018510 f i handles.obj
 0001:00017660       ??$write_int@V?$back_insert_iterator@V?$buffer@_W@detail@v6@fmt@@@std@@_WV<lambda_cb0155f587328621b8aee03f8219f50d>@@@detail@v6@fmt@@YA?AV?$back_insert_iterator@V?$buffer@_W@detail@v6@fmt@@@std@@V34@HV?$basic_string_view@D@12@ABU?$basic_format_specs@_W@12@V<lambda_cb0155f587328621b8aee03f8219f50d>@@@Z 10018660 f i handles.obj
 0001:000177a0       ??$write_int@V?$back_insert_iterator@V?$buffer@_W@detail@v6@fmt@@@std@@_WV<lambda_cc6251dcb89ce1d8f4de28763bbd722c>@@@detail@v6@fmt@@YA?AV?$back_insert_iterator@V?$buffer@_W@detail@v6@fmt@@@std@@V34@HV?$basic_string_view@D@12@ABU?$basic_format_specs@_W@12@V<lambda_cc6251dcb89ce1d8f4de28763bbd722c>@@@Z 100187a0 f i handles.obj
 0001:000178e0       ??$write_int@V?$back_insert_iterator@V?$buffer@_W@detail@v6@fmt@@@std@@_WV<lambda_ce6c92d8068300cd238b81597b5afbca>@@@detail@v6@fmt@@YA?AV?$back_insert_iterator@V?$buffer@_W@detail@v6@fmt@@@std@@V34@HV?$basic_string_view@D@12@ABU?$basic_format_specs@_W@12@V<lambda_ce6c92d8068300cd238b81597b5afbca>@@@Z 100188e0 f i handles.obj
 0001:00017a40       ??$write_nonfinite@_WV?$back_insert_iterator@V?$buffer@_W@detail@v6@fmt@@@std@@@detail@v6@fmt@@YA?AV?$back_insert_iterator@V?$buffer@_W@detail@v6@fmt@@@std@@V34@_NABU?$basic_format_specs@_W@12@ABUfloat_specs@012@@Z 10018a40 f i handles.obj
 0001:00017b40       ??$write_padded@$01V?$back_insert_iterator@V?$buffer@_W@detail@v6@fmt@@@std@@_WV?$float_writer@_W@detail@v6@fmt@@@detail@v6@fmt@@YA?AV?$back_insert_iterator@V?$buffer@_W@detail@v6@fmt@@@std@@V34@ABU?$basic_format_specs@_W@12@IABV?$float_writer@_W@012@@Z 10018b40 f i handles.obj
 0001:00017bf0       ??$write_ptr@_WV?$back_insert_iterator@V?$buffer@_W@detail@v6@fmt@@@std@@I@detail@v6@fmt@@YA?AV?$back_insert_iterator@V?$buffer@_W@detail@v6@fmt@@@std@@V34@IPBU?$basic_format_specs@_W@12@@Z 10018bf0 f i handles.obj
 0001:00017ce0       ??0?$basic_string@_WU?$char_traits@_W@std@@V?$allocator@_W@2@@std@@QAE@ABV01@@Z 10018ce0 f i handles.obj
 0001:00017d70       ??0?$float_writer@_W@detail@v6@fmt@@QAE@PBDHHUfloat_specs@123@_W@Z 10018d70 f i handles.obj
 0001:00017df0       ??1?$scoped_lock@VPerfThread@@@std@@QAE@XZ 10018df0 f i handles.obj
 0001:00017e20       ??1?$unique_ptr@$$BY0A@DU?$default_delete@$$BY0A@D@std@@@std@@QAE@XZ 10018e20 f i handles.obj
 0001:00017e20       ??1?$unique_ptr@$$BY0A@_WU?$default_delete@$$BY0A@_W@std@@@std@@QAE@XZ 10018e20 f i handles.obj
 0001:00017e30       ??1?$unique_ptr@USYSTEM_HANDLE_INFORMATION@@Uvirtual_deleter@@@std@@QAE@XZ 10018e30 f i handles.obj
 0001:00017e50       ??1?$unique_ptr@XUfree_deleter@@@std@@QAE@XZ 10018e50 f i handles.obj
 0001:00017e50       ??1?$unique_ptr@UPluginPanelItem@@Ufree_deleter@@@std@@QAE@XZ 10018e50 f i Pclass.obj
 0001:00017e60       ??1?$unique_ptr@XUhandle_closer@@@std@@QAE@XZ 10018e60 f i handles.obj
 0001:00017e70       ??1?$unique_ptr@_WUlocal_deleter@@@std@@QAE@XZ 10018e70 f i handles.obj
 0001:00017e80       ??1DebugToken@@QAE@XZ      10018e80 f i handles.obj
 0001:00018190       ??Rwriter@?1???$parse_format_string@$0A@_WAAU?$format_handler@V?$arg_formatter@V?$back_insert_iterator@V?$buffer@_W@detail@v6@fmt@@@std@@_W@detail@v6@fmt@@_WV?$basic_format_context@V?$back_insert_iterator@V?$buffer@_W@detail@v6@fmt@@@std@@_W@34@@detail@v6@fmt@@@detail@v6@fmt@@YAXV?$basic_string_view@_W@23@AAU?$format_handler@V?$arg_formatter@V?$back_insert_iterator@V?$buffer@_W@detail@v6@fmt@@@std@@_W@detail@v6@fmt@@_WV?$basic_format_context@V?$back_insert_iterator@V?$buffer@_W@detail@v6@fmt@@@std@@_W@34@@123@@Z@QAEXPB_W2@Z 10019190 f i handles.obj
 0001:000188b0       ?PrintHandleInfo@@YA_NKPAX_NPAVPerfThread@@@Z 100198b0 f   handles.obj
 0001:00018de0       ?_Xran@?$basic_string_view@_WU?$char_traits@_W@std@@@std@@CAXXZ 10019de0 f i handles.obj
 0001:00018df0       ?append@?$basic_string@_WU?$char_traits@_W@std@@V?$allocator@_W@2@@std@@QAEAAV12@QB_WI@Z 10019df0 f i handles.obj
 0001:00018f70       ?compare@?$_WChar_traits@_W@std@@SAHQB_W0I@Z 10019f70 f i handles.obj
 0001:000190f0       ?get@?$basic_format_args@V?$basic_format_context@V?$back_insert_iterator@V?$buffer@_W@detail@v6@fmt@@@std@@_W@v6@fmt@@@v6@fmt@@QBE?AV?$basic_format_arg@V?$basic_format_context@V?$back_insert_iterator@V?$buffer@_W@detail@v6@fmt@@@std@@_W@v6@fmt@@@23@H@Z 1001a0f0 f i handles.obj
 0001:00019190       ?get_arg@?$specs_handler@V?$basic_format_parse_context@_WUerror_handler@detail@v6@fmt@@@v6@fmt@@V?$basic_format_context@V?$back_insert_iterator@V?$buffer@_W@detail@v6@fmt@@@std@@_W@23@@detail@v6@fmt@@AAE?AV?$basic_format_arg@V?$basic_format_context@V?$back_insert_iterator@V?$buffer@_W@detail@v6@fmt@@@std@@_W@v6@fmt@@@34@V?$basic_string_view@_W@34@@Z 1001a190 f i handles.obj
 0001:00019210       ?on_char@char_spec_handler@?$arg_formatter_base@V?$back_insert_iterator@V?$buffer@_W@detail@v6@fmt@@@std@@_WUerror_handler@detail@v6@fmt@@@detail@v6@fmt@@QAEXXZ 1001a210 f i handles.obj
 0001:000192f0       ?on_dec@?$int_writer@V?$back_insert_iterator@V?$buffer@_W@detail@v6@fmt@@@std@@_WI@detail@v6@fmt@@QAEXXZ 1001a2f0 f i handles.obj
 0001:00019350       ?on_dec@?$int_writer@V?$back_insert_iterator@V?$buffer@_W@detail@v6@fmt@@@std@@_W_K@detail@v6@fmt@@QAEXXZ 1001a350 f i handles.obj
 0001:00019390       ?on_fill@?$specs_setter@_W@detail@v6@fmt@@QAEXV?$basic_string_view@_W@34@@Z 1001a390 f i handles.obj
 0001:00019480       ?on_num@?$int_writer@V?$back_insert_iterator@V?$buffer@_W@detail@v6@fmt@@@std@@_WI@detail@v6@fmt@@QAEXXZ 1001a480 f i handles.obj
 0001:00019770       ?on_num@?$int_writer@V?$back_insert_iterator@V?$buffer@_W@detail@v6@fmt@@@std@@_W_K@detail@v6@fmt@@QAEXXZ 1001a770 f i handles.obj
 0001:00019a90       ?on_replacement_field@?$format_handler@V?$arg_formatter@V?$back_insert_iterator@V?$buffer@_W@detail@v6@fmt@@@std@@_W@detail@v6@fmt@@_WV?$basic_format_context@V?$back_insert_iterator@V?$buffer@_W@detail@v6@fmt@@@std@@_W@34@@detail@v6@fmt@@QAEXHPB_W@Z 1001aa90 f i handles.obj
 0001:00019b10       ?on_text@?$format_handler@V?$arg_formatter@V?$back_insert_iterator@V?$buffer@_W@detail@v6@fmt@@@std@@_W@detail@v6@fmt@@_WV?$basic_format_context@V?$back_insert_iterator@V?$buffer@_W@detail@v6@fmt@@@std@@_W@34@@detail@v6@fmt@@QAEXPB_W0@Z 1001ab10 f i handles.obj
 0001:00019c40       ?write@?$arg_formatter_base@V?$back_insert_iterator@V?$buffer@_W@detail@v6@fmt@@@std@@_WUerror_handler@detail@v6@fmt@@@detail@v6@fmt@@IAEXPB_W@Z 1001ac40 f i handles.obj
 0001:00019d70       ?write@?$arg_formatter_base@V?$back_insert_iterator@V?$buffer@_W@detail@v6@fmt@@@std@@_WUerror_handler@detail@v6@fmt@@@detail@v6@fmt@@IAEX_N@Z 1001ad70 f i handles.obj
 0001:00019ef0       ??0PluginDialogBuilder@@QAE@ABUPluginStartupInfo@@ABU_GUID@@1HPB_WP6GHPAXHH3@Z3_K@Z 1001aef0 f i Pcfg.obj
 0001:00019ff0       ??1PluginDialogBuilder@@QAE@XZ 1001aff0 f i Pcfg.obj
 0001:0001a060       ??1PluginSettings@@QAE@XZ  1001b060 f i Pcfg.obj
 0001:0001a0a0       ??_GPluginEditFieldBinding@@UAEPAXI@Z 1001b0a0 f i Pclass.obj
 0001:0001a0a0       ??_EPluginEditFieldBinding@@UAEPAXI@Z 1001b0a0 f i Pclass.obj
 0001:0001a0a0       ??_EPluginCheckBoxBinding@@UAEPAXI@Z 1001b0a0 f i Pcfg.obj
 0001:0001a0a0       ??_GPluginCheckBoxBinding@@UAEPAXI@Z 1001b0a0 f i Pcfg.obj
 0001:0001a0c0       ?AddButtons@PluginDialogBuilder@@QAEXHPBHHH@Z 1001b0c0 f i Pcfg.obj
 0001:0001a2f0       ?AddCheckbox@PluginDialogBuilder@@QAEPAUFarDialogItem@@HPAHH_N@Z 1001b2f0 f i Pcfg.obj
 0001:0001a3e0       ?AddDialogItem@PluginDialogBuilder@@AAEPAUFarDialogItem@@W4FARDIALOGITEMTYPES@@PB_W@Z 1001b3e0 f i Pcfg.obj
 0001:0001a500       ?Config@@YAHXZ             1001b500 f   Pcfg.obj
 0001:0001a810       ?ItemWidth@PluginDialogBuilder@@CAHABUFarDialogItem@@@Z 1001b810 f i Pcfg.obj
 0001:0001a870       ?Read@options@@QAEXXZ      1001b870 f   Pcfg.obj
 0001:0001ab70       ?SaveValue@PluginCheckBoxBinding@@UAEXPBUFarDialogItem@@H@Z 1001bb70 f i Pcfg.obj
 0001:0001abb0       ?ShowDialog@PluginDialogBuilder@@QAE_NXZ 1001bbb0 f i Pcfg.obj
 0001:0001abe0       ?ShowDialogEx@PluginDialogBuilder@@QAEHXZ 1001bbe0 f i Pcfg.obj
 0001:0001ae30       ?Write@options@@QBEXXZ     1001be30 f   Pcfg.obj
 0001:0001b050       ??$?H_WU?$char_traits@_W@std@@V?$allocator@_W@1@@std@@YA?AV?$basic_string@_WU?$char_traits@_W@std@@V?$allocator@_W@2@@0@ABV10@$$QAV10@@Z 1001c050 f i Pclass.obj
 0001:0001b0c0       ??$_Assign_range@PBUmode@@@?$vector@Umode@@V?$allocator@Umode@@@std@@@std@@AAEXPBUmode@@0Uforward_iterator_tag@1@@Z 1001c0c0 f i Pclass.obj
 0001:0001b290       ??$_Copy_unchecked@PBUmode@@PAU1@@std@@YAPAUmode@@PBU1@0PAU1@@Z 1001c290 f i Pclass.obj
 0001:0001b2f0       ??$_Destroy_range@V?$allocator@V?$basic_string@_WU?$char_traits@_W@std@@V?$allocator@_W@2@@std@@@std@@@std@@YAXPAV?$basic_string@_WU?$char_traits@_W@std@@V?$allocator@_W@2@@0@QAV10@AAV?$allocator@V?$basic_string@_WU?$char_traits@_W@std@@V?$allocator@_W@2@@std@@@0@@Z 1001c2f0 f i Pclass.obj
 0001:0001b360       ??$_Emplace_reallocate@V?$basic_string@_WU?$char_traits@_W@std@@V?$allocator@_W@2@@std@@@?$vector@V?$basic_string@_WU?$char_traits@_W@std@@V?$allocator@_W@2@@std@@V?$allocator@V?$basic_string@_WU?$char_traits@_W@std@@V?$allocator@_W@2@@std@@@2@@std@@QAEPAV?$basic_string@_WU?$char_traits@_W@std@@V?$allocator@_W@2@@1@QAV21@$$QAV21@@Z 1001c360 f i Pclass.obj
 0001:0001b550       ??$_Find_last@K@?$_Hash@V?$_Umap_traits@KPAUHWND__@@V?$_Uhash_compare@KU?$hash@K@std@@U?$equal_to@K@2@@std@@V?$allocator@U?$pair@$$CBKPAUHWND__@@@std@@@3@$0A@@std@@@std@@IBE?AU?$_Hash_find_last_result@PAU?$_List_node@U?$pair@$$CBKPAUHWND__@@@std@@PAX@std@@@1@ABKI@Z 1001c550 f i Pclass.obj
 0001:0001b5c0       ??$_Resize_reallocate@U_Value_init_tag@std@@@?$vector@PB_WV?$allocator@PB_W@std@@@std@@AAEXIABU_Value_init_tag@1@@Z 1001c5c0 f i Pclass.obj
 0001:0001b6e0       ??$_Try_emplace@ABK$$V@?$_Hash@V?$_Umap_traits@KPAUHWND__@@V?$_Uhash_compare@KU?$hash@K@std@@U?$equal_to@K@2@@std@@V?$allocator@U?$pair@$$CBKPAUHWND__@@@std@@@3@$0A@@std@@@std@@IAE?AU?$pair@PAU?$_List_node@U?$pair@$$CBKPAUHWND__@@@std@@PAX@std@@_N@1@ABK@Z 1001c6e0 f i Pclass.obj
 0001:0001b8e0       ??$_Uninitialized_move@PAV?$basic_string@_WU?$char_traits@_W@std@@V?$allocator@_W@2@@std@@V?$allocator@V?$basic_string@_WU?$char_traits@_W@std@@V?$allocator@_W@2@@std@@@2@@std@@YAPAV?$basic_string@_WU?$char_traits@_W@std@@V?$allocator@_W@2@@0@QAV10@0PAV10@AAV?$allocator@V?$basic_string@_WU?$char_traits@_W@std@@V?$allocator@_W@2@@std@@@0@@Z 1001c8e0 f i Pclass.obj
 0001:0001b970       ??$format@PB_WAAPB_W@@YA?AV?$basic_string@_WU?$char_traits@_W@std@@V?$allocator@_W@2@@std@@$$QAPB_WAAPB_W@Z 1001c970 f i Pclass.obj
 0001:0001b9d0       ??$make_unique@VPerfThread@@$$V$0A@@std@@YA?AV?$unique_ptr@VPerfThread@@U?$default_delete@VPerfThread@@@std@@@0@XZ 1001c9d0 f i Pclass.obj
 0001:0001ba40       ??0?$basic_string@_WU?$char_traits@_W@std@@V?$allocator@_W@2@@std@@QAE@$$QAV01@@Z 1001ca40 f i Pclass.obj
 0001:0001ba90       ??0Plist@@QAE@XZ           1001ca90 f   Pclass.obj
 0001:0001bc70       ??1?$_List_node_emplace_op2@V?$allocator@U?$_List_node@U?$pair@$$CBKPAUHWND__@@@std@@PAX@std@@@std@@@std@@QAE@XZ 1001cc70 f i Pclass.obj
 0001:0001bc70       ??1?$_Alloc_construct_ptr@V?$allocator@U?$_List_node@U?$pair@$$CBKPAUHWND__@@@std@@PAX@std@@@std@@@std@@QAE@XZ 1001cc70 f i Pclass.obj
 0001:0001bc90       ??1?$_Hash@V?$_Umap_traits@KPAUHWND__@@V?$_Uhash_compare@KU?$hash@K@std@@U?$equal_to@K@2@@std@@V?$allocator@U?$pair@$$CBKPAUHWND__@@@std@@@3@$0A@@std@@@std@@QAE@XZ 1001cc90 f i Pclass.obj
 0001:0001bd20       ??1?$_Hash_vec@V?$allocator@V?$_List_unchecked_iterator@V?$_List_val@U?$_List_simple_types@U?$pair@$$CBKPAUHWND__@@@std@@@std@@@std@@@std@@@std@@@std@@QAE@XZ 1001cd20 f i Pclass.obj
 0001:0001bd70       ??1?$_Uninitialized_backout_al@V?$allocator@Umode@@@std@@@std@@QAE@XZ 1001cd70 f i Pclass.obj
 0001:0001bda0       ??1?$list@U?$pair@$$CBKPAUHWND__@@@std@@V?$allocator@U?$pair@$$CBKPAUHWND__@@@std@@@2@@std@@QAE@XZ 1001cda0 f i Pclass.obj
 0001:0001bde0       ??1?$pair@KV?$basic_string@_WU?$char_traits@_W@std@@V?$allocator@_W@2@@std@@@std@@QAE@XZ 1001cde0 f i Pclass.obj
 0001:0001bde0       ??1?$pair@JV?$basic_string@_WU?$char_traits@_W@std@@V?$allocator@_W@2@@std@@@std@@QAE@XZ 1001cde0 f i Pclass.obj
 0001:0001be40       ??1?$unique_ptr@VPerfThread@@U?$default_delete@VPerfThread@@@std@@@std@@QAE@XZ 1001ce40 f i Pclass.obj
 0001:0001be60       ??1?$unique_ptr@VWMIConnection@@U?$default_delete@VWMIConnection@@@std@@@std@@QAE@XZ 1001ce60 f i Pclass.obj
 0001:0001be80       ??1?$unordered_map@KPAUHWND__@@U?$hash@K@std@@U?$equal_to@K@3@V?$allocator@U?$pair@$$CBKPAUHWND__@@@std@@@3@@std@@QAE@XZ 1001ce80 f i Pclass.obj
 0001:0001be90       ??1?$vector@UFarMenuItem@@V?$allocator@UFarMenuItem@@@std@@@std@@QAE@XZ 1001ce90 f i Pclass.obj
 0001:0001bef0       ??1?$vector@V?$basic_string@_WU?$char_traits@_W@std@@V?$allocator@_W@2@@std@@V?$allocator@V?$basic_string@_WU?$char_traits@_W@std@@V?$allocator@_W@2@@std@@@2@@std@@QAE@XZ 1001cef0 f i Pclass.obj
 0001:0001bf00       ??1Plist@@QAE@XZ           1001cf00 f   Pclass.obj
 0001:0001bfe0       ??1ProcessData@@QAE@XZ     1001cfe0 f i Pclass.obj
 0001:0001c080       ??1StrTok@@QAE@XZ          1001d080 f i Pclass.obj
 0001:0001c090       ??4?$basic_string@_WU?$char_traits@_W@std@@V?$allocator@_W@2@@std@@QAEAAV01@$$QAV01@@Z 1001d090 f i Pclass.obj
 0001:0001c130       ??4?$basic_string@_WU?$char_traits@_W@std@@V?$allocator@_W@2@@std@@QAEAAV01@QB_W@Z 1001d130 f i Pclass.obj
 0001:0001c160       ??4columns@@QAEAAU0@ABU0@@Z 1001d160 f i Pclass.obj
 0001:0001c1c0       ?AddEditField@PluginDialogBuilder@@QAEPAUFarDialogItem@@PA_WHHPB_W_N@Z 1001d1c0 f i Pclass.obj
 0001:0001c2a0       ?Compare@Plist@@QBEHPBUPluginPanelItem@@0I@Z 1001d2a0 f   Pclass.obj
 0001:0001c470       ?Connect@Plist@@QAE_NPB_W00@Z 1001d470 f   Pclass.obj
 0001:0001c6f0       ?ConnectWMI@Plist@@AAE_NXZ 1001d6f0 f   Pclass.obj
 0001:0001c810       ?DeleteFiles@Plist@@QAEHPAUPluginPanelItem@@I_K@Z 1001d810 f   Pclass.obj
 0001:0001cd60       ?DumpNTCounters@@YAXPAXAAVPerfThread@@KK@Z 1001dd60 f   Pclass.obj
 0001:0001d310       ?DurationToText@@YA?AV?$basic_string@_WU?$char_traits@_W@std@@V?$allocator@_W@2@@std@@_K@Z 1001e310 f   Pclass.obj
 0001:0001d470       ?EnumWndProc@@YGHPAUHWND__@@J@Z 1001e470 f   Pclass.obj
 0001:0001d540       ?FreeFindData@Plist@@SAXPAUPluginPanelItem@@I@Z 1001e540 f   Pclass.obj
 0001:0001d610       ?GetFiles@Plist@@QAEHPAUPluginPanelItem@@IHPAPB_W_KAAUoptions@@@Z 1001e610 f   Pclass.obj
 0001:0001eef0       ?GetFindData@Plist@@QAEHAAPAUPluginPanelItem@@AAI_K@Z 1001fef0 f   Pclass.obj
 0001:0001fb10       ?GetOpenPanelInfo@Plist@@QAEXPAUOpenPanelInfo@@@Z 10020b10 f   Pclass.obj
 0001:0001fde0       ?GetVersionInfo@Plist@@SA_NPB_WAAV?$unique_ptr@$$BY0A@DU?$default_delete@$$BY0A@D@std@@@std@@AAPB_W2@Z 10020de0 f   Pclass.obj
 0001:00020110       ?InitializePanelModes@Plist@@SAXXZ 10021110 f   Pclass.obj
 0001:00021690       ?PrintOwnerInfo@Plist@@AAEXPAXK@Z 10022690 f   Pclass.obj
 0001:00021a60       ?PrintVersionInfo@Plist@@CAXPAXPB_W@Z 10022a60 f   Pclass.obj
 0001:00021c10       ?ProcessEvent@Plist@@QAEHHPAX@Z 10022c10 f   Pclass.obj
 0001:00021db0       ?ProcessKey@Plist@@QAEHPBU_INPUT_RECORD@@@Z 10022db0 f   Pclass.obj
 0001:00023500       ?Reread@Plist@@AAEXXZ      10024500 f   Pclass.obj
 0001:00023580       ?SavePanelModes@Plist@@SAXXZ 10024580 f   Pclass.obj
 0001:00023880       ?SaveValue@PluginEditFieldBinding@@UAEXPBUFarDialogItem@@H@Z 10024880 f i Pclass.obj
 0001:00024080       ?_Assign_grow@?$_Hash_vec@V?$allocator@V?$_List_unchecked_iterator@V?$_List_val@U?$_List_simple_types@U?$pair@$$CBKPAUHWND__@@@std@@@std@@@std@@@std@@@std@@@std@@QAEXIV?$_List_unchecked_iterator@V?$_List_val@U?$_List_simple_types@U?$pair@$$CBKPAUHWND__@@@std@@@std@@@std@@@2@@Z 10025080 f i Pclass.obj
 0001:00024170       ?_Clear_and_reserve_geometric@?$vector@Umode@@V?$allocator@Umode@@@std@@@std@@AAEXI@Z 10025170 f i Pclass.obj
 0001:000242b0       ?_Forced_rehash@?$_Hash@V?$_Umap_traits@KPAUHWND__@@V?$_Uhash_compare@KU?$hash@K@std@@U?$equal_to@K@2@@std@@V?$allocator@U?$pair@$$CBKPAUHWND__@@@std@@@3@$0A@@std@@@std@@IAEXI@Z 100252b0 f i Pclass.obj
 0001:00024410       ?_Tidy@?$vector@V?$basic_string@_WU?$char_traits@_W@std@@V?$allocator@_W@2@@std@@V?$allocator@V?$basic_string@_WU?$char_traits@_W@std@@V?$allocator@_W@2@@std@@@2@@std@@AAEXXZ 10025410 f i Pclass.obj
 0001:00024490       ?_Xlength@?$vector@Umode@@V?$allocator@Umode@@@std@@@std@@CAXXZ 10025490 f i Pclass.obj
 0001:00024490       ?_Xlength@?$vector@PB_WV?$allocator@PB_W@std@@@std@@CAXXZ 10025490 f i Pclass.obj
 0001:00024490       ?_Xlength@?$vector@_WV?$allocator@_W@std@@@std@@CAXXZ 10025490 f i perfthread.obj
 0001:00024490       ?_Xlength@?$vector@PAUHINSTANCE__@@V?$allocator@PAUHINSTANCE__@@@std@@@std@@CAXXZ 10025490 f i Plist.obj
 0001:00024490       ?_Xlength@?$vector@EV?$allocator@E@std@@@std@@CAXXZ 10025490 f i perfthread.obj
 0001:00024490       ?_Xlength@?$vector@V?$basic_string@_WU?$char_traits@_W@std@@V?$allocator@_W@2@@std@@V?$allocator@V?$basic_string@_WU?$char_traits@_W@std@@V?$allocator@_W@2@@std@@@2@@std@@CAXXZ 10025490 f i Pclass.obj
 0001:00024490       ?_Xlength@?$vector@UProcessPerfData@@V?$allocator@UProcessPerfData@@@std@@@std@@CAXXZ 10025490 f i perfthread.obj
 0001:000244a0       ?_Xran@?$_String_val@U?$_Simple_types@_W@std@@@std@@SAXXZ 100254a0 f i Pclass.obj
 0001:000244b0       ?append@?$basic_string@_WU?$char_traits@_W@std@@V?$allocator@_W@2@@std@@QAEAAV12@I_W@Z 100254b0 f i Pclass.obj
 0001:00024670       ?clear@?$basic_string@_WU?$char_traits@_W@std@@V?$allocator@_W@2@@std@@QAEXXZ 10025670 f i Pclass.obj
 0001:00024990       ?insert@?$basic_string@_WU?$char_traits@_W@std@@V?$allocator@_W@2@@std@@QAEAAV12@IQB_WI@Z 10025990 f i Pclass.obj
 0001:00024bc0       ?make@custom_data@@SA@$$QAV?$vector@V?$basic_string@_WU?$char_traits@_W@std@@V?$allocator@_W@2@@std@@V?$allocator@V?$basic_string@_WU?$char_traits@_W@std@@V?$allocator@_W@2@@std@@@2@@std@@@Z 10025bc0 f i Pclass.obj
 0001:00025930       ??$_Resize_reallocate@U_Value_init_tag@std@@@?$vector@EV?$allocator@E@std@@@std@@AAEXIABU_Value_init_tag@1@@Z 10026930 f i perfthread.obj
 0001:000259f0       ??0?$vector@UProcessPerfData@@V?$allocator@UProcessPerfData@@@std@@@std@@QAE@IABV?$allocator@UProcessPerfData@@@1@@Z 100269f0 f i perfthread.obj
 0001:00025bb0       ??0PerfThread@@QAE@PB_W00@Z 10026bb0 f   perfthread.obj
 0001:000264d0       ??1?$_Tidy_guard@V?$vector@UProcessPerfData@@V?$allocator@UProcessPerfData@@@std@@@std@@@std@@QAE@XZ 100274d0 f i perfthread.obj
 0001:000264e0       ??1?$_Uninitialized_backout_al@V?$allocator@UProcessPerfData@@@std@@@std@@QAE@XZ 100274e0 f i perfthread.obj
 0001:00026510       ??1?$vector@EV?$allocator@E@std@@@std@@QAE@XZ 10027510 f i perfthread.obj
 0001:00026560       ??1?$vector@UProcessPerfData@@V?$allocator@UProcessPerfData@@@std@@@std@@QAE@XZ 10027560 f i perfthread.obj
 0001:00026570       ??1?$vector@_WV?$allocator@_W@std@@@std@@QAE@XZ 10027570 f i perfthread.obj
 0001:000265d0       ??1PerfThread@@QAE@XZ      100275d0 f   perfthread.obj
 0001:000267b0       ??1ProcessPerfData@@QAE@XZ 100277b0 f i perfthread.obj
 0001:00026930       ??1RegKey@@QAE@XZ          10027930 f i perfthread.obj
 0001:00026940       ?GetProcessData@PerfThread@@QAEPAUProcessPerfData@@KK@Z 10027940 f   perfthread.obj
 0001:00026a20       ?Refresh@PerfThread@@AAEXXZ 10027a20 f   perfthread.obj
 0001:00027510       ?RefreshWMIData@PerfThread@@AAEXXZ 10028510 f   perfthread.obj
 0001:000279b0       ?SyncReread@PerfThread@@QAEXXZ 100289b0 f   perfthread.obj
 0001:000279e0       ?ThreadProc@PerfThread@@CGKPAX@Z 100289e0 f   perfthread.obj
 0001:00027ac0       ?_Tidy@?$vector@UProcessPerfData@@V?$allocator@UProcessPerfData@@@std@@@std@@AAEXXZ 10028ac0 f i perfthread.obj
 0001:00027b50       ?lock@PerfThread@@QAEXXZ   10028b50 f   perfthread.obj
 0001:00027b60       ?unlock@PerfThread@@QAEXXZ 10028b60 f   perfthread.obj
 0001:00027b70       ??$_Resize_reallocate@U_Value_init_tag@std@@@?$vector@PAUHINSTANCE__@@V?$allocator@PAUHINSTANCE__@@@std@@@std@@AAEXIABU_Value_init_tag@1@@Z 10028b70 f i Plist.obj
 0001:00027d90       ??0?$basic_string@_WU?$char_traits@_W@std@@V?$allocator@_W@2@@std@@QAE@I_W@Z 10028d90 f i Plist.obj
 0001:00027e50       ??0?$vector@UProcessPerfData@@V?$allocator@UProcessPerfData@@@std@@@std@@QAE@ABV01@@Z 10028e50 f i Plist.obj
 0001:00028090       ??1?$function@$$A6A_NPA_WI@Z@std@@QAE@XZ 10029090 f i Plist.obj
 0001:00028090       ??1?$function@$$A6AXABUtagVARIANT@@@Z@std@@QAE@XZ 10029090 f i WMI.obj
 0001:000280c0       ??1?$vector@PAUHINSTANCE__@@V?$allocator@PAUHINSTANCE__@@@std@@@std@@QAE@XZ 100290c0 f i Plist.obj
 0001:00028190       ?CreateToken@DebugToken@@SA_NXZ 10029190 f   Plist.obj
 0001:00028250       ?Enable@DebugToken@@QAE_NXZ 10029250 f   Plist.obj
 0001:000283a0       ?GetInternalProcessData@?$ipc_functions@$00@@SA_NPAXPAULDR_MODULE_64@detail@@AA_K2_N@Z 100293a0 f i Plist.obj
 0001:000284f0       ?GetInternalProcessData@?$ipc_functions@$0A@@@SA_NPAXPAULDR_MODULE_SAME@detail@@AAPBD2_N@Z 100294f0 f i Plist.obj
 0001:000285d0       ?GetList@@YA_NAAPAUPluginPanelItem@@AAIAAVPerfThread@@@Z 100295d0 f   Plist.obj
 0001:00028970       ?GetOpenProcessData@?$ipc_functions@$00@@SAXPAXPAV?$basic_string@_WU?$char_traits@_W@std@@V?$allocator@_W@2@@std@@1111@Z 10029970 f i Plist.obj
 0001:00028bc0       ?GetOpenProcessData@?$ipc_functions@$0A@@@SAXPAXPAV?$basic_string@_WU?$char_traits@_W@std@@V?$allocator@_W@2@@std@@1111@Z 10029bc0 f i Plist.obj
 0001:00028dd0       ?GetOpenProcessData@@YAXPAXPAV?$basic_string@_WU?$char_traits@_W@std@@V?$allocator@_W@2@@std@@1111@Z 10029dd0 f   Plist.obj
 0001:00028e70       ?GetPData@@YA_NAAUProcessData@@ABUProcessPerfData@@@Z 10029e70 f   Plist.obj
 0001:00029030       ?KillProcess@@YA_NKPAUHWND__@@@Z 1002a030 f   Plist.obj
 0001:000291a0       ?OpenProcessForced@@YAPAXPAVDebugToken@@KKH@Z 1002a1a0 f   Plist.obj
 0001:000291f0       ?PrintModules@?$ipc_functions@$00@@SAXPAX0AAUoptions@@@Z 1002a1f0 f i Plist.obj
 0001:000293f0       ?PrintModules@?$ipc_functions@$0A@@@SAXPAX0AAUoptions@@@Z 1002a3f0 f i Plist.obj
 0001:000294e0       ?PrintModules@@YAXPAXKAAUoptions@@@Z 1002a4e0 f   Plist.obj
 0001:000298c0       ?PrintNTCurDirAndEnv@@YAXPAX0H@Z 1002a8c0 f   Plist.obj
 0001:00029c10       ?Revert@DebugToken@@QAE_NXZ 1002ac10 f   Plist.obj
 0001:00029c70       ?_Move@?$_Func_impl_no_alloc@V<lambda_7407d5cd5d4425cb98b7ee1223d84907>@@_NPA_WI@std@@EAEPAV?$_Func_base@_NPA_WI@2@PAX@Z 1002ac70 f i Plist.obj
 0001:00029c70       ?_Copy@?$_Func_impl_no_alloc@V<lambda_7407d5cd5d4425cb98b7ee1223d84907>@@_NPA_WI@std@@EBEPAV?$_Func_base@_NPA_WI@2@PAX@Z 1002ac70 f i Plist.obj
 0001:00029c90       ?_Move@?$_Func_impl_no_alloc@V<lambda_ca95615ebb3c7b16132ff39b7c245039>@@_NPA_WI@std@@EAEPAV?$_Func_base@_NPA_WI@2@PAX@Z 1002ac90 f i Plist.obj
 0001:00029c90       ?_Copy@?$_Func_impl_no_alloc@V<lambda_ca95615ebb3c7b16132ff39b7c245039>@@_NPA_WI@std@@EBEPAV?$_Func_base@_NPA_WI@2@PAX@Z 1002ac90 f i Plist.obj
 0001:00029cb0       ?_Delete_this@?$_Func_impl_no_alloc@V<lambda_7407d5cd5d4425cb98b7ee1223d84907>@@_NPA_WI@std@@EAEX_N@Z 1002acb0 f   Plist.obj
 0001:00029cb0       ?_Delete_this@?$_Func_impl_no_alloc@V<lambda_ca95615ebb3c7b16132ff39b7c245039>@@_NPA_WI@std@@EAEX_N@Z 1002acb0 f   Plist.obj
 0001:00029d00       ?_Do_call@?$_Func_impl_no_alloc@V<lambda_7407d5cd5d4425cb98b7ee1223d84907>@@_NPA_WI@std@@EAE_N$$QAPA_W$$QAI@Z 1002ad00 f i Plist.obj
 0001:00029d60       ?_Do_call@?$_Func_impl_no_alloc@V<lambda_ca95615ebb3c7b16132ff39b7c245039>@@_NPA_WI@std@@EAE_N$$QAPA_W$$QAI@Z 1002ad60 f i Plist.obj
 0001:00029da0       ?_Get@?$_Func_impl_no_alloc@V<lambda_7407d5cd5d4425cb98b7ee1223d84907>@@_NPA_WI@std@@EBEPBXXZ 1002ada0 f   Plist.obj
 0001:00029da0       ?_Get@?$_Func_impl_no_alloc@V<lambda_ca95615ebb3c7b16132ff39b7c245039>@@_NPA_WI@std@@EBEPBXXZ 1002ada0 f   Plist.obj
 0001:00029dc0       ?_Target_type@?$_Func_impl_no_alloc@V<lambda_7407d5cd5d4425cb98b7ee1223d84907>@@_NPA_WI@std@@EBEABVtype_info@@XZ 1002adc0 f i Plist.obj
 0001:00029dd0       ?_Target_type@?$_Func_impl_no_alloc@V<lambda_ca95615ebb3c7b16132ff39b7c245039>@@_NPA_WI@std@@EBEABVtype_info@@XZ 1002add0 f i Plist.obj
 0001:00029de0       ?allocate@?$allocator@PAUHINSTANCE__@@@std@@QAEPAPAUHINSTANCE__@@I@Z 1002ade0 f i Plist.obj
 0001:0002a150       ?read_string@?$ipc_functions@$00@@SA?AV?$basic_string@_WU?$char_traits@_W@std@@V?$allocator@_W@2@@std@@PAXABUUNICODE_STRING_64@detail@@@Z 1002b150 f i Plist.obj
 0001:0002a240       ?read_string@?$ipc_functions@$00@@SA?AV?$basic_string@_WU?$char_traits@_W@std@@V?$allocator@_W@2@@std@@PAX_K@Z 1002b240 f i Plist.obj
 0001:0002a2b0       ?read_string@?$ipc_functions@$0A@@@SA?AV?$basic_string@_WU?$char_traits@_W@std@@V?$allocator@_W@2@@std@@PAXABUUNICODE_STRING_SAME@detail@@@Z 1002b2b0 f i Plist.obj
 0001:0002a360       ?read_string@?$ipc_functions@$0A@@@SA?AV?$basic_string@_WU?$char_traits@_W@std@@V?$allocator@_W@2@@std@@PAXQBX@Z 1002b360 f i Plist.obj
 0001:0002a3c0       ?ConvertDate@@YAXABU_FILETIME@@PA_W1@Z 1002b3c0 f   Pmix.obj
 0001:0002a450       ?GetMsg@@YAPB_WH@Z         1002b450 f   Pmix.obj
 0001:0002a470       ?WinError@@YAHPB_W@Z       1002b470 f   Pmix.obj
 0001:0002a840       ??0WMIConnection@@QAE@XZ   1002b840 f   WMI.obj
 0001:0002a8a0       ??1?$ptr_setter@V?$unique_ptr@UIWbemClassObject@@Ucom_closer@@@std@@@@QAE@XZ 1002b8a0 f i WMI.obj
 0001:0002a8e0       ??1?$unique_ptr@UIWbemClassObject@@Ucom_closer@@@std@@QAE@XZ 1002b8e0 f i WMI.obj
 0001:0002a8e0       ??1?$unique_ptr@UIWbemLocator@@Ucom_closer@@@std@@QAE@XZ 1002b8e0 f i WMI.obj
 0001:0002a920       ??1WMIConnection@@QAE@XZ   1002b920 f   WMI.obj
 0001:0002a980       ??1bstr@@QAE@XZ            1002b980 f i WMI.obj
 0001:0002a990       ?Connect@WMIConnection@@QAE_NPB_W00@Z 1002b990 f   WMI.obj
 0001:0002ab90       ?Disconnect@WMIConnection@@QAEXXZ 1002bb90 f   WMI.obj
 0001:0002abb0       ?ExecMethod@WMIConnection@@AAEHKPB_W0K@Z 1002bbb0 f   WMI.obj
 0001:0002ae70       ?GetProcessCommandLine@WMIConnection@@QAE?AV?$basic_string@_WU?$char_traits@_W@std@@V?$allocator@_W@2@@std@@K@Z 1002be70 f   WMI.obj
 0001:0002af10       ?GetProcessExecutablePath@WMIConnection@@QAE?AV?$basic_string@_WU?$char_traits@_W@std@@V?$allocator@_W@2@@std@@K@Z 1002bf10 f   WMI.obj
 0001:0002afb0       ?GetProcessOwner@WMIConnection@@QAE?AV?$basic_string@_WU?$char_traits@_W@std@@V?$allocator@_W@2@@std@@KPAV23@@Z 1002bfb0 f   WMI.obj
 0001:0002b1d0       ?GetProcessPriority@WMIConnection@@QAEKK@Z 1002c1d0 f   WMI.obj
 0001:0002b250       ?GetProcessProperty@WMIConnection@@AAE_NKPB_WABV?$function@$$A6AXABUtagVARIANT@@@Z@std@@@Z 1002c250 f   WMI.obj
 0001:0002b360       ?GetProcessSessionId@WMIConnection@@QAEKK@Z 1002c360 f   WMI.obj
 0001:0002b3e0       ?GetProcessUserSid@WMIConnection@@QAE?AV?$basic_string@_WU?$char_traits@_W@std@@V?$allocator@_W@2@@std@@K@Z 1002c3e0 f   WMI.obj
 0001:0002b650       ?SetProcessPriority@WMIConnection@@QAEHKK@Z 1002c650 f   WMI.obj
 0001:0002b670       ?TerminateProcess@WMIConnection@@QAEHK@Z 1002c670 f   WMI.obj
 0001:0002b7e0       ?Message@@YAHIPB_WPAPB_WII@Z 1002c7e0 f   Proclist.obj
 0001:0002b980       ?is_wow64_process@@YA_NPAX@Z 1002c980 f   Proclist.obj
 0001:0002b9b0       _ClosePanelW@4             1002c9b0 f   Proclist.obj
 0001:0002b9e0       _CompareW@4                1002c9e0 f   Proclist.obj
 0001:0002ba00       _ConfigureW@4              1002ca00 f   Proclist.obj
 0001:0002ba10       _DeleteFilesW@4            1002ca10 f   Proclist.obj
 0001:0002ba30       _ExitFARW@4                1002ca30 f   Proclist.obj
 0001:0002ba40       _FreeFindDataW@4           1002ca40 f   Proclist.obj
 0001:0002ba60       _GetFilesW@4               1002ca60 f   Proclist.obj
 0001:0002ba90       _GetFindDataW@4            1002ca90 f   Proclist.obj
 0001:0002bab0       _GetGlobalInfoW@4          1002cab0 f   Proclist.obj
 0001:0002bb40       _GetOpenPanelInfoW@4       1002cb40 f   Proclist.obj
 0001:0002bb50       _GetPluginInfoW@4          1002cb50 f   Proclist.obj
 0001:0002bc00       _OpenW@4                   1002cc00 f   Proclist.obj
 0001:0002bc80       _ProcessPanelEventW@4      1002cc80 f   Proclist.obj
 0001:0002bca0       _ProcessPanelInputW@4      1002cca0 f   Proclist.obj
 0001:0002bcc0       _SetStartupInfoW@4         1002ccc0 f   Proclist.obj
 0001:0002c0c0       _DecodePointerWrapper@4    1002d0c0 f   vc_crt_fix_impl.obj
 0001:0002c110       _EncodePointerWrapper@4    1002d110 f   vc_crt_fix_impl.obj
 0001:0002c160       _GetLogicalProcessorInformationWrapper@8 1002d160 f   vc_crt_fix_impl.obj
 0001:0002c1b0       _GetModuleHandleExWWrapper@12 1002d1b0 f   vc_crt_fix_impl.obj
 0001:0002c200       _GetNumaHighestNodeNumberWrapper@4 1002d200 f   vc_crt_fix_impl.obj
 0001:0002c250       _InitializeSListHeadWrapper@4 1002d250 f   vc_crt_fix_impl.obj
 0001:0002c2a0       _InterlockedFlushSListWrapper@4 1002d2a0 f   vc_crt_fix_impl.obj
 0001:0002c2f0       _InterlockedPopEntrySListWrapper@4 1002d2f0 f   vc_crt_fix_impl.obj
 0001:0002c340       _InterlockedPushEntrySListWrapper@8 1002d340 f   vc_crt_fix_impl.obj
 0001:0002c390       _InterlockedPushListSListExWrapper@16 1002d390 f   vc_crt_fix_impl.obj
 0001:0002c3e0       _QueryDepthSListWrapper@4  1002d3e0 f   vc_crt_fix_impl.obj
 0001:0002c430       _RtlFirstEntrySListWrapper@4 1002d430 f   vc_crt_fix_impl.obj
 0001:0002c480       _SetThreadStackGuaranteeWrapper@4 1002d480 f   vc_crt_fix_impl.obj
 0001:0002c4c3       _ConvertSidToStringSidW@8  1002d4c3 f   advapi32:ADVAPI32.dll
 0001:0002c4c9       _WNetAddConnection2W@16    1002d4c9 f   mpr:MPR.dll
 0001:0002c4cf       _WNetCancelConnection2W@12 1002d4cf f   mpr:MPR.dll
 0001:0002c4d5       _GetFileVersionInfoSizeW@8 1002d4d5 f   version:VERSION.dll
 0001:0002c4db       _GetFileVersionInfoW@16    1002d4db f   version:VERSION.dll
 0001:0002c4e1       _VerQueryValueW@16         1002d4e1 f   version:VERSION.dll
 0001:0002c4e7       _GetModuleFileNameExW@16   1002d4e7 f   psapi:PSAPI.DLL
 0001:0002c4ed       _GetModuleInformation@16   1002d4ed f   psapi:PSAPI.DLL
 0001:0002c4f3       ??0_Init_locks@std@@QAE@XZ 1002d4f3 f   libcpmt:xlock.obj
 0001:0002c520       ??0_Lockit@std@@QAE@H@Z    1002d520 f   libcpmt:xlock.obj
 0001:0002c551       ??1_Init_locks@std@@QAE@XZ 1002d551 f   libcpmt:xlock.obj
 0001:0002c578       ??1_Lockit@std@@QAE@XZ     1002d578 f   libcpmt:xlock.obj
 0001:0002c597       ??0bad_alloc@std@@QAE@XZ   1002d597 f i libcpmt:xthrow.obj
 0001:0002c5af       ??0bad_function_call@std@@QAE@ABV01@@Z 1002d5af f i libcpmt:xthrow.obj
 0001:0002c5ca       ??0bad_function_call@std@@QAE@XZ 1002d5ca f i libcpmt:xthrow.obj
 0001:0002c5db       ??0length_error@std@@QAE@ABV01@@Z 1002d5db f i libcpmt:xthrow.obj
 0001:0002c5f6       ??0length_error@std@@QAE@PBD@Z 1002d5f6 f i libcpmt:xthrow.obj
 0001:0002c615       ??0logic_error@std@@QAE@ABV01@@Z 1002d615 f i libcpmt:xthrow.obj
 0001:0002c630       ??0out_of_range@std@@QAE@ABV01@@Z 1002d630 f i libcpmt:xthrow.obj
 0001:0002c64b       ??0out_of_range@std@@QAE@PBD@Z 1002d64b f i libcpmt:xthrow.obj
 0001:0002c66a       ??_Elength_error@std@@UAEPAXI@Z 1002d66a f i libcpmt:xthrow.obj
 0001:0002c66a       ??_Gbad_exception@std@@UAEPAXI@Z 1002d66a f i libvcruntime:frame.obj
 0001:0002c66a       ??_Gbad_function_call@std@@UAEPAXI@Z 1002d66a f i libcpmt:xthrow.obj
 0001:0002c66a       ??_Glength_error@std@@UAEPAXI@Z 1002d66a f i libcpmt:xthrow.obj
 0001:0002c66a       ??_Glogic_error@std@@UAEPAXI@Z 1002d66a f i libcpmt:xthrow.obj
 0001:0002c66a       ??_Gout_of_range@std@@UAEPAXI@Z 1002d66a f i libcpmt:xthrow.obj
 0001:0002c66a       ??_Elogic_error@std@@UAEPAXI@Z 1002d66a f i libcpmt:xthrow.obj
 0001:0002c66a       ??_Ebad_function_call@std@@UAEPAXI@Z 1002d66a f i libcpmt:xthrow.obj
 0001:0002c66a       ??_Ebad_exception@std@@UAEPAXI@Z 1002d66a f i libvcruntime:frame.obj
 0001:0002c66a       ??_Eout_of_range@std@@UAEPAXI@Z 1002d66a f i libcpmt:xthrow.obj
 0001:0002c697       ?__scrt_throw_std_bad_alloc@@YAXXZ 1002d697 f   LIBCMT:throw_bad_alloc.obj
 0001:0002c697       ?_Xbad_alloc@std@@YAXXZ    1002d697 f   libcpmt:xthrow.obj
 0001:0002c6b4       ?_Xbad_function_call@std@@YAXXZ 1002d6b4 f   libcpmt:xthrow.obj
 0001:0002c6d1       ?_Xlength_error@std@@YAXPBD@Z 1002d6d1 f   libcpmt:xthrow.obj
 0001:0002c6f1       ?_Xout_of_range@std@@YAXPBD@Z 1002d6f1 f   libcpmt:xthrow.obj
 0001:0002c711       ?_Xruntime_error@std@@YAXPBD@Z 1002d711 f   libcpmt:xthrow.obj
 0001:0002c731       ?what@bad_function_call@std@@UBEPBDXZ 1002d731 f i libcpmt:xthrow.obj
 0001:0002c737       ??0_Locimp@locale@std@@AAE@_N@Z 1002d737 f i libcpmt:locale0.obj
 0001:0002c778       ??1_Fac_node@std@@QAE@XZ   1002d778 f i libcpmt:locale0.obj
 0001:0002c7a9       ??1_Fac_tidy_reg_t@std@@QAE@XZ 1002d7a9 f i libcpmt:locale0.obj
 0001:0002c7d0       ??1_Locimp@locale@std@@MAE@XZ 1002d7d0 f i libcpmt:locale0.obj
 0001:0002c7fb       ??4?$_Yarn@D@std@@QAEAAV01@PBD@Z 1002d7fb f i libcpmt:locale0.obj
 0001:0002c84f       ??_G_Locimp@locale@std@@MAEPAXI@Z 1002d84f f i libcpmt:locale0.obj
 0001:0002c84f       ??_E_Locimp@locale@std@@MAEPAXI@Z 1002d84f f i libcpmt:locale0.obj
 0001:0002c871       ?_Facet_Register@std@@YAXPAV_Facet_base@1@@Z 1002d871 f   libcpmt:locale0.obj
 0001:0002c89d       ?_Getgloballocale@locale@std@@CAPAV_Locimp@12@XZ 1002d89d f   libcpmt:locale0.obj
 0001:0002c8a3       ?_Init@locale@std@@CAPAV_Locimp@12@_N@Z 1002d8a3 f   libcpmt:locale0.obj
 0001:0002c933       ?_Locimp_dtor@_Locimp@locale@std@@CAXPAV123@@Z 1002d933 f   libcpmt:locale0.obj
 0001:0002c9a3       ?_Locinfo_ctor@_Locinfo@std@@SAXPAV12@PBD@Z 1002d9a3 f   libcpmt:locale0.obj
 0001:0002c9ee       ?_Locinfo_dtor@_Locinfo@std@@SAXPAV12@@Z 1002d9ee f   libcpmt:locale0.obj
 0001:0002ca08       ?_New_Locimp@_Locimp@locale@std@@CAPAV123@_N@Z 1002da08 f   libcpmt:locale0.obj
 0001:0002ca2b       ?_Setgloballocale@locale@std@@CAXPAX@Z 1002da2b f   libcpmt:locale0.obj
 0001:0002ca53       __Deletegloballocale       1002da53 f   libcpmt:locale0.obj
 0001:0002cab8       __Getcvt                   1002dab8 f   libcpmt:xwctomb.obj
 0001:0002cb2b       __Mbrtowc                  1002db2b f   libcpmt:xmbtowc.obj
 0001:0002ccb4       __Mtxdst                   1002dcb4 f   libcpmt:xmtx.obj
 0001:0002ccc2       __Mtxinit                  1002dcc2 f   libcpmt:xmtx.obj
 0001:0002ccd9       __Mtxlock                  1002dcd9 f   libcpmt:xmtx.obj
 0001:0002cce7       __Mtxunlock                1002dce7 f   libcpmt:xmtx.obj
 0001:0002ccf5       ??1_Init_atexit@@QAE@XZ    1002dcf5 f i libcpmt:iosptrs.obj
 0001:0002cd58       ?_Atexit@@YAXP6AXXZ@Z      1002dd58 f   libcpmt:iosptrs.obj
 0001:0002d041       ___crtInitializeCriticalSectionEx 1002e041 f   libcpmt:winapisupp.obj
 0001:0002d076       __freea_crt                1002e076 f i libcpmt:StlLCMapStringA.obj
 0001:0002d094       ??3@YAXPAXI@Z              1002e094 f   LIBCMT:delete_scalar_size.obj
 0001:0002d0e6       ___scrt_acquire_startup_lock 1002e0e6 f   LIBCMT:utility.obj
 0001:0002d118       ___scrt_dllmain_after_initialize_c 1002e118 f   LIBCMT:utility.obj
 0001:0002d143       ___scrt_dllmain_before_initialize_c 1002e143 f   LIBCMT:utility.obj
 0001:0002d151       ___scrt_dllmain_crt_thread_attach 1002e151 f   LIBCMT:utility.obj
 0001:0002d170       ___scrt_dllmain_crt_thread_detach 1002e170 f   LIBCMT:utility.obj
 0001:0002d17d       ___scrt_dllmain_exception_filter 1002e17d f   LIBCMT:utility.obj
 0001:0002d1b1       ___scrt_dllmain_uninitialize_c 1002e1b1 f   LIBCMT:utility.obj
 0001:0002d1d4       ___scrt_dllmain_uninitialize_critical 1002e1d4 f   LIBCMT:utility.obj
 0001:0002d1e1       ___scrt_initialize_crt     1002e1e1 f   LIBCMT:utility.obj
 0001:0002d21a       ___scrt_initialize_onexit_tables 1002e21a f   LIBCMT:utility.obj
 0001:0002d2a1       ___scrt_is_nonwritable_in_current_image 1002e2a1 f   LIBCMT:utility.obj
 0001:0002d335       ___scrt_release_startup_lock 1002e335 f   LIBCMT:utility.obj
 0001:0002d352       ___scrt_uninitialize_crt   1002e352 f   LIBCMT:utility.obj
 0001:0002d37a       __onexit                   1002e37a f   LIBCMT:utility.obj
 0001:0002d3a7       _atexit                    1002e3a7 f   LIBCMT:utility.obj
 0001:0002d3bc       ??2@YAPAXI@Z               1002e3bc f   LIBCMT:new_scalar.obj
 0001:0002d3f0       __allmul                   1002e3f0 f   LIBCMT:llmul.obj
 0001:0002d430       __allshl                   1002e430 f   LIBCMT:llshl.obj
 0001:0002d450       __aullshr                  1002e450 f   LIBCMT:ullshr.obj
 0001:0002d46f       ??_Etype_info@@UAEPAXI@Z   1002e46f f i LIBCMT:std_type_info_static.obj
 0001:0002d46f       ??_Gtype_info@@UAEPAXI@Z   1002e46f f i LIBCMT:std_type_info_static.obj
 0001:0002d492       ??_U@YAPAXI@Z              1002e492 f   LIBCMT:new_array.obj
 0001:0002d49b       ??_V@YAXPAX@Z              1002e49b f   LIBCMT:delete_array.obj
 0001:0002d4a0       ??_M@YGXPAXIIP6EX0@Z@Z     1002e4a0 f   LIBCMT:ehvecdtr.obj
 0001:0002d525       ?__ArrayUnwind@@YGXPAXIIP6EX0@Z@Z 1002e525 f   LIBCMT:ehvecdtr.obj
 0001:0002d5c0       __aulldiv                  1002e5c0 f   LIBCMT:ulldiv.obj
 0001:0002d630       __aulldvrm                 1002e630 f   LIBCMT:ulldvrm.obj
 0001:0002d6d0       __aullrem                  1002e6d0 f   LIBCMT:ullrem.obj
 0001:0002d750       __ftoi2                    1002e750 f   LIBCMT:ftol2.obj
 0001:0002d750       __ftol2_sse_excpt          1002e750     LIBCMT:ftol2.obj
 0001:0002d750       __ftol2_sse                1002e750     LIBCMT:ftol2.obj
 0001:0002d7d0       __ftoui2                   1002e7d0 f   LIBCMT:ftol2.obj
 0001:0002d880       __ftol2                    1002e880 f   LIBCMT:ftol2.obj
 0001:0002d930       __ftoul2                   1002e930 f   LIBCMT:ftol2.obj
 0001:0002d9f0       __alldiv                   1002e9f0 f   LIBCMT:lldiv.obj
 0001:0002ddd5       __DllMainCRTStartup@12     1002edd5 f   LIBCMT:dll_dllmain.obj
 0001:0002ddf8       @__security_check_cookie@4 1002edf8 f   LIBCMT:secchk.obj
 0001:0002de09       __EH_epilog3               1002ee09 f   LIBCMT:ehprolg3.obj
 0001:0002de1e       __EH_epilog3_GS            1002ee1e f   LIBCMT:ehprolg3.obj
 0001:0002de2f       __EH_prolog3               1002ee2f f   LIBCMT:ehprolg3.obj
 0001:0002de63       __EH_prolog3_GS            1002ee63 f   LIBCMT:ehprolg3.obj
 0001:0002de9a       __EH_prolog3_catch         1002ee9a f   LIBCMT:ehprolg3.obj
 0001:0002ded1       @_guard_check_icall_nop@4  1002eed1 f i LIBCMT:guard_support.obj
 0001:0002dee0       __alloca_probe_16          1002eee0 f   LIBCMT:alloca16.obj
 0001:0002def6       __alloca_probe_8           1002eef6     LIBCMT:alloca16.obj
 0001:0002df0c       ??3@YAXPAX@Z               1002ef0c f   LIBCMT:delete_scalar.obj
 0001:0002df11       ___isa_available_init      1002ef11 f   LIBCMT:cpu_disp.obj
 0001:0002e0e1       __get_startup_argv_mode    1002f0e1 f   LIBCMT:argv_mode.obj
 0001:0002e0e5       ___scrt_is_ucrt_dll_in_use 1002f0e5 f   LIBCMT:ucrt_detection.obj
 0001:0002e0f1       ___scrt_fastfail           1002f0f1 f   LIBCMT:utility_desktop.obj
 0001:0002e20b       __crt_debugger_hook        1002f20b f   LIBCMT:utility_desktop.obj
 0001:0002e220       __SEH_prolog4              1002f220 f   LIBCMT:sehprolg4.obj
 0001:0002e266       __SEH_epilog4              1002f266 f   LIBCMT:sehprolg4.obj
 0001:0002e27b       ?__scrt_throw_std_bad_array_new_length@@YAXXZ 1002f27b f   LIBCMT:throw_bad_alloc.obj
 0001:0002e2e5       ___security_init_cookie    1002f2e5 f   LIBCMT:gs_support.obj
 0001:0002e330       _DllMain@12                1002f330 f   LIBCMT:dll_dllmain_stub.obj
 0001:0002e336       ?__scrt_initialize_type_info@@YAXXZ 1002f336 f   LIBCMT:tncleanup.obj
 0001:0002e342       ?__scrt_uninitialize_type_info@@YAXXZ 1002f342 f   LIBCMT:tncleanup.obj
 0001:0002e34e       ___local_stdio_scanf_options 1002f34e f i LIBCMT:default_local_stdio_options.obj
 0001:0002e354       ___scrt_initialize_default_local_stdio_options 1002f354 f   LIBCMT:default_local_stdio_options.obj
 0001:0002e371       ___scrt_get_dyn_tls_init_callback 1002f371 f   LIBCMT:dyn_tls_init.obj
 0001:0002e377       __RTC_Initialize           1002f377 f   LIBCMT:initsect.obj
 0001:0002e3a3       __RTC_Terminate            1002f3a3 f   LIBCMT:initsect.obj
 0001:0002e3cf       ___raise_securityfailure   1002f3cf f   LIBCMT:gs_report.obj
 0001:0002e3f7       ___report_gsfailure        1002f3f7 f   LIBCMT:gs_report.obj
 0001:0002e4f0       ___report_rangecheckfailure 1002f4f0 f   LIBCMT:gs_report.obj
 0001:0002e4fc       ___report_securityfailure  1002f4fc f   LIBCMT:gs_report.obj
 0001:0002e5ca       __get_purecall_handler     1002f5ca f   libvcruntime:purevirt.obj
 0001:0002e5d0       __purecall                 1002f5d0 f   libvcruntime:purevirt.obj
 0001:0002e5ec       ___DestructExceptionObject 1002f5ec f   libvcruntime:ehhelpers.obj
 0001:0002e68d       ?_CallMemberFunction0@@YGXQAX0@Z 1002f68d f i libvcruntime:ehhelpers.obj
 0001:0002e6f2       __IsExceptionObjectToBeDestroyed 1002f6f2 f   libvcruntime:ehhelpers.obj
 0001:0002e718       ___AdjustPointer           1002f718 f   libvcruntime:ehhelpers.obj
 0001:0002e73d       ___FrameUnwindFilter       1002f73d f   libvcruntime:ehhelpers.obj
 0001:0002e793       ___current_exception       1002f793 f   libvcruntime:ehhelpers.obj
 0001:0002e79c       ___current_exception_context 1002f79c f   libvcruntime:ehhelpers.obj
 0001:0002e7a5       ___std_terminate           1002f7a5 f   libvcruntime:ehhelpers.obj
 0001:0002e7aa       ___std_exception_copy      1002f7aa f   libvcruntime:std_exception.obj
 0001:0002e80d       ___std_exception_destroy   1002f80d f   libvcruntime:std_exception.obj
 0001:0002e82c       __CxxThrowException@8      1002f82c f   libvcruntime:throw.obj
 0001:0002e898       ?GetRangeOfTrysToCheck@__FrameHandler3@@SA?AU?$pair@Viterator@TryBlockMap@__FrameHandler3@@V123@@std@@AAVTryBlockMap@1@HPAXPBU_s_FuncInfo@@H@Z 1002f898 f   libvcruntime:trnsctrl.obj
 0001:0002e908       ?_CallCatchBlock2@@YAPAXPAUEHRegistrationNode@@PBU_s_FuncInfo@@PAXHK@Z 1002f908 f   libvcruntime:trnsctrl.obj
 0001:0002e966       ?_CallSETranslator@@YAHPAUEHExceptionRecord@@PAUEHRegistrationNode@@PAX2PBU_s_FuncInfo@@H1@Z 1002f966 f   libvcruntime:trnsctrl.obj
 0001:0002ea4c       ?_JumpToContinuation@@YGXPAXPAUEHRegistrationNode@@@Z 1002fa4c f   libvcruntime:trnsctrl.obj
 0001:0002ea7c       ?_UnwindNestedFrames@@YGXPAUEHRegistrationNode@@PAUEHExceptionRecord@@@Z 1002fa7c f   libvcruntime:trnsctrl.obj
 0001:0002eacf       __CatchGuardHandler        1002facf f   libvcruntime:trnsctrl.obj
 0001:0002eb00       __CreateFrameInfo          1002fb00 f   libvcruntime:trnsctrl.obj
 0001:0002eb24       __FindAndUnlinkFrame       1002fb24 f   libvcruntime:trnsctrl.obj
 0001:0002eb6c       __TranslatorGuardHandler   1002fb6c f   libvcruntime:trnsctrl.obj
 0001:0002ec09       ___CxxFrameHandler3        1002fc09 f   libvcruntime:trnsctrl.obj
 0001:0002ec40       _memchr                    1002fc40 f   libvcruntime:memchr.obj
 0001:0002ecf0       _memcpy                    1002fcf0 f   libvcruntime:memcpy.obj
 0001:0002f270       _memmove                   10030270 f   libvcruntime:memmove.obj
 0001:0002f7f0       _memset                    100307f0 f   libvcruntime:memset.obj
 0001:0002f94a       _wcschr                    1003094a f   libvcruntime:wcschr.obj
 0001:0002fa11       _memcmp                    10030a11 f   libvcruntime:memcmp.obj
 0001:000309b5       ___vcrt_initialize         100319b5 f   libvcruntime:initialization.obj
 0001:000309d4       ___vcrt_thread_attach      100319d4 f   libvcruntime:initialization.obj
 0001:000309df       ___vcrt_thread_detach      100319df f   libvcruntime:initialization.obj
 0001:000309ea       ___vcrt_uninitialize       100319ea f   libvcruntime:initialization.obj
 0001:00030a01       ___vcrt_uninitialize_critical 10031a01 f   libvcruntime:initialization.obj
 0001:00030a50       __except_handler4          10031a50 f   libvcruntime:chandler4.obj
 0001:00030bae       ___std_type_info_compare   10031bae f   libvcruntime:std_type_info.obj
 0001:00030bea       ___std_type_info_destroy_list 10031bea f   libvcruntime:std_type_info.obj
 0001:00030c0d       ___vcrt_freefls@4          10031c0d f   libvcruntime:per_thread_data.obj
 0001:00030c29       ___vcrt_freeptd            10031c29 f   libvcruntime:per_thread_data.obj
 0001:00030c5f       ___vcrt_getptd             10031c5f f   libvcruntime:per_thread_data.obj
 0001:00030c6d       ___vcrt_getptd_noexit      10031c6d f   libvcruntime:per_thread_data.obj
 0001:00030cff       ___vcrt_initialize_ptd     10031cff f   libvcruntime:per_thread_data.obj
 0001:00030d32       ___vcrt_uninitialize_ptd   10031d32 f   libvcruntime:per_thread_data.obj
 0001:00031490       ??$TypeMatchHelper@V__FrameHandler3@@@@YAHPBU_s_HandlerType@@PBU_s_CatchableType@@PBU_s_ThrowInfo@@@Z 10032490 f i libvcruntime:frame.obj
 0001:0003151e       ??$__InternalCxxFrameHandler@V__FrameHandler3@@@@YA?AW4_EXCEPTION_DISPOSITION@@PAUEHExceptionRecord@@PAUEHRegistrationNode@@PAU_CONTEXT@@PAXPBU_s_FuncInfo@@H1E@Z 1003251e f i libvcruntime:frame.obj
 0001:00031620       ??0bad_exception@std@@QAE@ABV01@@Z 10032620 f i libvcruntime:frame.obj
 0001:0003163b       ??0bad_exception@std@@QAE@XZ 1003263b f i libvcruntime:frame.obj
 0001:00031653       ??8type_info@@QBE_NABV0@@Z 10032653 f i libvcruntime:frame.obj
 0001:000318ba       ?FrameUnwindToEmptyState@__FrameHandler3@@SAXPAUEHRegistrationNode@@PAXPBU_s_FuncInfo@@@Z 100328ba f   libvcruntime:frame.obj
 0001:000318d2       ?FrameUnwindToState@__FrameHandler3@@SAXPAUEHRegistrationNode@@PAXPBU_s_FuncInfo@@H@Z 100328d2 f   libvcruntime:frame.obj
 0001:00031a54       ?_CallMemberFunction1@@YGXQAX00@Z 10032a54 f i libvcruntime:frame.obj
 0001:00031a64       ?_CallMemberFunction2@@YGXQAX00H@Z 10032a64 f i libvcruntime:frame.obj
 0001:00031a77       ?getESTypes@__FrameHandler3@@SAPBU_s_ESTypeList@@PBU_s_FuncInfo@@@Z 10032a77 f i libvcruntime:frame.obj
 0001:00031a90       __CallSettingFrame@12      10032a90 f   libvcruntime:lowhelpr.obj
 0001:00031ab7       __NLG_Return               10032ab7     libvcruntime:lowhelpr.obj
 0001:00031adc       ___except_validate_context_record 10032adc f   libvcruntime:jbcxrval.obj
 0001:00031b0c       ___except_validate_jump_buffer 10032b0c f   libvcruntime:jbcxrval.obj
 0001:00031b39       ___vcrt_initialize_locks   10032b39 f   libvcruntime:locks.obj
 0001:00031b75       ___vcrt_uninitialize_locks 10032b75 f   libvcruntime:locks.obj
 0001:00031bb0       __local_unwind4            10032bb0 f   libvcruntime:exsup4.obj
 0001:00031c88       __seh_longjmp_unwind4@4    10032c88 f   libvcruntime:exsup4.obj
 0001:00031cb0       @_EH4_CallFilterFunc@8     10032cb0 f   libvcruntime:exsup4.obj
 0001:00031cc8       @_EH4_TransferToHandler@8  10032cc8 f   libvcruntime:exsup4.obj
 0001:00031ce4       @_EH4_GlobalUnwind2@8      10032ce4 f   libvcruntime:exsup4.obj
 0001:00031d00       @_EH4_LocalUnwind@16       10032d00 f   libvcruntime:exsup4.obj
 0001:00031e0c       ___vcrt_FlsAlloc           10032e0c f   libvcruntime:winapi_downlevel.obj
 0001:00031e47       ___vcrt_FlsFree            10032e47 f   libvcruntime:winapi_downlevel.obj
 0001:00031e82       ___vcrt_FlsGetValue        10032e82 f   libvcruntime:winapi_downlevel.obj
 0001:00031ebd       ___vcrt_FlsSetValue        10032ebd f   libvcruntime:winapi_downlevel.obj
 0001:00031efb       ___vcrt_InitializeCriticalSectionEx 10032efb f   libvcruntime:winapi_downlevel.obj
 0001:00031f42       _unexpected                10032f42 f   libvcruntime:unexpected.obj
 0001:00031f5f       ?GetCurrentState@__FrameHandler3@@SAHPAUEHRegistrationNode@@PAXPBU_s_FuncInfo@@@Z 10032f5f f   libvcruntime:ehstate.obj
 0001:00031f7c       ?SetState@__FrameHandler3@@SAXPAUEHRegistrationNode@@PBU_s_FuncInfo@@H@Z 10032f7c f   libvcruntime:ehstate.obj
 0001:00031f90       __global_unwind2           10032f90 f   libvcruntime:exsup.obj
 0001:00031ff6       __local_unwind2            10032ff6 f   libvcruntime:exsup.obj
 0001:0003207a       __abnormal_termination     1003307a f   libvcruntime:exsup.obj
 0001:000320a0       __NLG_Notify1              100330a0 f   libvcruntime:exsup.obj
 0001:000320ac       __NLG_Notify               100330ac f   libvcruntime:exsup.obj
 0001:000320c3       __NLG_Dispatch             100330c3     libvcruntime:exsup.obj
 0001:000320c3       __NLG_Dispatch2            100330c3     libvcruntime:exsup.obj
 0001:000320cb       __NLG_Call                 100330cb f   libvcruntime:exsup.obj
 0001:000320cd       __NLG_Return2              100330cd     libvcruntime:exsup.obj
 0001:000320ce       ___acrt_call_reportfault   100330ce f   libucrt:invalid_parameter.obj
 0001:00032207       ___acrt_initialize_invalid_parameter_handler 10033207 f   libucrt:invalid_parameter.obj
 0001:00032216       __invalid_parameter        10033216 f   libucrt:invalid_parameter.obj
 0001:0003227a       __invalid_parameter_noinfo 1003327a f   libucrt:invalid_parameter.obj
 0001:0003228a       __invalid_parameter_noinfo_noreturn 1003328a f   libucrt:invalid_parameter.obj
 0001:000322a7       __invoke_watson            100332a7 f   libucrt:invalid_parameter.obj
 0001:000322db       __dclass                   100332db f   libucrt:nan.obj
 0001:000322ec       __dsign                    100332ec f   libucrt:nan.obj
 0001:000322ec       __ldsign                   100332ec f   libucrt:nanl.obj
 0001:000322fc       __ldclass                  100332fc f   libucrt:nanl.obj
 0001:0003230d       __fdclass                  1003330d f   libucrt:nanf.obj
 0001:0003231e       __fdsign                   1003331e f   libucrt:nanf.obj
 0001:00032330       _calloc                    10033330 f   libucrt:calloc.obj
 0001:0003233b       _free                      1003333b f   libucrt:free.obj
 0001:00032356       ___acrt_errno_from_os_error 10033356 f   libucrt:errno.obj
 0001:00032399       ___acrt_errno_map_os_error 10033399 f   libucrt:errno.obj
 0001:000323bc       ___doserrno                100333bc f   libucrt:errno.obj
 0001:000323cf       __errno                    100333cf f   libucrt:errno.obj
 0001:000323e2       ___acrt_initialize_stdio   100333e2 f   libucrt:_file.obj
 0001:000324aa       ___acrt_uninitialize_stdio 100334aa f   libucrt:_file.obj
 0001:000324f6       __lock_file                100334f6 f   libucrt:_file.obj
 0001:0003250a       __unlock_file              1003350a f   libucrt:_file.obj
 0001:0003251e       __fileno                   1003351e f   libucrt:fileno.obj
 0001:000327ab       ??$count@D@formatting_buffer@__crt_stdio_output@@QBEIXZ 100337ab f i libucrt:output.obj
 0001:000327c3       ??$ensure_buffer_is_big_enough@D@formatting_buffer@__crt_stdio_output@@QAE_NI@Z 100337c3 f i libucrt:output.obj
 0001:00032840       ??$is_wide_character_specifier@D@__crt_stdio_output@@YA_N_KDW4length_modifier@0@@Z 10033840 f i libucrt:output.obj
 0001:00032871       ??$scratch_data@D@formatting_buffer@__crt_stdio_output@@QAEPADXZ 10033871 f i libucrt:output.obj
 0001:0003288f       ??$type_case_integer_parse_into_buffer@I@?$output_processor@DV?$string_output_adapter@D@__crt_stdio_output@@V?$format_validation_base@DV?$string_output_adapter@D@__crt_stdio_output@@@2@@__crt_stdio_output@@AAEXII_N@Z 1003388f f i libucrt:output.obj
 0001:00032902       ??$type_case_integer_parse_into_buffer@_K@?$output_processor@DV?$string_output_adapter@D@__crt_stdio_output@@V?$format_validation_base@DV?$string_output_adapter@D@__crt_stdio_output@@@2@@__crt_stdio_output@@AAEX_KI_N@Z 10033902 f i libucrt:output.obj
 0001:00032990       ??$write_multiple_characters@V?$string_output_adapter@D@__crt_stdio_output@@D@__crt_stdio_output@@YAXABV?$string_output_adapter@D@0@DHQAH@Z 10033990 f i libucrt:output.obj
 0001:000329bc       ??0?$common_data@D@__crt_stdio_output@@IAE@XZ 100339bc f i libucrt:output.obj
 0001:00032a01       ??0?$output_adapter_data@DV?$string_output_adapter@D@__crt_stdio_output@@@__crt_stdio_output@@IAE@ABV?$string_output_adapter@D@1@_KQBDQAU__crt_locale_pointers@@QAD@Z 10033a01 f i libucrt:output.obj
 0001:00032a3d       ??0_LocaleUpdate@@QAE@QAU__crt_locale_pointers@@@Z 10033a3d f i libucrt:output.obj
 0001:00032ac0       ??1_LocaleUpdate@@QAE@XZ   10033ac0 f i libucrt:output.obj
 0001:00032ad0       ??1formatting_buffer@__crt_stdio_output@@QAE@XZ 10033ad0 f i libucrt:output.obj
 0001:00032aea       ??4?$__crt_unique_heap_ptr@DU__crt_internal_free_policy@@@@QAEAAV0@$$QAV0@@Z 10033aea f i libucrt:output.obj
 0001:00032b0e       ?crop_zeroes@__crt_stdio_output@@YAXPADQAU__crt_locale_pointers@@@Z 10033b0e f i libucrt:output.obj
 0001:00032b6e       ?find_next_state@?$output_processor@DV?$string_output_adapter@D@__crt_stdio_output@@V?$format_validation_base@DV?$string_output_adapter@D@__crt_stdio_output@@@2@@__crt_stdio_output@@ABE?AW4state@2@DW432@@Z 10033b6e f i libucrt:output.obj
 0001:00032bae       ?force_decimal_point@__crt_stdio_output@@YAXPADQAU__crt_locale_pointers@@@Z 10033bae f i libucrt:output.obj
 0001:00032c0a       ?parse_int_from_format_string@?$output_processor@DV?$string_output_adapter@D@__crt_stdio_output@@V?$format_validation_base@DV?$string_output_adapter@D@__crt_stdio_output@@@2@@__crt_stdio_output@@AAE_NQAH@Z 10033c0a f i libucrt:output.obj
 0001:00032c7e       ?process@?$output_processor@DV?$string_output_adapter@D@__crt_stdio_output@@V?$format_validation_base@DV?$string_output_adapter@D@__crt_stdio_output@@@2@@__crt_stdio_output@@QAEHXZ 10033c7e f i libucrt:output.obj
 0001:00032da2       ?state_case_flag@?$output_processor@DV?$string_output_adapter@D@__crt_stdio_output@@V?$format_validation_base@DV?$string_output_adapter@D@__crt_stdio_output@@@2@@__crt_stdio_output@@AAE_NXZ 10033da2 f i libucrt:output.obj
 0001:00032ddf       ?state_case_normal@?$output_processor@DV?$string_output_adapter@D@__crt_stdio_output@@V?$format_validation_base@DV?$string_output_adapter@D@__crt_stdio_output@@@2@@__crt_stdio_output@@AAE_NXZ 10033ddf f i libucrt:output.obj
 0001:00032dfe       ?state_case_normal_common@?$output_processor@DV?$string_output_adapter@D@__crt_stdio_output@@V?$format_validation_base@DV?$string_output_adapter@D@__crt_stdio_output@@@2@@__crt_stdio_output@@AAE_NXZ 10033dfe f i libucrt:output.obj
 0001:00032e28       ?state_case_normal_tchar@?$output_processor@DV?$string_output_adapter@D@__crt_stdio_output@@V?$format_validation_base@DV?$string_output_adapter@D@__crt_stdio_output@@@2@@__crt_stdio_output@@AAE_ND@Z 10033e28 f i libucrt:output.obj
 0001:00032e8c       ?state_case_precision@?$output_processor@DV?$string_output_adapter@D@__crt_stdio_output@@V?$format_validation_base@DV?$string_output_adapter@D@__crt_stdio_output@@@2@@__crt_stdio_output@@AAE_NXZ 10033e8c f i libucrt:output.obj
 0001:00032eb2       ?state_case_size@?$output_processor@DV?$string_output_adapter@D@__crt_stdio_output@@V?$format_validation_base@DV?$string_output_adapter@D@__crt_stdio_output@@@2@@__crt_stdio_output@@AAE_NXZ 10033eb2 f i libucrt:output.obj
 0001:00033000       ?state_case_type@?$output_processor@DV?$string_output_adapter@D@__crt_stdio_output@@V?$format_validation_base@DV?$string_output_adapter@D@__crt_stdio_output@@@2@@__crt_stdio_output@@AAE_NXZ 10034000 f i libucrt:output.obj
 0001:00033232       ?state_case_width@?$output_processor@DV?$string_output_adapter@D@__crt_stdio_output@@V?$format_validation_base@DV?$string_output_adapter@D@__crt_stdio_output@@@2@@__crt_stdio_output@@AAE_NXZ 10034232 f i libucrt:output.obj
 0001:0003325d       ?to_integer_size@__crt_stdio_output@@YAIW4length_modifier@1@@Z 1003425d f i libucrt:output.obj
 0001:000332b1       ?type_case_Z@?$output_processor@DV?$string_output_adapter@D@__crt_stdio_output@@V?$format_validation_base@DV?$string_output_adapter@D@__crt_stdio_output@@@2@@__crt_stdio_output@@AAE_NXZ 100342b1 f i libucrt:output.obj
 0001:0003330b       ?type_case_a@?$output_processor@DV?$string_output_adapter@D@__crt_stdio_output@@V?$format_validation_base@DV?$string_output_adapter@D@__crt_stdio_output@@@2@@__crt_stdio_output@@AAE_NXZ 1003430b f i libucrt:output.obj
 0001:0003345a       ?type_case_c_tchar@?$output_processor@DV?$string_output_adapter@D@__crt_stdio_output@@V?$format_validation_base@DV?$string_output_adapter@D@__crt_stdio_output@@@2@@__crt_stdio_output@@AAE_ND@Z 1003445a f i libucrt:output.obj
 0001:000334ea       ?type_case_integer@?$output_processor@DV?$string_output_adapter@D@__crt_stdio_output@@V?$format_validation_base@DV?$string_output_adapter@D@__crt_stdio_output@@@2@@__crt_stdio_output@@AAE_NI_N@Z 100344ea f i libucrt:output.obj
 0001:0003363b       ?type_case_n@?$output_processor@DV?$string_output_adapter@D@__crt_stdio_output@@V?$format_validation_base@DV?$string_output_adapter@D@__crt_stdio_output@@@2@@__crt_stdio_output@@AAE_NXZ 1003463b f i libucrt:output.obj
 0001:000336af       ?type_case_o@?$output_processor@DV?$string_output_adapter@D@__crt_stdio_output@@V?$format_validation_base@DV?$string_output_adapter@D@__crt_stdio_output@@@2@@__crt_stdio_output@@AAE_NXZ 100346af f i libucrt:output.obj
 0001:000336ce       ?type_case_p@?$output_processor@DV?$string_output_adapter@D@__crt_stdio_output@@V?$format_validation_base@DV?$string_output_adapter@D@__crt_stdio_output@@@2@@__crt_stdio_output@@AAE_NXZ 100346ce f i libucrt:output.obj
 0001:000336e6       ?type_case_s@?$output_processor@DV?$string_output_adapter@D@__crt_stdio_output@@V?$format_validation_base@DV?$string_output_adapter@D@__crt_stdio_output@@@2@@__crt_stdio_output@@AAE_NXZ 100346e6 f i libucrt:output.obj
 0001:00033757       ?validate@?$c_string_character_source@D@__crt_strtox@@QBE_NXZ 10034757 f i libucrt:strtod.obj
 0001:00033757       ?validate@?$c_string_character_source@_W@__crt_strtox@@QBE_NXZ 10034757 f i libucrt:strtod.obj
 0001:00033757       ?validate@?$string_output_adapter@D@__crt_stdio_output@@QBE_NXZ 10034757 f i libucrt:output.obj
 0001:00033772       ?validate_and_update_state_at_end_of_format_string@?$format_validation_base@DV?$string_output_adapter@D@__crt_stdio_output@@@__crt_stdio_output@@IBE_NXZ 10034772 f i libucrt:output.obj
 0001:00033794       ?write_character@?$string_output_adapter@D@__crt_stdio_output@@QBE_NDQAH@Z 10034794 f i libucrt:output.obj
 0001:000337d6       ?write_stored_string_tchar@?$output_processor@DV?$string_output_adapter@D@__crt_stdio_output@@V?$format_validation_base@DV?$string_output_adapter@D@__crt_stdio_output@@@2@@__crt_stdio_output@@AAE_ND@Z 100347d6 f i libucrt:output.obj
 0001:0003387d       ?write_string@?$string_output_adapter@D@__crt_stdio_output@@QBEXQBDHQAHAAV__crt_deferred_errno_cache@@@Z 1003487d f i libucrt:output.obj
 0001:000338e4       ___acrt_locale_get_ctype_array_value 100348e4 f i libucrt:output.obj
 0001:00033906       ___stdio_common_vsnprintf_s 10034906 f   libucrt:output.obj
 0001:0003392d       _terminate                 1003492d f   libucrt:terminate.obj
 0001:00033969       _localeconv                10034969 f   libucrt:localeconv.obj
 0001:00033991       ___acrt_lowio_create_handle_array 10034991 f   libucrt:osfinfo.obj
 0001:00033a0c       ___acrt_lowio_destroy_handle_array 10034a0c f   libucrt:osfinfo.obj
 0001:00033a41       ___acrt_lowio_ensure_fh_exists 10034a41 f   libucrt:osfinfo.obj
 0001:00033adf       ___acrt_lowio_lock_fh      10034adf f   libucrt:osfinfo.obj
 0001:00033b02       ___acrt_lowio_unlock_fh    10034b02 f   libucrt:osfinfo.obj
 0001:00033b25       __free_osfhnd              10034b25 f   libucrt:osfinfo.obj
 0001:00033bb6       __get_osfhandle            10034bb6 f   libucrt:osfinfo.obj
 0001:00033c20       __isatty                   10034c20 f   libucrt:isatty.obj
 0001:00033c76       _malloc                    10034c76 f   libucrt:malloc.obj
 0001:00033c81       __dlog                     10034c81 f   libucrt:log2d.obj
 0001:00033dc8       _log2                      10034dc8 f   libucrt:log2d.obj
 0001:00033df0       _modf                      10034df0 f   libucrt:modf_pentium4.obj
 0001:00033e30       __modf_pentium4            10034e30 f   libucrt:modf_pentium4.obj
 0001:00033f38       _round                     10034f38 f   libucrt:round.obj
 0001:00033f89       __isleadbyte_l             10034f89 f i libucrt:_wctype.obj
 0001:00033fc3       _iswdigit                  10034fc3 f i libucrt:_wctype.obj
 0001:00033fd6       _wcscspn                   10034fd6 f   libucrt:wcscspn.obj
 0001:0003402f       _wcsncpy                   1003502f f   libucrt:wcsncpy.obj
 0001:00034072       _wcspbrk                   10035072 f   libucrt:wcspbrk.obj
 0001:000340c0       _wcstok                    100350c0 f   libucrt:wcstok.obj
 0001:000340f0       __CIlog10                  100350f0 f   libucrt:log10_impl.obj
 0001:0003412b       __CIlog10_default          1003512b f   libucrt:log10_impl.obj
 0001:0003413f       __log10_default            1003513f     libucrt:log10_impl.obj
 0001:00034200       __CIpow                    10035200 f   libucrt:pow_impl.obj
 0001:0003423b       __CIpow_default            1003523b f   libucrt:pow_impl.obj
 0001:00034254       __pow_default              10035254     libucrt:pow_impl.obj
 0001:00034450       _ceil                      10035450 f   libucrt:ceil_pentium4.obj
 0001:00034490       __ceil_pentium4            10035490 f   libucrt:ceil_pentium4.obj
 0001:0003456d       ___acrt_initialize_locks   1003556d f   libucrt:locks.obj
 0001:000345ae       ___acrt_lock               100355ae f   libucrt:locks.obj
 0001:000345c5       ___acrt_uninitialize_locks 100355c5 f   libucrt:locks.obj
 0001:000345f6       ___acrt_unlock             100355f6 f   libucrt:locks.obj
 0001:0003460d       __lock_locales             1003560d f   libucrt:locks.obj
 0001:0003461b       __unlock_locales           1003561b f   libucrt:locks.obj
 0001:0003487e       _setlocale                 1003587e f   libucrt:setlocale.obj
 0001:000348b6       ____lc_codepage_func       100358b6 f   libucrt:initctype.obj
 0001:000348db       ____lc_locale_name_func    100358db f   libucrt:initctype.obj
 0001:00034902       ____mb_cur_max_func        10035902 f   libucrt:initctype.obj
 0001:00034927       ___acrt_locale_initialize_ctype 10035927 f   libucrt:initctype.obj
 0001:00034d85       ___pctype_func             10035d85 f   libucrt:ctype.obj
 0001:00034da9       ??$make_c_string_character_source@DPAPAD@__crt_strtox@@YA?AV?$c_string_character_source@D@0@QBDQAPAD@Z 10035da9 f i libucrt:strtod.obj
 0001:00034dd0       ?divide@__crt_strtox@@YA_KAAUbig_integer@1@ABU21@@Z 10035dd0 f i libucrt:strtod.obj
 0001:00035268       ?unget@?$c_string_character_source@D@__crt_strtox@@QAEXD@Z 10036268 f i libucrt:strtod.obj
 0001:00035291       ?unget@?$c_string_character_source@_W@__crt_strtox@@QAEX_W@Z 10036291 f i libucrt:strtod.obj
 0001:000352bf       __ischartype_l             100362bf f i libucrt:strtod.obj
 0001:000353a0       _strcspn                   100363a0 f   libucrt:strcspn.obj
 0001:000353e6       _abort                     100363e6 f   libucrt:abort.obj
 0001:0003542a       _wcsdup                    1003642a f   libucrt:wcsdup.obj
 0001:0003542a       __wcsdup                   1003642a f   libucrt:wcsdup.obj
 0001:0003553b       ??$__acrt_mbs_to_wcs_cp@U__crt_win32_buffer_internal_dynamic_resizing@@@@YAHQBDAAV?$__crt_win32_buffer@_WU__crt_win32_buffer_internal_dynamic_resizing@@@@I@Z 1003653b f i libucrt:strftime.obj
 0001:00035558       ?_deallocate@?$__crt_win32_buffer@DU__crt_win32_buffer_internal_dynamic_resizing@@@@AAEXXZ 10036558 f i libucrt:argv_wildcards.obj
 0001:00035558       ?_deallocate@?$__crt_win32_buffer@_WU__crt_win32_buffer_internal_dynamic_resizing@@@@AAEXXZ 10036558 f i libucrt:strftime.obj
 0001:00035572       ?allocate@?$__crt_win32_buffer@DU__crt_win32_buffer_no_resizing@@@@QAEHI@Z 10036572 f i libucrt:strftime.obj
 0001:00035599       ?allocate@?$__crt_win32_buffer@_WU__crt_win32_buffer_internal_dynamic_resizing@@@@QAEHI@Z 10036599 f i libucrt:strftime.obj
 0001:000355d8       ?allocate@__crt_win32_buffer_internal_dynamic_resizing@@SAHQAPAXIABV__crt_win32_buffer_empty_debug_info@@@Z 100365d8 f i libucrt:strftime.obj
 0001:000355f7       ?set_to_nullptr@?$__crt_win32_buffer@DU__crt_win32_buffer_no_resizing@@@@QAEXXZ 100365f7 f i libucrt:strftime.obj
 0001:0003560b       ___strncnt                 1003660b f   libucrt:strncnt.obj
 0001:00035627       _wcscpy_s                  10036627 f   libucrt:wcscpy_s.obj
 0001:0003568b       _strnlen                   1003668b f   libucrt:strnlen.obj
 0001:000357ad       _wcsnlen                   100367ad f   libucrt:strnlen.obj
 0001:0003595d       __seh_filter_dll           1003695d f   libucrt:exception_filter.obj
 0001:0003597d       __seh_filter_exe           1003697d f   libucrt:exception_filter.obj
 0001:00035d4b       ___acrt_initialize_thread_local_exit_callback 10036d4b f   libucrt:exit.obj
 0001:00035d5a       __cexit                    10036d5a f   libucrt:exit.obj
 0001:00035d69       __exit                     10036d69 f   libucrt:exit.obj
 0001:00035d7f       __is_c_termination_complete 10036d7f f   libucrt:exit.obj
 0001:00036033       ___acrt_allocate_buffer_for_argv 10037033 f   libucrt:argv_parsing.obj
 0001:00036082       __configure_narrow_argv    10037082 f   libucrt:argv_parsing.obj
 0001:000361df       ??$uninitialize@A6AXAAPAPA_W@Z@?$dual_state_global@PAPA_W@__crt_state_management@@QAEXA6AXAAPAPA_W@Z@Z 100371df f i libucrt:environment_initialization.obj
 0001:000361df       ??$uninitialize@A6AXAAPAPAD@Z@?$dual_state_global@PAPAD@__crt_state_management@@QAEXA6AXAAPAPAD@Z@Z 100371df f i libucrt:environment_initialization.obj
 0001:0003623e       ___dcrt_uninitialize_environments_nolock 1003723e f   libucrt:environment_initialization.obj
 0001:00036275       __initialize_narrow_environment 10037275 f   libucrt:environment_initialization.obj
 0001:00036330       ??$__crt_fast_encode_pointer@PAP6AXXZ@@YAPAP6AXXZQAP6AXXZ@Z 10037330 f i libucrt:onexit.obj
 0001:00036330       ??$__crt_fast_encode_pointer@P6AHXZ@@YAP6AHXZQ6AHXZ@Z 10037330 f i libucrt:onexit.obj
 0001:00036330       ??$__crt_fast_encode_pointer@P6GHPA_WKJ@Z@@YAP6GHPA_WKJ@ZQ6GH0KJ@Z@Z 10037330 f i libucrt:winapi_thunks.obj
 0001:00036330       ??$__crt_fast_encode_pointer@PAX@@YAPAXQAX@Z 10037330 f i libucrt:initialization.obj
 0001:00036552       __crt_atexit               10037552 f   libucrt:onexit.obj
 0001:00036568       __execute_onexit_table     10037568 f   libucrt:onexit.obj
 0001:00036595       __initialize_onexit_table  10037595 f   libucrt:onexit.obj
 0001:000365be       __register_onexit_function 100375be f   libucrt:onexit.obj
 0001:000365f1       ___acrt_uninitialize_command_line 100375f1 f   libucrt:argv_data.obj
 0001:000366ef       ___acrt_initialize         100376ef f   libucrt:initialization.obj
 0001:00036701       ___acrt_thread_attach      10037701 f   libucrt:initialization.obj
 0001:0003670c       ___acrt_thread_detach      1003770c f   libucrt:initialization.obj
 0001:00036714       ___acrt_uninitialize       10037714 f   libucrt:initialization.obj
 0001:00036744       ___acrt_uninitialize_critical 10037744 f   libucrt:initialization.obj
 0001:00036756       ___initialize_lconv_for_unsigned_char 10037756 f   libucrt:lconv_unsigned_char_initialization.obj
 0001:00036784       ___acrt_initialize_new_handler 10037784 f   libucrt:new_handler.obj
 0001:00036793       __callnewh                 10037793 f   libucrt:new_handler.obj
 0001:000367c0       __query_new_handler        100377c0 f   libucrt:new_handler.obj
 0001:0003681c       __initterm                 1003781c f   libucrt:initterm.obj
 0001:00036861       __initterm_e               10037861 f   libucrt:initterm.obj
 0001:0003688f       _strcpy_s                  1003788f f   libucrt:strcpy_s.obj
 0001:000368e9       ??$is_overflow_condition@K@__crt_strtox@@YA_NIK@Z 100378e9 f i libucrt:atox.obj
 0001:0003691a       ??$parse_integer@KV?$c_string_character_source@D@__crt_strtox@@@__crt_strtox@@YAKQAU__crt_locale_pointers@@V?$c_string_character_source@D@0@H_N@Z 1003791a f i libucrt:atox.obj
 0001:00036b3f       ??$parse_integer@KV?$c_string_character_source@_W@__crt_strtox@@@__crt_strtox@@YAKQAU__crt_locale_pointers@@V?$c_string_character_source@_W@0@H_N@Z 10037b3f f i libucrt:atox.obj
 0001:00037147       __wtol                     10038147 f   libucrt:atox.obj
 0001:00037170       _strncmp                   10038170 f   libucrt:strncmp.obj
 0001:000371e8       _wcsncmp                   100381e8 f   libucrt:wcsncmp.obj
 0001:00037560       ___acrt_freeptd            10038560 f   libucrt:per_thread_data.obj
 0001:0003758c       ___acrt_getptd             1003858c f   libucrt:per_thread_data.obj
 0001:00037649       ___acrt_getptd_head        10038649 f   libucrt:per_thread_data.obj
 0001:000376e3       ___acrt_getptd_noexit      100386e3 f   libucrt:per_thread_data.obj
 0001:00037798       ___acrt_initialize_ptd     10038798 f   libucrt:per_thread_data.obj
 0001:000377c4       ___acrt_uninitialize_ptd   100387c4 f   libucrt:per_thread_data.obj
 0001:00037856       __d_int                    10038856 f   libucrt:_test.obj
 0001:0003795c       __dtest                    1003895c f   libucrt:_test.obj
 0001:000379c0       __fdtest                   100389c0 f   libucrt:_test.obj
 0001:00037a0e       __fperrraise               10038a0e f   libucrt:_test.obj
 0001:00037a2f       __ldtest                   10038a2f f   libucrt:_test.obj
 0001:00037a3a       __calloc_base              10038a3a f   libucrt:calloc_base.obj
 0001:00037a97       __free_base                10038a97 f   libucrt:free_base.obj
 0001:00037df1       ___acrt_AppPolicyGetProcessTerminationMethodInternal@4 10038df1 f   libucrt:winapi_thunks.obj
 0001:00037e31       ___acrt_AreFileApisANSI@0  10038e31 f   libucrt:winapi_thunks.obj
 0001:00037e50       ___acrt_EnumSystemLocalesEx@16 10038e50 f   libucrt:winapi_thunks.obj
 0001:00037ea4       ___acrt_FlsAlloc@4         10038ea4 f   libucrt:winapi_thunks.obj
 0001:00037ee3       ___acrt_FlsFree@4          10038ee3 f   libucrt:winapi_thunks.obj
 0001:00037f22       ___acrt_FlsGetValue@4      10038f22 f   libucrt:winapi_thunks.obj
 0001:00037f61       ___acrt_FlsSetValue@8      10038f61 f   libucrt:winapi_thunks.obj
 0001:00037fa3       ___acrt_GetLocaleInfoEx@16 10038fa3 f   libucrt:winapi_thunks.obj
 0001:00037fe5       ___acrt_GetUserDefaultLocaleName@8 10038fe5 f   libucrt:winapi_thunks.obj
 0001:00038021       ___acrt_InitializeCriticalSectionEx@12 10039021 f   libucrt:winapi_thunks.obj
 0001:0003806c       ___acrt_IsValidLocaleName@4 1003906c f   libucrt:winapi_thunks.obj
 0001:000380a4       ___acrt_LCIDToLocaleName@16 100390a4 f   libucrt:winapi_thunks.obj
 0001:000380e3       ___acrt_LCMapStringEx@36   100390e3 f   libucrt:winapi_thunks.obj
 0001:00038140       ___acrt_LocaleNameToLCID@8 10039140 f   libucrt:winapi_thunks.obj
 0001:00038171       ___acrt_can_use_vista_locale_apis 10039171 f   libucrt:winapi_thunks.obj
 0001:0003817c       ___acrt_eagerly_load_locale_apis 1003917c f   libucrt:winapi_thunks.obj
 0001:000381b3       ___acrt_initialize_winapi_thunks 100391b3 f   libucrt:winapi_thunks.obj
 0001:000381de       ___acrt_uninitialize_winapi_thunks 100391de f   libucrt:winapi_thunks.obj
 0001:00038214       __fcloseall                10039214 f   libucrt:closeall.obj
 0001:0003849c       ___acrt_stdio_flush_nolock 1003949c f   libucrt:fflush.obj
 0001:00038501       __fflush_nolock            10039501 f   libucrt:fflush.obj
 0001:00038549       __flushall                 10039549 f   libucrt:fflush.obj
 0001:00038552       ___acrt_stdio_free_buffer_nolock 10039552 f   libucrt:_freebuf.obj
 0001:000386fc       ___acrt_initialize_lowio   100396fc f   libucrt:ioinit.obj
 0001:0003875c       ___acrt_uninitialize_lowio 1003975c f   libucrt:ioinit.obj
 0001:00038f01       __write                    10039f01 f   libucrt:write.obj
 0001:00038ff3       __write_nolock             10039ff3 f   libucrt:write.obj
 0001:000391d5       __malloc_base              1003a1d5 f   libucrt:malloc_base.obj
 0001:00039223       _strtol                    1003a223 f   libucrt:strtox.obj
 0001:0003924d       __mbtowc_l                 1003a24d f   libucrt:mbtowc.obj
 0001:0003938f       _mbtowc                    1003a38f f   libucrt:mbtowc.obj
 0001:000393a9       __wctomb_s_l               1003a3a9 f   libucrt:wctomb.obj
 0001:00039504       _wctomb_s                  1003a504 f   libucrt:wctomb.obj
 0001:00039521       ___acrt_update_locale_info 1003a521 f   libucrt:locale_update.obj
 0001:0003954e       ___acrt_update_multibyte_info 1003a54e f   libucrt:locale_update.obj
 0001:0003957b       ?__acrt_fp_classify@@YA?AW4__acrt_fp_class@@ABN@Z 1003a57b f i libucrt:cvt.obj
 0001:00039dc6       ___acrt_fp_format          1003adc6 f   libucrt:cvt.obj
 0001:00039f01       __get_printf_count_output  1003af01 f   libucrt:printf_count_output.obj
 0001:0003a019       ??0_expandlocale_locale_name_cache@@QAE@QA_WIQAU__crt_qualified_locale_data@@@Z 1003b019 f i libucrt:wsetlocale.obj
 0001:0003a063       ??1_expandlocale_locale_name_cache@@QAE@XZ 1003b063 f i libucrt:wsetlocale.obj
 0001:0003a1fb       ?commit_locale_name@_expandlocale_locale_name_cache@@QAEXQB_WI@Z 1003b1fb f i libucrt:wsetlocale.obj
 0001:0003a23f       ?commit_locale_name_cache_already_updated@_expandlocale_locale_name_cache@@QAEXQB_WI@Z 1003b23f f i libucrt:wsetlocale.obj
 0001:0003a274       ___acrt_copy_locale_name   1003b274 f   libucrt:wsetlocale.obj
 0001:0003a2d4       ___acrt_set_locale_changed 1003b2d4 f   libucrt:wsetlocale.obj
 0001:0003a2df       ___acrt_uninitialize_locale 1003b2df f   libucrt:wsetlocale.obj
 0001:0003a306       ___lc_lctowcs              1003b306 f   libucrt:wsetlocale.obj
 0001:0003a376       ___lc_wcstolc              1003b376 f   libucrt:wsetlocale.obj
 0001:0003a8bb       __wcscats                  1003b8bb f   libucrt:wsetlocale.obj
 0001:0003a8fc       __wsetlocale               1003b8fc f   libucrt:wsetlocale.obj
 0001:0003b7a4       __mbstowcs_s_l             1003c7a4 f   libucrt:mbstowcs.obj
 0001:0003b884       _mbstowcs_s                1003c884 f   libucrt:mbstowcs.obj
 0001:0003b957       _strncpy_s                 1003c957 f   libucrt:strncpy_s.obj
 0001:0003b962       __query_app_type           1003c962 f   libucrt:report_runtime_error.obj
 0001:0003b968       __dunscale                 1003c968 f   libucrt:_unscale.obj
 0001:0003b9fe       ___acrt_initialize_sse2    1003c9fe f   libucrt:mathfcns.obj
 0001:0003ba0e       __modf_default             1003ca0e f   libucrt:modf.obj
 0001:0003bb14       ___libm_error_support      1003cb14 f   libucrt:libm_error.obj
 0001:0003bd08       _iswctype                  1003cd08 f   libucrt:iswctype.obj
 0001:0003bd71       ___acrt_wcstok_s_novalidation 1003cd71 f   libucrt:wcstok_s.obj
 0001:0003be50       __CIlog10_pentium4         1003ce50 f   libucrt:log10_pentium4.obj
 0001:0003be68       __log10_pentium4           1003ce68     libucrt:log10_pentium4.obj
 0001:0003c100       __fFEXP                    1003d100 f   libucrt:87tran.obj
 0001:0003c157       __rtinfpopse               1003d157     libucrt:87tran.obj
 0001:0003c159       __rtinfnpopse              1003d159     libucrt:87tran.obj
 0001:0003c169       __fFLN                     1003d169     libucrt:87tran.obj
 0001:0003c21e       __rtinfpop                 1003d21e     libucrt:87tran.obj
 0001:0003c220       __rtinfnpop                1003d220     libucrt:87tran.obj
 0001:0003c230       __rtforexpinf              1003d230 f   libucrt:87tran.obj
 0001:0003c23d       __ffexpm1                  1003d23d     libucrt:87tran.obj
 0001:0003c2f0       __trandisp1                1003d2f0 f   libucrt:87disp.obj
 0001:0003c365       __trandisp2                1003d365 f   libucrt:87disp.obj
 0001:0003c3ff       __rttospopde               1003d3ff     libucrt:87disp.obj
 0001:0003c404       __rttospop                 1003d404     libucrt:87disp.obj
 0001:0003c410       __rtnospop                 1003d410 f   libucrt:87disp.obj
 0001:0003c420       __rttosnpop                1003d420 f   libucrt:87disp.obj
 0001:0003c421       __rtnospopde               1003d421     libucrt:87disp.obj
 0001:0003c428       __rtzeropop                1003d428     libucrt:87disp.obj
 0001:0003c42a       __rtzeronpop               1003d42a     libucrt:87disp.obj
 0001:0003c430       __rtzerospop               1003d430 f   libucrt:87disp.obj
 0001:0003c43d       __rtonepop                 1003d43d     libucrt:87disp.obj
 0001:0003c440       __rtonenpop                1003d440 f   libucrt:87disp.obj
 0001:0003c450       __tosnan1                  1003d450 f   libucrt:87disp.obj
 0001:0003c480       __nosnan2                  1003d480 f   libucrt:87disp.obj
 0001:0003c490       __tosnan2                  1003d490 f   libucrt:87disp.obj
 0001:0003c4c0       __nan2                     1003d4c0 f   libucrt:87disp.obj
 0001:0003c500       __rtindfpop                1003d500 f   libucrt:87disp.obj
 0001:0003c502       __rtindfnpop               1003d502     libucrt:87disp.obj
 0001:0003c513       __rttosnpopde              1003d513     libucrt:87disp.obj
 0001:0003c520       __rtatan2inf               1003d520 f   libucrt:87disp.obj
 0001:0003c53d       __rtchsifneg               1003d53d     libucrt:87disp.obj
 0001:0003c550       __twoToTOS                 1003d550 f   libucrt:common.obj
 0001:0003c565       __load_CW                  1003d565 f   libucrt:common.obj
 0001:0003c57c       __convertTOStoQNaN         1003d57c f   libucrt:common.obj
 0001:0003c595       __fload_withFB             1003d595 f   libucrt:common.obj
 0001:0003c5d8       __checkTOS_withFB          1003d5d8 f   libucrt:common.obj
 0001:0003c5ee       __fast_exit                1003d5ee f   libucrt:common.obj
 0001:0003c5fb       __math_exit                1003d5fb f   libucrt:common.obj
 0001:0003c625       __check_overflow_exit      1003d625 f   libucrt:common.obj
 0001:0003c639       __check_range_exit         1003d639 f   libucrt:common.obj
 0001:0003c6e0       __startTwoArgErrorHandling 1003d6e0 f   libucrt:genexcep.obj
 0001:0003c6f7       __startOneArgErrorHandling 1003d6f7 f   libucrt:genexcep.obj
 0001:0003c740       __CIpow_pentium4           1003d740 f   libucrt:pow_pentium4.obj
 0001:0003c759       __pow_pentium4             1003d759     libucrt:pow_pentium4.obj
 0001:0003d260       __d_inttype                1003e260 f   libucrt:powhlp.obj
 0001:0003d2c8       __powhlp                   1003e2c8 f   libucrt:powhlp.obj
 0001:0003d3f3       __ceil_default             1003e3f3 f   libucrt:ceil.obj
 0001:0003d751       __wcstombs_s_l             1003e751 f   libucrt:wcstombs.obj
 0001:0003d8fb       ___acrt_GetLocaleInfoA     1003e8fb f   libucrt:getlocaleinfoa.obj
 0001:0003daab       ___acrt_GetStringTypeA     1003eaab f   libucrt:getstringtypea.obj
 0001:0003dd98       ___acrt_LCMapStringA       1003ed98 f   libucrt:lcmapstringa.obj
 0001:0003dde1       __errcode                  1003ede1 f   libucrt:fpexcept.obj
 0001:0003de15       __except1                  1003ee15 f   libucrt:fpexcept.obj
 0001:0003dee3       __handle_exc               1003eee3 f   libucrt:fpexcept.obj
 0001:0003e0ce       __raise_exc                1003f0ce f   libucrt:fpexcept.obj
 0001:0003e0f1       __raise_exc_ex             1003f0f1 f   libucrt:fpexcept.obj
 0001:0003e3e7       __set_errno_from_matherr   1003f3e7 f   libucrt:fpexcept.obj
 0001:0003e416       __umatherr                 1003f416 f   libucrt:fpexcept.obj
 0001:0003e4b6       __decomp                   1003f4b6 f   libucrt:util.obj
 0001:0003e588       __set_exp                  1003f588 f   libucrt:util.obj
 0001:0003e5b5       __sptype                   1003f5b5 f   libucrt:util.obj
 0001:0003e613       __clrfp                    1003f613 f   libucrt:fpctrl.obj
 0001:0003e624       __ctrlfp                   1003f624 f   libucrt:fpctrl.obj
 0001:0003e64e       __set_statfp               1003f64e f   libucrt:fpctrl.obj
 0001:0003e6a7       __statfp                   1003f6a7 f   libucrt:fpctrl.obj
 0001:0003e6b7       __copysign                 1003f6b7 f   libucrt:ieeemisc.obj
 0001:0003e6da       __fpclass                  1003f6da f   libucrt:ieeemisc.obj
 0001:0003e77e       __realloc_base             1003f77e f   libucrt:realloc_base.obj
 0001:0003e7e7       __isctype_l                1003f7e7 f   libucrt:isctype.obj
 0001:0003e980       ___acrt_get_sigabrt_handler 1003f980 f   libucrt:signal.obj
 0001:0003e9a7       ___acrt_initialize_signal_handlers 1003f9a7 f   libucrt:signal.obj
 0001:0003e9c5       ___fpecode                 1003f9c5 f   libucrt:signal.obj
 0001:0003e9ce       _raise                     1003f9ce f   libucrt:signal.obj
 0001:0003ebc9       ___acrt_MultiByteToWideChar 1003fbc9 f   libucrt:multibytetowidechar.obj
 0001:0003ec45       ___acrt_WideCharToMultiByte 1003fc45 f   libucrt:widechartomultibyte.obj
 0001:0003ecf2       ___ascii_wcsicmp           1003fcf2 f   libucrt:wcsicmp.obj
 0001:0003ed2f       __towlower_internal        1003fd2f f i libucrt:wcsicmp.obj
 0001:0003ed6e       __wcsicmp                  1003fd6e f   libucrt:wcsicmp.obj
 0001:0003edb7       __wcsicmp_l                1003fdb7 f   libucrt:wcsicmp.obj
 0001:0003ee6f       ___acrt_initialize_timeset 1003fe6f f   libucrt:timeset.obj
 0001:0003ee9a       ___acrt_get_process_end_policy 1003fe9a f   libucrt:win_policies.obj
 0001:0003f4a9       ?__acrt_get_utf8_acp_compatibility_codepage@@YAIXZ 100404a9 f i libucrt:argv_wildcards.obj
 0001:0003f4e8       ?allocate@?$__crt_win32_buffer@DU__crt_win32_buffer_internal_dynamic_resizing@@@@QAEHI@Z 100404e8 f i libucrt:argv_wildcards.obj
 0001:0003f5ab       ___acrt_expand_narrow_argv_wildcards 100405ab f   libucrt:argv_wildcards.obj
 0001:0003f67d       ___acrt_GetModuleFileNameA 1004067d f   libucrt:getmodulefilenamea.obj
 0001:0003fc3c       ___acrt_initialize_multibyte 10040c3c f   libucrt:mbctype.obj
 0001:0003fc84       ___acrt_update_thread_multibyte_data 10040c84 f   libucrt:mbctype.obj
 0001:0003fc97       __setmbcp_nolock           10040c97 f   libucrt:mbctype.obj
 0001:0003fee1       __ismbblead                10040ee1 f   libucrt:ismbbyte.obj
 0001:0003fef9       ___acrt_initialize_command_line 10040ef9 f   libucrt:argv_data.obj
 0001:0003ff49       ___dcrt_get_narrow_environment_from_os 10040f49 f   libucrt:get_environment_from_os.obj
 0001:0003ffcd       __recalloc_base            10040fcd f   libucrt:recalloc.obj
 0001:0004003a       ___acrt_initialize_heap    1004103a f   libucrt:heap_handle.obj
 0001:0004004b       ___acrt_uninitialize_heap  1004104b f   libucrt:heap_handle.obj
 0001:00040055       ___acrt_execute_initializers 10041055 f   libucrt:shared_initialization.obj
 0001:000400bd       ___acrt_execute_uninitializers 100410bd f   libucrt:shared_initialization.obj
 0001:000400ee       ___acrt_has_user_matherr   100410ee f   libucrt:matherr.obj
 0001:00040106       ___acrt_initialize_user_matherr 10041106 f   libucrt:matherr.obj
 0001:00040115       ___acrt_invoke_user_matherr 10041115 f   libucrt:matherr.obj
 0001:00040147       ___acrt_add_locale_ref     10041147 f   libucrt:locale_refcounting.obj
 0001:000401c4       ___acrt_free_locale        100411c4 f   libucrt:locale_refcounting.obj
 0001:0004030c       ___acrt_locale_add_lc_time_reference 1004130c f   libucrt:locale_refcounting.obj
 0001:00040335       ___acrt_locale_free_lc_time_if_unreferenced 10041335 f   libucrt:locale_refcounting.obj
 0001:00040366       ___acrt_locale_release_lc_time_reference 10041366 f   libucrt:locale_refcounting.obj
 0001:0004038f       ___acrt_release_locale_ref 1004138f f   libucrt:locale_refcounting.obj
 0001:00040410       ___acrt_update_thread_locale_data 10041410 f   libucrt:locale_refcounting.obj
 0001:00040491       __updatetlocinfoEx_nolock  10041491 f   libucrt:locale_refcounting.obj
 0001:000404e1       _fegetexceptflag           100414e1 f   libucrt:fegetexceptflag.obj
 0001:00040512       _fesetexceptflag           10041512 f   libucrt:fesetexceptflag.obj
 0001:00040878       ___acrt_fenv_get_control   10041878 f   libucrt:_fenvutils.obj
 0001:000408f8       ___acrt_fenv_get_fp_status_word_from_exception_mask 100418f8 f   libucrt:_fenvutils.obj
 0001:00040912       ___acrt_fenv_get_status    10041912 f   libucrt:_fenvutils.obj
 0001:000409ca       ___acrt_fenv_set_control   100419ca f   libucrt:_fenvutils.obj
 0001:00040a32       ___acrt_fenv_set_status    10041a32 f   libucrt:_fenvutils.obj
 0001:00040b29       __query_new_mode           10041b29 f   libucrt:new_mode.obj
 0001:00040b80       ___acrt_DownlevelLCIDToLocaleName 10041b80 f   libucrt:lcidtoname_downlevel.obj
 0001:00040c2a       ___acrt_DownlevelLocaleNameToLCID 10041c2a f   libucrt:lcidtoname_downlevel.obj
 0001:00040c56       __fclose_nolock            10041c56 f   libucrt:fclose.obj
 0001:00040ccd       _fclose                    10041ccd f   libucrt:fclose.obj
 0001:00040df3       __commit                   10041df3 f   libucrt:commit.obj
 0001:00040eec       __lseeki64_nolock          10041eec f   libucrt:lseek.obj
 0001:00040f33       ?__mbrtowc_utf8@__crt_mbstring@@YAIPA_WPBDIPAU_Mbstatet@@@Z 10041f33 f   libucrt:mbrtowc.obj
 0001:00040f73       ?__mbsrtowcs_utf8@__crt_mbstring@@YAIPA_WPAPBDIPAU_Mbstatet@@@Z 10041f73 f   libucrt:mbrtowc.obj
 0001:0004106e       __putwch_nolock            1004206e f   libucrt:putwch.obj
 0001:000410a0       ?__c32rtomb_utf8@__crt_mbstring@@YAIPAD_UPAU_Mbstatet@@@Z 100420a0 f   libucrt:c32rtomb.obj
 0001:0004114b       ?return_illegal_sequence@__crt_mbstring@@YAIPAU_Mbstatet@@@Z 1004214b f i libucrt:c32rtomb.obj
 0001:0004116a       _c32rtomb                  1004216a f   libucrt:c32rtomb.obj
 0001:00041175       ___acrt_fp_strflt_to_string 10042175 f   libucrt:_fptostr.obj
 0001:00041235       ___acrt_fltout             10042235 f   libucrt:cfout.obj
 0001:0004257f       ___acrt_locale_free_monetary 1004357f f   libucrt:initmon.obj
 0001:0004267d       ___acrt_locale_initialize_monetary 1004367d f   libucrt:initmon.obj
 0001:00042a34       ___acrt_locale_free_numeric 10043a34 f   libucrt:initnum.obj
 0001:00042a9d       ___acrt_locale_initialize_numeric 10043a9d f   libucrt:initnum.obj
 0001:00042f60       ___acrt_locale_free_time   10043f60 f   libucrt:inittime.obj
 0001:00043044       ___acrt_locale_initialize_time 10044044 f   libucrt:inittime.obj
 0001:000430bf       _wcscat_s                  100440bf f   libucrt:wcscat_s.obj
 0001:0004321b       _wcsncat_s                 1004421b f   libucrt:wcsncat_s.obj
 0001:000432f1       _wcsncpy_s                 100442f1 f   libucrt:wcsncpy_s.obj
 0001:000439f8       ___acrt_get_qualified_locale 100449f8 f   libucrt:get_qualified_locale.obj
 0001:00044359       ___acrt_get_qualified_locale_downlevel 10045359 f   libucrt:getqloc_downlevel.obj
 0001:0004454e       __dnorm                    1004554e f   libucrt:_norm.obj
 0001:000446e3       __frnd                     100456e3 f   libucrt:frnd.obj
 0001:000446f7       ___acrt_GetStringTypeW     100456f7 f   libucrt:getstringtypew.obj
 0001:00044710       __87except                 10045710 f   libucrt:87except.obj
 0001:0004481a       ?__wcsrtombs_utf8@__crt_mbstring@@YAIPADPAPB_WIPAU_Mbstatet@@@Z 1004581a f   libucrt:wcrtomb.obj
 0001:00044918       __towlower_l               10045918 f   libucrt:towlower.obj
 0001:00044a00       _qsort                     10045a00 f   libucrt:qsort.obj
 0001:00044e50       _strpbrk                   10045e50 f   libucrt:strpbrk.obj
 0001:00044e90       __mbsdec                   10045e90 f   libucrt:mbsdec.obj
 0001:00044ea7       __mbsdec_l                 10045ea7 f   libucrt:mbsdec.obj
 0001:00044f43       __msize_base               10045f43 f   libucrt:msize.obj
 0001:00044f76       _fetestexcept              10045f76 f   libucrt:fetestexcept.obj
 0001:00044f96       ___ascii_wcsnicmp          10045f96 f   libucrt:wcsnicmp.obj
 0001:00044fe5       __wcsnicmp                 10045fe5 f   libucrt:wcsnicmp.obj
 0001:00045031       __wcsnicmp_l               10046031 f   libucrt:wcsnicmp.obj
 0001:00045190       __close                    10046190 f   libucrt:close.obj
 0001:0004521d       __close_nolock             1004621d f   libucrt:close.obj
 0001:000452b9       ?__acrt_stdio_free_stream@@YAXV__crt_stdio_stream@@@Z 100462b9 f   libucrt:stream.obj
 0001:000452f4       ?__mbrtoc32_utf8@__crt_mbstring@@YAIPA_UPBDIPAU_Mbstatet@@@Z 100462f4 f   libucrt:mbrtoc32.obj
 0001:000454ba       ___dcrt_lowio_ensure_console_output_initialized 100464ba f   libucrt:initcon.obj
 0001:000454d9       ___dcrt_terminate_console_output 100464d9 f   libucrt:initcon.obj
 0001:000454f0       ___dcrt_write_console      100464f0 f   libucrt:initcon.obj
 0001:00045545       _fegetenv                  10046545 f   libucrt:fegetenv.obj
 0001:00045562       _fesetenv                  10046562 f   libucrt:fesetenv.obj
 0001:000455ad       _feholdexcept              100465ad f   libucrt:feholdexcept.obj
 0001:0004571f       __itow_s                   1004671f f   libucrt:xtoa.obj
 0001:00045752       ?__c16rtomb_utf8@__crt_mbstring@@YAIPAD_SPAU_Mbstatet@@@Z 10046752 f   libucrt:c16rtomb.obj
 0001:000457ec       ___acrt_LCMapStringW       100467ec f   libucrt:lcmapstringw.obj
 0001:0004582a       __clearfp                  1004682a f   libucrt:ieee87.obj
 0001:00045910       ___ascii_strnicmp          10046910 f   libucrt:_strnicm.obj
 0001:00045971       _IsProcessorFeaturePresent@4 10046971 f   kernel32:KERNEL32.dll
 0001:00045980       __FindPESection            10046980 f   LIBCMT:pesect.obj
 0001:000459d0       __IsNonwritableInCurrentImage 100469d0 f   LIBCMT:pesect.obj
 0001:00045a90       __ValidateImageBase        10046a90 f   LIBCMT:pesect.obj
 0001:00045ad0       __alldvrm                  10046ad0 f   LIBCMT:lldvrm.obj
 0001:00045bb0       _strrchr                   10046bb0 f   libvcruntime:strrchr.obj
 0001:00045cf0       _strchr                    10046cf0 f   libvcruntime:strchr.obj
 0001:00045d5e       ___from_strstr_to_strchr   10046d5e     libvcruntime:strchr.obj
 0001:00045e1b       __filter_x86_sse2_floating_point_exception_default 10046e1b f   LIBCMT:x86_exception_filter.obj
 0001:00045e1b       __filter_x86_sse2_floating_point_exception 10046e1b f   LIBCMT:x86_exception_filter.obj
 0001:00047248       __TI3?AVbad_array_new_length@std@@ 10048248     format.obj
 0001:00047258       __CTA3?AVbad_array_new_length@std@@ 10048258     format.obj
 0001:00047268       __CT??_R0?AVbad_array_new_length@std@@@8??0bad_array_new_length@std@@QAE@ABV01@@Z12 10048268     format.obj
 0001:00047284       __CT??_R0?AVbad_alloc@std@@@8??0bad_alloc@std@@QAE@ABV01@@Z12 10048284     format.obj
 0001:000472a0       __CT??_R0?AVexception@std@@@8??0exception@std@@QAE@ABV01@@Z12 100482a0     format.obj
 0001:000472bc       __CT??_R0?AVruntime_error@std@@@8??0runtime_error@std@@QAE@ABV01@@Z12 100482bc     format.obj
 0001:000472d8       __TI2?AVruntime_error@std@@ 100482d8     format.obj
 0001:000472e8       __CTA2?AVruntime_error@std@@ 100482e8     format.obj
 0001:000472f4       __TI3?AVformat_error@v6@fmt@@ 100482f4     format.obj
 0001:00047304       __CTA3?AVformat_error@v6@fmt@@ 10048304     format.obj
 0001:00047314       __CT??_R0?AVformat_error@v6@fmt@@@8??0format_error@v6@fmt@@QAE@ABV012@@Z12 10048314     format.obj
 0001:0004852c       __TI2?AVbad_alloc@std@@    1004952c     libcpmt:xthrow.obj
 0001:0004853c       __CTA2?AVbad_alloc@std@@   1004953c     libcpmt:xthrow.obj
 0001:00048548       __CT??_R0?AVlogic_error@std@@@8??0logic_error@std@@QAE@ABV01@@Z12 10049548     libcpmt:xthrow.obj
 0001:00048564       __TI3?AVlength_error@std@@ 10049564     libcpmt:xthrow.obj
 0001:00048574       __CTA3?AVlength_error@std@@ 10049574     libcpmt:xthrow.obj
 0001:00048584       __CT??_R0?AVlength_error@std@@@8??0length_error@std@@QAE@ABV01@@Z12 10049584     libcpmt:xthrow.obj
 0001:000485a0       __TI3?AVout_of_range@std@@ 100495a0     libcpmt:xthrow.obj
 0001:000485b0       __CTA3?AVout_of_range@std@@ 100495b0     libcpmt:xthrow.obj
 0001:000485c0       __CT??_R0?AVout_of_range@std@@@8??0out_of_range@std@@QAE@ABV01@@Z12 100495c0     libcpmt:xthrow.obj
 0001:000485dc       __TI2?AVbad_function_call@std@@ 100495dc     libcpmt:xthrow.obj
 0001:000485ec       __CTA2?AVbad_function_call@std@@ 100495ec     libcpmt:xthrow.obj
 0001:000485f8       __CT??_R0?AVbad_function_call@std@@@8??0bad_function_call@std@@QAE@ABV01@@Z12 100495f8     libcpmt:xthrow.obj
 0001:0004880c       __TI2?AVbad_exception@std@@ 1004980c     libvcruntime:frame.obj
 0001:0004881c       __CTA2?AVbad_exception@std@@ 1004981c     libvcruntime:frame.obj
 0001:00048828       __CT??_R0?AVbad_exception@std@@@8??0bad_exception@std@@QAE@ABV01@@Z12 10049828     libvcruntime:frame.obj
 0002:00000000       ?instantiate_format_float@v6@fmt@@3P6AHNHUfloat_specs@detail@12@AAV?$buffer@D@412@@ZA 1004a000     format.obj
 0002:0000006c       ?pNtQueryInformationProcess@@3P6GJPAXW4_PROCESSINFOCLASS@@0KPAK@ZA 1004a06c     Proclist.obj
 0002:00000070       ?pNtQueryInformationThread@@3P6GJPAXK0KPAK@ZA 1004a070     Proclist.obj
 0002:00000074       ?pNtQueryObject@@3P6GJPAXK0K0@ZA 1004a074     Proclist.obj
 0002:00000078       ?pNtQuerySystemInformation@@3P6GJKPAXKPAK@ZA 1004a078     Proclist.obj
 0002:0000007c       ?pNtQueryInformationFile@@3P6GJPAX00KK@ZA 1004a07c     Proclist.obj
 0002:00000080       ?pNtWow64QueryInformationProcess64@@3P6GJPAXW4_PROCESSINFOCLASS@@0KPAK@ZA 1004a080     Proclist.obj
 0002:00000084       ?pNtWow64ReadVirtualMemory64@@3P6GJPAX_K01PA_K@ZA 1004a084     Proclist.obj
 0002:00000088       ?pIsValidSid@@3P6GHPAX@ZA  1004a088     Proclist.obj
 0002:0000008c       ?pGetSidIdentifierAuthority@@3P6GPAU_SID_IDENTIFIER_AUTHORITY@@PAX@ZA 1004a08c     Proclist.obj
 0002:00000090       ?pGetSidSubAuthorityCount@@3P6GPAEPAX@ZA 1004a090     Proclist.obj
 0002:00000094       ?pGetSidSubAuthority@@3P6GPAKPAXK@ZA 1004a094     Proclist.obj
 0002:00000098       ?pIsWow64Process@@3P6GHPAXPAH@ZA 1004a098     Proclist.obj
 0002:0000009c       ?pGetGuiResources@@3P6GKPAXK@ZA 1004a09c     Proclist.obj
 0002:000000a0       ?pCoSetProxyBlanket@@3P6GJPAUIUnknown@@KKPA_WKKPAXK@ZA 1004a0a0     Proclist.obj
 0002:000000a4       ?pEnumProcessModulesEx@@3P6GHPAXPAPAUHINSTANCE__@@KPAKK@ZA 1004a0a4     Proclist.obj
 0002:000000b8       ___scrt_native_dllmain_reason 1004a0b8     LIBCMT:utility.obj
 0002:000000bc       ___do_unsigned_char_lconv_initialization 1004a0bc     LIBCMT:lconv_unsigned_char.obj
 0002:000000c0       __fltused                  1004a0c0     LIBCMT:fltused.obj
 0002:000000d0       ___security_cookie_complement 1004a0d0     LIBCMT:gs_cookie.obj
 0002:000000d4       ___security_cookie         1004a0d4     LIBCMT:gs_cookie.obj
 0002:000000e0       ___isa_enabled             1004a0e0     LIBCMT:cpu_disp.obj
 0002:00000100       __NLG_Destination          1004a100     libvcruntime:exsup.obj
 0002:00000118       __iob                      1004a118     libucrt:_file.obj
 0002:000001c0       ___acrt_lconv_c            1004a1c0     libucrt:localeconv.obj
 0002:00000210       ___acrt_lconv              1004a210     libucrt:localeconv.obj
 0002:00000214       ___acrt_lconv_static_decimal 1004a214     libucrt:localeconv.obj
 0002:00000218       ___acrt_lconv_static_W_decimal 1004a218     libucrt:localeconv.obj
 0002:00000220       __pctype                   1004a220     libucrt:ctype.obj
 0002:00000224       __pwctype                  1004a224     libucrt:ctype.obj
 0002:00000230       ___abort_behavior          1004a230     libucrt:abort.obj
 0002:00000248       ___acrt_initial_locale_data 1004a248     libucrt:nlsdata.obj
 0002:00000300       ___acrt_initial_locale_pointers 1004a300     libucrt:nlsdata.obj
 0002:00000308       ___acrt_wide_c_locale_string 1004a308     libucrt:nlsdata.obj
 0002:0000030c       ___mb_cur_max              1004a30c     libucrt:nlsdata.obj
 0002:00000320       ___globallocalestatus      1004a320     libucrt:glstatus.obj
 0002:000003b0       ___acrt_initial_multibyte_data 1004a3b0     libucrt:mbctype.obj
 0002:000008d0       __lookuptrailbytes         1004a8d0     libucrt:read.obj
 0002:000009e0       ??_R0?AVbad_array_new_length@std@@@8 1004a9e0     format.obj
 0002:00000a08       ??_R0?AVbad_alloc@std@@@8  1004aa08     format.obj
 0002:00000a24       ??_R0?AVexception@std@@@8  1004aa24     format.obj
 0002:00000a40       ??_R0?AVruntime_error@std@@@8 1004aa40     format.obj
 0002:00000a60       ??_R0?AVformat_error@v6@fmt@@@8 1004aa60     format.obj
 0002:00000a84       ??_R0?AV<lambda_7407d5cd5d4425cb98b7ee1223d84907>@@@8 1004aa84     Plist.obj
 0002:00000abc       ??_R0?AV<lambda_ca95615ebb3c7b16132ff39b7c245039>@@@8 1004aabc     Plist.obj
 0002:00000b9c       ??_R0?AVlogic_error@std@@@8 1004ab9c     libcpmt:xthrow.obj
 0002:00000bbc       ??_R0?AVlength_error@std@@@8 1004abbc     libcpmt:xthrow.obj
 0002:00000bdc       ??_R0?AVout_of_range@std@@@8 1004abdc     libcpmt:xthrow.obj
 0002:00000bfc       ??_R0?AVbad_function_call@std@@@8 1004abfc     libcpmt:xthrow.obj
 0002:00000c20       ??_R0?AV_Facet_base@std@@@8 1004ac20     libcpmt:locale0.obj
 0002:00000c40       ??_R0?AV_Locimp@locale@std@@@8 1004ac40     libcpmt:locale0.obj
 0002:00000c64       ??_R0?AVfacet@locale@std@@@8 1004ac64     libcpmt:locale0.obj
 0002:00000c84       ??_R0?AU_Crt_new_delete@std@@@8 1004ac84     libcpmt:locale0.obj
 0002:00000ca8       ??_R0?AV?$numpunct@_W@std@@@8 1004aca8     libcpmt:wlocale.obj
 0002:00000cc8       ??_R0?AVtype_info@@@8      1004acc8     LIBCMT:std_type_info_static.obj
 0002:00000ce0       ??_R0?AVbad_exception@std@@@8 1004ace0     libvcruntime:frame.obj
 0002:00000d00       ?m_PanelModesDataLocal@Plist@@0V?$vector@Umode@@V?$allocator@Umode@@@std@@@std@@A 1004ad00     fileio.obj
 0002:00000d0c       ?m_PanelModesDataRemote@Plist@@0V?$vector@Umode@@V?$allocator@Umode@@@std@@@std@@A 1004ad0c     fileio.obj
 0002:00000d18       ?_OptionsStorage@?1??__local_stdio_printf_options@@9@4_KA 1004ad18     format.obj
 0002:00000d20       ?id@?$numpunct@_W@std@@2V0locale@2@A 1004ad20     format.obj
 0002:00000d24       ?id@?$numpunct@D@std@@2V0locale@2@A 1004ad24     format.obj
 0002:00000d28       ?_Psave@?$_Facetptr@V?$numpunct@_W@std@@@std@@2PBVfacet@locale@2@B 1004ad28     format.obj
 0002:00001968       ?Info@@3UPluginStartupInfo@@A 1004b968     Proclist.obj
 0002:000019f4       ?Opt@@3Uoptions@@A         1004b9f4     Proclist.obj
 0002:00001a18       ?FSF@@3UFarStandardFunctions@@A 1004ba18     Proclist.obj
 0002:00001aec       ?Ptr@?1???R<lambda_1af49d8e19f959e583a46d83b89ae789>@@QBE@XZ@4PAXA 1004baec     vc_crt_fix_impl.obj
 0002:00001c50       ?_Id_cnt@id@locale@std@@0HA 1004bc50     libcpmt:locale0.obj
 0002:00001c54       ?_Clocptr@_Locimp@locale@std@@0PAV123@A 1004bc54     libcpmt:locale0.obj
 0002:00001c58       ?id@?$ctype@G@std@@2V0locale@2@A 1004bc58     libcpmt:locale0.obj
 0002:00001c5c       ?id@?$codecvt@_WDU_Mbstatet@@@std@@2V0locale@2@A 1004bc5c     libcpmt:locale0.obj
 0002:00001c60       ?id@?$codecvt@GDU_Mbstatet@@@std@@2V0locale@2@A 1004bc60     libcpmt:locale0.obj
 0002:00001c64       ?id@?$ctype@_W@std@@2V0locale@2@A 1004bc64     libcpmt:locale0.obj
 0002:00001c68       ?id@?$ctype@D@std@@2V0locale@2@A 1004bc68     libcpmt:locale0.obj
 0002:00001c84       ?id@?$num_get@DV?$istreambuf_iterator@DU?$char_traits@D@std@@@std@@@std@@2V0locale@2@A 1004bc84     libcpmt:locale.obj
 0002:00001c88       ?id@?$num_put@DV?$ostreambuf_iterator@DU?$char_traits@D@std@@@std@@@std@@2V0locale@2@A 1004bc88     libcpmt:locale.obj
 0002:00001c8c       ?id@?$codecvt@DDU_Mbstatet@@@std@@2V0locale@2@A 1004bc8c     libcpmt:locale.obj
 0002:00001c90       ?_Ptr_cin@std@@3PAV?$basic_istream@DU?$char_traits@D@std@@@1@A 1004bc90     libcpmt:iosptrs.obj
 0002:00001c94       ?_Ptr_cout@std@@3PAV?$basic_ostream@DU?$char_traits@D@std@@@1@A 1004bc94     libcpmt:iosptrs.obj
 0002:00001c98       ?_Ptr_cerr@std@@3PAV?$basic_ostream@DU?$char_traits@D@std@@@1@A 1004bc98     libcpmt:iosptrs.obj
 0002:00001c9c       ?_Ptr_clog@std@@3PAV?$basic_ostream@DU?$char_traits@D@std@@@1@A 1004bc9c     libcpmt:iosptrs.obj
 0002:00001ca0       ?_Ptr_wcin@std@@3PAV?$basic_istream@_WU?$char_traits@_W@std@@@1@A 1004bca0     libcpmt:iosptrs.obj
 0002:00001ca4       ?_Ptr_wcout@std@@3PAV?$basic_ostream@_WU?$char_traits@_W@std@@@1@A 1004bca4     libcpmt:iosptrs.obj
 0002:00001ca8       ?_Ptr_wcerr@std@@3PAV?$basic_ostream@_WU?$char_traits@_W@std@@@1@A 1004bca8     libcpmt:iosptrs.obj
 0002:00001cac       ?_Ptr_wclog@std@@3PAV?$basic_ostream@_WU?$char_traits@_W@std@@@1@A 1004bcac     libcpmt:iosptrs.obj
 0002:00001ce0       ___KERNEL32Functions       1004bce0     libcpmt:winapisupp.obj
 0002:00001d80       ?id@?$time_put@_WV?$ostreambuf_iterator@_WU?$char_traits@_W@std@@@std@@@std@@2V0locale@2@A 1004bd80     libcpmt:wlocale.obj
 0002:00001d84       ?id@?$num_get@_WV?$istreambuf_iterator@_WU?$char_traits@_W@std@@@std@@@std@@2V0locale@2@A 1004bd84     libcpmt:wlocale.obj
 0002:00001d88       ?id@?$num_put@_WV?$ostreambuf_iterator@_WU?$char_traits@_W@std@@@std@@@std@@2V0locale@2@A 1004bd88     libcpmt:wlocale.obj
 0002:00001d8c       ?id@?$collate@_W@std@@2V0locale@2@A 1004bd8c     libcpmt:wlocale.obj
 0002:00001d90       ?id@?$messages@_W@std@@2V0locale@2@A 1004bd90     libcpmt:wlocale.obj
 0002:00001d94       ?id@?$money_get@_WV?$istreambuf_iterator@_WU?$char_traits@_W@std@@@std@@@std@@2V0locale@2@A 1004bd94     libcpmt:wlocale.obj
 0002:00001d98       ?id@?$money_put@_WV?$ostreambuf_iterator@_WU?$char_traits@_W@std@@@std@@@std@@2V0locale@2@A 1004bd98     libcpmt:wlocale.obj
 0002:00001d9c       ?id@?$moneypunct@_W$0A@@std@@2V0locale@2@A 1004bd9c     libcpmt:wlocale.obj
 0002:00001da0       ?id@?$moneypunct@_W$00@std@@2V0locale@2@A 1004bda0     libcpmt:wlocale.obj
 0002:00001da4       ?id@?$time_get@_WV?$istreambuf_iterator@_WU?$char_traits@_W@std@@@std@@@std@@2V0locale@2@A 1004bda4     libcpmt:wlocale.obj
 0002:00001da8       ?id@?$num_get@GV?$istreambuf_iterator@GU?$char_traits@G@std@@@std@@@std@@2V0locale@2@A 1004bda8     libcpmt:wlocale.obj
 0002:00001dac       ?id@?$num_put@GV?$ostreambuf_iterator@GU?$char_traits@G@std@@@std@@@std@@2V0locale@2@A 1004bdac     libcpmt:wlocale.obj
 0002:00001db0       ?id@?$numpunct@G@std@@2V0locale@2@A 1004bdb0     libcpmt:wlocale.obj
 0002:00001db4       ?id@?$collate@G@std@@2V0locale@2@A 1004bdb4     libcpmt:wlocale.obj
 0002:00001db8       ?id@?$messages@G@std@@2V0locale@2@A 1004bdb8     libcpmt:wlocale.obj
 0002:00001dbc       ?id@?$money_get@GV?$istreambuf_iterator@GU?$char_traits@G@std@@@std@@@std@@2V0locale@2@A 1004bdbc     libcpmt:wlocale.obj
 0002:00001dc0       ?id@?$money_put@GV?$ostreambuf_iterator@GU?$char_traits@G@std@@@std@@@std@@2V0locale@2@A 1004bdc0     libcpmt:wlocale.obj
 0002:00001dc4       ?id@?$moneypunct@G$0A@@std@@2V0locale@2@A 1004bdc4     libcpmt:wlocale.obj
 0002:00001dc8       ?id@?$moneypunct@G$00@std@@2V0locale@2@A 1004bdc8     libcpmt:wlocale.obj
 0002:00001dcc       ?id@?$time_get@GV?$istreambuf_iterator@GU?$char_traits@G@std@@@std@@@std@@2V0locale@2@A 1004bdcc     libcpmt:wlocale.obj
 0002:00001dd0       ?id@?$time_put@GV?$ostreambuf_iterator@GU?$char_traits@G@std@@@std@@@std@@2V0locale@2@A 1004bdd0     libcpmt:wlocale.obj
 0002:00001dd4       ?id@?$collate@D@std@@2V0locale@2@A 1004bdd4     libcpmt:xlocale.obj
 0002:00001dd8       ?id@?$messages@D@std@@2V0locale@2@A 1004bdd8     libcpmt:xlocale.obj
 0002:00001ddc       ?id@?$money_get@DV?$istreambuf_iterator@DU?$char_traits@D@std@@@std@@@std@@2V0locale@2@A 1004bddc     libcpmt:xlocale.obj
 0002:00001de0       ?id@?$money_put@DV?$ostreambuf_iterator@DU?$char_traits@D@std@@@std@@@std@@2V0locale@2@A 1004bde0     libcpmt:xlocale.obj
 0002:00001de4       ?id@?$moneypunct@D$0A@@std@@2V0locale@2@A 1004bde4     libcpmt:xlocale.obj
 0002:00001de8       ?id@?$moneypunct@D$00@std@@2V0locale@2@A 1004bde8     libcpmt:xlocale.obj
 0002:00001dec       ?id@?$time_get@DV?$istreambuf_iterator@DU?$char_traits@D@std@@@std@@@std@@2V0locale@2@A 1004bdec     libcpmt:xlocale.obj
 0002:00001df0       ?id@?$time_put@DV?$ostreambuf_iterator@DU?$char_traits@D@std@@@std@@@std@@2V0locale@2@A 1004bdf0     libcpmt:xlocale.obj
 0002:00001df4       ___scrt_current_native_startup_state 1004bdf4     LIBCMT:utility.obj
 0002:00001df8       ___scrt_native_startup_lock 1004bdf8     LIBCMT:utility.obj
 0002:00001e1c       ___isa_available           1004be1c     LIBCMT:cpu_disp.obj
 0002:00001e20       ___favor                   1004be20     LIBCMT:cpu_disp.obj
 0002:00001e24       ___scrt_debugger_hook_flag 1004be24     LIBCMT:utility_desktop.obj
 0002:00001e28       ?__type_info_root_node@@3U__type_info_node@@A 1004be28     LIBCMT:tncleanup.obj
 0002:00001e30       ?_OptionsStorage@?1??__local_stdio_scanf_options@@9@4_KA 1004be30     LIBCMT:default_local_stdio_options.obj
 0002:00002154       ?__WinRTOutOfMemoryExceptionCallback@@3P6GPAXXZA 1004c154     libvcruntime:ehhelpers.obj
 0002:00002158       ___pPurecall               1004c158     libvcruntime:purevirt_data.obj
 0002:000021a0       ?pArgList@UnDecorator@@0PAVReplicator@@A 1004c1a0     libvcruntime:undname.obj
 0002:000021a4       ?pZNameList@UnDecorator@@0PAVReplicator@@A 1004c1a4     libvcruntime:undname.obj
 0002:000021a8       ?pTemplateArgList@UnDecorator@@0PAVReplicator@@A 1004c1a8     libvcruntime:undname.obj
 0002:000021ac       ?gName@UnDecorator@@0PBDB  1004c1ac     libvcruntime:undname.obj
 0002:000021b0       ?name@UnDecorator@@0PBDB   1004c1b0     libvcruntime:undname.obj
 0002:000021b4       ?disableFlags@UnDecorator@@0KA 1004c1b4     libvcruntime:undname.obj
 0002:000021b8       ?fExplicitTemplateParams@UnDecorator@@0_NA 1004c1b8     libvcruntime:undname.obj
 0002:000021b9       ?fGetTemplateArgumentList@UnDecorator@@0_NA 1004c1b9     libvcruntime:undname.obj
 0002:000021bc       ?m_pGetParameter@UnDecorator@@0P6APADJ@ZA 1004c1bc     libvcruntime:undname.obj
 0002:000021c0       ?m_CHPENameOffset@UnDecorator@@0KA 1004c1c0     libvcruntime:undname.obj
 0002:000021c4       ?m_recursionLevel@UnDecorator@@0KA 1004c1c4     libvcruntime:undname.obj
 0002:00002200       __nstream                  1004c200     libucrt:_file.obj
 0002:00002204       ___piob                    1004c204     libucrt:_file.obj
 0002:00002208       ___acrt_lconv_static_null  1004c208     libucrt:localeconv.obj
 0002:0000220c       ___acrt_lconv_static_W_null 1004c20c     libucrt:localeconv.obj
 0002:0000236c       ?c_exit_complete@?1???R<lambda_6e4b09c48022b2350581041d5f6b0c4c>@@QBE@XZ@4_NA 1004c36c     libucrt:exit.obj
 0002:00002478       __environ_table            1004c478     libucrt:environment_initialization.obj
 0002:0000247c       __wenviron_table           1004c47c     libucrt:environment_initialization.obj
 0002:00002480       ___dcrt_initial_wide_environment 1004c480     libucrt:environment_initialization.obj
 0002:00002484       ___dcrt_initial_narrow_environment 1004c484     libucrt:environment_initialization.obj
 0002:00002488       ___acrt_atexit_table       1004c488     libucrt:onexit.obj
 0002:00002494       ___acrt_at_quick_exit_table 1004c494     libucrt:onexit.obj
 0002:00002588       ___pioinfo                 1004c588     libucrt:ioinit.obj
 0002:00002788       __nhandle                  1004c788     libucrt:ioinit.obj
 0002:0000278c       ___acrt_stdout_buffer      1004c78c     libucrt:_sftbuf.obj
 0002:00002790       ___acrt_stderr_buffer      1004c790     libucrt:_sftbuf.obj
 0002:000027a0       ___acrt_locale_changed_data 1004c7a0     libucrt:wsetlocale.obj
 0002:000027a4       ___acrt_current_locale_data 1004c7a4     libucrt:nlsdata.obj
 0002:000027b0       ___fastflag                1004c7b0     libucrt:fp_flags.obj
 0002:000027c4       ?_timezone@@3V?$dual_state_global@J@__crt_state_management@@A 1004c7c4     libucrt:timeset.obj
 0002:000027c8       ?_daylight@@3V?$dual_state_global@H@__crt_state_management@@A 1004c7c8     libucrt:timeset.obj
 0002:000027cc       ?_dstbias@@3V?$dual_state_global@J@__crt_state_management@@A 1004c7cc     libucrt:timeset.obj
 0002:0000288c       __mbctype                  1004c88c     libucrt:mbctype.obj
 0002:00002890       __mbcasemap                1004c890     libucrt:mbctype.obj
 0002:00002894       ___acrt_current_multibyte_data 1004c894     libucrt:mbctype.obj
 0002:000028a0       __pgmptr                   1004c8a0     libucrt:argv_data.obj
 0002:000028a4       ___argc                    1004c8a4     libucrt:argv_data.obj
 0002:000028a8       ___argv                    1004c8a8     libucrt:argv_data.obj
 0002:000028ac       ___wargv                   1004c8ac     libucrt:argv_data.obj
 0002:000028b0       __acmdln                   1004c8b0     libucrt:argv_data.obj
 0002:000028b4       __wcmdln                   1004c8b4     libucrt:argv_data.obj
 0002:000028b8       ___acrt_heap               1004c8b8     libucrt:heap_handle.obj
 0002:000028d4       ___dyn_tls_init_callback   1004c8d4     <common>
 0002:000028d8       ___scrt_ucrt_dll_is_in_use 1004c8d8     <common>
 0002:000028dc       __pmatherr                 1004c8dc     <common>
 0002:000028e0       ___use_sse2_mathfcns       1004c8e0     <common>
 0003:00000000       __imp__AdjustTokenPrivileges@24 1004d000     advapi32:ADVAPI32.dll
 0003:00000004       __imp__LookupPrivilegeValueW@12 1004d004     advapi32:ADVAPI32.dll
 0003:00000008       __imp__DuplicateTokenEx@24 1004d008     advapi32:ADVAPI32.dll
 0003:0000000c       __imp__OpenThreadToken@16  1004d00c     advapi32:ADVAPI32.dll
 0003:00000010       __imp__OpenProcessToken@12 1004d010     advapi32:ADVAPI32.dll
 0003:00000014       __imp__SetThreadToken@8    1004d014     advapi32:ADVAPI32.dll
 0003:00000018       __imp__RegQueryValueExW@24 1004d018     advapi32:ADVAPI32.dll
 0003:0000001c       __imp__RegOpenKeyExW@20    1004d01c     advapi32:ADVAPI32.dll
 0003:00000020       __imp__RegConnectRegistryW@12 1004d020     advapi32:ADVAPI32.dll
 0003:00000024       __imp__RegCloseKey@4       1004d024     advapi32:ADVAPI32.dll
 0003:00000028       __imp__ConvertSidToStringSidW@8 1004d028     advapi32:ADVAPI32.dll
 0003:0000002c       __imp__GetUserNameW@8      1004d02c     advapi32:ADVAPI32.dll
 0003:00000030       __imp__LookupAccountNameW@28 1004d030     advapi32:ADVAPI32.dll
 0003:00000034       \177ADVAPI32_NULL_THUNK_DATA 1004d034     advapi32:ADVAPI32.dll
 0003:00000038       __imp__CreateFileW@28      1004d038     kernel32:KERNEL32.dll
 0003:0000003c       __imp__SetLastError@4      1004d03c     kernel32:KERNEL32.dll
 0003:00000040       __imp__SetEvent@4          1004d040     kernel32:KERNEL32.dll
 0003:00000044       __imp__GetCurrentThreadId@0 1004d044     kernel32:KERNEL32.dll
 0003:00000048       __imp__SetPriorityClass@8  1004d048     kernel32:KERNEL32.dll
 0003:0000004c       __imp__GetPriorityClass@4  1004d04c     kernel32:KERNEL32.dll
 0003:00000050       __imp__GetSystemTimeAsFileTime@4 1004d050     kernel32:KERNEL32.dll
 0003:00000054       __imp__GetLocalTime@4      1004d054     kernel32:KERNEL32.dll
 0003:00000058       __imp__GetTickCount@0      1004d058     kernel32:KERNEL32.dll
 0003:0000005c       __imp__lstrcmpW@8          1004d05c     kernel32:KERNEL32.dll
 0003:00000060       __imp__lstrcpynW@12        1004d060     kernel32:KERNEL32.dll
 0003:00000064       __imp__SystemTimeToTzSpecificLocalTime@12 1004d064     kernel32:KERNEL32.dll
 0003:00000068       __imp__FileTimeToSystemTime@8 1004d068     kernel32:KERNEL32.dll
 0003:0000006c       __imp__ResetEvent@4        1004d06c     kernel32:KERNEL32.dll
 0003:00000070       __imp__ReleaseMutex@4      1004d070     kernel32:KERNEL32.dll
 0003:00000074       __imp__CreateMutexW@12     1004d074     kernel32:KERNEL32.dll
 0003:00000078       __imp__CreateEventW@16     1004d078     kernel32:KERNEL32.dll
 0003:0000007c       __imp__WaitForMultipleObjects@16 1004d07c     kernel32:KERNEL32.dll
 0003:00000080       __imp__GetProcessTimes@20  1004d080     kernel32:KERNEL32.dll
 0003:00000084       __imp__GetLastError@0      1004d084     kernel32:KERNEL32.dll
 0003:00000088       __imp__TerminateProcess@8  1004d088     kernel32:KERNEL32.dll
 0003:0000008c       __imp__GetCurrentThread@0  1004d08c     kernel32:KERNEL32.dll
 0003:00000090       __imp__OpenProcess@12      1004d090     kernel32:KERNEL32.dll
 0003:00000094       __imp__ReadProcessMemory@20 1004d094     kernel32:KERNEL32.dll
 0003:00000098       __imp__FileTimeToLocalFileTime@8 1004d098     kernel32:KERNEL32.dll
 0003:0000009c       __imp__GetModuleHandleW@4  1004d09c     kernel32:KERNEL32.dll
 0003:000000a0       __imp__lstrlenW@4          1004d0a0     kernel32:KERNEL32.dll
 0003:000000a4       __imp__GetDateFormatW@24   1004d0a4     kernel32:KERNEL32.dll
 0003:000000a8       __imp__GetTimeFormatW@24   1004d0a8     kernel32:KERNEL32.dll
 0003:000000ac       __imp__GetProcAddress@8    1004d0ac     kernel32:KERNEL32.dll
 0003:000000b0       __imp__InitializeCriticalSection@4 1004d0b0     kernel32:KERNEL32.dll
 0003:000000b4       __imp__EnterCriticalSection@4 1004d0b4     kernel32:KERNEL32.dll
 0003:000000b8       __imp__LeaveCriticalSection@4 1004d0b8     kernel32:KERNEL32.dll
 0003:000000bc       __imp__DeleteCriticalSection@4 1004d0bc     kernel32:KERNEL32.dll
 0003:000000c0       __imp__GetThreadTimes@20   1004d0c0     kernel32:KERNEL32.dll
 0003:000000c4       __imp__VirtualQuery@12     1004d0c4     kernel32:KERNEL32.dll
 0003:000000c8       __imp__GetModuleFileNameW@12 1004d0c8     kernel32:KERNEL32.dll
 0003:000000cc       __imp__LoadLibraryW@4      1004d0cc     kernel32:KERNEL32.dll
 0003:000000d0       __imp__FlushFileBuffers@4  1004d0d0     kernel32:KERNEL32.dll
 0003:000000d4       __imp__GetProcessHeap@0    1004d0d4     kernel32:KERNEL32.dll
 0003:000000d8       __imp__FreeEnvironmentStringsW@4 1004d0d8     kernel32:KERNEL32.dll
 0003:000000dc       __imp__GetEnvironmentStringsW@0 1004d0dc     kernel32:KERNEL32.dll
 0003:000000e0       __imp__GetCommandLineW@0   1004d0e0     kernel32:KERNEL32.dll
 0003:000000e4       __imp__GetCommandLineA@0   1004d0e4     kernel32:KERNEL32.dll
 0003:000000e8       __imp__GetOEMCP@0          1004d0e8     kernel32:KERNEL32.dll
 0003:000000ec       __imp__GetACP@0            1004d0ec     kernel32:KERNEL32.dll
 0003:000000f0       __imp__IsValidCodePage@4   1004d0f0     kernel32:KERNEL32.dll
 0003:000000f4       __imp__FindNextFileW@8     1004d0f4     kernel32:KERNEL32.dll
 0003:000000f8       __imp__LocalFree@4         1004d0f8     kernel32:KERNEL32.dll
 0003:000000fc       __imp__VirtualFree@12      1004d0fc     kernel32:KERNEL32.dll
 0003:00000100       __imp__VirtualAlloc@16     1004d100     kernel32:KERNEL32.dll
 0003:00000104       __imp__TerminateThread@8   1004d104     kernel32:KERNEL32.dll
 0003:00000108       __imp__CreateThread@24     1004d108     kernel32:KERNEL32.dll
 0003:0000010c       __imp__GetCurrentProcessId@0 1004d10c     kernel32:KERNEL32.dll
 0003:00000110       __imp__GetCurrentProcess@0 1004d110     kernel32:KERNEL32.dll
 0003:00000114       __imp__WaitForSingleObject@8 1004d114     kernel32:KERNEL32.dll
 0003:00000118       __imp__DuplicateHandle@28  1004d118     kernel32:KERNEL32.dll
 0003:0000011c       __imp__CloseHandle@4       1004d11c     kernel32:KERNEL32.dll
 0003:00000120       __imp__WriteFile@20        1004d120     kernel32:KERNEL32.dll
 0003:00000124       __imp__GetFileType@4       1004d124     kernel32:KERNEL32.dll
 0003:00000128       __imp__WriteConsoleW@20    1004d128     kernel32:KERNEL32.dll
 0003:0000012c       __imp__FormatMessageW@28   1004d12c     kernel32:KERNEL32.dll
 0003:00000130       __imp__FindFirstFileExW@24 1004d130     kernel32:KERNEL32.dll
 0003:00000134       __imp__FindClose@4         1004d134     kernel32:KERNEL32.dll
 0003:00000138       __imp__HeapReAlloc@16      1004d138     kernel32:KERNEL32.dll
 0003:0000013c       __imp__GetConsoleMode@8    1004d13c     kernel32:KERNEL32.dll
 0003:00000140       __imp__GetConsoleCP@0      1004d140     kernel32:KERNEL32.dll
 0003:00000144       __imp__SetFilePointerEx@20 1004d144     kernel32:KERNEL32.dll
 0003:00000148       __imp__GetStdHandle@4      1004d148     kernel32:KERNEL32.dll
 0003:0000014c       __imp__EnumSystemLocalesW@8 1004d14c     kernel32:KERNEL32.dll
 0003:00000150       __imp__GetUserDefaultLCID@0 1004d150     kernel32:KERNEL32.dll
 0003:00000154       __imp__IsValidLocale@8     1004d154     kernel32:KERNEL32.dll
 0003:00000158       __imp__HeapFree@12         1004d158     kernel32:KERNEL32.dll
 0003:0000015c       __imp__HeapAlloc@12        1004d15c     kernel32:KERNEL32.dll
 0003:00000160       __imp__ExitProcess@4       1004d160     kernel32:KERNEL32.dll
 0003:00000164       __imp__SetStdHandle@8      1004d164     kernel32:KERNEL32.dll
 0003:00000168       __imp__LoadLibraryExW@12   1004d168     kernel32:KERNEL32.dll
 0003:0000016c       __imp__WideCharToMultiByte@32 1004d16c     kernel32:KERNEL32.dll
 0003:00000170       __imp__MultiByteToWideChar@24 1004d170     kernel32:KERNEL32.dll
 0003:00000174       __imp__InitializeCriticalSectionAndSpinCount@8 1004d174     kernel32:KERNEL32.dll
 0003:00000178       __imp__TlsAlloc@0          1004d178     kernel32:KERNEL32.dll
 0003:0000017c       __imp__TlsGetValue@4       1004d17c     kernel32:KERNEL32.dll
 0003:00000180       __imp__TlsSetValue@8       1004d180     kernel32:KERNEL32.dll
 0003:00000184       __imp__TlsFree@4           1004d184     kernel32:KERNEL32.dll
 0003:00000188       __imp__GetStringTypeW@16   1004d188     kernel32:KERNEL32.dll
 0003:0000018c       __imp__LCMapStringW@24     1004d18c     kernel32:KERNEL32.dll
 0003:00000190       __imp__GetLocaleInfoW@16   1004d190     kernel32:KERNEL32.dll
 0003:00000194       __imp__GetCPInfo@8         1004d194     kernel32:KERNEL32.dll
 0003:00000198       __imp__IsProcessorFeaturePresent@4 1004d198     kernel32:KERNEL32.dll
 0003:0000019c       __imp__IsDebuggerPresent@0 1004d19c     kernel32:KERNEL32.dll
 0003:000001a0       __imp__UnhandledExceptionFilter@4 1004d1a0     kernel32:KERNEL32.dll
 0003:000001a4       __imp__SetUnhandledExceptionFilter@4 1004d1a4     kernel32:KERNEL32.dll
 0003:000001a8       __imp__GetStartupInfoW@4   1004d1a8     kernel32:KERNEL32.dll
 0003:000001ac       __imp__QueryPerformanceCounter@4 1004d1ac     kernel32:KERNEL32.dll
 0003:000001b0       __imp__RaiseException@16   1004d1b0     kernel32:KERNEL32.dll
 0003:000001b4       __imp__RtlUnwind@16        1004d1b4     kernel32:KERNEL32.dll
 0003:000001b8       __imp__FreeLibrary@4       1004d1b8     kernel32:KERNEL32.dll
 0003:000001bc       __imp__HeapSize@12         1004d1bc     kernel32:KERNEL32.dll
 0003:000001c0       \177KERNEL32_NULL_THUNK_DATA 1004d1c0     kernel32:KERNEL32.dll
 0003:000001c4       __imp__WNetAddConnection2W@16 1004d1c4     mpr:MPR.dll
 0003:000001c8       __imp__WNetCancelConnection2W@12 1004d1c8     mpr:MPR.dll
 0003:000001cc       \177MPR_NULL_THUNK_DATA    1004d1cc     mpr:MPR.dll
 0003:000001d0       __imp__VariantClear@4      1004d1d0     oleaut32:OLEAUT32.dll
 0003:000001d4       __imp__SysAllocString@4    1004d1d4     oleaut32:OLEAUT32.dll
 0003:000001d8       __imp__SysFreeString@4     1004d1d8     oleaut32:OLEAUT32.dll
 0003:000001dc       \177OLEAUT32_NULL_THUNK_DATA 1004d1dc     oleaut32:OLEAUT32.dll
 0003:000001e0       __imp__GetModuleInformation@16 1004d1e0     psapi:PSAPI.DLL
 0003:000001e4       __imp__GetModuleFileNameExW@16 1004d1e4     psapi:PSAPI.DLL
 0003:000001e8       \177PSAPI_NULL_THUNK_DATA  1004d1e8     psapi:PSAPI.DLL
 0003:000001ec       __imp__EnumWindows@8       1004d1ec     user32:USER32.dll
 0003:000001f0       __imp__SetForegroundWindow@4 1004d1f0     user32:USER32.dll
 0003:000001f4       __imp__ShowWindowAsync@8   1004d1f4     user32:USER32.dll
 0003:000001f8       __imp__IsWindowVisible@4   1004d1f8     user32:USER32.dll
 0003:000001fc       __imp__GetWindowTextW@12   1004d1fc     user32:USER32.dll
 0003:00000200       __imp__IsIconic@4          1004d200     user32:USER32.dll
 0003:00000204       __imp__GetWindowLongW@8    1004d204     user32:USER32.dll
 0003:00000208       __imp__GetAncestor@8       1004d208     user32:USER32.dll
 0003:0000020c       __imp__GetLastActivePopup@4 1004d20c     user32:USER32.dll
 0003:00000210       __imp__GetWindowThreadProcessId@8 1004d210     user32:USER32.dll
 0003:00000214       __imp__GetParent@4         1004d214     user32:USER32.dll
 0003:00000218       __imp__CharUpperBuffW@8    1004d218     user32:USER32.dll
 0003:0000021c       \177USER32_NULL_THUNK_DATA 1004d21c     user32:USER32.dll
 0003:00000220       __imp__GetFileVersionInfoW@16 1004d220     version:VERSION.dll
 0003:00000224       __imp__VerQueryValueW@16   1004d224     version:VERSION.dll
 0003:00000228       __imp__GetFileVersionInfoSizeW@8 1004d228     version:VERSION.dll
 0003:0000022c       \177VERSION_NULL_THUNK_DATA 1004d22c     version:VERSION.dll
 0003:00000230       __imp__CoInitialize@4      1004d230     ole32:ole32.dll
 0003:00000234       __imp__CoCreateInstance@20 1004d234     ole32:ole32.dll
 0003:00000238       __imp__CoUninitialize@0    1004d238     ole32:ole32.dll
 0003:0000023c       \177ole32_NULL_THUNK_DATA  1004d23c     ole32:ole32.dll
 0003:00000240       ___guard_check_icall_fptr  1004d240     LIBCMT:guard_support.obj
 0003:00000244       __IMPORT_DESCRIPTOR_KERNEL32 1004d244     kernel32:KERNEL32.dll
 0003:00000258       __IMPORT_DESCRIPTOR_USER32 1004d258     user32:USER32.dll
 0003:0000026c       __IMPORT_DESCRIPTOR_ADVAPI32 1004d26c     advapi32:ADVAPI32.dll
 0003:00000280       __IMPORT_DESCRIPTOR_ole32  1004d280     ole32:ole32.dll
 0003:00000294       __IMPORT_DESCRIPTOR_MPR    1004d294     mpr:MPR.dll
 0003:000002a8       __IMPORT_DESCRIPTOR_VERSION 1004d2a8     version:VERSION.dll
 0003:000002bc       __IMPORT_DESCRIPTOR_OLEAUT32 1004d2bc     oleaut32:OLEAUT32.dll
 0003:000002d0       __IMPORT_DESCRIPTOR_PSAPI  1004d2d0     psapi:PSAPI.DLL
 0003:000002e4       __NULL_IMPORT_DESCRIPTOR   1004d2e4     kernel32:KERNEL32.dll

 entry point at        0001:0002ddd5

 Static symbols

 0001:00000004       ?initlocks$initializer$@std@@3P6AXXZA 10001004     libcpmt:xlock.obj
 0001:00000008       ?initlocks$initializer$@std@@3P6AXXZA 10001008     libcpmt:iosptrs.obj
 0001:0000000c       ?init_atexit$initializer$@@3P6AXXZA 1000100c     libcpmt:iosptrs.obj
 0001:00000010       ?_Fac_tidy_reg$initializer$@std@@3P6AXXZA 10001010     libcpmt:locale0.obj
 0001:00000014       ?classic_locale$initializer$@std@@3P6AXXZA 10001014     libcpmt:locale0.obj
 0001:00000018       ??m_PanelModesDataLocal$initializer$@Plist@@0P6AXXZA@@3P6AXXZA 10001018     fileio.obj
 0001:0000001c       ??m_PanelModesDataRemote$initializer$@Plist@@0P6AXXZA@@3P6AXXZA 1000101c     fileio.obj
 0001:00000020       ?hDebugToken$initializer$@@3P6AXXZA 10001020     Plist.obj
 0001:0000002c       ?pinit@@3P6AHXZA           1000102c     libcpmt:winapisupp.obj
 0001:00000030       _pinit                     10001030     LIBCMT:lconv_unsigned_char.obj
 0001:00000960       ?constStrTypes@@3QBQB_WB   10001960     handles.obj
 0001:00000d28       ?StatusCols@?1??InitializePanelModes@Plist@@SAXXZ@4QB_WB 10001d28     Pclass.obj
 0001:00000d38       ?StatusWidths@?1??InitializePanelModes@Plist@@SAXXZ@4QB_WB 10001d38     Pclass.obj
 0001:0000155c       ?invalid_chars@?1??GetFiles@Plist@@QAEHPAUPluginPanelItem@@IHPAPB_W_KAAUoptions@@@Z@4QB_WB 1000255c     Pclass.obj
 0001:00001694       ?PrClasses@?EH@??ProcessKey@Plist@@QAEHPBU_INPUT_RECORD@@@Z@4QBGB 10002694     Pclass.obj
 0001:000016a0       ?Pr@?HF@??ProcessKey@Plist@@QAEHPBU_INPUT_RECORD@@@Z@4QBEB 100026a0     Pclass.obj
 0001:00001f34       ??_7?$_Func_impl_no_alloc@V<lambda_2188c710c02002b0eab1052a0acb7023>@@_NPA_WI@std@@6B@ 10002f34     Plist.obj
 0001:00002140       ??_7?$_Func_impl_no_alloc@V<lambda_8364a2c8b43a2a1256754ccc435293aa>@@XABUtagVARIANT@@@std@@6B@ 10003140     WMI.obj
 0001:00002158       ??_7?$_Func_impl_no_alloc@V<lambda_d3397212bd5e450c6dbd36f327bf5553>@@XABUtagVARIANT@@@std@@6B@ 10003158     WMI.obj
 0001:00002424       ?kernel32@modules@@3QB_WB  10003424     vc_crt_fix_impl.obj
 0001:00002438       ?ntdll@modules@@3QB_WB     10003438     vc_crt_fix_impl.obj
 0001:000029e4       _digits                    100039e4     libcpmt:xstoul.obj
 0001:00002a0c       _ndigs                     10003a0c     libcpmt:xstoul.obj
 0001:00002a34       _digits                    10003a34     libcpmt:xstoull.obj
 0001:00002a5c       _ndigs                     10003a5c     libcpmt:xstoull.obj
 0001:00002a88       ?LcidToLocaleNameTable@@3QBULcidToLocaleName@@B 10003a88     libcpmt:winapinls.obj
 0001:000031a8       ?LocaleNameToIndexTable@@3QBULocaleNameIndex@@B 100041a8     libcpmt:winapinls.obj
 0001:00004b40       two32                      10005b40     LIBCMT:ftol2.obj
 0001:00004b44       two63                      10005b44     LIBCMT:ftol2.obj
 0001:00004b48       _NaN                       10005b48     LIBCMT:ftol2.obj
 0001:00004b50       _GS_ExceptionPointers      10005b50     LIBCMT:gs_report.obj
 0001:00004b78       ?tokenTable@@3QBUStringLiteral@@B 10005b78     libvcruntime:undname.obj
 0001:00004bf8       ?nameTable@@3QBUStringLiteral@@B 10005bf8     libvcruntime:undname.obj
 0001:00004e90       ?rttiTable@@3QBUStringLiteral@@B 10005e90     libvcruntime:undname.obj
 0001:00004eb8       ?IndirectionName@@3QBUStringLiteral@@B 10005eb8     libvcruntime:undname.obj
 0001:00004ee8       ?PrefixName@@3QBUStringLiteral@@B 10005ee8     libvcruntime:undname.obj
 0001:00005510       ?module_names@?A0x1172487b@@3QBQB_WB 10006510     libvcruntime:winapi_downlevel.obj
 0001:000055a4       ?candidate_modules@?1??try_get_FlsAlloc@@YAP6GKP6GXPAX@Z@ZXZ@4QBW4module_id@?A0x1172487b@@B 100065a4     libvcruntime:winapi_downlevel.obj
 0001:000055ac       ?candidate_modules@?1??try_get_FlsFree@@YAP6GHK@ZXZ@4QBW4module_id@?A0x1172487b@@B 100065ac     libvcruntime:winapi_downlevel.obj
 0001:000055b4       ?candidate_modules@?1??try_get_FlsGetValue@@YAP6GPAXK@ZXZ@4QBW4module_id@?A0x1172487b@@B 100065b4     libvcruntime:winapi_downlevel.obj
 0001:000055bc       ?candidate_modules@?1??try_get_FlsSetValue@@YAP6GHKPAX@ZXZ@4QBW4module_id@?A0x1172487b@@B 100065bc     libvcruntime:winapi_downlevel.obj
 0001:000055c4       ?candidate_modules@?1??try_get_InitializeCriticalSectionEx@@YAP6GHPAU_RTL_CRITICAL_SECTION@@KK@ZXZ@4QBW4module_id@?A0x1172487b@@B 100065c4     libvcruntime:winapi_downlevel.obj
 0001:000055d0       ?errtable@@3QBUerrentry@?A0x31fdb9ec@@B 100065d0     libucrt:errno.obj
 0001:00005850       _Mantissa                  10006850     libucrt:modf_pentium4.obj
 0001:00005860       _Bns                       10006860     libucrt:modf_pentium4.obj
 0001:00005870       _Sign                      10006870     libucrt:modf_pentium4.obj
 0001:00005880       _Zero                      10006880     libucrt:modf_pentium4.obj
 0001:00005890       LOG_name                   10006890     libucrt:log10_impl.obj
 0001:000058a0       POW_name                   100068a0     libucrt:pow_impl.obj
 0001:000058b0       _One                       100068b0     libucrt:ceil_pentium4.obj
 0001:000058c0       _Bns                       100068c0     libucrt:ceil_pentium4.obj
 0001:000058d0       _Zero                      100068d0     libucrt:ceil_pentium4.obj
 0001:000058e0       _S                         100068e0     libucrt:ceil_pentium4.obj
 0001:000058f0       _NegZero                   100068f0     libucrt:ceil_pentium4.obj
 0001:00006af8       ___acrt_initializers       10007af8     libucrt:initialization.obj
 0001:00006b78       ?mask@?P@??_d_int@@9@4QBGB 10007b78     libucrt:_test.obj
 0001:00006b98       ?sub@?P@??_d_int@@9@4QBIB  10007b98     libucrt:_test.obj
 0001:00006bb8       ?module_names@?A0x391cf84c@@3QBQB_WB 10007bb8     libucrt:winapi_thunks.obj
 0001:00007000       ?candidate_modules@?1??try_get_AreFileApisANSI@@YAP6GHXZXZ@4QBW4module_id@?A0x391cf84c@@B 10008000     libucrt:winapi_thunks.obj
 0001:00007014       ?candidate_modules@?1??try_get_CompareStringEx@@YAP6GHPB_WK0H0HPAU_nlsversioninfo@@PAXJ@ZXZ@4QBW4module_id@?A0x391cf84c@@B 10008014     libucrt:winapi_thunks.obj
 0001:0000701c       ?candidate_modules@?1??try_get_EnumSystemLocalesEx@@YAP6GHP6GHPA_WKJ@ZKJPAX@ZXZ@4QBW4module_id@?A0x391cf84c@@B 1000801c     libucrt:winapi_thunks.obj
 0001:00007038       ?candidate_modules@?1??try_get_FlsAlloc@@YAP6GKP6GXPAX@Z@ZXZ@4QBW4module_id@?A0x391cf84c@@B 10008038     libucrt:winapi_thunks.obj
 0001:00007040       ?candidate_modules@?1??try_get_FlsFree@@YAP6GHK@ZXZ@4QBW4module_id@?A0x391cf84c@@B 10008040     libucrt:winapi_thunks.obj
 0001:00007048       ?candidate_modules@?1??try_get_FlsGetValue@@YAP6GPAXK@ZXZ@4QBW4module_id@?A0x391cf84c@@B 10008048     libucrt:winapi_thunks.obj
 0001:00007050       ?candidate_modules@?1??try_get_FlsSetValue@@YAP6GHKPAX@ZXZ@4QBW4module_id@?A0x391cf84c@@B 10008050     libucrt:winapi_thunks.obj
 0001:00007058       ?candidate_modules@?1??try_get_GetDateFormatEx@@YAP6GHPB_WKPBU_SYSTEMTIME@@0PA_WH0@ZXZ@4QBW4module_id@?A0x391cf84c@@B 10008058     libucrt:winapi_thunks.obj
 0001:00007070       ?candidate_modules@?1??try_get_GetLocaleInfoEx@@YAP6GHPB_WKPA_WH@ZXZ@4QBW4module_id@?A0x391cf84c@@B 10008070     libucrt:winapi_thunks.obj
 0001:00007078       ?candidate_modules@?1??try_get_GetTimeFormatEx@@YAP6GHPB_WKPBU_SYSTEMTIME@@0PA_WH@ZXZ@4QBW4module_id@?A0x391cf84c@@B 10008078     libucrt:winapi_thunks.obj
 0001:00007090       ?candidate_modules@?1??try_get_GetUserDefaultLocaleName@@YAP6GHPA_WH@ZXZ@4QBW4module_id@?A0x391cf84c@@B 10008090     libucrt:winapi_thunks.obj
 0001:000070b4       ?candidate_modules@?1??try_get_InitializeCriticalSectionEx@@YAP6GHPAU_RTL_CRITICAL_SECTION@@KK@ZXZ@4QBW4module_id@?A0x391cf84c@@B 100080b4     libucrt:winapi_thunks.obj
 0001:000070bc       ?candidate_modules@?1??try_get_IsValidLocaleName@@YAP6GHPB_W@ZXZ@4QBW4module_id@?A0x391cf84c@@B 100080bc     libucrt:winapi_thunks.obj
 0001:000070d8       ?candidate_modules@?1??try_get_LCMapStringEx@@YAP6GHPB_WK0HPA_WHPAU_nlsversioninfo@@PAXJ@ZXZ@4QBW4module_id@?A0x391cf84c@@B 100080d8     libucrt:winapi_thunks.obj
 0001:000070e0       ?candidate_modules@?1??try_get_LCIDToLocaleName@@YAP6GHKPA_WHK@ZXZ@4QBW4module_id@?A0x391cf84c@@B 100080e0     libucrt:winapi_thunks.obj
 0001:000070fc       ?candidate_modules@?1??try_get_LocaleNameToLCID@@YAP6GKPB_WK@ZXZ@4QBW4module_id@?A0x391cf84c@@B 100080fc     libucrt:winapi_thunks.obj
 0001:00007118       ?candidate_modules@?1??try_get_AppPolicyGetProcessTerminationMethod@@YAP6GJPAXPAW4AppPolicyProcessTerminationMethod@@@ZXZ@4QBW4module_id@?A0x391cf84c@@B 10008118     libucrt:winapi_thunks.obj
 0001:00007148       ?strings@?1??fp_format_nan_or_infinity@@YAHW4__acrt_fp_class@@_NPADI1@Z@4QAY03QBDA 10008148     libucrt:cvt.obj
 0001:000071c0       __first_127char            100081c0     libucrt:wsetlocale.obj
 0001:00007810       emask                      10008810     libucrt:log10_pentium4.obj
 0001:00007820       CC                         10008820     libucrt:log10_pentium4.obj
 0001:00007830       Magic                      10008830     libucrt:log10_pentium4.obj
 0001:00007840       hi_mask                    10008840     libucrt:log10_pentium4.obj
 0001:00007850       LOG10_2                    10008850     libucrt:log10_pentium4.obj
 0001:00007860       place_L                    10008860     libucrt:log10_pentium4.obj
 0001:00007880       One                        10008880     libucrt:log10_pentium4.obj
 0001:00007890       Zero                       10008890     libucrt:log10_pentium4.obj
 0001:000078a0       Two52                      100088a0     libucrt:log10_pentium4.obj
 0001:000078b0       Infs                       100088b0     libucrt:log10_pentium4.obj
 0001:000078c0       NaN                        100088c0     libucrt:log10_pentium4.obj
 0001:000078d0       coeff                      100088d0     libucrt:log10_pentium4.obj
 0001:0000792e       _log2max                   1000892e     libucrt:87tran.obj
 0001:00007938       _smallarg                  10008938     libucrt:87tran.obj
 0001:00007942       _half                      10008942     libucrt:87tran.obj
 0001:0000798e       One                        1000898e     libucrt:87disp.obj
 0001:00007996       Three                      10008996     libucrt:87disp.obj
 0001:0000799e       XAMtoTagTab                1000899e     libucrt:87disp.obj
 0001:000079b0       One                        100089b0     libucrt:common.obj
 0001:000079c4       DblMax                     100089c4     libucrt:common.obj
 0001:000079cc       DblMin                     100089cc     libucrt:common.obj
 0001:000079d4       IeeeAdjO                   100089d4     libucrt:common.obj
 0001:000079dc       IeeeAdjU                   100089dc     libucrt:common.obj
 0001:000079e4       _infinity                  100089e4     libucrt:common.obj
 0001:000079ec       _zero                      100089ec     libucrt:common.obj
 0001:00007a00       Shifter                    10008a00     libucrt:pow_pentium4.obj
 0001:00007a10       SIGMASK                    10008a10     libucrt:pow_pentium4.obj
 0001:00007a20       ONEMASK                    10008a20     libucrt:pow_pentium4.obj
 0001:00007a30       ABSVALMASK                 10008a30     libucrt:pow_pentium4.obj
 0001:00007a40       cev                        10008a40     libucrt:pow_pentium4.obj
 0001:00007a68       HALFSIG                    10008a68     libucrt:pow_pentium4.obj
 0001:00007a70       LHN                        10008a70     libucrt:pow_pentium4.obj
 0001:00007a78       sNaN                       10008a78     libucrt:pow_pentium4.obj
 0001:00007a80       INF                        10008a80     libucrt:pow_pentium4.obj
 0001:00007a88       NEG_INF                    10008a88     libucrt:pow_pentium4.obj
 0001:00007a90       NEG_ZERO                   10008a90     libucrt:pow_pentium4.obj
 0001:00007a98       NEG_BIG                    10008a98     libucrt:pow_pentium4.obj
 0001:00007aa0       POS_BIG                    10008aa0     libucrt:pow_pentium4.obj
 0001:00007aa8       EMIN                       10008aa8     libucrt:pow_pentium4.obj
 0001:00007ab0       QIND                       10008ab0     libucrt:pow_pentium4.obj
 0001:00007ac8       ?_names@?1??_get_fname@@9@9 10008ac8     libucrt:fpexcept.obj
 0001:00007c70       _over                      10008c70     libucrt:fpctrl.obj
 0001:00007c7c       _under                     10008c7c     libucrt:fpctrl.obj
 0001:00007c88       ?_mb_locale_names@@3QBQB_WB 10008c88     libucrt:mbctype.obj
 0001:00007c98       ?LcidToLocaleNameTable@?A0x881e4c05@@3QBULcidToLocaleName@1@B 10008c98     libucrt:lcidtoname_downlevel.obj
 0001:000083b8       ?LocaleNameToIndexTable@?A0x881e4c05@@3QBULocaleNameIndex@1@B 100093b8     libucrt:lcidtoname_downlevel.obj
 0001:00008ad8       ?large_power_indices@?1??multiply_by_power_of_ten@__crt_strtox@@YA_NAAUbig_integer@2@I@Z@4QBUunpack_index@?1??12@YA_N0I@Z@B 10009ad8     libucrt:cfout.obj
 0001:0000e390       ??__E?m_PanelModesDataLocal@Plist@@0V?$vector@Umode@@V?$allocator@Umode@@@std@@@std@@A@@YAXXZ 1000f390 f   fileio.obj
 0001:0000e3a0       ??__E?m_PanelModesDataRemote@Plist@@0V?$vector@Umode@@V?$allocator@Umode@@@std@@@std@@A@@YAXXZ 1000f3a0 f   fileio.obj
 0001:0000e3b0       ??__EhDebugToken@@YAXXZ    1000f3b0 f   Plist.obj
 0001:0000e3bc       ??__Einitlocks@std@@YAXXZ  1000f3bc f   libcpmt:xlock.obj
 0001:0000e3d2       ??__E_Fac_tidy_reg@std@@YAXXZ 1000f3d2 f   libcpmt:locale0.obj
 0001:0000e3de       ??__Eclassic_locale@std@@YAXXZ 1000f3de f   libcpmt:locale0.obj
 0001:0000e3ea       ??__Einit_atexit@@YAXXZ    1000f3ea f   libcpmt:iosptrs.obj
 0001:0000e3f6       ??__Einitlocks@std@@YAXXZ  1000f3f6 f   libcpmt:iosptrs.obj
 0001:0000e410       $$000000                   1000f410     chkstk.obj
 0001:00010430       $LN118                     10011430     format.obj
 0001:00010674       $LN64                      10011674     format.obj
 0001:00012f04       $LN65                      10013f04     handles.obj
 0001:00012fd4       $LN65                      10013fd4     handles.obj
 0001:00013360       $LN93                      10014360     handles.obj
 0001:0001337c       $LN92                      1001437c     handles.obj
 0001:00013668       $LN93                      10014668     handles.obj
 0001:00013684       $LN92                      10014684     handles.obj
 0001:00013e88       $LN17                      10014e88     handles.obj
 0001:00013eb4       $LN16                      10014eb4     handles.obj
 0001:00014894       $LN135                     10015894     handles.obj
 0001:000148a0       $LN134                     100158a0     handles.obj
 0001:00015324       $LN199                     10016324     handles.obj
 0001:00015994       $LN191                     10016994     handles.obj
 0001:00017ec0       ??R<lambda_890e54932aec59752afe9828b9159bfd>@@QBEPA_WPA_W@Z 10018ec0 f   handles.obj
 0001:00017f10       ??R<lambda_c3630acb37279cf92411e07a2b271fdf>@@QBE?AV?$basic_string@_WU?$char_traits@_W@std@@V?$allocator@_W@2@@std@@XZ 10018f10 f   handles.obj
 0001:00018120       ??R<lambda_d7ff147dc01dcbc9a9a648dbdce06a58>@@QBE_NV?$basic_string_view@_WU?$char_traits@_W@std@@@std@@0@Z 10019120 f   handles.obj
 0001:00018290       ?GetFileNameThread@test@?4??GetFileName@@YA?AV?$basic_string@_WU?$char_traits@_W@std@@V?$allocator@_W@2@@std@@PAX@Z@SGK0@Z 10019290 f   handles.obj
 0001:000182c0       ?GetNameByType@@YA?AV?$basic_string@_WU?$char_traits@_W@std@@V?$allocator@_W@2@@std@@PAXGPAVPerfThread@@@Z 100192c0 f   handles.obj
 0001:00018894       $LN450                     10019894     handles.obj
 0001:00018fc0       ?duplicate_handle@@YA?AV?$unique_ptr@XUhandle_closer@@@std@@PAXK@Z 10019fc0 f   handles.obj
 0001:00019b60       ?query_object@@YA?AV?$unique_ptr@$$BY0A@DU?$default_delete@$$BY0A@D@std@@@std@@PAXW4OBJECT_INFORMATION_CLASS@@@Z 1001ab60 f   handles.obj
 0001:0001a2cc       $LN47                      1001b2cc     Pcfg.obj
 0001:0001a2dc       $LN46                      1001b2dc     Pcfg.obj
 0001:0001a84c       $LN14                      1001b84c     Pcfg.obj
 0001:0001a85c       $LN13                      1001b85c     Pcfg.obj
 0001:0001ae0c       $LN70                      1001be0c     Pcfg.obj
 0001:0001ae1c       $LN69                      1001be1c     Pcfg.obj
 0001:0001cd40       $LN271                     1001dd40     Pclass.obj
 0001:0001faa4       $LN766                     10020aa4     Pclass.obj
 0001:0001fab8       $LN765                     10020ab8     Pclass.obj
 0001:0001fad0       $LN769                     10020ad0     Pclass.obj
 0001:0001faf0       $LN768                     10020af0     Pclass.obj
 0001:000219b0       ?PrintTitle@@YA?AV?$basic_string@_WU?$char_traits@_W@std@@V?$allocator@_W@2@@std@@H@Z 100229b0 f   Pclass.obj
 0001:00021a10       ?PrintTitle@@YA?AV?$basic_string@_WU?$char_traits@_W@std@@V?$allocator@_W@2@@std@@V?$basic_string_view@_WU?$char_traits@_W@std@@@2@@Z 10022a10 f   Pclass.obj
 0001:000234d8       $LN1062                    100244d8     Pclass.obj
 0001:000234e8       $LN1061                    100244e8     Pclass.obj
 0001:000238b0       ?TranslateMode@@YA_NABV?$basic_string@_WU?$char_traits@_W@std@@V?$allocator@_W@2@@std@@AAV12@@Z 100248b0 f   Pclass.obj
 0001:00024040       $LN480                     10025040     Pclass.obj
 0001:00024048       $LN479                     10025048     Pclass.obj
 0001:00024060       $LN482                     10025060     Pclass.obj
 0001:00024068       $LN481                     10025068     Pclass.obj
 0001:00024690       ?convert_panel_modes@@YAXABV?$vector@Umode@@V?$allocator@Umode@@@std@@@std@@AAV?$array@UPanelMode@@$09@2@@Z 10025690 f   Pclass.obj
 0001:00024730       ?generate_titles@@YAXABV?$basic_string@_WU?$char_traits@_W@std@@V?$allocator@_W@2@@std@@AAUPanelMode@@@Z 10025730 f   Pclass.obj
 0001:0002492c       $LN86                      1002592c     Pclass.obj
 0001:00024940       $LN85                      10025940     Pclass.obj
 0001:00024958       $LN88                      10025958     Pclass.obj
 0001:00024978       $LN87                      10025978     Pclass.obj
 0001:00024d90       ?ui64toa_width@@YA?AV?$basic_string@_WU?$char_traits@_W@std@@V?$allocator@_W@2@@std@@_KI_N@Z 10025d90 f   Pclass.obj
 0001:00025260       ?window_ex_style@@YA@PAUHWND__@@@Z 10026260 f   Pclass.obj
 0001:000255f0       ?window_style@@YA@PAUHWND__@@@Z 100265f0 f   Pclass.obj
 0001:00027c50       ??$print_module@PAX@@YAXQAXPAXKAAUoptions@@ABV?$function@$$A6A_NPA_WI@Z@std@@@Z 10028c50 f   Plist.obj
 0001:00028120       ??R<lambda_dfa89da47ba22f95c142cf8e3e15cf1d>@@QBEXXZ 10029120 f   Plist.obj
 0001:000282e0       ?FreeUserData@@YGXQAXQBUFarPanelItemFreeInfo@@@Z 100292e0 f   Plist.obj
 0001:00029c50       ?_Copy@?$_Func_impl_no_alloc@V<lambda_2188c710c02002b0eab1052a0acb7023>@@_NPA_WI@std@@EBEPAV?$_Func_base@_NPA_WI@2@PAX@Z 1002ac50 f   Plist.obj
 0001:00029c50       ?_Move@?$_Func_impl_no_alloc@V<lambda_2188c710c02002b0eab1052a0acb7023>@@_NPA_WI@std@@EAEPAV?$_Func_base@_NPA_WI@2@PAX@Z 1002ac50 f   Plist.obj
 0001:00029cb0       ?_Delete_this@?$_Func_impl_no_alloc@V<lambda_2188c710c02002b0eab1052a0acb7023>@@_NPA_WI@std@@EAEX_N@Z 1002acb0 f   Plist.obj
 0001:00029cd0       ?_Do_call@?$_Func_impl_no_alloc@V<lambda_2188c710c02002b0eab1052a0acb7023>@@_NPA_WI@std@@EAE_N$$QAPA_W$$QAI@Z 1002acd0 f   Plist.obj
 0001:00029da0       ?_Get@?$_Func_impl_no_alloc@V<lambda_2188c710c02002b0eab1052a0acb7023>@@_NPA_WI@std@@EBEPBXXZ 1002ada0 f   Plist.obj
 0001:00029da0       ?_Get@?$_Func_impl_no_alloc@V<lambda_8364a2c8b43a2a1256754ccc435293aa>@@XABUtagVARIANT@@@std@@EBEPBXXZ 1002ada0 f   WMI.obj
 0001:00029da0       ?_Get@?$_Func_impl_no_alloc@V<lambda_d3397212bd5e450c6dbd36f327bf5553>@@XABUtagVARIANT@@@std@@EBEPBXXZ 1002ada0 f   WMI.obj
 0001:00029db0       ?_Target_type@?$_Func_impl_no_alloc@V<lambda_2188c710c02002b0eab1052a0acb7023>@@_NPA_WI@std@@EBEABVtype_info@@XZ 1002adb0 f   Plist.obj
 0001:00029e40       ?is_wow64_itself@@YA_NXZ   1002ae40 f   Plist.obj
 0001:00029eb0       ?print_module_impl@@YAXQAXABV?$basic_string@_WU?$char_traits@_W@std@@V?$allocator@_W@2@@std@@KABUoptions@@ABV?$function@$$A6A_NPA_WI@Z@2@@Z 1002aeb0 f   Plist.obj
 0001:0002b5a0       ?ProcessPath@@YA@K@Z       1002c5a0 f   WMI.obj
 0001:0002b690       ?_Copy@?$_Func_impl_no_alloc@V<lambda_8364a2c8b43a2a1256754ccc435293aa>@@XABUtagVARIANT@@@std@@EBEPAV?$_Func_base@XABUtagVARIANT@@@2@PAX@Z 1002c690 f   WMI.obj
 0001:0002b690       ?_Move@?$_Func_impl_no_alloc@V<lambda_8364a2c8b43a2a1256754ccc435293aa>@@XABUtagVARIANT@@@std@@EAEPAV?$_Func_base@XABUtagVARIANT@@@2@PAX@Z 1002c690 f   WMI.obj
 0001:0002b6b0       ?_Copy@?$_Func_impl_no_alloc@V<lambda_d3397212bd5e450c6dbd36f327bf5553>@@XABUtagVARIANT@@@std@@EBEPAV?$_Func_base@XABUtagVARIANT@@@2@PAX@Z 1002c6b0 f   WMI.obj
 0001:0002b6b0       ?_Move@?$_Func_impl_no_alloc@V<lambda_d3397212bd5e450c6dbd36f327bf5553>@@XABUtagVARIANT@@@std@@EAEPAV?$_Func_base@XABUtagVARIANT@@@2@PAX@Z 1002c6b0 f   WMI.obj
 0001:0002b6d0       ?_Delete_this@?$_Func_impl_no_alloc@V<lambda_8364a2c8b43a2a1256754ccc435293aa>@@XABUtagVARIANT@@@std@@EAEX_N@Z 1002c6d0 f   WMI.obj
 0001:0002b6d0       ?_Delete_this@?$_Func_impl_no_alloc@V<lambda_d3397212bd5e450c6dbd36f327bf5553>@@XABUtagVARIANT@@@std@@EAEX_N@Z 1002c6d0 f   WMI.obj
 0001:0002b6f0       ?_Do_call@?$_Func_impl_no_alloc@V<lambda_8364a2c8b43a2a1256754ccc435293aa>@@XABUtagVARIANT@@@std@@EAEXABUtagVARIANT@@@Z 1002c6f0 f   WMI.obj
 0001:0002b710       ?_Do_call@?$_Func_impl_no_alloc@V<lambda_d3397212bd5e450c6dbd36f327bf5553>@@XABUtagVARIANT@@@std@@EAEXABUtagVARIANT@@@Z 1002c710 f   WMI.obj
 0001:0002b750       ?_Target_type@?$_Func_impl_no_alloc@V<lambda_8364a2c8b43a2a1256754ccc435293aa>@@XABUtagVARIANT@@@std@@EBEABVtype_info@@XZ 1002c750 f   WMI.obj
 0001:0002b760       ?_Target_type@?$_Func_impl_no_alloc@V<lambda_d3397212bd5e450c6dbd36f327bf5553>@@XABUtagVARIANT@@@std@@EBEABVtype_info@@XZ 1002c760 f   WMI.obj
 0001:0002b770       ?fNtQueryInformationFile@@YGJPAX00KK@Z 1002c770 f   Proclist.obj
 0001:0002b770       ?fNtQueryInformationProcess@@YGJPAXW4_PROCESSINFOCLASS@@0KPAK@Z 1002c770 f   Proclist.obj
 0001:0002b770       ?fNtQueryInformationThread@@YGJPAXK0KPAK@Z 1002c770 f   Proclist.obj
 0001:0002b770       ?fNtQueryObject@@YGJPAXK0K0@Z 1002c770 f   Proclist.obj
 0001:0002b770       ?fNtWow64QueryInformationProcess64@@YGJPAXW4_PROCESSINFOCLASS@@0KPAK@Z 1002c770 f   Proclist.obj
 0001:0002b780       ?fNtQuerySystemInformation@@YGJKPAXKPAK@Z 1002c780 f   Proclist.obj
 0001:0002b790       ?fNtWow64ReadVirtualMemory64@@YGJPAX_K01PA_K@Z 1002c790 f   Proclist.obj
 0001:0002b7a0       ?fGetGuiResources@@YGKPAXK@Z 1002c7a0 f   Proclist.obj
 0001:0002b7a0       ?fGetSidSubAuthority@@YGPAKPAXK@Z 1002c7a0 f   Proclist.obj
 0001:0002b7a0       ?fIsWow64Process@@YGHPAXPAH@Z 1002c7a0 f   Proclist.obj
 0001:0002b7b0       ?fGetSidIdentifierAuthority@@YGPAU_SID_IDENTIFIER_AUTHORITY@@PAX@Z 1002c7b0 f   Proclist.obj
 0001:0002b7b0       ?fGetSidSubAuthorityCount@@YGPAEPAX@Z 1002c7b0 f   Proclist.obj
 0001:0002b7b0       ?fIsValidSid@@YGHPAX@Z     1002c7b0 f   Proclist.obj
 0001:0002b7c0       ?fCoSetProxyBlanket@@YGJPAUIUnknown@@KKPA_WKKPAXK@Z 1002c7c0 f   Proclist.obj
 0001:0002b7d0       ?fEnumProcessModulesEx@@YGHPAXPAPAUHINSTANCE__@@KPAKK@Z 1002c7d0 f   Proclist.obj
 0001:0002b810       ?dynamic_bind@@YAXXZ       1002c810 f   Proclist.obj
 0001:0002bd10       ?DecodePointer@implementation@?1??DecodePointerWrapper@@YGPAXPAX@Z@SGPAX0@Z 1002cd10 f   vc_crt_fix_impl.obj
 0001:0002bd10       ?EncodePointer@implementation@?1??EncodePointerWrapper@@YGPAXPAX@Z@SGPAX0@Z 1002cd10 f   vc_crt_fix_impl.obj
 0001:0002bd20       ?GetLogicalProcessorInformation@implementation@?1??GetLogicalProcessorInformationWrapper@@YGHPAU_SYSTEM_LOGICAL_PROCESSOR_INFORMATION@@PAK@Z@SGH01@Z 1002cd20 f   vc_crt_fix_impl.obj
 0001:0002bd30       ?GetModuleHandleExW@implementation@?1??GetModuleHandleExWWrapper@@YGHKPB_WPAPAUHINSTANCE__@@@Z@SGHK01@Z 1002cd30 f   vc_crt_fix_impl.obj
 0001:0002be00       ?GetNumaHighestNodeNumber@implementation@?1??GetNumaHighestNodeNumberWrapper@@YGHPAK@Z@SGH0@Z 1002ce00 f   vc_crt_fix_impl.obj
 0001:0002be20       ?InitializeSListHead@implementation@slist@@YGXPAT_SLIST_HEADER@@@Z 1002ce20 f   vc_crt_fix_impl.obj
 0001:0002bee0       ?InterlockedFlushSList@implementation@slist@@YGPAU_SINGLE_LIST_ENTRY@@PAT_SLIST_HEADER@@@Z 1002cee0 f   vc_crt_fix_impl.obj
 0001:0002bf10       ?InterlockedPopEntrySList@implementation@slist@@YGPAU_SINGLE_LIST_ENTRY@@PAT_SLIST_HEADER@@@Z 1002cf10 f   vc_crt_fix_impl.obj
 0001:0002bf60       ?InterlockedPushEntrySList@implementation@slist@@YGPAU_SINGLE_LIST_ENTRY@@PAT_SLIST_HEADER@@PAU3@@Z 1002cf60 f   vc_crt_fix_impl.obj
 0001:0002bfa0       ?InterlockedPushListSListEx@implementation@slist@@YGPAU_SINGLE_LIST_ENTRY@@PAT_SLIST_HEADER@@PAU3@1K@Z 1002cfa0 f   vc_crt_fix_impl.obj
 0001:0002bfe0       ?QueryDepthSList@implementation@slist@@YGGPAT_SLIST_HEADER@@@Z 1002cfe0 f   vc_crt_fix_impl.obj
 0001:0002c010       ?RtlFirstEntrySList@implementation@slist@@YGPAU_SINGLE_LIST_ENTRY@@PAT_SLIST_HEADER@@@Z 1002d010 f   vc_crt_fix_impl.obj
 0001:0002c040       ?SetThreadStackGuarantee@implementation@?1??SetThreadStackGuaranteeWrapper@@YGHPAK@Z@SGH0@Z 1002d040 f   vc_crt_fix_impl.obj
 0001:0002c050       ?XorPointer@@YAPAXPAX@Z    1002d050 f   vc_crt_fix_impl.obj
 0001:0002ca8e       _tidy_global               1002da8e f   libcpmt:locale0.obj
 0001:0002cc5d       __Utf8_trailing_byte_count 1002dc5d f   libcpmt:xmbtowc.obj
 0001:0002cd87       ?initialize_pointers@@YAHXZ 1002dd87 f   libcpmt:winapisupp.obj
 0001:0002d0a2       ?find_pe_section@@YAPAU_IMAGE_SECTION_HEADER@@QAEI@Z 1002e0a2 f   LIBCMT:utility.obj
 0001:0002d3f0       $$000000                   1002e3f0     LIBCMT:llmul.obj
 0001:0002d430       $$000000                   1002e430     LIBCMT:llshl.obj
 0001:0002d450       $$000000                   1002e450     LIBCMT:ullshr.obj
 0001:0002d5c0       $$000000                   1002e5c0     LIBCMT:ulldiv.obj
 0001:0002d630       $$000000                   1002e630     LIBCMT:ulldvrm.obj
 0001:0002d6d0       $$000000                   1002e6d0     LIBCMT:ullrem.obj
 0001:0002d750       $$000000                   1002e750     LIBCMT:ftol2.obj
 0001:0002d9f0       $$000000                   1002e9f0     LIBCMT:lldiv.obj
 0001:0002da9a       ?dllmain_crt_dispatch@@YGHQAUHINSTANCE__@@KQAX@Z 1002ea9a f   LIBCMT:dll_dllmain.obj
 0001:0002daed       ?dllmain_crt_process_attach@@YAHQAUHINSTANCE__@@QAX@Z 1002eaed f   LIBCMT:dll_dllmain.obj
 0001:0002dbf4       ?dllmain_crt_process_detach@@YAH_N@Z 1002ebf4 f   LIBCMT:dll_dllmain.obj
 0001:0002dca4       ?dllmain_dispatch@@YAHQAUHINSTANCE__@@KQAX@Z 1002eca4 f   LIBCMT:dll_dllmain.obj
 0001:0002ddaa       ?dllmain_raw@@YGHQAUHINSTANCE__@@KQAX@Z 1002edaa f   LIBCMT:dll_dllmain.obj
 0001:0002dee0       $$000000                   1002eee0     LIBCMT:alloca16.obj
 0001:0002e220       $$000000                   1002f220     LIBCMT:sehprolg4.obj
 0001:0002e298       ___get_entropy             1002f298 f   LIBCMT:gs_support.obj
 0001:0002e69a       ?_FilterSetCurrentException@@YAKPAU_EXCEPTION_POINTERS@@E@Z 1002f69a f   libvcruntime:ehhelpers.obj
 0001:0002ec40       $$000000                   1002fc40     libvcruntime:memchr.obj
 0001:0002ecf0       $$000000                   1002fcf0     libvcruntime:memcpy.obj
 0001:0002ef54       TrailingUpVec              1002ff54     libvcruntime:memcpy.obj
 0001:0002f000       TrailingDownVec            10030000     libvcruntime:memcpy.obj
 0001:0002f270       $$000000                   10030270     libvcruntime:memmove.obj
 0001:0002f4d4       TrailingUpVec              100304d4     libvcruntime:memmove.obj
 0001:0002f580       TrailingDownVec            10030580     libvcruntime:memmove.obj
 0001:0002f7f0       $$000000                   100307f0     libvcruntime:memset.obj
 0001:00030935       $LN1241                    10031935     libvcruntime:memcmp.obj
 0001:00030a10       _ValidateLocalCookies      10031a10 f   libvcruntime:chandler4.obj
 0001:00030d4d       ??$BuildCatchObjectHelperInternal@V__FrameHandler3@@@@YAHPAUEHExceptionRecord@@PAXPBU_s_HandlerType@@PBU_s_CatchableType@@@Z 10031d4d f   libvcruntime:frame.obj
 0001:00030e8b       ??$BuildCatchObjectInternal@V__FrameHandler3@@@@YAXPAUEHExceptionRecord@@PAXPBU_s_HandlerType@@PBU_s_CatchableType@@@Z 10031e8b f   libvcruntime:frame.obj
 0001:00030f24       ??$CatchIt@V__FrameHandler3@@@@YAXPAUEHExceptionRecord@@PAUEHRegistrationNode@@PAU_CONTEXT@@PAXPBU_s_FuncInfo@@PBU_s_HandlerType@@PBU_s_CatchableType@@PBU_s_TryBlockMapEntry@@H1EE@Z 10031f24 f   libvcruntime:frame.obj
 0001:00030fa4       ??$FindHandler@V__FrameHandler3@@@@YAXPAUEHExceptionRecord@@PAUEHRegistrationNode@@PAU_CONTEXT@@PAXPBU_s_FuncInfo@@EH1@Z 10031fa4 f   libvcruntime:frame.obj
 0001:0003135a       ??$FindHandlerForForeignException@V__FrameHandler3@@@@YAXPAUEHExceptionRecord@@PAUEHRegistrationNode@@PAU_CONTEXT@@PAXPBU_s_FuncInfo@@HH1@Z 1003235a f   libvcruntime:frame.obj
 0001:00031672       ?CallCatchBlock@@YAPAXPAUEHExceptionRecord@@PAUEHRegistrationNode@@PAU_CONTEXT@@PBU_s_FuncInfo@@PAXHK@Z 10032672 f   libvcruntime:frame.obj
 0001:00031836       ?CallUnexpected@@YAXPBU_s_ESTypeList@@@Z 10032836 f   libvcruntime:frame.obj
 0001:00031856       __catch$?CallUnexpected@@YAXPBU_s_ESTypeList@@@Z$0 10032856 f   libvcruntime:frame.obj
 0001:00031870       ?ExFilterRethrow@@YAHPAU_EXCEPTION_POINTERS@@@Z 10032870 f   libvcruntime:frame.obj
 0001:000319ba       ?IsInExceptionSpec@@YAEPAUEHExceptionRecord@@PBU_s_ESTypeList@@@Z 100329ba f   libvcruntime:frame.obj
 0001:00031a90       $$000000                   10032a90     libvcruntime:lowhelpr.obj
 0001:00031bb0       $$000000                   10032bb0     libvcruntime:exsup4.obj
 0001:00031c40       __unwind_handler4          10032c40 f   libvcruntime:exsup4.obj
 0001:00031d17       ?try_get_first_available_module@@YAPAUHINSTANCE__@@QBW4module_id@?A0x1172487b@@0@Z 10032d17 f   libvcruntime:winapi_downlevel.obj
 0001:00031dc3       ?try_get_function@@YAPAXW4function_id@?A0x1172487b@@QBDQBW4module_id@2@2@Z 10032dc3 f   libvcruntime:winapi_downlevel.obj
 0001:00031f90       $$000000                   10032f90     libvcruntime:exsup.obj
 0001:00031fb1       __unwind_handler           10032fb1 f   libvcruntime:exsup.obj
 0001:00032545       ??$common_vsnprintf_s@D@@YAH_KQADIIQBDQAU__crt_locale_pointers@@1@Z 10033545 f   libucrt:output.obj
 0001:0003262d       ??$common_vsprintf@Vformat_validation_base@__crt_stdio_output@@D@@YAH_KQADIQBDQAU__crt_locale_pointers@@1@Z 1003362d f   libucrt:output.obj
 0001:00032d82       $LN51                      10033d82     libucrt:output.obj
 0001:00033291       $LN20                      10034291     libucrt:output.obj
 0001:000332a5       $LN17                      100342a5     libucrt:output.obj
 0001:00033df0       $$000000                   10034df0     libucrt:modf_pentium4.obj
 0001:000340f0       $$000000                   100350f0     libucrt:log10_impl.obj
 0001:00034200       $$000000                   10035200     libucrt:pow_impl.obj
 0001:00034450       $$000000                   10035450     libucrt:ceil_pentium4.obj
 0001:00034624       ??$?RV<lambda_646e26742ed01d5bc03234f44bb6d3d3>@@AAV<lambda_b37934c380d97b75fd242ea49540127a>@@V<lambda_bbd9d45274666fbb50f81a29ad795c13>@@@?$__crt_seh_guarded_call@PAD@@QAEPAD$$QAV<lambda_646e26742ed01d5bc03234f44bb6d3d3>@@AAV<lambda_b37934c380d97b75fd242ea49540127a>@@$$QAV<lambda_bbd9d45274666fbb50f81a29ad795c13>@@@Z 10035624 f   libucrt:setlocale.obj
 0001:0003467f       ??R<lambda_b37934c380d97b75fd242ea49540127a>@@QBEPADXZ 1003567f f   libucrt:setlocale.obj
 0001:000347e3       _call_wsetlocale           100357e3 f   libucrt:setlocale.obj
 0001:00035313       _memcpy_s                  10036313 f   libucrt:cfout.obj
 0001:00035313       _memcpy_s                  10036313 f   libucrt:strtod.obj
 0001:00035313       _memcpy_s                  10036313 f   libucrt:mbctype.obj
 0001:000353a0       $$000000                   100363a0     libucrt:strcspn.obj
 0001:00035489       ??$__acrt_convert_wcs_mbs_cp@D_WV<lambda_62f6974d9771e494a5ea317cc32e971c>@@U__crt_win32_buffer_internal_dynamic_resizing@@@@YAHQBDAAV?$__crt_win32_buffer@_WU__crt_win32_buffer_internal_dynamic_resizing@@@@ABV<lambda_62f6974d9771e494a5ea317cc32e971c>@@I@Z 10036489 f   libucrt:strftime.obj
 0001:00035ad5       ??$?RV<lambda_03b1d95aef87969028cfba75ccab2455>@@AAV<lambda_6e4b09c48022b2350581041d5f6b0c4c>@@V<lambda_22bdf7517842c4b3e53723af5aa32b9e>@@@?$__crt_seh_guarded_call@X@@QAEX$$QAV<lambda_03b1d95aef87969028cfba75ccab2455>@@AAV<lambda_6e4b09c48022b2350581041d5f6b0c4c>@@$$QAV<lambda_22bdf7517842c4b3e53723af5aa32b9e>@@@Z 10036ad5 f   libucrt:exit.obj
 0001:00035b22       ??R<lambda_6e4b09c48022b2350581041d5f6b0c4c>@@QBE@XZ 10036b22 f   libucrt:exit.obj
 0001:00035bfc       ?atexit_exception_filter@@YAHK@Z 10036bfc f   libucrt:exit.obj
 0001:00035c0f       ?common_exit@@YAXHW4_crt_exit_cleanup_mode@@W4_crt_exit_return_mode@@@Z 10036c0f f   libucrt:exit.obj
 0001:00035c73       ?exit_or_terminate_process@@YAXI@Z 10036c73 f   libucrt:exit.obj
 0001:00035cb5       ?is_managed_app@@YA_NXZ    10036cb5 f   libucrt:exit.obj
 0001:00035cf8       ?try_cor_exit_process@@YAXI@Z 10036cf8 f   libucrt:exit.obj
 0001:00035d86       ??$common_configure_argv@D@@YAHW4_crt_argv_mode@@@Z 10036d86 f   libucrt:argv_parsing.obj
 0001:00035ebc       ??$parse_command_line@D@@YAXPADPAPAD0PAI2@Z 10036ebc f   libucrt:argv_parsing.obj
 0001:0003608d       ??$common_initialize_environment_nolock@D@@YAHXZ 1003708d f   libucrt:environment_initialization.obj
 0001:000360e0       ??$create_environment@D@@YAQAPADQAD@Z 100370e0 f   libucrt:environment_initialization.obj
 0001:000361b0       ??$free_environment@D@@YAXQAPAD@Z 100371b0 f   libucrt:environment_initialization.obj
 0001:000361b0       ??$free_environment@_W@@YAXQAPA_W@Z 100371b0 f   libucrt:environment_initialization.obj
 0001:00036208       ??$uninitialize_environment_internal@D@@YAXAAPAPAD@Z 10037208 f   libucrt:environment_initialization.obj
 0001:00036223       ??$uninitialize_environment_internal@_W@@YAXAAPAPA_W@Z 10037223 f   libucrt:environment_initialization.obj
 0001:0003627a       ??$?RV<lambda_69a2805e680e0e292e8ba93315fe43a8>@@AAV<lambda_f03950bc5685219e0bcd2087efbe011e>@@V<lambda_03fcd07e894ec930e3f35da366ca99d6>@@@?$__crt_seh_guarded_call@H@@QAEH$$QAV<lambda_69a2805e680e0e292e8ba93315fe43a8>@@AAV<lambda_f03950bc5685219e0bcd2087efbe011e>@@$$QAV<lambda_03fcd07e894ec930e3f35da366ca99d6>@@@Z 1003727a f   libucrt:onexit.obj
 0001:000362d5       ??$?RV<lambda_8e746cf0007f6ed984d6f78af1fec997>@@AAV<lambda_22ebabd17bc4fa466a2aca6d8deb888d>@@V<lambda_18ed0c0b38a6dc0daf1e7ac6d6adf05e>@@@?$__crt_seh_guarded_call@H@@QAEH$$QAV<lambda_8e746cf0007f6ed984d6f78af1fec997>@@AAV<lambda_22ebabd17bc4fa466a2aca6d8deb888d>@@$$QAV<lambda_18ed0c0b38a6dc0daf1e7ac6d6adf05e>@@@Z 100372d5 f   libucrt:onexit.obj
 0001:0003634f       ??R<lambda_22ebabd17bc4fa466a2aca6d8deb888d>@@QBEHXZ 1003734f f   libucrt:onexit.obj
 0001:00036478       ??R<lambda_f03950bc5685219e0bcd2087efbe011e>@@QBEHXZ 10037478 f   libucrt:onexit.obj
 0001:000365f1       _initialize_environment    100375f1 f   libucrt:initialization.obj
 0001:000365f1       _initialize_global_state_isolation 100375f1 f   libucrt:initialization.obj
 0001:000365f1       _report_memory_leaks       100375f1 f   libucrt:initialization.obj
 0001:000365f1       _uninitialize_c            100375f1 f   libucrt:initialization.obj
 0001:000365f1       _uninitialize_global_state_isolation 100375f1 f   libucrt:initialization.obj
 0001:000365f4       _initialize_global_variables 100375f4 f   libucrt:initialization.obj
 0001:00036601       _initialize_c              10037601 f   libucrt:initialization.obj
 0001:0003661b       _uninitialize_environment  1003761b f   libucrt:initialization.obj
 0001:00036623       _initialize_pointers       10037623 f   libucrt:initialization.obj
 0001:00036651       _uninitialize_vcruntime    10037651 f   libucrt:initialization.obj
 0001:0003665a       _uninitialize_allocated_memory 1003765a f   libucrt:initialization.obj
 0001:00036671       _uninitialize_allocated_io_buffers 10037671 f   libucrt:initialization.obj
 0001:000366c1       ??R<lambda_af42a3ee9806e9a7305d451646e05244>@@QBEXAAPAU__crt_multibyte_data@@@Z 100376c1 f   libucrt:initialization.obj
 0001:00037170       $$000000                   10038170     libucrt:strncmp.obj
 0001:00037222       ??$?RV<lambda_15ade71b0218206bbe3333a0c9b79046>@@AAV<lambda_da44e0f8b0f19ba52fefafb335991732>@@V<lambda_207f2d024fc103971653565357d6cd41>@@@?$__crt_seh_guarded_call@X@@QAEX$$QAV<lambda_15ade71b0218206bbe3333a0c9b79046>@@AAV<lambda_da44e0f8b0f19ba52fefafb335991732>@@$$QAV<lambda_207f2d024fc103971653565357d6cd41>@@@Z 10038222 f   libucrt:per_thread_data.obj
 0001:00037274       ??$?RV<lambda_38edbb1296d33220d7e4dd0ed76b244a>@@AAV<lambda_5ce1d447e08cb34b2473517608e21441>@@V<lambda_fb385d3da700c9147fc39e65dd577a8c>@@@?$__crt_seh_guarded_call@X@@QAEX$$QAV<lambda_38edbb1296d33220d7e4dd0ed76b244a>@@AAV<lambda_5ce1d447e08cb34b2473517608e21441>@@$$QAV<lambda_fb385d3da700c9147fc39e65dd577a8c>@@@Z 10038274 f   libucrt:per_thread_data.obj
 0001:000372df       ??$?RV<lambda_6affb1475c98b40b75cdec977db92e3c>@@AAV<lambda_b8d4b9c228a6ecc3f80208dbb4b4a104>@@V<lambda_608742c3c92a14382c1684fc64f96c88>@@@?$__crt_seh_guarded_call@X@@QAEX$$QAV<lambda_6affb1475c98b40b75cdec977db92e3c>@@AAV<lambda_b8d4b9c228a6ecc3f80208dbb4b4a104>@@$$QAV<lambda_608742c3c92a14382c1684fc64f96c88>@@@Z 100382df f   libucrt:per_thread_data.obj
 0001:00037334       ??$?RV<lambda_a7e850c220f1c8d1e6efeecdedd162c6>@@AAV<lambda_46720907175c18b6c9d2717bc0d2d362>@@V<lambda_9048902d66e8d99359bc9897bbb930a8>@@@?$__crt_seh_guarded_call@X@@QAEX$$QAV<lambda_a7e850c220f1c8d1e6efeecdedd162c6>@@AAV<lambda_46720907175c18b6c9d2717bc0d2d362>@@$$QAV<lambda_9048902d66e8d99359bc9897bbb930a8>@@@Z 10038334 f   libucrt:per_thread_data.obj
 0001:0003738e       ?construct_ptd@@YAXQAU__acrt_ptd@@QAPAU__crt_locale_data@@@Z 1003838e f   libucrt:per_thread_data.obj
 0001:00037427       ?destroy_fls@@YGXPAX@Z     10038427 f   libucrt:per_thread_data.obj
 0001:00037448       ?destroy_ptd@@YAXQAU__acrt_ptd@@@Z 10038448 f   libucrt:per_thread_data.obj
 0001:00037515       ?replace_current_thread_locale_nolock@@YAXQAU__acrt_ptd@@QAU__crt_locale_data@@@Z 10038515 f   libucrt:per_thread_data.obj
 0001:000377de       ?fperrraise_with@@YAXHK@Z  100387de f   libucrt:_test.obj
 0001:00037ad1       ?<lambda_invoker_stdcall>@<lambda_29d3c280b90b41c2ae070ffca879996a>@@CGHPA_W@Z 10038ad1 f   libucrt:winapi_thunks.obj
 0001:00037ade       ??$?RV<lambda_6b4b7855443974f2b4b77000ea21c99c>@@AAV<lambda_8f7d3b162ab39427f4fa9995c67a7986>@@V<lambda_cc9a5ba8a5d8428b9634eab82665e5dc>@@@?$__crt_seh_guarded_call@H@@QAEH$$QAV<lambda_6b4b7855443974f2b4b77000ea21c99c>@@AAV<lambda_8f7d3b162ab39427f4fa9995c67a7986>@@$$QAV<lambda_cc9a5ba8a5d8428b9634eab82665e5dc>@@@Z 10038ade f   libucrt:winapi_thunks.obj
 0001:00037b5a       ??R<lambda_29d3c280b90b41c2ae070ffca879996a>@@QBEHPA_W@Z 10038b5a f   libucrt:winapi_thunks.obj
 0001:00037b89       ?try_get_AreFileApisANSI@@YAP6GHXZXZ 10038b89 f   libucrt:winapi_thunks.obj
 0001:00037ba3       ?try_get_CompareStringEx@@YAP6GHPB_WK0H0HPAU_nlsversioninfo@@PAXJ@ZXZ 10038ba3 f   libucrt:winapi_thunks.obj
 0001:00037bbd       ?try_get_EnumSystemLocalesEx@@YAP6GHP6GHPA_WKJ@ZKJPAX@ZXZ 10038bbd f   libucrt:winapi_thunks.obj
 0001:00037bd7       ?try_get_GetDateFormatEx@@YAP6GHPB_WKPBU_SYSTEMTIME@@0PA_WH0@ZXZ 10038bd7 f   libucrt:winapi_thunks.obj
 0001:00037bf1       ?try_get_GetLocaleInfoEx@@YAP6GHPB_WKPA_WH@ZXZ 10038bf1 f   libucrt:winapi_thunks.obj
 0001:00037c0b       ?try_get_GetTimeFormatEx@@YAP6GHPB_WKPBU_SYSTEMTIME@@0PA_WH@ZXZ 10038c0b f   libucrt:winapi_thunks.obj
 0001:00037c25       ?try_get_GetUserDefaultLocaleName@@YAP6GHPA_WH@ZXZ 10038c25 f   libucrt:winapi_thunks.obj
 0001:00037c3f       ?try_get_IsValidLocaleName@@YAP6GHPB_W@ZXZ 10038c3f f   libucrt:winapi_thunks.obj
 0001:00037c59       ?try_get_LCIDToLocaleName@@YAP6GHKPA_WHK@ZXZ 10038c59 f   libucrt:winapi_thunks.obj
 0001:00037c73       ?try_get_LCMapStringEx@@YAP6GHPB_WK0HPA_WHPAU_nlsversioninfo@@PAXJ@ZXZ 10038c73 f   libucrt:winapi_thunks.obj
 0001:00037c8d       ?try_get_LocaleNameToLCID@@YAP6GKPB_WK@ZXZ 10038c8d f   libucrt:winapi_thunks.obj
 0001:00037ca7       ?try_get_first_available_module@@YAPAUHINSTANCE__@@QBW4module_id@?A0x391cf84c@@0@Z 10038ca7 f   libucrt:winapi_thunks.obj
 0001:00037d6e       ?try_get_function@@YAPAXW4function_id@?A0x391cf84c@@QBDQBW4module_id@2@2@Z 10038d6e f   libucrt:winapi_thunks.obj
 0001:000382bf       ??$?RV<lambda_2866be3712abc81a800a822484c830d8>@@AAV<lambda_39ca0ed439415581b5b15c265174cece>@@V<lambda_2b24c74d71094a6cd0cb82e44167d71b>@@@?$__crt_seh_guarded_call@X@@QAEX$$QAV<lambda_2866be3712abc81a800a822484c830d8>@@AAV<lambda_39ca0ed439415581b5b15c265174cece>@@$$QAV<lambda_2b24c74d71094a6cd0cb82e44167d71b>@@@Z 100392bf f   libucrt:fflush.obj
 0001:0003834b       ??$?RV<lambda_2cc53f568c5a2bb6f192f930a45d44ea>@@AAV<lambda_ab61a845afdef5b7c387490eaf3616ee>@@V<lambda_c2ffc0b7726aa6be21d5f0026187e748>@@@?$__crt_seh_guarded_call@X@@QAEX$$QAV<lambda_2cc53f568c5a2bb6f192f930a45d44ea>@@AAV<lambda_ab61a845afdef5b7c387490eaf3616ee>@@$$QAV<lambda_c2ffc0b7726aa6be21d5f0026187e748>@@@Z 1003934b f   libucrt:fflush.obj
 0001:000383f7       ?common_flush_all@@YAH_N@Z 100393f7 f   libucrt:fflush.obj
 0001:00038444       ?common_flush_all_should_try_to_flush_stream@@YA_NV__crt_stdio_stream@@QAH@Z 10039444 f   libucrt:fflush.obj
 0001:00038477       ?is_stream_flushable_or_commitable@@YA_NJ@Z 10039477 f   libucrt:fflush.obj
 0001:00038592       ?initialize_inherited_file_handles_nolock@@YAXXZ 10039592 f   libucrt:ioinit.obj
 0001:00038648       ?initialize_stdio_handles_nolock@@YAXXZ 10039648 f   libucrt:ioinit.obj
 0001:00038788       ?write_double_translated_ansi_nolock@@YA?AUwrite_result@?A0x17268360@@HQBDI@Z 10039788 f   libucrt:write.obj
 0001:00038b32       ?write_double_translated_unicode_nolock@@YA?AUwrite_result@?A0x17268360@@QBDI@Z 10039b32 f   libucrt:write.obj
 0001:00038b9a       ?write_requires_double_translation_nolock@@YA_NH@Z 10039b9a f   libucrt:write.obj
 0001:00038c0b       ?write_text_ansi_nolock@@YA?AUwrite_result@?A0x17268360@@HQBDI@Z 10039c0b f   libucrt:write.obj
 0001:00038ce6       ?write_text_utf16le_nolock@@YA?AUwrite_result@?A0x17268360@@HQBDI@Z 10039ce6 f   libucrt:write.obj
 0001:00038dcf       ?write_text_utf8_nolock@@YA?AUwrite_result@?A0x17268360@@HQBDI@Z 10039dcf f   libucrt:write.obj
 0001:000395dd       ?fp_format_a@@YAHQBNPADIQADIH_NIQAU__crt_locale_pointers@@@Z 1003a5dd f   libucrt:cvt.obj
 0001:000398f6       ?fp_format_e@@YAHQBNQADI1IH_NIQAU__crt_locale_pointers@@@Z 1003a8f6 f   libucrt:cvt.obj
 0001:00039998       ?fp_format_e_internal@@YAHQADIH_NIQAU_strflt@@1QAU__crt_locale_pointers@@@Z 1003a998 f   libucrt:cvt.obj
 0001:00039ae0       ?fp_format_f@@YAHQBNQADI1IHQAU__crt_locale_pointers@@@Z 1003aae0 f   libucrt:cvt.obj
 0001:00039b6b       ?fp_format_f_internal@@YAHQADIHQAU_strflt@@_NQAU__crt_locale_pointers@@@Z 1003ab6b f   libucrt:cvt.obj
 0001:00039c3c       ?fp_format_g@@YAHQBNQADI1IH_NIQAU__crt_locale_pointers@@@Z 1003ac3c f   libucrt:cvt.obj
 0001:00039cfd       ?fp_format_nan_or_infinity@@YAHW4__acrt_fp_class@@_NPADI1@Z 1003acfd f   libucrt:cvt.obj
 0001:00039d92       ?shift_bytes@@YAXQADI0H@Z  1003ad92 f   libucrt:cvt.obj
 0001:00039f16       _no_op_initialize          1003af16 f   libucrt:wsetlocale.obj
 0001:00039f19       ??$?RV<lambda_135d2772fca65dc1248eeaa1b56e886a>@@AAV<lambda_2a444430fde8c29194d880d93eed5e8f>@@AAV<lambda_8dff2cf36a5417162780cd64fa2883ef>@@@?$__crt_seh_guarded_call@X@@QAEX$$QAV<lambda_135d2772fca65dc1248eeaa1b56e886a>@@AAV<lambda_2a444430fde8c29194d880d93eed5e8f>@@AAV<lambda_8dff2cf36a5417162780cd64fa2883ef>@@@Z 1003af19 f   libucrt:wsetlocale.obj
 0001:00039f5e       ??$?RV<lambda_4fdada1b837b2abbf20876fac97688ad>@@AAV<lambda_b57350f2640456a0859d250846f69caf>@@V<lambda_eed5e4f92b5b7d55fa22c48c484aaa54>@@@?$__crt_seh_guarded_call@X@@QAEX$$QAV<lambda_4fdada1b837b2abbf20876fac97688ad>@@AAV<lambda_b57350f2640456a0859d250846f69caf>@@$$QAV<lambda_eed5e4f92b5b7d55fa22c48c484aaa54>@@@Z 1003af5e f   libucrt:wsetlocale.obj
 0001:00039fab       ??$?RV<lambda_e5124f882df8998aaf41531e079ba474>@@AAV<lambda_3e16ef9562a7dcce91392c22ab16ea36>@@V<lambda_e25ca0880e6ef98be67edffd8c599615>@@@?$__crt_seh_guarded_call@X@@QAEX$$QAV<lambda_e5124f882df8998aaf41531e079ba474>@@AAV<lambda_3e16ef9562a7dcce91392c22ab16ea36>@@$$QAV<lambda_e25ca0880e6ef98be67edffd8c599615>@@@Z 1003afab f   libucrt:wsetlocale.obj
 0001:0003a093       ??R<lambda_2a444430fde8c29194d880d93eed5e8f>@@QBE@XZ 1003b093 f   libucrt:wsetlocale.obj
 0001:0003a0fd       ??R<lambda_b57350f2640456a0859d250846f69caf>@@QBEXXZ 1003b0fd f   libucrt:wsetlocale.obj
 0001:0003a4c6       __copytlocinfo_nolock      1003b4c6 f   libucrt:wsetlocale.obj
 0001:0003a4f5       __expandlocale             1003b4f5 f   libucrt:wsetlocale.obj
 0001:0003a97f       __wsetlocale_get_all       1003b97f f   libucrt:wsetlocale.obj
 0001:0003ab1a       __wsetlocale_nolock        1003bb1a f   libucrt:wsetlocale.obj
 0001:0003ae0a       __wsetlocale_set_cat       1003be0a f   libucrt:wsetlocale.obj
 0001:0003b1d1       _get_default_code_page     1003c1d1 f   libucrt:wsetlocale.obj
 0001:0003b200       _parse_bcp47               1003c200 f   libucrt:wsetlocale.obj
 0001:0003b3ea       _parse_bcp47_code_page     1003c3ea f   libucrt:wsetlocale.obj
 0001:0003b429       _parse_bcp47_language      1003c429 f   libucrt:wsetlocale.obj
 0001:0003b49b       _parse_bcp47_region        1003c49b f   libucrt:wsetlocale.obj
 0001:0003b554       _parse_bcp47_script        1003c554 f   libucrt:wsetlocale.obj
 0001:0003b5c4       _string_is_alpha           1003c5c4 f   libucrt:wsetlocale.obj
 0001:0003b601       ?_mbstowcs_l_helper@@YAIPA_WPBDIPAU__crt_locale_pointers@@@Z 1003c601 f   libucrt:mbstowcs.obj
 0001:0003b8a4       ??$common_tcsncpy_s@D@@YAHQADIQBDI@Z 1003c8a4 f   libucrt:strncpy_s.obj
 0001:0003be50       $$000000                   1003ce50     libucrt:log10_pentium4.obj
 0001:0003c0e0       $$000000                   1003d0e0     libucrt:87tran.obj
 0001:0003c2f0       $$000000                   1003d2f0     libucrt:87disp.obj
 0001:0003c550       $$000000                   1003d550     libucrt:common.obj
 0001:0003c6e0       $$000000                   1003d6e0     libucrt:genexcep.obj
 0001:0003c740       $$000000                   1003d740     libucrt:pow_pentium4.obj
 0001:0003d4a8       ?_wcstombs_l_helper@@YAIPADPB_WIPAU__crt_locale_pointers@@@Z 1003e4a8 f   libucrt:wcstombs.obj
 0001:0003d81c       ?InternalGetLocaleInfoA@@YAHQAU__crt_locale_pointers@@QB_WKQADH@Z 1003e81c f   libucrt:getlocaleinfoa.obj
 0001:0003dbae       ?__acrt_LCMapStringA_stat@@YAHPAU__crt_locale_pointers@@PB_WKPBDHPADHHH@Z 1003ebae f   libucrt:lcmapstringa.obj
 0001:0003e8b2       ??$?RV<lambda_cbab9ec6f41b0180b23cc171c22676b0>@@AAV<lambda_44731a7d0e6d81c3e6aa82d741081786>@@V<lambda_4b292cb8dd18144e164572427af410ab>@@@?$__crt_seh_guarded_call@P6AXH@Z@@QAEP6AXH@Z$$QAV<lambda_cbab9ec6f41b0180b23cc171c22676b0>@@AAV<lambda_44731a7d0e6d81c3e6aa82d741081786>@@$$QAV<lambda_4b292cb8dd18144e164572427af410ab>@@@Z 1003f8b2 f   libucrt:signal.obj
 0001:0003e916       ?get_global_action_nolock@@YAPAP6AXH@ZH@Z 1003f916 f   libucrt:signal.obj
 0001:0003e958       ?siglookup@@YAPAU__crt_signal_action_t@@HQAU1@@Z 1003f958 f   libucrt:signal.obj
 0001:0003eecb       ?<lambda_invoker_cdecl>@<lambda_838c7f62c73c983481e27c09e84b0b5d>@@CAHPBX0@Z 1003fecb f   libucrt:argv_wildcards.obj
 0001:0003eee3       ??$__acrt_convert_wcs_mbs_cp@_WDV<lambda_28bda7af82a03b66c1cb3803a755f95d>@@U__crt_win32_buffer_internal_dynamic_resizing@@@@YAHQB_WAAV?$__crt_win32_buffer@DU__crt_win32_buffer_internal_dynamic_resizing@@@@ABV<lambda_28bda7af82a03b66c1cb3803a755f95d>@@I@Z 1003fee3 f   libucrt:argv_wildcards.obj
 0001:0003efb2       ??$common_expand_argv_wildcards@D@@YAHQAPADQAPAPAD@Z 1003ffb2 f   libucrt:argv_wildcards.obj
 0001:0003f1a1       ??$copy_and_add_argument_to_buffer@D@@YAHQBD0IAAV?$argument_list@D@?A0x5f5c8891@@@Z 100401a1 f   libucrt:argv_wildcards.obj
 0001:0003f252       ??$expand_argument_wildcards@D@@YAHQAD0AAV?$argument_list@D@?A0x5f5c8891@@@Z 10040252 f   libucrt:argv_wildcards.obj
 0001:0003f524       ?expand_if_necessary@?$argument_list@D@?A0x5f5c8891@@AAEHXZ 10040524 f   libucrt:argv_wildcards.obj
 0001:0003f5b6       ??$__acrt_convert_wcs_mbs_cp@_WDV<lambda_0fec1a7b3f42a53036604e18c2d5e07e>@@U__crt_win32_buffer_no_resizing@@@@YAHQB_WAAV?$__crt_win32_buffer@DU__crt_win32_buffer_no_resizing@@@@ABV<lambda_0fec1a7b3f42a53036604e18c2d5e07e>@@I@Z 100405b6 f   libucrt:getmodulefilenamea.obj
 0001:0003f71e       ??$?RV<lambda_ceb1ee4838e85a9d631eb091e2fbe199>@@AAV<lambda_ae742caa10f662c28703da3d2ea5e57e>@@V<lambda_cd08b5d6af4937fe54fc07d0c9bf6b37>@@@?$__crt_seh_guarded_call@X@@QAEX$$QAV<lambda_ceb1ee4838e85a9d631eb091e2fbe199>@@AAV<lambda_ae742caa10f662c28703da3d2ea5e57e>@@$$QAV<lambda_cd08b5d6af4937fe54fc07d0c9bf6b37>@@@Z 1004071e f   libucrt:mbctype.obj
 0001:0003f76b       ??R<lambda_ae742caa10f662c28703da3d2ea5e57e>@@QBEXXZ 1004076b f   libucrt:mbctype.obj
 0001:0003f7ee       ?CPtoLocaleName@@YAPB_WH@Z 100407ee f   libucrt:mbctype.obj
 0001:0003f82c       ?getSystemCP@@YAHH@Z       1004082c f   libucrt:mbctype.obj
 0001:0003f89d       ?setSBCS@@YAXPAU__crt_multibyte_data@@@Z 1004089d f   libucrt:mbctype.obj
 0001:0003f902       ?setSBUpLow@@YAXPAU__crt_multibyte_data@@@Z 10040902 f   libucrt:mbctype.obj
 0001:0003fa83       ?setmbcp_internal@@YAHH_NQAU__acrt_ptd@@QAPAU__crt_multibyte_data@@@Z 10040a83 f   libucrt:mbctype.obj
 0001:0003fb9c       ?update_thread_multibyte_data_internal@@YAPAU__crt_multibyte_data@@QAU__acrt_ptd@@QAPAU1@@Z 10040b9c f   libucrt:mbctype.obj
 0001:0003fe8a       ?x_ismbbtype_l@@YAHPAU__crt_locale_pointers@@IHH@Z 10040e8a f   libucrt:ismbbyte.obj
 0001:0003ff12       ?find_end_of_double_null_terminated_sequence@@YAPB_WQB_W@Z 10040f12 f   libucrt:get_environment_from_os.obj
 0001:0004056b       ?to_abstract_control@@YA?AW4__acrt_fenv_abstract_control@@W4__acrt_fenv_machine_sse_control@@@Z 1004156b f   libucrt:_fenvutils.obj
 0001:00040627       ?to_abstract_control@@YA?AW4__acrt_fenv_abstract_control@@W4__acrt_fenv_machine_x87_control@@@Z 10041627 f   libucrt:_fenvutils.obj
 0001:000406e0       ?to_machine_sse_control@@YA?AW4__acrt_fenv_machine_sse_control@@W4__acrt_fenv_abstract_control@@@Z 100416e0 f   libucrt:_fenvutils.obj
 0001:000407ad       ?to_machine_x87_control@@YA?AW4__acrt_fenv_machine_x87_control@@W4__acrt_fenv_abstract_control@@@Z 100417ad f   libucrt:_fenvutils.obj
 0001:00040b30       ?GetTableIndexFromLocaleName@@YAHPB_W@Z 10041b30 f   libucrt:lcidtoname_downlevel.obj
 0001:00040d51       ??$?RV<lambda_9e9de3de5fa147e2223d7db92bc10aa6>@@AAV<lambda_38ce7e780aa69e748d6df282ebc68efe>@@V<lambda_8ca6da459f0f6780f1cff60fdc3d00e5>@@@?$__crt_seh_guarded_call@H@@QAEH$$QAV<lambda_9e9de3de5fa147e2223d7db92bc10aa6>@@AAV<lambda_38ce7e780aa69e748d6df282ebc68efe>@@$$QAV<lambda_8ca6da459f0f6780f1cff60fdc3d00e5>@@@Z 10041d51 f   libucrt:commit.obj
 0001:00040e70       ??$common_lseek_nolock@_J@@YA_JH_JH@Z 10041e70 f   libucrt:lseek.obj
 0001:00040f07       ??R<lambda_3d301b9e52f5099be73030e1f0bf487e>@@QBEIPBD@Z 10041f07 f   libucrt:mbrtowc.obj
 0001:00042cac       ?free_crt_array_internal@@YAXQAPBXI@Z 10043cac f   libucrt:inittime.obj
 0001:00042ce4       ?initialize_lc_time@@YA_NQAU__crt_lc_time_data@@QAU__crt_locale_data@@@Z 10043ce4 f   libucrt:inittime.obj
 0001:00043134       ??$common_tcsncat_s@_W@@YAHQA_WIQB_WI@Z 10044134 f   libucrt:wcsncat_s.obj
 0001:00043226       ??$common_tcsncpy_s@_W@@YAHQA_WIQB_WI@Z 10044226 f   libucrt:wcsncpy_s.obj
 0001:000432fc       _GetLocaleNameFromDefault  100442fc f   libucrt:get_qualified_locale.obj
 0001:00043383       _GetLocaleNameFromLangCountry 10044383 f   libucrt:get_qualified_locale.obj
 0001:0004341c       _GetLocaleNameFromLanguage 1004441c f   libucrt:get_qualified_locale.obj
 0001:00043475       _GetPrimaryLen             10044475 f   libucrt:get_qualified_locale.obj
 0001:000434a9       _LangCountryEnumProcEx@12  100444a9 f   libucrt:get_qualified_locale.obj
 0001:00043789       _LanguageEnumProcEx@12     10044789 f   libucrt:get_qualified_locale.obj
 0001:00043848       _ProcessCodePage           10044848 f   libucrt:get_qualified_locale.obj
 0001:0004393e       _TestDefaultCountry        1004493e f   libucrt:get_qualified_locale.obj
 0001:0004398b       _TranslateName             1004498b f   libucrt:get_qualified_locale.obj
 0001:00043bf3       _CountryEnumProc@4         10044bf3 f   libucrt:getqloc_downlevel.obj
 0001:00043c9a       _GetLcidFromCountry        10044c9a f   libucrt:getqloc_downlevel.obj
 0001:00043ce5       _GetLcidFromLangCountry    10044ce5 f   libucrt:getqloc_downlevel.obj
 0001:00043d80       _GetLcidFromLanguage       10044d80 f   libucrt:getqloc_downlevel.obj
 0001:00043ddf       _GetPrimaryLen             10044ddf f   libucrt:getqloc_downlevel.obj
 0001:00043e0b       _LangCountryEnumProc@4     10044e0b f   libucrt:getqloc_downlevel.obj
 0001:0004405e       _LanguageEnumProc@4        1004505e f   libucrt:getqloc_downlevel.obj
 0001:00044133       _LcidFromHexString         10045133 f   libucrt:getqloc_downlevel.obj
 0001:00044184       _ProcessCodePage           10045184 f   libucrt:getqloc_downlevel.obj
 0001:00044265       _TestDefaultCountry        10045265 f   libucrt:getqloc_downlevel.obj
 0001:0004428a       _TestDefaultLanguage       1004528a f   libucrt:getqloc_downlevel.obj
 0001:000442f8       _TranslateName             100452f8 f   libucrt:getqloc_downlevel.obj
 0001:000449c0       ?swap@@YAXPAD0I@Z          100459c0 f   libucrt:qsort.obj
 0001:00044e50       $$000000                   10045e50     libucrt:strpbrk.obj
 0001:00044f34       ?initialize_multibyte@@YAHXZ 10045f34 f   libucrt:multibyte_initializer.obj
 0001:00045104       ??$?RV<lambda_218ce3db14220d0be481dae8ef3383b6>@@AAV<lambda_628dfdc04ba53c8bfc02c9951375f3f5>@@V<lambda_57dc472bd5c9d5f3b2cbca59b8a843ae>@@@?$__crt_seh_guarded_call@H@@QAEH$$QAV<lambda_218ce3db14220d0be481dae8ef3383b6>@@AAV<lambda_628dfdc04ba53c8bfc02c9951375f3f5>@@$$QAV<lambda_57dc472bd5c9d5f3b2cbca59b8a843ae>@@@Z 10046104 f   libucrt:close.obj
 0001:0004549b       ?__dcrt_lowio_initialize_console_output@@YAXXZ 1004649b f   libucrt:initcon.obj
 0001:000455fa       ??$common_xtox@K_W@@YAHKQA_WII_N@Z 100465fa f   libucrt:xtoa.obj
 0001:000456ad       ??$common_xtox_s@K_W@@YAHKQA_WII_N@Z 100466ad f   libucrt:xtoa.obj
 0001:00045910       $$000000                   10046910     libucrt:_strnicm.obj
 0001:00045ad0       $$000000                   10046ad0     LIBCMT:lldvrm.obj
 0001:00045bb0       $$000000                   10046bb0     libvcruntime:strrchr.obj
 0001:00045cf0       $$000000                   10046cf0     libvcruntime:strchr.obj
 0001:00045ea0       __unwindfunclet$??$decimal_point_impl@_W@detail@v6@fmt@@YA_WVlocale_ref@012@@Z$0 10046ea0 f   format.obj
 0001:00045ea0       __unwindfunclet$??$grouping_impl@_W@detail@v6@fmt@@YA?AV?$basic_string@DU?$char_traits@D@std@@V?$allocator@D@2@@std@@Vlocale_ref@012@@Z$0 10046ea0 f   format.obj
 0001:00045ea0       __unwindfunclet$??$thousands_sep_impl@_W@detail@v6@fmt@@YA_WVlocale_ref@012@@Z$0 10046ea0 f   format.obj
 0001:00045ea8       __ehhandler$??$decimal_point_impl@_W@detail@v6@fmt@@YA_WVlocale_ref@012@@Z 10046ea8 f   format.obj
 0001:00045ea8       __ehhandler$??$grouping_impl@_W@detail@v6@fmt@@YA?AV?$basic_string@DU?$char_traits@D@std@@V?$allocator@D@2@@std@@Vlocale_ref@012@@Z 10046ea8 f   format.obj
 0001:00045ea8       __ehhandler$??$thousands_sep_impl@_W@detail@v6@fmt@@YA_WVlocale_ref@012@@Z 10046ea8 f   format.obj
 0001:00045ec0       __unwindfunclet$??$fallback_format@N@detail@v6@fmt@@YAXNAAV?$buffer@D@012@AAH@Z$0 10046ec0 f   format.obj
 0001:00045ec0       __unwindfunclet$??$fallback_format@O@detail@v6@fmt@@YAXOAAV?$buffer@D@012@AAH@Z$0 10046ec0 f   format.obj
 0001:00045ecb       __unwindfunclet$??$fallback_format@N@detail@v6@fmt@@YAXNAAV?$buffer@D@012@AAH@Z$1 10046ecb f   format.obj
 0001:00045ecb       __unwindfunclet$??$fallback_format@O@detail@v6@fmt@@YAXOAAV?$buffer@D@012@AAH@Z$1 10046ecb f   format.obj
 0001:00045ed6       __unwindfunclet$??$fallback_format@N@detail@v6@fmt@@YAXNAAV?$buffer@D@012@AAH@Z$2 10046ed6 f   format.obj
 0001:00045ed6       __unwindfunclet$??$fallback_format@O@detail@v6@fmt@@YAXOAAV?$buffer@D@012@AAH@Z$2 10046ed6 f   format.obj
 0001:00045ee1       __unwindfunclet$??$fallback_format@N@detail@v6@fmt@@YAXNAAV?$buffer@D@012@AAH@Z$3 10046ee1 f   format.obj
 0001:00045ee1       __unwindfunclet$??$fallback_format@O@detail@v6@fmt@@YAXOAAV?$buffer@D@012@AAH@Z$3 10046ee1 f   format.obj
 0001:00045eec       __ehhandler$??$fallback_format@N@detail@v6@fmt@@YAXNAAV?$buffer@D@012@AAH@Z 10046eec f   format.obj
 0001:00045eec       __ehhandler$??$fallback_format@O@detail@v6@fmt@@YAXOAAV?$buffer@D@012@AAH@Z 10046eec f   format.obj
 0001:00045f00       __ehhandler$??$get@Vlocale@std@@@locale_ref@detail@v6@fmt@@QBE?AVlocale@std@@XZ 10046f00 f   format.obj
 0001:00045f10       __unwindfunclet$??$use_facet@V?$numpunct@_W@std@@@std@@YAABV?$numpunct@_W@0@ABVlocale@0@@Z$0 10046f10 f   format.obj
 0001:00045f18       __unwindfunclet$??$use_facet@V?$numpunct@_W@std@@@std@@YAABV?$numpunct@_W@0@ABVlocale@0@@Z$2 10046f18 f   format.obj
 0001:00045f27       __unwindfunclet$??$use_facet@V?$numpunct@_W@std@@@std@@YAABV?$numpunct@_W@0@ABVlocale@0@@Z$3 10046f27 f   format.obj
 0001:00045f40       __unwindfunclet$??$use_facet@V?$numpunct@_W@std@@@std@@YAABV?$numpunct@_W@0@ABVlocale@0@@Z$4 10046f40 f   format.obj
 0001:00045f48       __unwindfunclet$??$use_facet@V?$numpunct@_W@std@@@std@@YAABV?$numpunct@_W@0@ABVlocale@0@@Z$5 10046f48 f   format.obj
 0001:00045f50       __unwindfunclet$??$use_facet@V?$numpunct@_W@std@@@std@@YAABV?$numpunct@_W@0@ABVlocale@0@@Z$1 10046f50 f   format.obj
 0001:00045f58       __ehhandler$??$use_facet@V?$numpunct@_W@std@@@std@@YAABV?$numpunct@_W@0@ABVlocale@0@@Z 10046f58 f   format.obj
 0001:00045f70       __unwindfunclet$??0_Locinfo@std@@QAE@PBD@Z$0 10046f70 f   format.obj
 0001:00045f78       __unwindfunclet$??0_Locinfo@std@@QAE@PBD@Z$1 10046f78 f   format.obj
 0001:00045f83       __unwindfunclet$??0_Locinfo@std@@QAE@PBD@Z$2 10046f83 f   format.obj
 0001:00045f8e       __unwindfunclet$??0_Locinfo@std@@QAE@PBD@Z$3 10046f8e f   format.obj
 0001:00045f99       __unwindfunclet$??0_Locinfo@std@@QAE@PBD@Z$4 10046f99 f   format.obj
 0001:00045fa4       __unwindfunclet$??0_Locinfo@std@@QAE@PBD@Z$5 10046fa4 f   format.obj
 0001:00045faf       __unwindfunclet$??0_Locinfo@std@@QAE@PBD@Z$6 10046faf f   format.obj
 0001:00045fba       __ehhandler$??0_Locinfo@std@@QAE@PBD@Z 10046fba f   format.obj
 0001:00045fd0       __ehhandler$??1PluginDialogBuilder@@QAE@XZ 10046fd0 f   Pcfg.obj
 0001:00045fd0       __ehhandler$??1PluginSettings@@QAE@XZ 10046fd0 f   Pcfg.obj
 0001:00045fd0       __ehhandler$??1?$unique_ptr@UIWbemClassObject@@Ucom_closer@@@std@@QAE@XZ 10046fd0 f   WMI.obj
 0001:00045fd0       __ehhandler$??1?$unique_ptr@UIWbemLocator@@Ucom_closer@@@std@@QAE@XZ 10046fd0 f   WMI.obj
 0001:00045fd0       __ehhandler$??1_Locinfo@std@@QAE@XZ 10046fd0 f   format.obj
 0001:00045fd0       __ehhandler$??1?$scoped_lock@VPerfThread@@@std@@QAE@XZ 10046fd0 f   handles.obj
 0001:00045fd0       __ehhandler$??1DebugToken@@QAE@XZ 10046fd0 f   handles.obj
 0001:00045fe0       __unwindfunclet$?on_error@error_handler@detail@v6@fmt@@QAEXPBD@Z$0 10046fe0 f   format.obj
 0001:00045fe0       __unwindfunclet$??$handle_int_type_spec@AAU?$int_writer@V?$back_insert_iterator@V?$buffer@_W@detail@v6@fmt@@@std@@_WI@detail@v6@fmt@@@detail@v6@fmt@@YAXDAAU?$int_writer@V?$back_insert_iterator@V?$buffer@_W@detail@v6@fmt@@@std@@_WI@012@@Z$0 10046fe0 f   handles.obj
 0001:00045fe0       __unwindfunclet$??$handle_int_type_spec@AAU?$int_writer@V?$back_insert_iterator@V?$buffer@_W@detail@v6@fmt@@@std@@_W_K@detail@v6@fmt@@@detail@v6@fmt@@YAXDAAU?$int_writer@V?$back_insert_iterator@V?$buffer@_W@detail@v6@fmt@@@std@@_W_K@012@@Z$0 10046fe0 f   handles.obj
 0001:00045fe0       __unwindfunclet$??$visit_format_arg@U?$default_arg_formatter@V?$back_insert_iterator@V?$buffer@_W@detail@v6@fmt@@@std@@_W@detail@v6@fmt@@V?$basic_format_context@V?$back_insert_iterator@V?$buffer@_W@detail@v6@fmt@@@std@@_W@34@@v6@fmt@@YA?AV?$back_insert_iterator@V?$buffer@_W@detail@v6@fmt@@@std@@$$QAU?$default_arg_formatter@V?$back_insert_iterator@V?$buffer@_W@detail@v6@fmt@@@std@@_W@detail@01@ABV?$basic_format_arg@V?$basic_format_context@V?$back_insert_iterator@V?$buffer@_W@detail@v6@fmt@@@std@@_W@v6@fmt@@@01@@Z$0 10046fe0 f   handles.obj
 0001:00045fe0       __unwindfunclet$?write@?$arg_formatter_base@V?$back_insert_iterator@V?$buffer@_W@detail@v6@fmt@@@std@@_WUerror_handler@detail@v6@fmt@@@detail@v6@fmt@@IAEXPB_W@Z$0 10046fe0 f   handles.obj
 0001:00045fe8       __ehhandler$?on_error@error_handler@detail@v6@fmt@@QAEXPBD@Z 10046fe8 f   format.obj
 0001:00045fe8       __ehhandler$??$handle_int_type_spec@AAU?$int_writer@V?$back_insert_iterator@V?$buffer@_W@detail@v6@fmt@@@std@@_WI@detail@v6@fmt@@@detail@v6@fmt@@YAXDAAU?$int_writer@V?$back_insert_iterator@V?$buffer@_W@detail@v6@fmt@@@std@@_WI@012@@Z 10046fe8 f   handles.obj
 0001:00045fe8       __ehhandler$??$handle_int_type_spec@AAU?$int_writer@V?$back_insert_iterator@V?$buffer@_W@detail@v6@fmt@@@std@@_W_K@detail@v6@fmt@@@detail@v6@fmt@@YAXDAAU?$int_writer@V?$back_insert_iterator@V?$buffer@_W@detail@v6@fmt@@@std@@_W_K@012@@Z 10046fe8 f   handles.obj
 0001:00045fe8       __ehhandler$??$visit_format_arg@U?$default_arg_formatter@V?$back_insert_iterator@V?$buffer@_W@detail@v6@fmt@@@std@@_W@detail@v6@fmt@@V?$basic_format_context@V?$back_insert_iterator@V?$buffer@_W@detail@v6@fmt@@@std@@_W@34@@v6@fmt@@YA?AV?$back_insert_iterator@V?$buffer@_W@detail@v6@fmt@@@std@@$$QAU?$default_arg_formatter@V?$back_insert_iterator@V?$buffer@_W@detail@v6@fmt@@@std@@_W@detail@01@ABV?$basic_format_arg@V?$basic_format_context@V?$back_insert_iterator@V?$buffer@_W@detail@v6@fmt@@@std@@_W@v6@fmt@@@01@@Z 10046fe8 f   handles.obj
 0001:00045fe8       __ehhandler$?write@?$arg_formatter_base@V?$back_insert_iterator@V?$buffer@_W@detail@v6@fmt@@@std@@_WUerror_handler@detail@v6@fmt@@@detail@v6@fmt@@IAEXPB_W@Z 10046fe8 f   handles.obj
 0001:00046000       __unwindfunclet$?square@bigint@detail@v6@fmt@@QAEXXZ$0 10047000 f   format.obj
 0001:0004600b       __ehhandler$?square@bigint@detail@v6@fmt@@QAEXXZ 1004700b f   format.obj
 0001:00046020       __unwindfunclet$??$vformat@_W$0A@@detail@v6@fmt@@YA?AV?$basic_string@_WU?$char_traits@_W@std@@V?$allocator@_W@2@@std@@V?$basic_string_view@_W@12@V?$basic_format_args@V?$basic_format_context@V?$back_insert_iterator@V?$buffer@_W@detail@v6@fmt@@@std@@_W@v6@fmt@@@12@@Z$0 10047020 f   handles.obj
 0001:0004602b       __ehhandler$??$vformat@_W$0A@@detail@v6@fmt@@YA?AV?$basic_string@_WU?$char_traits@_W@std@@V?$allocator@_W@2@@std@@V?$basic_string_view@_W@12@V?$basic_format_args@V?$basic_format_context@V?$back_insert_iterator@V?$buffer@_W@detail@v6@fmt@@@std@@_W@v6@fmt@@@12@@Z 1004702b f   handles.obj
 0001:00046040       __unwindfunclet$??$write@_WV?$back_insert_iterator@V?$buffer@_W@detail@v6@fmt@@@std@@M$0A@@detail@v6@fmt@@YA?AV?$back_insert_iterator@V?$buffer@_W@detail@v6@fmt@@@std@@V34@M@Z$0 10047040 f   handles.obj
 0001:0004604b       __ehhandler$??$write@_WV?$back_insert_iterator@V?$buffer@_W@detail@v6@fmt@@@std@@M$0A@@detail@v6@fmt@@YA?AV?$back_insert_iterator@V?$buffer@_W@detail@v6@fmt@@@std@@V34@M@Z 1004704b f   handles.obj
 0001:00046060       __unwindfunclet$??$write@_WV?$back_insert_iterator@V?$buffer@_W@detail@v6@fmt@@@std@@M$0A@@detail@v6@fmt@@YA?AV?$back_insert_iterator@V?$buffer@_W@detail@v6@fmt@@@std@@V34@MU?$basic_format_specs@_W@12@Vlocale_ref@012@@Z$0 10047060 f   handles.obj
 0001:0004606b       __unwindfunclet$??$write@_WV?$back_insert_iterator@V?$buffer@_W@detail@v6@fmt@@@std@@M$0A@@detail@v6@fmt@@YA?AV?$back_insert_iterator@V?$buffer@_W@detail@v6@fmt@@@std@@V34@MU?$basic_format_specs@_W@12@Vlocale_ref@012@@Z$1 1004706b f   handles.obj
 0001:00046073       __ehhandler$??$write@_WV?$back_insert_iterator@V?$buffer@_W@detail@v6@fmt@@@std@@M$0A@@detail@v6@fmt@@YA?AV?$back_insert_iterator@V?$buffer@_W@detail@v6@fmt@@@std@@V34@MU?$basic_format_specs@_W@12@Vlocale_ref@012@@Z 10047073 f   handles.obj
 0001:00046080       __unwindfunclet$??$write@_WV?$back_insert_iterator@V?$buffer@_W@detail@v6@fmt@@@std@@N$0A@@detail@v6@fmt@@YA?AV?$back_insert_iterator@V?$buffer@_W@detail@v6@fmt@@@std@@V34@N@Z$0 10047080 f   handles.obj
 0001:00046080       __unwindfunclet$??$write@_WV?$back_insert_iterator@V?$buffer@_W@detail@v6@fmt@@@std@@O$0A@@detail@v6@fmt@@YA?AV?$back_insert_iterator@V?$buffer@_W@detail@v6@fmt@@@std@@V34@O@Z$0 10047080 f   handles.obj
 0001:0004608b       __ehhandler$??$write@_WV?$back_insert_iterator@V?$buffer@_W@detail@v6@fmt@@@std@@N$0A@@detail@v6@fmt@@YA?AV?$back_insert_iterator@V?$buffer@_W@detail@v6@fmt@@@std@@V34@N@Z 1004708b f   handles.obj
 0001:0004608b       __ehhandler$??$write@_WV?$back_insert_iterator@V?$buffer@_W@detail@v6@fmt@@@std@@O$0A@@detail@v6@fmt@@YA?AV?$back_insert_iterator@V?$buffer@_W@detail@v6@fmt@@@std@@V34@O@Z 1004708b f   handles.obj
 0001:000460a0       __unwindfunclet$??$write@_WV?$back_insert_iterator@V?$buffer@_W@detail@v6@fmt@@@std@@N$0A@@detail@v6@fmt@@YA?AV?$back_insert_iterator@V?$buffer@_W@detail@v6@fmt@@@std@@V34@NU?$basic_format_specs@_W@12@Vlocale_ref@012@@Z$0 100470a0 f   handles.obj
 0001:000460a0       __unwindfunclet$??$write@_WV?$back_insert_iterator@V?$buffer@_W@detail@v6@fmt@@@std@@O$0A@@detail@v6@fmt@@YA?AV?$back_insert_iterator@V?$buffer@_W@detail@v6@fmt@@@std@@V34@OU?$basic_format_specs@_W@12@Vlocale_ref@012@@Z$0 100470a0 f   handles.obj
 0001:000460ab       __unwindfunclet$??$write@_WV?$back_insert_iterator@V?$buffer@_W@detail@v6@fmt@@@std@@N$0A@@detail@v6@fmt@@YA?AV?$back_insert_iterator@V?$buffer@_W@detail@v6@fmt@@@std@@V34@NU?$basic_format_specs@_W@12@Vlocale_ref@012@@Z$1 100470ab f   handles.obj
 0001:000460ab       __unwindfunclet$??$write@_WV?$back_insert_iterator@V?$buffer@_W@detail@v6@fmt@@@std@@O$0A@@detail@v6@fmt@@YA?AV?$back_insert_iterator@V?$buffer@_W@detail@v6@fmt@@@std@@V34@OU?$basic_format_specs@_W@12@Vlocale_ref@012@@Z$1 100470ab f   handles.obj
 0001:000460b3       __ehhandler$??$write@_WV?$back_insert_iterator@V?$buffer@_W@detail@v6@fmt@@@std@@N$0A@@detail@v6@fmt@@YA?AV?$back_insert_iterator@V?$buffer@_W@detail@v6@fmt@@@std@@V34@NU?$basic_format_specs@_W@12@Vlocale_ref@012@@Z 100470b3 f   handles.obj
 0001:000460b3       __ehhandler$??$write@_WV?$back_insert_iterator@V?$buffer@_W@detail@v6@fmt@@@std@@O$0A@@detail@v6@fmt@@YA?AV?$back_insert_iterator@V?$buffer@_W@detail@v6@fmt@@@std@@V34@OU?$basic_format_specs@_W@12@Vlocale_ref@012@@Z 100470b3 f   handles.obj
 0001:000460c0       __unwindfunclet$??R<lambda_c3630acb37279cf92411e07a2b271fdf>@@QBE?AV?$basic_string@_WU?$char_traits@_W@std@@V?$allocator@_W@2@@std@@XZ$1 100470c0 f   handles.obj
 0001:000460c8       __unwindfunclet$??R<lambda_c3630acb37279cf92411e07a2b271fdf>@@QBE?AV?$basic_string@_WU?$char_traits@_W@std@@V?$allocator@_W@2@@std@@XZ$2 100470c8 f   handles.obj
 0001:000460d0       __unwindfunclet$??R<lambda_c3630acb37279cf92411e07a2b271fdf>@@QBE?AV?$basic_string@_WU?$char_traits@_W@std@@V?$allocator@_W@2@@std@@XZ$3 100470d0 f   handles.obj
 0001:000460d8       __ehhandler$??R<lambda_c3630acb37279cf92411e07a2b271fdf>@@QBE?AV?$basic_string@_WU?$char_traits@_W@std@@V?$allocator@_W@2@@std@@XZ 100470d8 f   handles.obj
 0001:000460f0       __unwindfunclet$?GetNameByType@@YA?AV?$basic_string@_WU?$char_traits@_W@std@@V?$allocator@_W@2@@std@@PAXGPAVPerfThread@@@Z$1 100470f0 f   handles.obj
 0001:000460f8       __unwindfunclet$?GetNameByType@@YA?AV?$basic_string@_WU?$char_traits@_W@std@@V?$allocator@_W@2@@std@@PAXGPAVPerfThread@@@Z$12 100470f8 f   handles.obj
 0001:00046100       __unwindfunclet$?GetNameByType@@YA?AV?$basic_string@_WU?$char_traits@_W@std@@V?$allocator@_W@2@@std@@PAXGPAVPerfThread@@@Z$14 10047100 f   handles.obj
 0001:00046108       __unwindfunclet$?GetNameByType@@YA?AV?$basic_string@_WU?$char_traits@_W@std@@V?$allocator@_W@2@@std@@PAXGPAVPerfThread@@@Z$2 10047108 f   handles.obj
 0001:00046110       __unwindfunclet$?GetNameByType@@YA?AV?$basic_string@_WU?$char_traits@_W@std@@V?$allocator@_W@2@@std@@PAXGPAVPerfThread@@@Z$20 10047110 f   handles.obj
 0001:0004611e       __unwindfunclet$?GetNameByType@@YA?AV?$basic_string@_WU?$char_traits@_W@std@@V?$allocator@_W@2@@std@@PAXGPAVPerfThread@@@Z$3 1004711e f   handles.obj
 0001:00046126       __ehhandler$?GetNameByType@@YA?AV?$basic_string@_WU?$char_traits@_W@std@@V?$allocator@_W@2@@std@@PAXGPAVPerfThread@@@Z 10047126 f   handles.obj
 0001:00046130       __unwindfunclet$?PrintHandleInfo@@YA_NKPAX_NPAVPerfThread@@@Z$0 10047130 f   handles.obj
 0001:00046138       __unwindfunclet$?PrintHandleInfo@@YA_NKPAX_NPAVPerfThread@@@Z$2 10047138 f   handles.obj
 0001:00046140       __unwindfunclet$?PrintHandleInfo@@YA_NKPAX_NPAVPerfThread@@@Z$3 10047140 f   handles.obj
 0001:00046148       __unwindfunclet$?PrintHandleInfo@@YA_NKPAX_NPAVPerfThread@@@Z$20 10047148 f   handles.obj
 0001:00046150       __unwindfunclet$?PrintHandleInfo@@YA_NKPAX_NPAVPerfThread@@@Z$5 10047150 f   handles.obj
 0001:00046158       __unwindfunclet$?PrintHandleInfo@@YA_NKPAX_NPAVPerfThread@@@Z$6 10047158 f   handles.obj
 0001:00046160       __unwindfunclet$?PrintHandleInfo@@YA_NKPAX_NPAVPerfThread@@@Z$7 10047160 f   handles.obj
 0001:0004616b       __ehhandler$?PrintHandleInfo@@YA_NKPAX_NPAVPerfThread@@@Z 1004716b f   handles.obj
 0001:00046180       __unwindfunclet$?duplicate_handle@@YA?AV?$unique_ptr@XUhandle_closer@@@std@@PAXK@Z$0 10047180 f   handles.obj
 0001:00046188       __ehhandler$?duplicate_handle@@YA?AV?$unique_ptr@XUhandle_closer@@@std@@PAXK@Z 10047188 f   handles.obj
 0001:000461a0       __unwindfunclet$?on_fill@?$specs_setter@_W@detail@v6@fmt@@QAEXV?$basic_string_view@_W@34@@Z$0 100471a0 f   handles.obj
 0001:000461a8       __ehhandler$?on_fill@?$specs_setter@_W@detail@v6@fmt@@QAEXV?$basic_string_view@_W@34@@Z 100471a8 f   handles.obj
 0001:000461c0       __unwindfunclet$?on_num@?$int_writer@V?$back_insert_iterator@V?$buffer@_W@detail@v6@fmt@@@std@@_WI@detail@v6@fmt@@QAEXXZ$0 100471c0 f   handles.obj
 0001:000461c8       __unwindfunclet$?on_num@?$int_writer@V?$back_insert_iterator@V?$buffer@_W@detail@v6@fmt@@@std@@_WI@detail@v6@fmt@@QAEXXZ$1 100471c8 f   handles.obj
 0001:000461d3       __ehhandler$?on_num@?$int_writer@V?$back_insert_iterator@V?$buffer@_W@detail@v6@fmt@@@std@@_WI@detail@v6@fmt@@QAEXXZ 100471d3 f   handles.obj
 0001:000461e0       __unwindfunclet$?on_num@?$int_writer@V?$back_insert_iterator@V?$buffer@_W@detail@v6@fmt@@@std@@_W_K@detail@v6@fmt@@QAEXXZ$0 100471e0 f   handles.obj
 0001:000461e8       __unwindfunclet$?on_num@?$int_writer@V?$back_insert_iterator@V?$buffer@_W@detail@v6@fmt@@@std@@_W_K@detail@v6@fmt@@QAEXXZ$1 100471e8 f   handles.obj
 0001:000461f3       __ehhandler$?on_num@?$int_writer@V?$back_insert_iterator@V?$buffer@_W@detail@v6@fmt@@@std@@_W_K@detail@v6@fmt@@QAEXXZ 100471f3 f   handles.obj
 0001:00046200       __unwindfunclet$?query_object@@YA?AV?$unique_ptr@$$BY0A@DU?$default_delete@$$BY0A@D@std@@@std@@PAXW4OBJECT_INFORMATION_CLASS@@@Z$0 10047200 f   handles.obj
 0001:00046208       __ehhandler$?query_object@@YA?AV?$unique_ptr@$$BY0A@DU?$default_delete@$$BY0A@D@std@@@std@@PAXW4OBJECT_INFORMATION_CLASS@@@Z 10047208 f   handles.obj
 0001:00046220       __unwindfunclet$?Config@@YAHXZ$0 10047220 f   Pcfg.obj
 0001:00046228       __ehhandler$?Config@@YAHXZ 10047228 f   Pcfg.obj
 0001:00046240       __unwindfunclet$?Read@options@@QAEXXZ$0 10047240 f   Pcfg.obj
 0001:00046240       __unwindfunclet$?Write@options@@QBEXXZ$0 10047240 f   Pcfg.obj
 0001:00046248       __ehhandler$?Read@options@@QAEXXZ 10047248 f   Pcfg.obj
 0001:00046248       __ehhandler$?Write@options@@QBEXXZ 10047248 f   Pcfg.obj
 0001:00046260       __unwindfunclet$??$_Assign_range@PBUmode@@@?$vector@Umode@@V?$allocator@Umode@@@std@@@std@@AAEXPBUmode@@0Uforward_iterator_tag@1@@Z$0 10047260 f   Pclass.obj
 0001:00046268       __unwindfunclet$??$_Assign_range@PBUmode@@@?$vector@Umode@@V?$allocator@Umode@@@std@@@std@@AAEXPBUmode@@0Uforward_iterator_tag@1@@Z$3 10047268 f   Pclass.obj
 0001:00046270       __unwindfunclet$??$_Assign_range@PBUmode@@@?$vector@Umode@@V?$allocator@Umode@@@std@@@std@@AAEXPBUmode@@0Uforward_iterator_tag@1@@Z$4 10047270 f   Pclass.obj
 0001:0004627b       __unwindfunclet$??$_Assign_range@PBUmode@@@?$vector@Umode@@V?$allocator@Umode@@@std@@@std@@AAEXPBUmode@@0Uforward_iterator_tag@1@@Z$1 1004727b f   Pclass.obj
 0001:00046283       __unwindfunclet$??$_Assign_range@PBUmode@@@?$vector@Umode@@V?$allocator@Umode@@@std@@@std@@AAEXPBUmode@@0Uforward_iterator_tag@1@@Z$6 10047283 f   Pclass.obj
 0001:0004628b       __unwindfunclet$??$_Assign_range@PBUmode@@@?$vector@Umode@@V?$allocator@Umode@@@std@@@std@@AAEXPBUmode@@0Uforward_iterator_tag@1@@Z$7 1004728b f   Pclass.obj
 0001:00046296       __ehhandler$??$_Assign_range@PBUmode@@@?$vector@Umode@@V?$allocator@Umode@@@std@@@std@@AAEXPBUmode@@0Uforward_iterator_tag@1@@Z 10047296 f   Pclass.obj
 0001:000462a0       __unwindfunclet$??$_Try_emplace@ABK$$V@?$_Hash@V?$_Umap_traits@KPAUHWND__@@V?$_Uhash_compare@KU?$hash@K@std@@U?$equal_to@K@2@@std@@V?$allocator@U?$pair@$$CBKPAUHWND__@@@std@@@3@$0A@@std@@@std@@IAE?AU?$pair@PAU?$_List_node@U?$pair@$$CBKPAUHWND__@@@std@@PAX@std@@_N@1@ABK@Z$1 100472a0 f   Pclass.obj
 0001:000462a8       __unwindfunclet$??$_Try_emplace@ABK$$V@?$_Hash@V?$_Umap_traits@KPAUHWND__@@V?$_Uhash_compare@KU?$hash@K@std@@U?$equal_to@K@2@@std@@V?$allocator@U?$pair@$$CBKPAUHWND__@@@std@@@3@$0A@@std@@@std@@IAE?AU?$pair@PAU?$_List_node@U?$pair@$$CBKPAUHWND__@@@std@@PAX@std@@_N@1@ABK@Z$0 100472a8 f   Pclass.obj
 0001:000462b0       __ehhandler$??$_Try_emplace@ABK$$V@?$_Hash@V?$_Umap_traits@KPAUHWND__@@V?$_Uhash_compare@KU?$hash@K@std@@U?$equal_to@K@2@@std@@V?$allocator@U?$pair@$$CBKPAUHWND__@@@std@@@3@$0A@@std@@@std@@IAE?AU?$pair@PAU?$_List_node@U?$pair@$$CBKPAUHWND__@@@std@@PAX@std@@_N@1@ABK@Z 100472b0 f   Pclass.obj
 0001:000462c0       __unwindfunclet$??$make_unique@VPerfThread@@$$V$0A@@std@@YA?AV?$unique_ptr@VPerfThread@@U?$default_delete@VPerfThread@@@std@@@0@XZ$0 100472c0 f   Pclass.obj
 0001:000462d2       __ehhandler$??$make_unique@VPerfThread@@$$V$0A@@std@@YA?AV?$unique_ptr@VPerfThread@@U?$default_delete@VPerfThread@@@std@@@0@XZ 100472d2 f   Pclass.obj
 0001:000462e0       __unwindfunclet$??0Plist@@QAE@XZ$0 100472e0 f   Pclass.obj
 0001:000462eb       __unwindfunclet$??0Plist@@QAE@XZ$1 100472eb f   Pclass.obj
 0001:000462f6       __unwindfunclet$??0Plist@@QAE@XZ$2 100472f6 f   Pclass.obj
 0001:00046301       __unwindfunclet$??0Plist@@QAE@XZ$3 10047301 f   Pclass.obj
 0001:00046309       __unwindfunclet$??0Plist@@QAE@XZ$7 10047309 f   Pclass.obj
 0001:0004631b       __ehhandler$??0Plist@@QAE@XZ 1004731b f   Pclass.obj
 0001:00046330       __unwindfunclet$?Compare@Plist@@QBEHPBUPluginPanelItem@@0I@Z$0 10047330 f   Pclass.obj
 0001:00046338       __ehhandler$?Compare@Plist@@QBEHPBUPluginPanelItem@@0I@Z 10047338 f   Pclass.obj
 0001:00046350       __unwindfunclet$?Connect@Plist@@QAE_NPB_W00@Z$0 10047350 f   Pclass.obj
 0001:00046358       __unwindfunclet$?Connect@Plist@@QAE_NPB_W00@Z$3 10047358 f   Pclass.obj
 0001:0004636a       __unwindfunclet$?Connect@Plist@@QAE_NPB_W00@Z$1 1004736a f   Pclass.obj
 0001:00046372       __ehhandler$?Connect@Plist@@QAE_NPB_W00@Z 10047372 f   Pclass.obj
 0001:00046380       __unwindfunclet$?ConnectWMI@Plist@@AAE_NXZ$1 10047380 f   Pclass.obj
 0001:0004638f       __ehhandler$?ConnectWMI@Plist@@AAE_NXZ 1004738f f   Pclass.obj
 0001:000463a0       __unwindfunclet$?DeleteFiles@Plist@@QAEHPAUPluginPanelItem@@I_K@Z$0 100473a0 f   Pclass.obj
 0001:000463a8       __unwindfunclet$?DeleteFiles@Plist@@QAEHPAUPluginPanelItem@@I_K@Z$3 100473a8 f   Pclass.obj
 0001:000463b0       __ehhandler$?DeleteFiles@Plist@@QAEHPAUPluginPanelItem@@I_K@Z 100473b0 f   Pclass.obj
 0001:000463c0       __unwindfunclet$?DumpNTCounters@@YAXPAXAAVPerfThread@@KK@Z$0 100473c0 f   Pclass.obj
 0001:000463cb       __unwindfunclet$?DumpNTCounters@@YAXPAXAAVPerfThread@@KK@Z$1 100473cb f   Pclass.obj
 0001:000463d3       __unwindfunclet$?DumpNTCounters@@YAXPAXAAVPerfThread@@KK@Z$2 100473d3 f   Pclass.obj
 0001:000463db       __unwindfunclet$?DumpNTCounters@@YAXPAXAAVPerfThread@@KK@Z$3 100473db f   Pclass.obj
 0001:000463e3       __unwindfunclet$?DumpNTCounters@@YAXPAXAAVPerfThread@@KK@Z$4 100473e3 f   Pclass.obj
 0001:000463eb       __unwindfunclet$?DumpNTCounters@@YAXPAXAAVPerfThread@@KK@Z$5 100473eb f   Pclass.obj
 0001:000463f3       __unwindfunclet$?DumpNTCounters@@YAXPAXAAVPerfThread@@KK@Z$6 100473f3 f   Pclass.obj
 0001:000463fb       __unwindfunclet$?DumpNTCounters@@YAXPAXAAVPerfThread@@KK@Z$7 100473fb f   Pclass.obj
 0001:00046403       __ehhandler$?DumpNTCounters@@YAXPAXAAVPerfThread@@KK@Z 10047403 f   Pclass.obj
 0001:00046410       __unwindfunclet$?GetFiles@Plist@@QAEHPAUPluginPanelItem@@IHPAPB_W_KAAUoptions@@@Z$0 10047410 f   Pclass.obj
 0001:0004641b       __unwindfunclet$?GetFiles@Plist@@QAEHPAUPluginPanelItem@@IHPAPB_W_KAAUoptions@@@Z$1 1004741b f   Pclass.obj
 0001:00046423       __unwindfunclet$?GetFiles@Plist@@QAEHPAUPluginPanelItem@@IHPAPB_W_KAAUoptions@@@Z$2 10047423 f   Pclass.obj
 0001:0004642b       __unwindfunclet$?GetFiles@Plist@@QAEHPAUPluginPanelItem@@IHPAPB_W_KAAUoptions@@@Z$3 1004742b f   Pclass.obj
 0001:00046433       __unwindfunclet$?GetFiles@Plist@@QAEHPAUPluginPanelItem@@IHPAPB_W_KAAUoptions@@@Z$4 10047433 f   Pclass.obj
 0001:0004643b       __unwindfunclet$?GetFiles@Plist@@QAEHPAUPluginPanelItem@@IHPAPB_W_KAAUoptions@@@Z$5 1004743b f   Pclass.obj
 0001:00046443       __unwindfunclet$?GetFiles@Plist@@QAEHPAUPluginPanelItem@@IHPAPB_W_KAAUoptions@@@Z$6 10047443 f   Pclass.obj
 0001:0004644b       __unwindfunclet$?GetFiles@Plist@@QAEHPAUPluginPanelItem@@IHPAPB_W_KAAUoptions@@@Z$7 1004744b f   Pclass.obj
 0001:00046453       __unwindfunclet$?GetFiles@Plist@@QAEHPAUPluginPanelItem@@IHPAPB_W_KAAUoptions@@@Z$8 10047453 f   Pclass.obj
 0001:0004645b       __unwindfunclet$?GetFiles@Plist@@QAEHPAUPluginPanelItem@@IHPAPB_W_KAAUoptions@@@Z$9 1004745b f   Pclass.obj
 0001:00046463       __unwindfunclet$?GetFiles@Plist@@QAEHPAUPluginPanelItem@@IHPAPB_W_KAAUoptions@@@Z$10 10047463 f   Pclass.obj
 0001:0004646b       __unwindfunclet$?GetFiles@Plist@@QAEHPAUPluginPanelItem@@IHPAPB_W_KAAUoptions@@@Z$11 1004746b f   Pclass.obj
 0001:00046473       __unwindfunclet$?GetFiles@Plist@@QAEHPAUPluginPanelItem@@IHPAPB_W_KAAUoptions@@@Z$12 10047473 f   Pclass.obj
 0001:0004647b       __unwindfunclet$?GetFiles@Plist@@QAEHPAUPluginPanelItem@@IHPAPB_W_KAAUoptions@@@Z$13 1004747b f   Pclass.obj
 0001:00046483       __unwindfunclet$?GetFiles@Plist@@QAEHPAUPluginPanelItem@@IHPAPB_W_KAAUoptions@@@Z$14 10047483 f   Pclass.obj
 0001:0004648b       __unwindfunclet$?GetFiles@Plist@@QAEHPAUPluginPanelItem@@IHPAPB_W_KAAUoptions@@@Z$15 1004748b f   Pclass.obj
 0001:00046493       __unwindfunclet$?GetFiles@Plist@@QAEHPAUPluginPanelItem@@IHPAPB_W_KAAUoptions@@@Z$16 10047493 f   Pclass.obj
 0001:0004649b       __unwindfunclet$?GetFiles@Plist@@QAEHPAUPluginPanelItem@@IHPAPB_W_KAAUoptions@@@Z$19 1004749b f   Pclass.obj
 0001:000464a3       __unwindfunclet$?GetFiles@Plist@@QAEHPAUPluginPanelItem@@IHPAPB_W_KAAUoptions@@@Z$20 100474a3 f   Pclass.obj
 0001:000464ab       __unwindfunclet$?GetFiles@Plist@@QAEHPAUPluginPanelItem@@IHPAPB_W_KAAUoptions@@@Z$17 100474ab f   Pclass.obj
 0001:000464b6       __unwindfunclet$?GetFiles@Plist@@QAEHPAUPluginPanelItem@@IHPAPB_W_KAAUoptions@@@Z$18 100474b6 f   Pclass.obj
 0001:000464be       __unwindfunclet$?GetFiles@Plist@@QAEHPAUPluginPanelItem@@IHPAPB_W_KAAUoptions@@@Z$21 100474be f   Pclass.obj
 0001:000464c6       __unwindfunclet$?GetFiles@Plist@@QAEHPAUPluginPanelItem@@IHPAPB_W_KAAUoptions@@@Z$22 100474c6 f   Pclass.obj
 0001:000464d1       __unwindfunclet$?GetFiles@Plist@@QAEHPAUPluginPanelItem@@IHPAPB_W_KAAUoptions@@@Z$23 100474d1 f   Pclass.obj
 0001:000464d9       __unwindfunclet$?GetFiles@Plist@@QAEHPAUPluginPanelItem@@IHPAPB_W_KAAUoptions@@@Z$24 100474d9 f   Pclass.obj
 0001:000464e1       __unwindfunclet$?GetFiles@Plist@@QAEHPAUPluginPanelItem@@IHPAPB_W_KAAUoptions@@@Z$25 100474e1 f   Pclass.obj
 0001:000464e9       __unwindfunclet$?GetFiles@Plist@@QAEHPAUPluginPanelItem@@IHPAPB_W_KAAUoptions@@@Z$26 100474e9 f   Pclass.obj
 0001:000464f1       __unwindfunclet$?GetFiles@Plist@@QAEHPAUPluginPanelItem@@IHPAPB_W_KAAUoptions@@@Z$27 100474f1 f   Pclass.obj
 0001:000464fc       __unwindfunclet$?GetFiles@Plist@@QAEHPAUPluginPanelItem@@IHPAPB_W_KAAUoptions@@@Z$28 100474fc f   Pclass.obj
 0001:00046507       __unwindfunclet$?GetFiles@Plist@@QAEHPAUPluginPanelItem@@IHPAPB_W_KAAUoptions@@@Z$29 10047507 f   Pclass.obj
 0001:0004650f       __unwindfunclet$?GetFiles@Plist@@QAEHPAUPluginPanelItem@@IHPAPB_W_KAAUoptions@@@Z$30 1004750f f   Pclass.obj
 0001:0004651a       __unwindfunclet$?GetFiles@Plist@@QAEHPAUPluginPanelItem@@IHPAPB_W_KAAUoptions@@@Z$31 1004751a f   Pclass.obj
 0001:00046522       __unwindfunclet$?GetFiles@Plist@@QAEHPAUPluginPanelItem@@IHPAPB_W_KAAUoptions@@@Z$32 10047522 f   Pclass.obj
 0001:0004652d       __unwindfunclet$?GetFiles@Plist@@QAEHPAUPluginPanelItem@@IHPAPB_W_KAAUoptions@@@Z$33 1004752d f   Pclass.obj
 0001:00046535       __unwindfunclet$?GetFiles@Plist@@QAEHPAUPluginPanelItem@@IHPAPB_W_KAAUoptions@@@Z$34 10047535 f   Pclass.obj
 0001:00046540       __unwindfunclet$?GetFiles@Plist@@QAEHPAUPluginPanelItem@@IHPAPB_W_KAAUoptions@@@Z$35 10047540 f   Pclass.obj
 0001:00046548       __unwindfunclet$?GetFiles@Plist@@QAEHPAUPluginPanelItem@@IHPAPB_W_KAAUoptions@@@Z$36 10047548 f   Pclass.obj
 0001:00046553       __unwindfunclet$?GetFiles@Plist@@QAEHPAUPluginPanelItem@@IHPAPB_W_KAAUoptions@@@Z$37 10047553 f   Pclass.obj
 0001:0004655e       __unwindfunclet$?GetFiles@Plist@@QAEHPAUPluginPanelItem@@IHPAPB_W_KAAUoptions@@@Z$38 1004755e f   Pclass.obj
 0001:00046566       __unwindfunclet$?GetFiles@Plist@@QAEHPAUPluginPanelItem@@IHPAPB_W_KAAUoptions@@@Z$39 10047566 f   Pclass.obj
 0001:00046571       __unwindfunclet$?GetFiles@Plist@@QAEHPAUPluginPanelItem@@IHPAPB_W_KAAUoptions@@@Z$40 10047571 f   Pclass.obj
 0001:0004657c       __unwindfunclet$?GetFiles@Plist@@QAEHPAUPluginPanelItem@@IHPAPB_W_KAAUoptions@@@Z$41 1004757c f   Pclass.obj
 0001:00046584       __unwindfunclet$?GetFiles@Plist@@QAEHPAUPluginPanelItem@@IHPAPB_W_KAAUoptions@@@Z$42 10047584 f   Pclass.obj
 0001:0004658c       __ehhandler$?GetFiles@Plist@@QAEHPAUPluginPanelItem@@IHPAPB_W_KAAUoptions@@@Z 1004758c f   Pclass.obj
 0001:000465a0       __unwindfunclet$?GetFindData@Plist@@QAEHAAPAUPluginPanelItem@@AAI_K@Z$0 100475a0 f   Pclass.obj
 0001:000465ab       __unwindfunclet$?GetFindData@Plist@@QAEHAAPAUPluginPanelItem@@AAI_K@Z$13 100475ab f   Pclass.obj
 0001:000465b6       __unwindfunclet$?GetFindData@Plist@@QAEHAAPAUPluginPanelItem@@AAI_K@Z$14 100475b6 f   Pclass.obj
 0001:000465c1       __unwindfunclet$?GetFindData@Plist@@QAEHAAPAUPluginPanelItem@@AAI_K@Z$1 100475c1 f   Pclass.obj
 0001:000465cc       __unwindfunclet$?GetFindData@Plist@@QAEHAAPAUPluginPanelItem@@AAI_K@Z$2 100475cc f   Pclass.obj
 0001:000465d4       __unwindfunclet$?GetFindData@Plist@@QAEHAAPAUPluginPanelItem@@AAI_K@Z$3 100475d4 f   Pclass.obj
 0001:000465dc       __unwindfunclet$?GetFindData@Plist@@QAEHAAPAUPluginPanelItem@@AAI_K@Z$4 100475dc f   Pclass.obj
 0001:000465e7       __unwindfunclet$?GetFindData@Plist@@QAEHAAPAUPluginPanelItem@@AAI_K@Z$5 100475e7 f   Pclass.obj
 0001:000465ef       __unwindfunclet$?GetFindData@Plist@@QAEHAAPAUPluginPanelItem@@AAI_K@Z$6 100475ef f   Pclass.obj
 0001:000465fa       __unwindfunclet$?GetFindData@Plist@@QAEHAAPAUPluginPanelItem@@AAI_K@Z$7 100475fa f   Pclass.obj
 0001:00046602       __ehhandler$?GetFindData@Plist@@QAEHAAPAUPluginPanelItem@@AAI_K@Z 10047602 f   Pclass.obj
 0001:00046610       __unwindfunclet$?GetVersionInfo@Plist@@SA_NPB_WAAV?$unique_ptr@$$BY0A@DU?$default_delete@$$BY0A@D@std@@@std@@AAPB_W2@Z$1 10047610 f   Pclass.obj
 0001:00046618       __unwindfunclet$?GetVersionInfo@Plist@@SA_NPB_WAAV?$unique_ptr@$$BY0A@DU?$default_delete@$$BY0A@D@std@@@std@@AAPB_W2@Z$2 10047618 f   Pclass.obj
 0001:00046620       __unwindfunclet$?GetVersionInfo@Plist@@SA_NPB_WAAV?$unique_ptr@$$BY0A@DU?$default_delete@$$BY0A@D@std@@@std@@AAPB_W2@Z$4 10047620 f   Pclass.obj
 0001:00046628       __ehhandler$?GetVersionInfo@Plist@@SA_NPB_WAAV?$unique_ptr@$$BY0A@DU?$default_delete@$$BY0A@D@std@@@std@@AAPB_W2@Z 10047628 f   Pclass.obj
 0001:00046640       __unwindfunclet$?InitializePanelModes@Plist@@SAXXZ$0 10047640 f   Pclass.obj
 0001:0004664b       __unwindfunclet$?InitializePanelModes@Plist@@SAXXZ$8 1004764b f   Pclass.obj
 0001:00046656       __unwindfunclet$?InitializePanelModes@Plist@@SAXXZ$9 10047656 f   Pclass.obj
 0001:00046661       __unwindfunclet$?InitializePanelModes@Plist@@SAXXZ$17 10047661 f   Pclass.obj
 0001:0004666c       __unwindfunclet$?InitializePanelModes@Plist@@SAXXZ$18 1004766c f   Pclass.obj
 0001:00046677       __unwindfunclet$?InitializePanelModes@Plist@@SAXXZ$26 10047677 f   Pclass.obj
 0001:00046682       __unwindfunclet$?InitializePanelModes@Plist@@SAXXZ$27 10047682 f   Pclass.obj
 0001:0004668d       __unwindfunclet$?InitializePanelModes@Plist@@SAXXZ$35 1004768d f   Pclass.obj
 0001:00046698       __unwindfunclet$?InitializePanelModes@Plist@@SAXXZ$36 10047698 f   Pclass.obj
 0001:000466a3       __unwindfunclet$?InitializePanelModes@Plist@@SAXXZ$44 100476a3 f   Pclass.obj
 0001:000466ae       __unwindfunclet$?InitializePanelModes@Plist@@SAXXZ$45 100476ae f   Pclass.obj
 0001:000466b9       __unwindfunclet$?InitializePanelModes@Plist@@SAXXZ$53 100476b9 f   Pclass.obj
 0001:000466c4       __unwindfunclet$?InitializePanelModes@Plist@@SAXXZ$54 100476c4 f   Pclass.obj
 0001:000466cf       __unwindfunclet$?InitializePanelModes@Plist@@SAXXZ$62 100476cf f   Pclass.obj
 0001:000466da       __unwindfunclet$?InitializePanelModes@Plist@@SAXXZ$63 100476da f   Pclass.obj
 0001:000466e5       __unwindfunclet$?InitializePanelModes@Plist@@SAXXZ$71 100476e5 f   Pclass.obj
 0001:000466f0       __unwindfunclet$?InitializePanelModes@Plist@@SAXXZ$72 100476f0 f   Pclass.obj
 0001:000466fb       __unwindfunclet$?InitializePanelModes@Plist@@SAXXZ$80 100476fb f   Pclass.obj
 0001:00046706       __unwindfunclet$?InitializePanelModes@Plist@@SAXXZ$81 10047706 f   Pclass.obj
 0001:00046711       __unwindfunclet$?InitializePanelModes@Plist@@SAXXZ$90 10047711 f   Pclass.obj
 0001:0004672a       __unwindfunclet$?InitializePanelModes@Plist@@SAXXZ$91 1004772a f   Pclass.obj
 0001:00046735       __unwindfunclet$?InitializePanelModes@Plist@@SAXXZ$99 10047735 f   Pclass.obj
 0001:00046740       __unwindfunclet$?InitializePanelModes@Plist@@SAXXZ$100 10047740 f   Pclass.obj
 0001:0004674b       __unwindfunclet$?InitializePanelModes@Plist@@SAXXZ$108 1004774b f   Pclass.obj
 0001:00046756       __unwindfunclet$?InitializePanelModes@Plist@@SAXXZ$109 10047756 f   Pclass.obj
 0001:00046761       __unwindfunclet$?InitializePanelModes@Plist@@SAXXZ$117 10047761 f   Pclass.obj
 0001:0004676c       __unwindfunclet$?InitializePanelModes@Plist@@SAXXZ$118 1004776c f   Pclass.obj
 0001:00046777       __unwindfunclet$?InitializePanelModes@Plist@@SAXXZ$126 10047777 f   Pclass.obj
 0001:00046782       __unwindfunclet$?InitializePanelModes@Plist@@SAXXZ$127 10047782 f   Pclass.obj
 0001:0004678d       __unwindfunclet$?InitializePanelModes@Plist@@SAXXZ$135 1004778d f   Pclass.obj
 0001:00046798       __unwindfunclet$?InitializePanelModes@Plist@@SAXXZ$136 10047798 f   Pclass.obj
 0001:000467a3       __unwindfunclet$?InitializePanelModes@Plist@@SAXXZ$144 100477a3 f   Pclass.obj
 0001:000467ae       __unwindfunclet$?InitializePanelModes@Plist@@SAXXZ$145 100477ae f   Pclass.obj
 0001:000467b9       __unwindfunclet$?InitializePanelModes@Plist@@SAXXZ$153 100477b9 f   Pclass.obj
 0001:000467c4       __unwindfunclet$?InitializePanelModes@Plist@@SAXXZ$154 100477c4 f   Pclass.obj
 0001:000467cf       __unwindfunclet$?InitializePanelModes@Plist@@SAXXZ$162 100477cf f   Pclass.obj
 0001:000467da       __unwindfunclet$?InitializePanelModes@Plist@@SAXXZ$163 100477da f   Pclass.obj
 0001:000467e5       __unwindfunclet$?InitializePanelModes@Plist@@SAXXZ$171 100477e5 f   Pclass.obj
 0001:000467f0       __unwindfunclet$?InitializePanelModes@Plist@@SAXXZ$172 100477f0 f   Pclass.obj
 0001:000467fb       __unwindfunclet$?InitializePanelModes@Plist@@SAXXZ$181 100477fb f   Pclass.obj
 0001:00046814       __unwindfunclet$?InitializePanelModes@Plist@@SAXXZ$182 10047814 f   Pclass.obj
 0001:0004681c       __unwindfunclet$?InitializePanelModes@Plist@@SAXXZ$183 1004781c f   Pclass.obj
 0001:00046824       __ehhandler$?InitializePanelModes@Plist@@SAXXZ 10047824 f   Pclass.obj
 0001:00046830       __unwindfunclet$?PrintOwnerInfo@Plist@@AAEXPAXK@Z$0 10047830 f   Pclass.obj
 0001:00046838       __unwindfunclet$?PrintOwnerInfo@Plist@@AAEXPAXK@Z$1 10047838 f   Pclass.obj
 0001:00046843       __unwindfunclet$?PrintOwnerInfo@Plist@@AAEXPAXK@Z$2 10047843 f   Pclass.obj
 0001:0004684b       __unwindfunclet$?PrintOwnerInfo@Plist@@AAEXPAXK@Z$3 1004784b f   Pclass.obj
 0001:00046853       __unwindfunclet$?PrintOwnerInfo@Plist@@AAEXPAXK@Z$4 10047853 f   Pclass.obj
 0001:0004685b       __unwindfunclet$?PrintOwnerInfo@Plist@@AAEXPAXK@Z$5 1004785b f   Pclass.obj
 0001:00046863       __unwindfunclet$?PrintOwnerInfo@Plist@@AAEXPAXK@Z$6 10047863 f   Pclass.obj
 0001:0004686e       __unwindfunclet$?PrintOwnerInfo@Plist@@AAEXPAXK@Z$7 1004786e f   Pclass.obj
 0001:00046876       __ehhandler$?PrintOwnerInfo@Plist@@AAEXPAXK@Z 10047876 f   Pclass.obj
 0001:00046880       __unwindfunclet$?PrintVersionInfo@Plist@@CAXPAXPB_W@Z$0 10047880 f   Pclass.obj
 0001:00046888       __unwindfunclet$?PrintVersionInfo@Plist@@CAXPAXPB_W@Z$1 10047888 f   Pclass.obj
 0001:00046890       __unwindfunclet$?PrintVersionInfo@Plist@@CAXPAXPB_W@Z$2 10047890 f   Pclass.obj
 0001:00046898       __unwindfunclet$?PrintVersionInfo@Plist@@CAXPAXPB_W@Z$3 10047898 f   Pclass.obj
 0001:000468a0       __unwindfunclet$?PrintVersionInfo@Plist@@CAXPAXPB_W@Z$4 100478a0 f   Pclass.obj
 0001:000468a8       __ehhandler$?PrintVersionInfo@Plist@@CAXPAXPB_W@Z 100478a8 f   Pclass.obj
 0001:000468c0       __unwindfunclet$?ProcessEvent@Plist@@QAEHHPAX@Z$0 100478c0 f   Pclass.obj
 0001:000468c8       __ehhandler$?ProcessEvent@Plist@@QAEHHPAX@Z 100478c8 f   Pclass.obj
 0001:000468e0       __unwindfunclet$?ProcessKey@Plist@@QAEHPBU_INPUT_RECORD@@@Z$0 100478e0 f   Pclass.obj
 0001:000468e8       __unwindfunclet$?ProcessKey@Plist@@QAEHPBU_INPUT_RECORD@@@Z$4 100478e8 f   Pclass.obj
 0001:000468f3       __unwindfunclet$?ProcessKey@Plist@@QAEHPBU_INPUT_RECORD@@@Z$16 100478f3 f   Pclass.obj
 0001:00046905       __unwindfunclet$?ProcessKey@Plist@@QAEHPBU_INPUT_RECORD@@@Z$1 10047905 f   Pclass.obj
 0001:0004690d       __unwindfunclet$?ProcessKey@Plist@@QAEHPBU_INPUT_RECORD@@@Z$2 1004790d f   Pclass.obj
 0001:00046918       __unwindfunclet$?ProcessKey@Plist@@QAEHPBU_INPUT_RECORD@@@Z$3 10047918 f   Pclass.obj
 0001:00046920       __unwindfunclet$?ProcessKey@Plist@@QAEHPBU_INPUT_RECORD@@@Z$7 10047920 f   Pclass.obj
 0001:00046928       __unwindfunclet$?ProcessKey@Plist@@QAEHPBU_INPUT_RECORD@@@Z$8 10047928 f   Pclass.obj
 0001:00046930       __unwindfunclet$?ProcessKey@Plist@@QAEHPBU_INPUT_RECORD@@@Z$9 10047930 f   Pclass.obj
 0001:00046938       __unwindfunclet$?ProcessKey@Plist@@QAEHPBU_INPUT_RECORD@@@Z$10 10047938 f   Pclass.obj
 0001:00046940       __unwindfunclet$?ProcessKey@Plist@@QAEHPBU_INPUT_RECORD@@@Z$20 10047940 f   Pclass.obj
 0001:0004694b       __unwindfunclet$?ProcessKey@Plist@@QAEHPBU_INPUT_RECORD@@@Z$11 1004794b f   Pclass.obj
 0001:00046953       __unwindfunclet$?ProcessKey@Plist@@QAEHPBU_INPUT_RECORD@@@Z$12 10047953 f   Pclass.obj
 0001:0004695b       __ehhandler$?ProcessKey@Plist@@QAEHPBU_INPUT_RECORD@@@Z 1004795b f   Pclass.obj
 0001:00046970       __unwindfunclet$?SavePanelModes@Plist@@SAXXZ$0 10047970 f   Pclass.obj
 0001:00046978       __unwindfunclet$?SavePanelModes@Plist@@SAXXZ$1 10047978 f   Pclass.obj
 0001:00046980       __ehhandler$?SavePanelModes@Plist@@SAXXZ 10047980 f   Pclass.obj
 0001:00046990       __unwindfunclet$?TranslateMode@@YA_NABV?$basic_string@_WU?$char_traits@_W@std@@V?$allocator@_W@2@@std@@AAV12@@Z$0 10047990 f   Pclass.obj
 0001:00046998       __ehhandler$?TranslateMode@@YA_NABV?$basic_string@_WU?$char_traits@_W@std@@V?$allocator@_W@2@@std@@AAV12@@Z 10047998 f   Pclass.obj
 0001:000469b0       __unwindfunclet$?generate_titles@@YAXABV?$basic_string@_WU?$char_traits@_W@std@@V?$allocator@_W@2@@std@@AAUPanelMode@@@Z$0 100479b0 f   Pclass.obj
 0001:000469b8       __ehhandler$?generate_titles@@YAXABV?$basic_string@_WU?$char_traits@_W@std@@V?$allocator@_W@2@@std@@AAUPanelMode@@@Z 100479b8 f   Pclass.obj
 0001:000469d0       __unwindfunclet$?ui64toa_width@@YA?AV?$basic_string@_WU?$char_traits@_W@std@@V?$allocator@_W@2@@std@@_KI_N@Z$0 100479d0 f   Pclass.obj
 0001:000469d0       __unwindfunclet$?read_string@?$ipc_functions@$00@@SA?AV?$basic_string@_WU?$char_traits@_W@std@@V?$allocator@_W@2@@std@@PAXABUUNICODE_STRING_64@detail@@@Z$0 100479d0 f   Plist.obj
 0001:000469d8       __ehhandler$?ui64toa_width@@YA?AV?$basic_string@_WU?$char_traits@_W@std@@V?$allocator@_W@2@@std@@_KI_N@Z 100479d8 f   Pclass.obj
 0001:000469d8       __ehhandler$?read_string@?$ipc_functions@$00@@SA?AV?$basic_string@_WU?$char_traits@_W@std@@V?$allocator@_W@2@@std@@PAXABUUNICODE_STRING_64@detail@@@Z 100479d8 f   Plist.obj
 0001:000469f0       __unwindfunclet$?window_ex_style@@YA@PAUHWND__@@@Z$0 100479f0 f   Pclass.obj
 0001:000469f0       __unwindfunclet$?window_style@@YA@PAUHWND__@@@Z$0 100479f0 f   Pclass.obj
 0001:000469f8       __ehhandler$?window_ex_style@@YA@PAUHWND__@@@Z 100479f8 f   Pclass.obj
 0001:000469f8       __ehhandler$?window_style@@YA@PAUHWND__@@@Z 100479f8 f   Pclass.obj
 0001:00046a10       __unwindfunclet$??0PerfThread@@QAE@PB_W00@Z$16 10047a10 f   perfthread.obj
 0001:00046a1e       __unwindfunclet$??0PerfThread@@QAE@PB_W00@Z$0 10047a1e f   perfthread.obj
 0001:00046a29       __unwindfunclet$??0PerfThread@@QAE@PB_W00@Z$1 10047a29 f   perfthread.obj
 0001:00046a34       __unwindfunclet$??0PerfThread@@QAE@PB_W00@Z$2 10047a34 f   perfthread.obj
 0001:00046a3f       __unwindfunclet$??0PerfThread@@QAE@PB_W00@Z$3 10047a3f f   perfthread.obj
 0001:00046a4a       __unwindfunclet$??0PerfThread@@QAE@PB_W00@Z$4 10047a4a f   perfthread.obj
 0001:00046a55       __unwindfunclet$??0PerfThread@@QAE@PB_W00@Z$5 10047a55 f   perfthread.obj
 0001:00046a60       __unwindfunclet$??0PerfThread@@QAE@PB_W00@Z$6 10047a60 f   perfthread.obj
 0001:00046a6b       __unwindfunclet$??0PerfThread@@QAE@PB_W00@Z$7 10047a6b f   perfthread.obj
 0001:00046a76       __unwindfunclet$??0PerfThread@@QAE@PB_W00@Z$8 10047a76 f   perfthread.obj
 0001:00046a81       __unwindfunclet$??0PerfThread@@QAE@PB_W00@Z$9 10047a81 f   perfthread.obj
 0001:00046a8f       __unwindfunclet$??0PerfThread@@QAE@PB_W00@Z$10 10047a8f f   perfthread.obj
 0001:00046a9d       __unwindfunclet$??0PerfThread@@QAE@PB_W00@Z$11 10047a9d f   perfthread.obj
 0001:00046aa5       __unwindfunclet$??0PerfThread@@QAE@PB_W00@Z$13 10047aa5 f   perfthread.obj
 0001:00046aad       __unwindfunclet$??0PerfThread@@QAE@PB_W00@Z$14 10047aad f   perfthread.obj
 0001:00046ab5       __ehhandler$??0PerfThread@@QAE@PB_W00@Z 10047ab5 f   perfthread.obj
 0001:00046ac0       __unwindfunclet$?Refresh@PerfThread@@AAEXXZ$0 10047ac0 f   perfthread.obj
 0001:00046ac8       __unwindfunclet$?Refresh@PerfThread@@AAEXXZ$1 10047ac8 f   perfthread.obj
 0001:00046ad0       __unwindfunclet$?Refresh@PerfThread@@AAEXXZ$2 10047ad0 f   perfthread.obj
 0001:00046ad8       __unwindfunclet$?Refresh@PerfThread@@AAEXXZ$5 10047ad8 f   perfthread.obj
 0001:00046ae0       __ehhandler$?Refresh@PerfThread@@AAEXXZ 10047ae0 f   perfthread.obj
 0001:00046af0       __unwindfunclet$?RefreshWMIData@PerfThread@@AAEXXZ$2 10047af0 f   perfthread.obj
 0001:00046af8       __ehhandler$?RefreshWMIData@PerfThread@@AAEXXZ 10047af8 f   perfthread.obj
 0001:00046b10       __unwindfunclet$??$print_module@PAX@@YAXQAXPAXKAAUoptions@@ABV?$function@$$A6A_NPA_WI@Z@std@@@Z$0 10047b10 f   Plist.obj
 0001:00046b18       __ehhandler$??$print_module@PAX@@YAXQAXPAXKAAUoptions@@ABV?$function@$$A6A_NPA_WI@Z@std@@@Z 10047b18 f   Plist.obj
 0001:00046b30       __unwindfunclet$??0?$vector@UProcessPerfData@@V?$allocator@UProcessPerfData@@@std@@@std@@QAE@ABV01@@Z$0 10047b30 f   Plist.obj
 0001:00046b38       __unwindfunclet$??0?$vector@UProcessPerfData@@V?$allocator@UProcessPerfData@@@std@@@std@@QAE@ABV01@@Z$1 10047b38 f   Plist.obj
 0001:00046b40       __unwindfunclet$??0?$vector@UProcessPerfData@@V?$allocator@UProcessPerfData@@@std@@@std@@QAE@ABV01@@Z$2 10047b40 f   Plist.obj
 0001:00046b4e       __unwindfunclet$??0?$vector@UProcessPerfData@@V?$allocator@UProcessPerfData@@@std@@@std@@QAE@ABV01@@Z$3 10047b4e f   Plist.obj
 0001:00046b5c       __unwindfunclet$??0?$vector@UProcessPerfData@@V?$allocator@UProcessPerfData@@@std@@@std@@QAE@ABV01@@Z$4 10047b5c f   Plist.obj
 0001:00046b6a       __ehhandler$??0?$vector@UProcessPerfData@@V?$allocator@UProcessPerfData@@@std@@@std@@QAE@ABV01@@Z 10047b6a f   Plist.obj
 0001:00046b80       __unwindfunclet$?GetList@@YA_NAAPAUPluginPanelItem@@AAIAAVPerfThread@@@Z$0 10047b80 f   Plist.obj
 0001:00046b88       __ehhandler$?GetList@@YA_NAAPAUPluginPanelItem@@AAIAAVPerfThread@@@Z 10047b88 f   Plist.obj
 0001:00046ba0       __unwindfunclet$?GetOpenProcessData@@YAXPAXPAV?$basic_string@_WU?$char_traits@_W@std@@V?$allocator@_W@2@@std@@1111@Z$0 10047ba0 f   Plist.obj
 0001:00046ba0       __unwindfunclet$?is_wow64_itself@@YA_NXZ$0 10047ba0 f   Plist.obj
 0001:00046bae       __ehhandler$?GetOpenProcessData@@YAXPAXPAV?$basic_string@_WU?$char_traits@_W@std@@V?$allocator@_W@2@@std@@1111@Z 10047bae f   Plist.obj
 0001:00046bae       __ehhandler$?is_wow64_itself@@YA_NXZ 10047bae f   Plist.obj
 0001:00046bc0       __unwindfunclet$?KillProcess@@YA_NKPAUHWND__@@@Z$0 10047bc0 f   Plist.obj
 0001:00046bc8       __unwindfunclet$?KillProcess@@YA_NKPAUHWND__@@@Z$1 10047bc8 f   Plist.obj
 0001:00046bd0       __ehhandler$?KillProcess@@YA_NKPAUHWND__@@@Z 10047bd0 f   Plist.obj
 0001:00046be0       __unwindfunclet$?PrintModules@?$ipc_functions@$00@@SAXPAX0AAUoptions@@@Z$0 10047be0 f   Plist.obj
 0001:00046be8       __unwindfunclet$?PrintModules@?$ipc_functions@$00@@SAXPAX0AAUoptions@@@Z$1 10047be8 f   Plist.obj
 0001:00046bf0       __ehhandler$?PrintModules@?$ipc_functions@$00@@SAXPAX0AAUoptions@@@Z 10047bf0 f   Plist.obj
 0001:00046c00       __unwindfunclet$?PrintModules@?$ipc_functions@$0A@@@SAXPAX0AAUoptions@@@Z$0 10047c00 f   Plist.obj
 0001:00046c08       __ehhandler$?PrintModules@?$ipc_functions@$0A@@@SAXPAX0AAUoptions@@@Z 10047c08 f   Plist.obj
 0001:00046c20       __unwindfunclet$?PrintModules@@YAXPAXKAAUoptions@@@Z$0 10047c20 f   Plist.obj
 0001:00046c28       __unwindfunclet$?PrintModules@@YAXPAXKAAUoptions@@@Z$1 10047c28 f   Plist.obj
 0001:00046c30       __unwindfunclet$?PrintModules@@YAXPAXKAAUoptions@@@Z$2 10047c30 f   Plist.obj
 0001:00046c38       __unwindfunclet$?PrintModules@@YAXPAXKAAUoptions@@@Z$3 10047c38 f   Plist.obj
 0001:00046c40       __ehhandler$?PrintModules@@YAXPAXKAAUoptions@@@Z 10047c40 f   Plist.obj
 0001:00046c50       __unwindfunclet$?PrintNTCurDirAndEnv@@YAXPAX0H@Z$0 10047c50 f   Plist.obj
 0001:00046c58       __unwindfunclet$?PrintNTCurDirAndEnv@@YAXPAX0H@Z$1 10047c58 f   Plist.obj
 0001:00046c60       __unwindfunclet$?PrintNTCurDirAndEnv@@YAXPAX0H@Z$7 10047c60 f   Plist.obj
 0001:00046c6e       __unwindfunclet$?PrintNTCurDirAndEnv@@YAXPAX0H@Z$2 10047c6e f   Plist.obj
 0001:00046c76       __unwindfunclet$?PrintNTCurDirAndEnv@@YAXPAX0H@Z$3 10047c76 f   Plist.obj
 0001:00046c7e       __unwindfunclet$?PrintNTCurDirAndEnv@@YAXPAX0H@Z$4 10047c7e f   Plist.obj
 0001:00046c86       __ehhandler$?PrintNTCurDirAndEnv@@YAXPAX0H@Z 10047c86 f   Plist.obj
 0001:00046c90       __unwindfunclet$?print_module_impl@@YAXQAXABV?$basic_string@_WU?$char_traits@_W@std@@V?$allocator@_W@2@@std@@KABUoptions@@ABV?$function@$$A6A_NPA_WI@Z@2@@Z$0 10047c90 f   Plist.obj
 0001:00046c98       __unwindfunclet$?print_module_impl@@YAXQAXABV?$basic_string@_WU?$char_traits@_W@std@@V?$allocator@_W@2@@std@@KABUoptions@@ABV?$function@$$A6A_NPA_WI@Z@2@@Z$1 10047c98 f   Plist.obj
 0001:00046ca0       __unwindfunclet$?print_module_impl@@YAXQAXABV?$basic_string@_WU?$char_traits@_W@std@@V?$allocator@_W@2@@std@@KABUoptions@@ABV?$function@$$A6A_NPA_WI@Z@2@@Z$2 10047ca0 f   Plist.obj
 0001:00046ca8       __ehhandler$?print_module_impl@@YAXQAXABV?$basic_string@_WU?$char_traits@_W@std@@V?$allocator@_W@2@@std@@KABUoptions@@ABV?$function@$$A6A_NPA_WI@Z@2@@Z 10047ca8 f   Plist.obj
 0001:00046cc0       __unwindfunclet$?WinError@@YAHPB_W@Z$0 10047cc0 f   Pmix.obj
 0001:00046cc8       __unwindfunclet$?WinError@@YAHPB_W@Z$1 10047cc8 f   Pmix.obj
 0001:00046cd0       __ehhandler$?WinError@@YAHPB_W@Z 10047cd0 f   Pmix.obj
 0001:00046ce0       __unwindfunclet$??0WMIConnection@@QAE@XZ$0 10047ce0 f   WMI.obj
 0001:00046ce8       __ehhandler$??0WMIConnection@@QAE@XZ 10047ce8 f   WMI.obj
 0001:00046d00       __ehhandler$??1?$ptr_setter@V?$unique_ptr@UIWbemClassObject@@Ucom_closer@@@std@@@@QAE@XZ 10047d00 f   WMI.obj
 0001:00046d00       __ehhandler$??1WMIConnection@@QAE@XZ 10047d00 f   WMI.obj
 0001:00046d10       __unwindfunclet$?Connect@WMIConnection@@QAE_NPB_W00@Z$0 10047d10 f   WMI.obj
 0001:00046d18       __unwindfunclet$?Connect@WMIConnection@@QAE_NPB_W00@Z$2 10047d18 f   WMI.obj
 0001:00046d20       __unwindfunclet$?Connect@WMIConnection@@QAE_NPB_W00@Z$3 10047d20 f   WMI.obj
 0001:00046d28       __unwindfunclet$?Connect@WMIConnection@@QAE_NPB_W00@Z$4 10047d28 f   WMI.obj
 0001:00046d30       __unwindfunclet$?Connect@WMIConnection@@QAE_NPB_W00@Z$5 10047d30 f   WMI.obj
 0001:00046d38       __ehhandler$?Connect@WMIConnection@@QAE_NPB_W00@Z 10047d38 f   WMI.obj
 0001:00046d50       __unwindfunclet$?ExecMethod@WMIConnection@@AAEHKPB_W0K@Z$0 10047d50 f   WMI.obj
 0001:00046d58       __unwindfunclet$?ExecMethod@WMIConnection@@AAEHKPB_W0K@Z$1 10047d58 f   WMI.obj
 0001:00046d60       __unwindfunclet$?ExecMethod@WMIConnection@@AAEHKPB_W0K@Z$2 10047d60 f   WMI.obj
 0001:00046d68       __unwindfunclet$?ExecMethod@WMIConnection@@AAEHKPB_W0K@Z$3 10047d68 f   WMI.obj
 0001:00046d70       __unwindfunclet$?ExecMethod@WMIConnection@@AAEHKPB_W0K@Z$4 10047d70 f   WMI.obj
 0001:00046d78       __unwindfunclet$?ExecMethod@WMIConnection@@AAEHKPB_W0K@Z$5 10047d78 f   WMI.obj
 0001:00046d80       __unwindfunclet$?ExecMethod@WMIConnection@@AAEHKPB_W0K@Z$6 10047d80 f   WMI.obj
 0001:00046d88       __unwindfunclet$?ExecMethod@WMIConnection@@AAEHKPB_W0K@Z$7 10047d88 f   WMI.obj
 0001:00046d90       __unwindfunclet$?ExecMethod@WMIConnection@@AAEHKPB_W0K@Z$8 10047d90 f   WMI.obj
 0001:00046d98       __unwindfunclet$?ExecMethod@WMIConnection@@AAEHKPB_W0K@Z$9 10047d98 f   WMI.obj
 0001:00046da0       __unwindfunclet$?ExecMethod@WMIConnection@@AAEHKPB_W0K@Z$10 10047da0 f   WMI.obj
 0001:00046da8       __ehhandler$?ExecMethod@WMIConnection@@AAEHKPB_W0K@Z 10047da8 f   WMI.obj
 0001:00046dc0       __unwindfunclet$?GetProcessCommandLine@WMIConnection@@QAE?AV?$basic_string@_WU?$char_traits@_W@std@@V?$allocator@_W@2@@std@@K@Z$1 10047dc0 f   WMI.obj
 0001:00046dc0       __unwindfunclet$?GetProcessExecutablePath@WMIConnection@@QAE?AV?$basic_string@_WU?$char_traits@_W@std@@V?$allocator@_W@2@@std@@K@Z$1 10047dc0 f   WMI.obj
 0001:00046dd9       __unwindfunclet$?GetProcessCommandLine@WMIConnection@@QAE?AV?$basic_string@_WU?$char_traits@_W@std@@V?$allocator@_W@2@@std@@K@Z$2 10047dd9 f   WMI.obj
 0001:00046dd9       __unwindfunclet$?GetProcessExecutablePath@WMIConnection@@QAE?AV?$basic_string@_WU?$char_traits@_W@std@@V?$allocator@_W@2@@std@@K@Z$2 10047dd9 f   WMI.obj
 0001:00046de1       __ehhandler$?GetProcessCommandLine@WMIConnection@@QAE?AV?$basic_string@_WU?$char_traits@_W@std@@V?$allocator@_W@2@@std@@K@Z 10047de1 f   WMI.obj
 0001:00046de1       __ehhandler$?GetProcessExecutablePath@WMIConnection@@QAE?AV?$basic_string@_WU?$char_traits@_W@std@@V?$allocator@_W@2@@std@@K@Z 10047de1 f   WMI.obj
 0001:00046df0       __unwindfunclet$?GetProcessOwner@WMIConnection@@QAE?AV?$basic_string@_WU?$char_traits@_W@std@@V?$allocator@_W@2@@std@@KPAV23@@Z$0 10047df0 f   WMI.obj
 0001:00046df0       __unwindfunclet$?GetProcessUserSid@WMIConnection@@QAE?AV?$basic_string@_WU?$char_traits@_W@std@@V?$allocator@_W@2@@std@@K@Z$0 10047df0 f   WMI.obj
 0001:00046df8       __unwindfunclet$?GetProcessOwner@WMIConnection@@QAE?AV?$basic_string@_WU?$char_traits@_W@std@@V?$allocator@_W@2@@std@@KPAV23@@Z$1 10047df8 f   WMI.obj
 0001:00046df8       __unwindfunclet$?GetProcessUserSid@WMIConnection@@QAE?AV?$basic_string@_WU?$char_traits@_W@std@@V?$allocator@_W@2@@std@@K@Z$1 10047df8 f   WMI.obj
 0001:00046e00       __unwindfunclet$?GetProcessOwner@WMIConnection@@QAE?AV?$basic_string@_WU?$char_traits@_W@std@@V?$allocator@_W@2@@std@@KPAV23@@Z$2 10047e00 f   WMI.obj
 0001:00046e00       __unwindfunclet$?GetProcessUserSid@WMIConnection@@QAE?AV?$basic_string@_WU?$char_traits@_W@std@@V?$allocator@_W@2@@std@@K@Z$2 10047e00 f   WMI.obj
 0001:00046e08       __unwindfunclet$?GetProcessOwner@WMIConnection@@QAE?AV?$basic_string@_WU?$char_traits@_W@std@@V?$allocator@_W@2@@std@@KPAV23@@Z$3 10047e08 f   WMI.obj
 0001:00046e08       __unwindfunclet$?GetProcessUserSid@WMIConnection@@QAE?AV?$basic_string@_WU?$char_traits@_W@std@@V?$allocator@_W@2@@std@@K@Z$3 10047e08 f   WMI.obj
 0001:00046e10       __unwindfunclet$?GetProcessOwner@WMIConnection@@QAE?AV?$basic_string@_WU?$char_traits@_W@std@@V?$allocator@_W@2@@std@@KPAV23@@Z$5 10047e10 f   WMI.obj
 0001:00046e10       __unwindfunclet$?GetProcessUserSid@WMIConnection@@QAE?AV?$basic_string@_WU?$char_traits@_W@std@@V?$allocator@_W@2@@std@@K@Z$5 10047e10 f   WMI.obj
 0001:00046e18       __ehhandler$?GetProcessOwner@WMIConnection@@QAE?AV?$basic_string@_WU?$char_traits@_W@std@@V?$allocator@_W@2@@std@@KPAV23@@Z 10047e18 f   WMI.obj
 0001:00046e18       __ehhandler$?GetProcessUserSid@WMIConnection@@QAE?AV?$basic_string@_WU?$char_traits@_W@std@@V?$allocator@_W@2@@std@@K@Z 10047e18 f   WMI.obj
 0001:00046e30       __unwindfunclet$?GetProcessPriority@WMIConnection@@QAEKK@Z$0 10047e30 f   WMI.obj
 0001:00046e30       __unwindfunclet$?GetProcessSessionId@WMIConnection@@QAEKK@Z$0 10047e30 f   WMI.obj
 0001:00046e38       __ehhandler$?GetProcessPriority@WMIConnection@@QAEKK@Z 10047e38 f   WMI.obj
 0001:00046e38       __ehhandler$?GetProcessSessionId@WMIConnection@@QAEKK@Z 10047e38 f   WMI.obj
 0001:00046e50       __unwindfunclet$?GetProcessProperty@WMIConnection@@AAE_NKPB_WABV?$function@$$A6AXABUtagVARIANT@@@Z@std@@@Z$0 10047e50 f   WMI.obj
 0001:00046e58       __unwindfunclet$?GetProcessProperty@WMIConnection@@AAE_NKPB_WABV?$function@$$A6AXABUtagVARIANT@@@Z@std@@@Z$1 10047e58 f   WMI.obj
 0001:00046e60       __unwindfunclet$?GetProcessProperty@WMIConnection@@AAE_NKPB_WABV?$function@$$A6AXABUtagVARIANT@@@Z@std@@@Z$2 10047e60 f   WMI.obj
 0001:00046e68       __ehhandler$?GetProcessProperty@WMIConnection@@AAE_NKPB_WABV?$function@$$A6AXABUtagVARIANT@@@Z@std@@@Z 10047e68 f   WMI.obj
 0001:00046e72       __unwindfunclet$?_Init@locale@std@@CAPAV_Locimp@12@_N@Z$0 10047e72 f   libcpmt:locale0.obj
 0001:00046e7a       __ehhandler$?_Init@locale@std@@CAPAV_Locimp@12@_N@Z 10047e7a f   libcpmt:locale0.obj
 0001:00046e95       __ehhandler$??1_Init_atexit@@QAE@XZ 10047e95 f   libcpmt:iosptrs.obj
 0001:00046eb0       __ehhandler$?CallUnexpected@@YAXPBU_s_ESTypeList@@@Z 10047eb0 f   libvcruntime:frame.obj
 0001:00046ecb       __unwindfunclet$?_wcstombs_l_helper@@YAIPADPB_WIPAU__crt_locale_pointers@@@Z$0 10047ecb f   libucrt:wcstombs.obj
 0001:00046ed3       __ehhandler$?_wcstombs_l_helper@@YAIPADPB_WIPAU__crt_locale_pointers@@@Z 10047ed3 f   libucrt:wcstombs.obj
 0001:00046f00       ??__F?m_PanelModesDataLocal@Plist@@0V?$vector@Umode@@V?$allocator@Umode@@@std@@@std@@A@@YAXXZ 10047f00 f   fileio.obj
 0001:00046f10       ??__F?m_PanelModesDataRemote@Plist@@0V?$vector@Umode@@V?$allocator@Umode@@@std@@@std@@A@@YAXXZ 10047f10 f   fileio.obj
 0001:00046f20       ??__FUserAccountID@?1??GetUserAccountID@@YA@XZ@YAXXZ 10047f20 f   handles.obj
 0001:00046f80       ??__FTitle@?1??GetOpenPanelInfo@Plist@@QAEXPAUOpenPanelInfo@@@Z@YAXXZ 10047f80 f   Pclass.obj
 0001:00046fe0       ??__FhDebugToken@@YAXXZ    10047fe0 f   Plist.obj
 0001:00047000       ??__FDeleter@?1??InitializeSListHead@implementation@slist@@YGXPAT_SLIST_HEADER@@@Z@YAXXZ 10048000 f   vc_crt_fix_impl.obj
 0001:0004703d       ??__Finitlocks@std@@YAXXZ  1004803d f   libcpmt:xlock.obj
 0001:00047047       ??__F_Fac_tidy_reg@std@@YAXXZ 10048047 f   libcpmt:locale0.obj
 0001:00047051       ??__Fclassic_locale@std@@YAXXZ 10048051 f   libcpmt:locale0.obj
 0001:0004705b       ??__Finit_atexit@@YAXXZ    1004805b f   libcpmt:iosptrs.obj
 0001:00047065       ??__Finitlocks@std@@YAXXZ  10048065 f   libcpmt:iosptrs.obj
 0001:00047070       __ehfuncinfo$??0_Locinfo@std@@QAE@PBD@Z 10048070     format.obj
 0001:00047094       __unwindtable$??0_Locinfo@std@@QAE@PBD@Z 10048094     format.obj
 0001:000470cc       __ehfuncinfo$??1PluginDialogBuilder@@QAE@XZ 100480cc     Pcfg.obj
 0001:000470cc       __ehfuncinfo$??1PluginSettings@@QAE@XZ 100480cc     Pcfg.obj
 0001:000470cc       __ehfuncinfo$??1?$unique_ptr@UIWbemClassObject@@Ucom_closer@@@std@@QAE@XZ 100480cc     WMI.obj
 0001:000470cc       __ehfuncinfo$??1?$unique_ptr@UIWbemLocator@@Ucom_closer@@@std@@QAE@XZ 100480cc     WMI.obj
 0001:000470cc       __ehfuncinfo$??1_Locinfo@std@@QAE@XZ 100480cc     format.obj
 0001:000470cc       __ehfuncinfo$??1?$scoped_lock@VPerfThread@@@std@@QAE@XZ 100480cc     handles.obj
 0001:000470cc       __ehfuncinfo$??1DebugToken@@QAE@XZ 100480cc     handles.obj
 0001:000470cc       __ehfuncinfo$??1_Init_atexit@@QAE@XZ 100480cc     libcpmt:iosptrs.obj
 0001:000470f0       __unwindtable$?on_error@error_handler@detail@v6@fmt@@QAEXPBD@Z 100480f0     format.obj
 0001:000470f0       __unwindtable$??$handle_int_type_spec@AAU?$int_writer@V?$back_insert_iterator@V?$buffer@_W@detail@v6@fmt@@@std@@_WI@detail@v6@fmt@@@detail@v6@fmt@@YAXDAAU?$int_writer@V?$back_insert_iterator@V?$buffer@_W@detail@v6@fmt@@@std@@_WI@012@@Z 100480f0     handles.obj
 0001:000470f0       __unwindtable$??$handle_int_type_spec@AAU?$int_writer@V?$back_insert_iterator@V?$buffer@_W@detail@v6@fmt@@@std@@_W_K@detail@v6@fmt@@@detail@v6@fmt@@YAXDAAU?$int_writer@V?$back_insert_iterator@V?$buffer@_W@detail@v6@fmt@@@std@@_W_K@012@@Z 100480f0     handles.obj
 0001:000470f0       __unwindtable$??$visit_format_arg@U?$default_arg_formatter@V?$back_insert_iterator@V?$buffer@_W@detail@v6@fmt@@@std@@_W@detail@v6@fmt@@V?$basic_format_context@V?$back_insert_iterator@V?$buffer@_W@detail@v6@fmt@@@std@@_W@34@@v6@fmt@@YA?AV?$back_insert_iterator@V?$buffer@_W@detail@v6@fmt@@@std@@$$QAU?$default_arg_formatter@V?$back_insert_iterator@V?$buffer@_W@detail@v6@fmt@@@std@@_W@detail@01@ABV?$basic_format_arg@V?$basic_format_context@V?$back_insert_iterator@V?$buffer@_W@detail@v6@fmt@@@std@@_W@v6@fmt@@@01@@Z 100480f0     handles.obj
 0001:000470f0       __unwindtable$?write@?$arg_formatter_base@V?$back_insert_iterator@V?$buffer@_W@detail@v6@fmt@@@std@@_WUerror_handler@detail@v6@fmt@@@detail@v6@fmt@@IAEXPB_W@Z 100480f0     handles.obj
 0001:000470f8       __ehfuncinfo$?on_error@error_handler@detail@v6@fmt@@QAEXPBD@Z 100480f8     format.obj
 0001:000470f8       __ehfuncinfo$??$handle_int_type_spec@AAU?$int_writer@V?$back_insert_iterator@V?$buffer@_W@detail@v6@fmt@@@std@@_WI@detail@v6@fmt@@@detail@v6@fmt@@YAXDAAU?$int_writer@V?$back_insert_iterator@V?$buffer@_W@detail@v6@fmt@@@std@@_WI@012@@Z 100480f8     handles.obj
 0001:000470f8       __ehfuncinfo$??$handle_int_type_spec@AAU?$int_writer@V?$back_insert_iterator@V?$buffer@_W@detail@v6@fmt@@@std@@_W_K@detail@v6@fmt@@@detail@v6@fmt@@YAXDAAU?$int_writer@V?$back_insert_iterator@V?$buffer@_W@detail@v6@fmt@@@std@@_W_K@012@@Z 100480f8     handles.obj
 0001:000470f8       __ehfuncinfo$??$visit_format_arg@U?$default_arg_formatter@V?$back_insert_iterator@V?$buffer@_W@detail@v6@fmt@@@std@@_W@detail@v6@fmt@@V?$basic_format_context@V?$back_insert_iterator@V?$buffer@_W@detail@v6@fmt@@@std@@_W@34@@v6@fmt@@YA?AV?$back_insert_iterator@V?$buffer@_W@detail@v6@fmt@@@std@@$$QAU?$default_arg_formatter@V?$back_insert_iterator@V?$buffer@_W@detail@v6@fmt@@@std@@_W@detail@01@ABV?$basic_format_arg@V?$basic_format_context@V?$back_insert_iterator@V?$buffer@_W@detail@v6@fmt@@@std@@_W@v6@fmt@@@01@@Z 100480f8     handles.obj
 0001:000470f8       __ehfuncinfo$?write@?$arg_formatter_base@V?$back_insert_iterator@V?$buffer@_W@detail@v6@fmt@@@std@@_WUerror_handler@detail@v6@fmt@@@detail@v6@fmt@@IAEXPB_W@Z 100480f8     handles.obj
 0001:0004711c       __unwindtable$??$decimal_point_impl@_W@detail@v6@fmt@@YA_WVlocale_ref@012@@Z 1004811c     format.obj
 0001:0004711c       __unwindtable$??$grouping_impl@_W@detail@v6@fmt@@YA?AV?$basic_string@DU?$char_traits@D@std@@V?$allocator@D@2@@std@@Vlocale_ref@012@@Z 1004811c     format.obj
 0001:0004711c       __unwindtable$??$thousands_sep_impl@_W@detail@v6@fmt@@YA_WVlocale_ref@012@@Z 1004811c     format.obj
 0001:00047124       __ehfuncinfo$??$decimal_point_impl@_W@detail@v6@fmt@@YA_WVlocale_ref@012@@Z 10048124     format.obj
 0001:00047124       __ehfuncinfo$??$grouping_impl@_W@detail@v6@fmt@@YA?AV?$basic_string@DU?$char_traits@D@std@@V?$allocator@D@2@@std@@Vlocale_ref@012@@Z 10048124     format.obj
 0001:00047124       __ehfuncinfo$??$thousands_sep_impl@_W@detail@v6@fmt@@YA_WVlocale_ref@012@@Z 10048124     format.obj
 0001:00047148       __unwindtable$?square@bigint@detail@v6@fmt@@QAEXXZ 10048148     format.obj
 0001:00047158       __ehfuncinfo$?square@bigint@detail@v6@fmt@@QAEXXZ 10048158     format.obj
 0001:0004717c       __unwindtable$??$get@Vlocale@std@@@locale_ref@detail@v6@fmt@@QBE?AVlocale@std@@XZ 1004817c     format.obj
 0001:00047184       __ehfuncinfo$??$get@Vlocale@std@@@locale_ref@detail@v6@fmt@@QBE?AVlocale@std@@XZ 10048184     format.obj
 0001:000471a8       __ehfuncinfo$??$use_facet@V?$numpunct@_W@std@@@std@@YAABV?$numpunct@_W@0@ABVlocale@0@@Z 100481a8     format.obj
 0001:000471cc       __unwindtable$??$use_facet@V?$numpunct@_W@std@@@std@@YAABV?$numpunct@_W@0@ABVlocale@0@@Z 100481cc     format.obj
 0001:00047204       __unwindtable$??$fallback_format@N@detail@v6@fmt@@YAXNAAV?$buffer@D@012@AAH@Z 10048204     format.obj
 0001:00047204       __unwindtable$??$fallback_format@O@detail@v6@fmt@@YAXOAAV?$buffer@D@012@AAH@Z 10048204     format.obj
 0001:00047224       __ehfuncinfo$??$fallback_format@N@detail@v6@fmt@@YAXNAAV?$buffer@D@012@AAH@Z 10048224     format.obj
 0001:00047224       __ehfuncinfo$??$fallback_format@O@detail@v6@fmt@@YAXOAAV?$buffer@D@012@AAH@Z 10048224     format.obj
 0001:00047330       __ehfuncinfo$?PrintHandleInfo@@YA_NKPAX_NPAVPerfThread@@@Z 10048330     handles.obj
 0001:00047354       __unwindtable$?PrintHandleInfo@@YA_NKPAX_NPAVPerfThread@@@Z 10048354     handles.obj
 0001:0004738c       __unwindtable$?query_object@@YA?AV?$unique_ptr@$$BY0A@DU?$default_delete@$$BY0A@D@std@@@std@@PAXW4OBJECT_INFORMATION_CLASS@@@Z 1004838c     handles.obj
 0001:00047394       __ehfuncinfo$?query_object@@YA?AV?$unique_ptr@$$BY0A@DU?$default_delete@$$BY0A@D@std@@@std@@PAXW4OBJECT_INFORMATION_CLASS@@@Z 10048394     handles.obj
 0001:000473b8       __unwindtable$??R<lambda_c3630acb37279cf92411e07a2b271fdf>@@QBE?AV?$basic_string@_WU?$char_traits@_W@std@@V?$allocator@_W@2@@std@@XZ 100483b8     handles.obj
 0001:000473d0       __ehfuncinfo$??R<lambda_c3630acb37279cf92411e07a2b271fdf>@@QBE?AV?$basic_string@_WU?$char_traits@_W@std@@V?$allocator@_W@2@@std@@XZ 100483d0     handles.obj
 0001:000473f4       __ehfuncinfo$?GetNameByType@@YA?AV?$basic_string@_WU?$char_traits@_W@std@@V?$allocator@_W@2@@std@@PAXGPAVPerfThread@@@Z 100483f4     handles.obj
 0001:00047418       __unwindtable$?GetNameByType@@YA?AV?$basic_string@_WU?$char_traits@_W@std@@V?$allocator@_W@2@@std@@PAXGPAVPerfThread@@@Z 10048418     handles.obj
 0001:00047450       __unwindtable$?duplicate_handle@@YA?AV?$unique_ptr@XUhandle_closer@@@std@@PAXK@Z 10048450     handles.obj
 0001:00047470       __ehfuncinfo$?duplicate_handle@@YA?AV?$unique_ptr@XUhandle_closer@@@std@@PAXK@Z 10048470     handles.obj
 0001:00047494       __unwindtable$??$vformat@_W$0A@@detail@v6@fmt@@YA?AV?$basic_string@_WU?$char_traits@_W@std@@V?$allocator@_W@2@@std@@V?$basic_string_view@_W@12@V?$basic_format_args@V?$basic_format_context@V?$back_insert_iterator@V?$buffer@_W@detail@v6@fmt@@@std@@_W@v6@fmt@@@12@@Z 10048494     handles.obj
 0001:0004749c       __ehfuncinfo$??$vformat@_W$0A@@detail@v6@fmt@@YA?AV?$basic_string@_WU?$char_traits@_W@std@@V?$allocator@_W@2@@std@@V?$basic_string_view@_W@12@V?$basic_format_args@V?$basic_format_context@V?$back_insert_iterator@V?$buffer@_W@detail@v6@fmt@@@std@@_W@v6@fmt@@@12@@Z 1004849c     handles.obj
 0001:000474c0       __unwindtable$?on_fill@?$specs_setter@_W@detail@v6@fmt@@QAEXV?$basic_string_view@_W@34@@Z 100484c0     handles.obj
 0001:000474c8       __ehfuncinfo$?on_fill@?$specs_setter@_W@detail@v6@fmt@@QAEXV?$basic_string_view@_W@34@@Z 100484c8     handles.obj
 0001:000474ec       __unwindtable$??$write@_WV?$back_insert_iterator@V?$buffer@_W@detail@v6@fmt@@@std@@M$0A@@detail@v6@fmt@@YA?AV?$back_insert_iterator@V?$buffer@_W@detail@v6@fmt@@@std@@V34@M@Z 100484ec     handles.obj
 0001:000474f4       __ehfuncinfo$??$write@_WV?$back_insert_iterator@V?$buffer@_W@detail@v6@fmt@@@std@@M$0A@@detail@v6@fmt@@YA?AV?$back_insert_iterator@V?$buffer@_W@detail@v6@fmt@@@std@@V34@M@Z 100484f4     handles.obj
 0001:00047518       __unwindtable$??$write@_WV?$back_insert_iterator@V?$buffer@_W@detail@v6@fmt@@@std@@N$0A@@detail@v6@fmt@@YA?AV?$back_insert_iterator@V?$buffer@_W@detail@v6@fmt@@@std@@V34@N@Z 10048518     handles.obj
 0001:00047518       __unwindtable$??$write@_WV?$back_insert_iterator@V?$buffer@_W@detail@v6@fmt@@@std@@O$0A@@detail@v6@fmt@@YA?AV?$back_insert_iterator@V?$buffer@_W@detail@v6@fmt@@@std@@V34@O@Z 10048518     handles.obj
 0001:00047520       __ehfuncinfo$??$write@_WV?$back_insert_iterator@V?$buffer@_W@detail@v6@fmt@@@std@@N$0A@@detail@v6@fmt@@YA?AV?$back_insert_iterator@V?$buffer@_W@detail@v6@fmt@@@std@@V34@N@Z 10048520     handles.obj
 0001:00047520       __ehfuncinfo$??$write@_WV?$back_insert_iterator@V?$buffer@_W@detail@v6@fmt@@@std@@O$0A@@detail@v6@fmt@@YA?AV?$back_insert_iterator@V?$buffer@_W@detail@v6@fmt@@@std@@V34@O@Z 10048520     handles.obj
 0001:00047544       __unwindtable$??$write@_WV?$back_insert_iterator@V?$buffer@_W@detail@v6@fmt@@@std@@M$0A@@detail@v6@fmt@@YA?AV?$back_insert_iterator@V?$buffer@_W@detail@v6@fmt@@@std@@V34@MU?$basic_format_specs@_W@12@Vlocale_ref@012@@Z 10048544     handles.obj
 0001:00047554       __ehfuncinfo$??$write@_WV?$back_insert_iterator@V?$buffer@_W@detail@v6@fmt@@@std@@M$0A@@detail@v6@fmt@@YA?AV?$back_insert_iterator@V?$buffer@_W@detail@v6@fmt@@@std@@V34@MU?$basic_format_specs@_W@12@Vlocale_ref@012@@Z 10048554     handles.obj
 0001:00047578       __unwindtable$??$write@_WV?$back_insert_iterator@V?$buffer@_W@detail@v6@fmt@@@std@@N$0A@@detail@v6@fmt@@YA?AV?$back_insert_iterator@V?$buffer@_W@detail@v6@fmt@@@std@@V34@NU?$basic_format_specs@_W@12@Vlocale_ref@012@@Z 10048578     handles.obj
 0001:00047578       __unwindtable$??$write@_WV?$back_insert_iterator@V?$buffer@_W@detail@v6@fmt@@@std@@O$0A@@detail@v6@fmt@@YA?AV?$back_insert_iterator@V?$buffer@_W@detail@v6@fmt@@@std@@V34@OU?$basic_format_specs@_W@12@Vlocale_ref@012@@Z 10048578     handles.obj
 0001:00047588       __ehfuncinfo$??$write@_WV?$back_insert_iterator@V?$buffer@_W@detail@v6@fmt@@@std@@N$0A@@detail@v6@fmt@@YA?AV?$back_insert_iterator@V?$buffer@_W@detail@v6@fmt@@@std@@V34@NU?$basic_format_specs@_W@12@Vlocale_ref@012@@Z 10048588     handles.obj
 0001:00047588       __ehfuncinfo$??$write@_WV?$back_insert_iterator@V?$buffer@_W@detail@v6@fmt@@@std@@O$0A@@detail@v6@fmt@@YA?AV?$back_insert_iterator@V?$buffer@_W@detail@v6@fmt@@@std@@V34@OU?$basic_format_specs@_W@12@Vlocale_ref@012@@Z 10048588     handles.obj
 0001:000475ac       __unwindtable$?on_num@?$int_writer@V?$back_insert_iterator@V?$buffer@_W@detail@v6@fmt@@@std@@_WI@detail@v6@fmt@@QAEXXZ 100485ac     handles.obj
 0001:000475bc       __ehfuncinfo$?on_num@?$int_writer@V?$back_insert_iterator@V?$buffer@_W@detail@v6@fmt@@@std@@_WI@detail@v6@fmt@@QAEXXZ 100485bc     handles.obj
 0001:000475e0       __unwindtable$?on_num@?$int_writer@V?$back_insert_iterator@V?$buffer@_W@detail@v6@fmt@@@std@@_W_K@detail@v6@fmt@@QAEXXZ 100485e0     handles.obj
 0001:000475f0       __ehfuncinfo$?on_num@?$int_writer@V?$back_insert_iterator@V?$buffer@_W@detail@v6@fmt@@@std@@_W_K@detail@v6@fmt@@QAEXXZ 100485f0     handles.obj
 0001:00047614       __unwindtable$?Read@options@@QAEXXZ 10048614     Pcfg.obj
 0001:00047614       __unwindtable$?Write@options@@QBEXXZ 10048614     Pcfg.obj
 0001:00047624       __ehfuncinfo$?Read@options@@QAEXXZ 10048624     Pcfg.obj
 0001:00047624       __ehfuncinfo$?Write@options@@QBEXXZ 10048624     Pcfg.obj
 0001:00047648       __unwindtable$?Config@@YAHXZ 10048648     Pcfg.obj
 0001:00047658       __ehfuncinfo$?Config@@YAHXZ 10048658     Pcfg.obj
 0001:0004767c       __ehfuncinfo$??0Plist@@QAE@XZ 1004867c     Pclass.obj
 0001:000476a0       __unwindtable$??0Plist@@QAE@XZ 100486a0     Pclass.obj
 0001:000476d0       __unwindtable$?Connect@Plist@@QAE_NPB_W00@Z 100486d0     Pclass.obj
 0001:000476e8       __ehfuncinfo$?Connect@Plist@@QAE_NPB_W00@Z 100486e8     Pclass.obj
 0001:0004770c       __ehfuncinfo$?GetFindData@Plist@@QAEHAAPAUPluginPanelItem@@AAI_K@Z 1004870c     Pclass.obj
 0001:00047730       __unwindtable$?GetFindData@Plist@@QAEHAAPAUPluginPanelItem@@AAI_K@Z 10048730     Pclass.obj
 0001:00047790       __ehfuncinfo$?GetFiles@Plist@@QAEHPAUPluginPanelItem@@IHPAPB_W_KAAUoptions@@@Z 10048790     Pclass.obj
 0001:000477b4       __unwindtable$?GetFiles@Plist@@QAEHPAUPluginPanelItem@@IHPAPB_W_KAAUoptions@@@Z 100487b4     Pclass.obj
 0001:00047924       __unwindtable$?DeleteFiles@Plist@@QAEHPAUPluginPanelItem@@I_K@Z 10048924     Pclass.obj
 0001:00047934       __ehfuncinfo$?DeleteFiles@Plist@@QAEHPAUPluginPanelItem@@I_K@Z 10048934     Pclass.obj
 0001:00047958       __unwindtable$?ProcessEvent@Plist@@QAEHHPAX@Z 10048958     Pclass.obj
 0001:00047968       __ehfuncinfo$?ProcessEvent@Plist@@QAEHHPAX@Z 10048968     Pclass.obj
 0001:0004798c       __unwindtable$?Compare@Plist@@QBEHPBUPluginPanelItem@@0I@Z 1004898c     Pclass.obj
 0001:000479ac       __ehfuncinfo$?Compare@Plist@@QBEHPBUPluginPanelItem@@0I@Z 100489ac     Pclass.obj
 0001:000479d0       __ehfuncinfo$?ProcessKey@Plist@@QAEHPBU_INPUT_RECORD@@@Z 100489d0     Pclass.obj
 0001:000479f4       __unwindtable$?ProcessKey@Plist@@QAEHPBU_INPUT_RECORD@@@Z 100489f4     Pclass.obj
 0001:00047a64       __unwindtable$?GetVersionInfo@Plist@@SA_NPB_WAAV?$unique_ptr@$$BY0A@DU?$default_delete@$$BY0A@D@std@@@std@@AAPB_W2@Z 10048a64     Pclass.obj
 0001:00047a7c       __ehfuncinfo$?GetVersionInfo@Plist@@SA_NPB_WAAV?$unique_ptr@$$BY0A@DU?$default_delete@$$BY0A@D@std@@@std@@AAPB_W2@Z 10048a7c     Pclass.obj
 0001:00047aa0       __unwindtable$?SavePanelModes@Plist@@SAXXZ 10048aa0     Pclass.obj
 0001:00047ab8       __ehfuncinfo$?SavePanelModes@Plist@@SAXXZ 10048ab8     Pclass.obj
 0001:00047adc       __ehfuncinfo$?InitializePanelModes@Plist@@SAXXZ 10048adc     Pclass.obj
 0001:00047b00       __unwindtable$?InitializePanelModes@Plist@@SAXXZ 10048b00     Pclass.obj
 0001:00047c58       __ehfuncinfo$?PrintVersionInfo@Plist@@CAXPAXPB_W@Z 10048c58     Pclass.obj
 0001:00047c7c       __unwindtable$?PrintVersionInfo@Plist@@CAXPAXPB_W@Z 10048c7c     Pclass.obj
 0001:00047ca4       __ehfuncinfo$?PrintOwnerInfo@Plist@@AAEXPAXK@Z 10048ca4     Pclass.obj
 0001:00047cc8       __unwindtable$?PrintOwnerInfo@Plist@@AAEXPAXK@Z 10048cc8     Pclass.obj
 0001:00047d08       __unwindtable$?ConnectWMI@Plist@@AAE_NXZ 10048d08     Pclass.obj
 0001:00047d10       __ehfuncinfo$?ConnectWMI@Plist@@AAE_NXZ 10048d10     Pclass.obj
 0001:00047d34       __unwindtable$?ui64toa_width@@YA?AV?$basic_string@_WU?$char_traits@_W@std@@V?$allocator@_W@2@@std@@_KI_N@Z 10048d34     Pclass.obj
 0001:00047d34       __unwindtable$?read_string@?$ipc_functions@$00@@SA?AV?$basic_string@_WU?$char_traits@_W@std@@V?$allocator@_W@2@@std@@PAXABUUNICODE_STRING_64@detail@@@Z 10048d34     Plist.obj
 0001:00047d3c       __ehfuncinfo$?ui64toa_width@@YA?AV?$basic_string@_WU?$char_traits@_W@std@@V?$allocator@_W@2@@std@@_KI_N@Z 10048d3c     Pclass.obj
 0001:00047d3c       __ehfuncinfo$?read_string@?$ipc_functions@$00@@SA?AV?$basic_string@_WU?$char_traits@_W@std@@V?$allocator@_W@2@@std@@PAXABUUNICODE_STRING_64@detail@@@Z 10048d3c     Plist.obj
 0001:00047d60       __unwindtable$??$make_unique@VPerfThread@@$$V$0A@@std@@YA?AV?$unique_ptr@VPerfThread@@U?$default_delete@VPerfThread@@@std@@@0@XZ 10048d60     Pclass.obj
 0001:00047d68       __ehfuncinfo$??$make_unique@VPerfThread@@$$V$0A@@std@@YA?AV?$unique_ptr@VPerfThread@@U?$default_delete@VPerfThread@@@std@@@0@XZ 10048d68     Pclass.obj
 0001:00047d8c       __unwindtable$?TranslateMode@@YA_NABV?$basic_string@_WU?$char_traits@_W@std@@V?$allocator@_W@2@@std@@AAV12@@Z 10048d8c     Pclass.obj
 0001:00047d94       __ehfuncinfo$?TranslateMode@@YA_NABV?$basic_string@_WU?$char_traits@_W@std@@V?$allocator@_W@2@@std@@AAV12@@Z 10048d94     Pclass.obj
 0001:00047db8       __unwindtable$?generate_titles@@YAXABV?$basic_string@_WU?$char_traits@_W@std@@V?$allocator@_W@2@@std@@AAUPanelMode@@@Z 10048db8     Pclass.obj
 0001:00047dc0       __ehfuncinfo$?generate_titles@@YAXABV?$basic_string@_WU?$char_traits@_W@std@@V?$allocator@_W@2@@std@@AAUPanelMode@@@Z 10048dc0     Pclass.obj
 0001:00047de4       __unwindtable$?window_ex_style@@YA@PAUHWND__@@@Z 10048de4     Pclass.obj
 0001:00047de4       __unwindtable$?window_style@@YA@PAUHWND__@@@Z 10048de4     Pclass.obj
 0001:00047dec       __ehfuncinfo$?window_ex_style@@YA@PAUHWND__@@@Z 10048dec     Pclass.obj
 0001:00047dec       __ehfuncinfo$?window_style@@YA@PAUHWND__@@@Z 10048dec     Pclass.obj
 0001:00047e10       __ehfuncinfo$?DumpNTCounters@@YAXPAXAAVPerfThread@@KK@Z 10048e10     Pclass.obj
 0001:00047e34       __unwindtable$?DumpNTCounters@@YAXPAXAAVPerfThread@@KK@Z 10048e34     Pclass.obj
 0001:00047e84       __unwindtable$??$_Try_emplace@ABK$$V@?$_Hash@V?$_Umap_traits@KPAUHWND__@@V?$_Uhash_compare@KU?$hash@K@std@@U?$equal_to@K@2@@std@@V?$allocator@U?$pair@$$CBKPAUHWND__@@@std@@@3@$0A@@std@@@std@@IAE?AU?$pair@PAU?$_List_node@U?$pair@$$CBKPAUHWND__@@@std@@PAX@std@@_N@1@ABK@Z 10048e84     Pclass.obj
 0001:00047e94       __ehfuncinfo$??$_Try_emplace@ABK$$V@?$_Hash@V?$_Umap_traits@KPAUHWND__@@V?$_Uhash_compare@KU?$hash@K@std@@U?$equal_to@K@2@@std@@V?$allocator@U?$pair@$$CBKPAUHWND__@@@std@@@3@$0A@@std@@@std@@IAE?AU?$pair@PAU?$_List_node@U?$pair@$$CBKPAUHWND__@@@std@@PAX@std@@_N@1@ABK@Z 10048e94     Pclass.obj
 0001:00047eb8       __ehfuncinfo$??$_Assign_range@PBUmode@@@?$vector@Umode@@V?$allocator@Umode@@@std@@@std@@AAEXPBUmode@@0Uforward_iterator_tag@1@@Z 10048eb8     Pclass.obj
 0001:00047edc       __unwindtable$??$_Assign_range@PBUmode@@@?$vector@Umode@@V?$allocator@Umode@@@std@@@std@@AAEXPBUmode@@0Uforward_iterator_tag@1@@Z 10048edc     Pclass.obj
 0001:00047f0c       __ehfuncinfo$??0PerfThread@@QAE@PB_W00@Z 10048f0c     perfthread.obj
 0001:00047f30       __unwindtable$??0PerfThread@@QAE@PB_W00@Z 10048f30     perfthread.obj
 0001:00047fa8       __ehfuncinfo$?Refresh@PerfThread@@AAEXXZ 10048fa8     perfthread.obj
 0001:00047fcc       __unwindtable$?Refresh@PerfThread@@AAEXXZ 10048fcc     perfthread.obj
 0001:00047ffc       __unwindtable$?RefreshWMIData@PerfThread@@AAEXXZ 10048ffc     perfthread.obj
 0001:00048004       __ehfuncinfo$?RefreshWMIData@PerfThread@@AAEXXZ 10049004     perfthread.obj
 0001:00048028       __unwindtable$?GetList@@YA_NAAPAUPluginPanelItem@@AAIAAVPerfThread@@@Z 10049028     Plist.obj
 0001:00048030       __ehfuncinfo$?GetList@@YA_NAAPAUPluginPanelItem@@AAIAAVPerfThread@@@Z 10049030     Plist.obj
 0001:00048054       __unwindtable$?KillProcess@@YA_NKPAUHWND__@@@Z 10049054     Plist.obj
 0001:00048064       __ehfuncinfo$?KillProcess@@YA_NKPAUHWND__@@@Z 10049064     Plist.obj
 0001:00048088       __unwindtable$?GetOpenProcessData@@YAXPAXPAV?$basic_string@_WU?$char_traits@_W@std@@V?$allocator@_W@2@@std@@1111@Z 10049088     Plist.obj
 0001:00048088       __unwindtable$?is_wow64_itself@@YA_NXZ 10049088     Plist.obj
 0001:00048090       __ehfuncinfo$?GetOpenProcessData@@YAXPAXPAV?$basic_string@_WU?$char_traits@_W@std@@V?$allocator@_W@2@@std@@1111@Z 10049090     Plist.obj
 0001:00048090       __ehfuncinfo$?is_wow64_itself@@YA_NXZ 10049090     Plist.obj
 0001:000480b4       __ehfuncinfo$?PrintNTCurDirAndEnv@@YAXPAX0H@Z 100490b4     Plist.obj
 0001:000480d8       __unwindtable$?PrintNTCurDirAndEnv@@YAXPAX0H@Z 100490d8     Plist.obj
 0001:00048108       __unwindtable$?PrintModules@@YAXPAXKAAUoptions@@@Z 10049108     Plist.obj
 0001:00048128       __ehfuncinfo$?PrintModules@@YAXPAXKAAUoptions@@@Z 10049128     Plist.obj
 0001:0004814c       __ehfuncinfo$??0?$vector@UProcessPerfData@@V?$allocator@UProcessPerfData@@@std@@@std@@QAE@ABV01@@Z 1004914c     Plist.obj
 0001:00048170       __unwindtable$??0?$vector@UProcessPerfData@@V?$allocator@UProcessPerfData@@@std@@@std@@QAE@ABV01@@Z 10049170     Plist.obj
 0001:00048198       __unwindtable$?PrintModules@?$ipc_functions@$00@@SAXPAX0AAUoptions@@@Z 10049198     Plist.obj
 0001:000481a8       __ehfuncinfo$?PrintModules@?$ipc_functions@$00@@SAXPAX0AAUoptions@@@Z 100491a8     Plist.obj
 0001:000481cc       __unwindtable$?PrintModules@?$ipc_functions@$0A@@@SAXPAX0AAUoptions@@@Z 100491cc     Plist.obj
 0001:000481d4       __ehfuncinfo$?PrintModules@?$ipc_functions@$0A@@@SAXPAX0AAUoptions@@@Z 100491d4     Plist.obj
 0001:000481f8       __unwindtable$?print_module_impl@@YAXQAXABV?$basic_string@_WU?$char_traits@_W@std@@V?$allocator@_W@2@@std@@KABUoptions@@ABV?$function@$$A6A_NPA_WI@Z@2@@Z 100491f8     Plist.obj
 0001:00048210       __ehfuncinfo$?print_module_impl@@YAXQAXABV?$basic_string@_WU?$char_traits@_W@std@@V?$allocator@_W@2@@std@@KABUoptions@@ABV?$function@$$A6A_NPA_WI@Z@2@@Z 10049210     Plist.obj
 0001:00048234       __unwindtable$??$print_module@PAX@@YAXQAXPAXKAAUoptions@@ABV?$function@$$A6A_NPA_WI@Z@std@@@Z 10049234     Plist.obj
 0001:0004823c       __ehfuncinfo$??$print_module@PAX@@YAXQAXPAXKAAUoptions@@ABV?$function@$$A6A_NPA_WI@Z@std@@@Z 1004923c     Plist.obj
 0001:00048260       __unwindtable$?WinError@@YAHPB_W@Z 10049260     Pmix.obj
 0001:00048270       __ehfuncinfo$?WinError@@YAHPB_W@Z 10049270     Pmix.obj
 0001:00048294       __unwindtable$??0WMIConnection@@QAE@XZ 10049294     WMI.obj
 0001:0004829c       __ehfuncinfo$??0WMIConnection@@QAE@XZ 1004929c     WMI.obj
 0001:000482c0       __unwindtable$??1?$ptr_setter@V?$unique_ptr@UIWbemClassObject@@Ucom_closer@@@std@@@@QAE@XZ 100492c0     WMI.obj
 0001:000482c0       __unwindtable$??1WMIConnection@@QAE@XZ 100492c0     WMI.obj
 0001:000482c8       __ehfuncinfo$??1?$ptr_setter@V?$unique_ptr@UIWbemClassObject@@Ucom_closer@@@std@@@@QAE@XZ 100492c8     WMI.obj
 0001:000482c8       __ehfuncinfo$??1WMIConnection@@QAE@XZ 100492c8     WMI.obj
 0001:000482ec       __ehfuncinfo$?Connect@WMIConnection@@QAE_NPB_W00@Z 100492ec     WMI.obj
 0001:00048310       __unwindtable$?Connect@WMIConnection@@QAE_NPB_W00@Z 10049310     WMI.obj
 0001:00048348       __unwindtable$?GetProcessPriority@WMIConnection@@QAEKK@Z 10049348     WMI.obj
 0001:00048348       __unwindtable$?GetProcessSessionId@WMIConnection@@QAEKK@Z 10049348     WMI.obj
 0001:00048350       __ehfuncinfo$?GetProcessPriority@WMIConnection@@QAEKK@Z 10049350     WMI.obj
 0001:00048350       __ehfuncinfo$?GetProcessSessionId@WMIConnection@@QAEKK@Z 10049350     WMI.obj
 0001:00048374       __ehfuncinfo$?GetProcessOwner@WMIConnection@@QAE?AV?$basic_string@_WU?$char_traits@_W@std@@V?$allocator@_W@2@@std@@KPAV23@@Z 10049374     WMI.obj
 0001:00048374       __ehfuncinfo$?GetProcessUserSid@WMIConnection@@QAE?AV?$basic_string@_WU?$char_traits@_W@std@@V?$allocator@_W@2@@std@@K@Z 10049374     WMI.obj
 0001:00048398       __unwindtable$?GetProcessOwner@WMIConnection@@QAE?AV?$basic_string@_WU?$char_traits@_W@std@@V?$allocator@_W@2@@std@@KPAV23@@Z 10049398     WMI.obj
 0001:00048398       __unwindtable$?GetProcessUserSid@WMIConnection@@QAE?AV?$basic_string@_WU?$char_traits@_W@std@@V?$allocator@_W@2@@std@@K@Z 10049398     WMI.obj
 0001:000483d8       __unwindtable$?GetProcessCommandLine@WMIConnection@@QAE?AV?$basic_string@_WU?$char_traits@_W@std@@V?$allocator@_W@2@@std@@K@Z 100493d8     WMI.obj
 0001:000483d8       __unwindtable$?GetProcessExecutablePath@WMIConnection@@QAE?AV?$basic_string@_WU?$char_traits@_W@std@@V?$allocator@_W@2@@std@@K@Z 100493d8     WMI.obj
 0001:000483e8       __ehfuncinfo$?GetProcessCommandLine@WMIConnection@@QAE?AV?$basic_string@_WU?$char_traits@_W@std@@V?$allocator@_W@2@@std@@K@Z 100493e8     WMI.obj
 0001:000483e8       __ehfuncinfo$?GetProcessExecutablePath@WMIConnection@@QAE?AV?$basic_string@_WU?$char_traits@_W@std@@V?$allocator@_W@2@@std@@K@Z 100493e8     WMI.obj
 0001:0004840c       __ehfuncinfo$?ExecMethod@WMIConnection@@AAEHKPB_W0K@Z 1004940c     WMI.obj
 0001:00048430       __unwindtable$?ExecMethod@WMIConnection@@AAEHKPB_W0K@Z 10049430     WMI.obj
 0001:000484d0       __ehfuncinfo$?GetProcessProperty@WMIConnection@@AAE_NKPB_WABV?$function@$$A6AXABUtagVARIANT@@@Z@std@@@Z 100494d0     WMI.obj
 0001:000484f4       __unwindtable$?GetProcessProperty@WMIConnection@@AAE_NKPB_WABV?$function@$$A6AXABUtagVARIANT@@@Z@std@@@Z 100494f4     WMI.obj
 0001:00048614       __unwindtable$?_Init@locale@std@@CAPAV_Locimp@12@_N@Z 10049614     libcpmt:locale0.obj
 0001:0004861c       __ehfuncinfo$?_Init@locale@std@@CAPAV_Locimp@12@_N@Z 1004961c     libcpmt:locale0.obj
 0001:00048640       __sehtable$___scrt_is_nonwritable_in_current_image 10049640     LIBCMT:utility.obj
 0001:00048660       __sehtable$??_M@YGXPAXIIP6EX0@Z@Z 10049660     LIBCMT:ehvecdtr.obj
 0001:00048680       __sehtable$?__ArrayUnwind@@YGXPAXIIP6EX0@Z@Z 10049680     LIBCMT:ehvecdtr.obj
 0001:000486a0       __sehtable$?dllmain_crt_process_attach@@YAHQAUHINSTANCE__@@QAX@Z 100496a0     LIBCMT:dll_dllmain.obj
 0001:000486c0       __sehtable$?dllmain_crt_process_detach@@YAH_N@Z 100496c0     LIBCMT:dll_dllmain.obj
 0001:000486e8       __sehtable$?dllmain_dispatch@@YAHQAUHINSTANCE__@@KQAX@Z 100496e8     LIBCMT:dll_dllmain.obj
 0001:00048708       __sehtable$___DestructExceptionObject 10049708     libvcruntime:ehhelpers.obj
 0001:00048728       __sehtable$?FrameUnwindToState@__FrameHandler3@@SAXPAUEHRegistrationNode@@PAXPBU_s_FuncInfo@@H@Z 10049728     libvcruntime:frame.obj
 0001:00048750       __sehtable$?CallCatchBlock@@YAPAXPAUEHExceptionRecord@@PAUEHRegistrationNode@@PAU_CONTEXT@@PBU_s_FuncInfo@@PAXHK@Z 10049750     libvcruntime:frame.obj
 0001:00048778       __catchsym$?CallUnexpected@@YAXPBU_s_ESTypeList@@@Z$2 10049778     libvcruntime:frame.obj
 0001:00048788       __unwindtable$?CallUnexpected@@YAXPBU_s_ESTypeList@@@Z 10049788     libvcruntime:frame.obj
 0001:00048798       __tryblocktable$?CallUnexpected@@YAXPBU_s_ESTypeList@@@Z 10049798     libvcruntime:frame.obj
 0001:000487ac       __ehfuncinfo$?CallUnexpected@@YAXPBU_s_ESTypeList@@@Z 100497ac     libvcruntime:frame.obj
 0001:000487d0       __sehtable$??$BuildCatchObjectHelperInternal@V__FrameHandler3@@@@YAHPAUEHExceptionRecord@@PAXPBU_s_HandlerType@@PBU_s_CatchableType@@@Z 100497d0     libvcruntime:frame.obj
 0001:000487f0       __sehtable$??$BuildCatchObjectInternal@V__FrameHandler3@@@@YAXPAUEHExceptionRecord@@PAXPBU_s_HandlerType@@PBU_s_CatchableType@@@Z 100497f0     libvcruntime:frame.obj
 0001:00048848       __sehtable$_terminate      10049848     libucrt:terminate.obj
 0001:00048868       __sehtable$___acrt_lowio_ensure_fh_exists 10049868     libucrt:osfinfo.obj
 0001:00048888       __sehtable$??$?RV<lambda_646e26742ed01d5bc03234f44bb6d3d3>@@AAV<lambda_b37934c380d97b75fd242ea49540127a>@@V<lambda_bbd9d45274666fbb50f81a29ad795c13>@@@?$__crt_seh_guarded_call@PAD@@QAEPAD$$QAV<lambda_646e26742ed01d5bc03234f44bb6d3d3>@@AAV<lambda_b37934c380d97b75fd242ea49540127a>@@$$QAV<lambda_bbd9d45274666fbb50f81a29ad795c13>@@@Z 10049888     libucrt:setlocale.obj
 0001:000488a8       __sehtable$??R<lambda_6e4b09c48022b2350581041d5f6b0c4c>@@QBE@XZ 100498a8     libucrt:exit.obj
 0001:000488c8       __sehtable$??$?RV<lambda_03b1d95aef87969028cfba75ccab2455>@@AAV<lambda_6e4b09c48022b2350581041d5f6b0c4c>@@V<lambda_22bdf7517842c4b3e53723af5aa32b9e>@@@?$__crt_seh_guarded_call@X@@QAEX$$QAV<lambda_03b1d95aef87969028cfba75ccab2455>@@AAV<lambda_6e4b09c48022b2350581041d5f6b0c4c>@@$$QAV<lambda_22bdf7517842c4b3e53723af5aa32b9e>@@@Z 100498c8     libucrt:exit.obj
 0001:000488e8       __sehtable$??$?RV<lambda_8e746cf0007f6ed984d6f78af1fec997>@@AAV<lambda_22ebabd17bc4fa466a2aca6d8deb888d>@@V<lambda_18ed0c0b38a6dc0daf1e7ac6d6adf05e>@@@?$__crt_seh_guarded_call@H@@QAEH$$QAV<lambda_8e746cf0007f6ed984d6f78af1fec997>@@AAV<lambda_22ebabd17bc4fa466a2aca6d8deb888d>@@$$QAV<lambda_18ed0c0b38a6dc0daf1e7ac6d6adf05e>@@@Z 100498e8     libucrt:onexit.obj
 0001:00048908       __sehtable$??$?RV<lambda_69a2805e680e0e292e8ba93315fe43a8>@@AAV<lambda_f03950bc5685219e0bcd2087efbe011e>@@V<lambda_03fcd07e894ec930e3f35da366ca99d6>@@@?$__crt_seh_guarded_call@H@@QAEH$$QAV<lambda_69a2805e680e0e292e8ba93315fe43a8>@@AAV<lambda_f03950bc5685219e0bcd2087efbe011e>@@$$QAV<lambda_03fcd07e894ec930e3f35da366ca99d6>@@@Z 10049908     libucrt:onexit.obj
 0001:00048928       __sehtable$__query_new_handler 10049928     libucrt:new_handler.obj
 0001:00048948       __sehtable$??$?RV<lambda_15ade71b0218206bbe3333a0c9b79046>@@AAV<lambda_da44e0f8b0f19ba52fefafb335991732>@@V<lambda_207f2d024fc103971653565357d6cd41>@@@?$__crt_seh_guarded_call@X@@QAEX$$QAV<lambda_15ade71b0218206bbe3333a0c9b79046>@@AAV<lambda_da44e0f8b0f19ba52fefafb335991732>@@$$QAV<lambda_207f2d024fc103971653565357d6cd41>@@@Z 10049948     libucrt:per_thread_data.obj
 0001:00048968       __sehtable$??$?RV<lambda_a7e850c220f1c8d1e6efeecdedd162c6>@@AAV<lambda_46720907175c18b6c9d2717bc0d2d362>@@V<lambda_9048902d66e8d99359bc9897bbb930a8>@@@?$__crt_seh_guarded_call@X@@QAEX$$QAV<lambda_a7e850c220f1c8d1e6efeecdedd162c6>@@AAV<lambda_46720907175c18b6c9d2717bc0d2d362>@@$$QAV<lambda_9048902d66e8d99359bc9897bbb930a8>@@@Z 10049968     libucrt:per_thread_data.obj
 0001:00048988       __sehtable$??$?RV<lambda_38edbb1296d33220d7e4dd0ed76b244a>@@AAV<lambda_5ce1d447e08cb34b2473517608e21441>@@V<lambda_fb385d3da700c9147fc39e65dd577a8c>@@@?$__crt_seh_guarded_call@X@@QAEX$$QAV<lambda_38edbb1296d33220d7e4dd0ed76b244a>@@AAV<lambda_5ce1d447e08cb34b2473517608e21441>@@$$QAV<lambda_fb385d3da700c9147fc39e65dd577a8c>@@@Z 10049988     libucrt:per_thread_data.obj
 0001:000489a8       __sehtable$??$?RV<lambda_6affb1475c98b40b75cdec977db92e3c>@@AAV<lambda_b8d4b9c228a6ecc3f80208dbb4b4a104>@@V<lambda_608742c3c92a14382c1684fc64f96c88>@@@?$__crt_seh_guarded_call@X@@QAEX$$QAV<lambda_6affb1475c98b40b75cdec977db92e3c>@@AAV<lambda_b8d4b9c228a6ecc3f80208dbb4b4a104>@@$$QAV<lambda_608742c3c92a14382c1684fc64f96c88>@@@Z 100499a8     libucrt:per_thread_data.obj
 0001:000489c8       __sehtable$??$?RV<lambda_6b4b7855443974f2b4b77000ea21c99c>@@AAV<lambda_8f7d3b162ab39427f4fa9995c67a7986>@@V<lambda_cc9a5ba8a5d8428b9634eab82665e5dc>@@@?$__crt_seh_guarded_call@H@@QAEH$$QAV<lambda_6b4b7855443974f2b4b77000ea21c99c>@@AAV<lambda_8f7d3b162ab39427f4fa9995c67a7986>@@$$QAV<lambda_cc9a5ba8a5d8428b9634eab82665e5dc>@@@Z 100499c8     libucrt:winapi_thunks.obj
 0001:000489e8       __sehtable$__fcloseall     100499e8     libucrt:closeall.obj
 0001:00048a08       __sehtable$??$?RV<lambda_2866be3712abc81a800a822484c830d8>@@AAV<lambda_39ca0ed439415581b5b15c265174cece>@@V<lambda_2b24c74d71094a6cd0cb82e44167d71b>@@@?$__crt_seh_guarded_call@X@@QAEX$$QAV<lambda_2866be3712abc81a800a822484c830d8>@@AAV<lambda_39ca0ed439415581b5b15c265174cece>@@$$QAV<lambda_2b24c74d71094a6cd0cb82e44167d71b>@@@Z 10049a08     libucrt:fflush.obj
 0001:00048a28       __sehtable$??$?RV<lambda_2cc53f568c5a2bb6f192f930a45d44ea>@@AAV<lambda_ab61a845afdef5b7c387490eaf3616ee>@@V<lambda_c2ffc0b7726aa6be21d5f0026187e748>@@@?$__crt_seh_guarded_call@X@@QAEX$$QAV<lambda_2cc53f568c5a2bb6f192f930a45d44ea>@@AAV<lambda_ab61a845afdef5b7c387490eaf3616ee>@@$$QAV<lambda_c2ffc0b7726aa6be21d5f0026187e748>@@@Z 10049a28     libucrt:fflush.obj
 0001:00048a48       __sehtable$___acrt_initialize_lowio 10049a48     libucrt:ioinit.obj
 0001:00048a68       __sehtable$__write         10049a68     libucrt:write.obj
 0001:00048a88       __sehtable$??$?RV<lambda_e5124f882df8998aaf41531e079ba474>@@AAV<lambda_3e16ef9562a7dcce91392c22ab16ea36>@@V<lambda_e25ca0880e6ef98be67edffd8c599615>@@@?$__crt_seh_guarded_call@X@@QAEX$$QAV<lambda_e5124f882df8998aaf41531e079ba474>@@AAV<lambda_3e16ef9562a7dcce91392c22ab16ea36>@@$$QAV<lambda_e25ca0880e6ef98be67edffd8c599615>@@@Z 10049a88     libucrt:wsetlocale.obj
 0001:00048aa8       __sehtable$??$?RV<lambda_4fdada1b837b2abbf20876fac97688ad>@@AAV<lambda_b57350f2640456a0859d250846f69caf>@@V<lambda_eed5e4f92b5b7d55fa22c48c484aaa54>@@@?$__crt_seh_guarded_call@X@@QAEX$$QAV<lambda_4fdada1b837b2abbf20876fac97688ad>@@AAV<lambda_b57350f2640456a0859d250846f69caf>@@$$QAV<lambda_eed5e4f92b5b7d55fa22c48c484aaa54>@@@Z 10049aa8     libucrt:wsetlocale.obj
 0001:00048ac8       __sehtable$??$?RV<lambda_135d2772fca65dc1248eeaa1b56e886a>@@AAV<lambda_2a444430fde8c29194d880d93eed5e8f>@@AAV<lambda_8dff2cf36a5417162780cd64fa2883ef>@@@?$__crt_seh_guarded_call@X@@QAEX$$QAV<lambda_135d2772fca65dc1248eeaa1b56e886a>@@AAV<lambda_2a444430fde8c29194d880d93eed5e8f>@@AAV<lambda_8dff2cf36a5417162780cd64fa2883ef>@@@Z 10049ac8     libucrt:wsetlocale.obj
 0001:00048ae4       __unwindtable$?_wcstombs_l_helper@@YAIPADPB_WIPAU__crt_locale_pointers@@@Z 10049ae4     libucrt:wcstombs.obj
 0001:00048aec       __ehfuncinfo$?_wcstombs_l_helper@@YAIPADPB_WIPAU__crt_locale_pointers@@@Z 10049aec     libucrt:wcstombs.obj
 0001:00048b10       __sehtable$_raise          10049b10     libucrt:signal.obj
 0001:00048b30       __sehtable$??$?RV<lambda_cbab9ec6f41b0180b23cc171c22676b0>@@AAV<lambda_44731a7d0e6d81c3e6aa82d741081786>@@V<lambda_4b292cb8dd18144e164572427af410ab>@@@?$__crt_seh_guarded_call@P6AXH@Z@@QAEP6AXH@Z$$QAV<lambda_cbab9ec6f41b0180b23cc171c22676b0>@@AAV<lambda_44731a7d0e6d81c3e6aa82d741081786>@@$$QAV<lambda_4b292cb8dd18144e164572427af410ab>@@@Z 10049b30     libucrt:signal.obj
 0001:00048b50       __sehtable$?update_thread_multibyte_data_internal@@YAPAU__crt_multibyte_data@@QAU__acrt_ptd@@QAPAU1@@Z 10049b50     libucrt:mbctype.obj
 0001:00048b70       __sehtable$??$?RV<lambda_ceb1ee4838e85a9d631eb091e2fbe199>@@AAV<lambda_ae742caa10f662c28703da3d2ea5e57e>@@V<lambda_cd08b5d6af4937fe54fc07d0c9bf6b37>@@@?$__crt_seh_guarded_call@X@@QAEX$$QAV<lambda_ceb1ee4838e85a9d631eb091e2fbe199>@@AAV<lambda_ae742caa10f662c28703da3d2ea5e57e>@@$$QAV<lambda_cd08b5d6af4937fe54fc07d0c9bf6b37>@@@Z 10049b70     libucrt:mbctype.obj
 0001:00048b90       __sehtable$___acrt_update_thread_locale_data 10049b90     libucrt:locale_refcounting.obj
 0001:00048bb0       __sehtable$_fclose         10049bb0     libucrt:fclose.obj
 0001:00048bd0       __sehtable$??$?RV<lambda_9e9de3de5fa147e2223d7db92bc10aa6>@@AAV<lambda_38ce7e780aa69e748d6df282ebc68efe>@@V<lambda_8ca6da459f0f6780f1cff60fdc3d00e5>@@@?$__crt_seh_guarded_call@H@@QAEH$$QAV<lambda_9e9de3de5fa147e2223d7db92bc10aa6>@@AAV<lambda_38ce7e780aa69e748d6df282ebc68efe>@@$$QAV<lambda_8ca6da459f0f6780f1cff60fdc3d00e5>@@@Z 10049bd0     libucrt:commit.obj
 0001:00048bf0       __sehtable$??$?RV<lambda_218ce3db14220d0be481dae8ef3383b6>@@AAV<lambda_628dfdc04ba53c8bfc02c9951375f3f5>@@V<lambda_57dc472bd5c9d5f3b2cbca59b8a843ae>@@@?$__crt_seh_guarded_call@H@@QAEH$$QAV<lambda_218ce3db14220d0be481dae8ef3383b6>@@AAV<lambda_628dfdc04ba53c8bfc02c9951375f3f5>@@$$QAV<lambda_57dc472bd5c9d5f3b2cbca59b8a843ae>@@@Z 10049bf0     libucrt:close.obj
 0001:00048c10       __sehtable$__IsNonwritableInCurrentImage 10049c10     LIBCMT:pesect.obj
 0001:00048c30       .edata                     10049c30     ProcList.exp
 0001:00048c58       rgpv                       10049c58     ProcList.exp
 0001:00048c94       rgszName                   10049c94     ProcList.exp
 0001:00048cd0       rgwOrd                     10049cd0     ProcList.exp
 0001:00048cee       szName                     10049cee     ProcList.exp
 0001:00048cfb       $N00001                    10049cfb     ProcList.exp
 0001:00048d07       $N00002                    10049d07     ProcList.exp
 0001:00048d10       $N00003                    10049d10     ProcList.exp
 0001:00048d1b       $N00004                    10049d1b     ProcList.exp
 0001:00048d28       $N00005                    10049d28     ProcList.exp
 0001:00048d31       $N00006                    10049d31     ProcList.exp
 0001:00048d3f       $N00007                    10049d3f     ProcList.exp
 0001:00048d49       $N00008                    10049d49     ProcList.exp
 0001:00048d56       $N00009                    10049d56     ProcList.exp
 0001:00048d65       $N00010                    10049d65     ProcList.exp
 0001:00048d77       $N00011                    10049d77     ProcList.exp
 0001:00048d86       $N00012                    10049d86     ProcList.exp
 0001:00048d8c       $N00013                    10049d8c     ProcList.exp
 0001:00048d9f       $N00014                    10049d9f     ProcList.exp
 0001:00048db2       $N00015                    10049db2     ProcList.exp
 0002:00000008       ?FKeys@?1??GetOpenPanelInfo@Plist@@QAEXPAUOpenPanelInfo@@@Z@4PAGA 1004a008     Pclass.obj
 0002:0000004c       ?nr@?7??Connect@Plist@@QAE_NPB_W00@Z@4U_NETRESOURCEW@@A 1004a04c     Pclass.obj
 0002:000000b0       ?init@std@@3JA             1004a0b0     libcpmt:xlock.obj
 0002:000000b4       ?atcount_cdecl@@3IA        1004a0b4     libcpmt:iosptrs.obj
 0002:000000f0       ?__vcrt_flsindex@@3KA      1004a0f0     libvcruntime:per_thread_data.obj
 0002:00000110       ?errno_no_memory@@3HA      1004a110     libucrt:errno.obj
 0002:00000114       ?doserrno_no_memory@@3KA   1004a114     libucrt:errno.obj
 0002:00000240       ?__acrt_flsindex@@3KA      1004a240     libucrt:per_thread_data.obj
 0002:00000244       __ctype_loc_style          1004a244     libucrt:wsetlocale.obj
 0002:00000310       _newcw                     1004a310     libucrt:modf.obj
 0002:00000328       ?tzstd_program@@3PADA      1004a328     libucrt:timeset.obj
 0002:00000368       ?tzdst_program@@3PADA      1004a368     libucrt:timeset.obj
 0002:000003a8       ?tzname_states@@3PAY01PADA 1004a3a8     libucrt:timeset.obj
 0002:000005d0       __mbctypes                 1004a5d0     libucrt:mbctype.obj
 0002:000006d8       __mbcasemaps               1004a6d8     libucrt:mbctype.obj
 0002:000007d8       ?__rgctypeflag@@3PADA      1004a7d8     libucrt:mbctype.obj
 0002:000007e0       ?__rgcode_page_info@@3PAUcode_page_info@@A 1004a7e0     libucrt:mbctype.obj
 0002:000009d0       ?__dcrt_lowio_console_output_handle@@3PAXA 1004a9d0     libucrt:initcon.obj
 0002:00000af4       ??_R0?AV<lambda_2188c710c02002b0eab1052a0acb7023>@@@8 1004aaf4     Plist.obj
 0002:00000b2c       ??_R0?AV<lambda_d3397212bd5e450c6dbd36f327bf5553>@@@8 1004ab2c     WMI.obj
 0002:00000b64       ??_R0?AV<lambda_8364a2c8b43a2a1256754ccc435293aa>@@@8 1004ab64     WMI.obj
 0002:00000d2c       ?UserAccountID@?1??GetUserAccountID@@YA@XZ@4V?$basic_string@_WU?$char_traits@_W@std@@V?$allocator@_W@2@@std@@B 1004ad2c     handles.obj
 0002:00000d44       ?$S1@?1??GetUserAccountID@@YA@XZ@4IA 1004ad44     handles.obj
 0002:00000d48       ?TitlesLocal@?1??PanelModes@Plist@@QAEPAUPanelMode@@AAI@Z@4V?$array@V?$array@PA_W$0BI@@std@@$09@std@@A 1004ad48     Pclass.obj
 0002:00001108       ?TitlesRemote@?1??PanelModes@Plist@@QAEPAUPanelMode@@AAI@Z@4V?$array@V?$array@PA_W$0BI@@std@@$09@std@@A 1004b108     Pclass.obj
 0002:000014c8       ?PanelModesLocal@?1??PanelModes@Plist@@QAEPAUPanelMode@@AAI@Z@4V?$array@UPanelMode@@$09@std@@A 1004b4c8     Pclass.obj
 0002:00001608       ?PanelModesRemote@?1??PanelModes@Plist@@QAEPAUPanelMode@@AAI@Z@4V?$array@UPanelMode@@$09@std@@A 1004b608     Pclass.obj
 0002:00001748       ?ArraysInited@?2??PanelModes@Plist@@QAEPAUPanelMode@@AAI@Z@4_NA 1004b748     Pclass.obj
 0002:0000174c       ?Title@?1??GetOpenPanelInfo@Plist@@QAEXPAUOpenPanelInfo@@@Z@4V?$basic_string@_WU?$char_traits@_W@std@@V?$allocator@_W@2@@std@@A 1004b74c     Pclass.obj
 0002:00001764       ?$S1@?1??GetOpenPanelInfo@Plist@@QAEXPAUOpenPanelInfo@@@Z@4IA 1004b764     Pclass.obj
 0002:00001768       ?kbl@?1??GetOpenPanelInfo@Plist@@QAEXPAUOpenPanelInfo@@@Z@4PAUKeyBarLabel@@A 1004b768     Pclass.obj
 0002:00001818       ?kbt@?1??GetOpenPanelInfo@Plist@@QAEXPAUOpenPanelInfo@@@Z@4UKeyBarTitles@@A 1004b818     Pclass.obj
 0002:00001820       ?$S2@?1??GetOpenPanelInfo@Plist@@QAEXPAUOpenPanelInfo@@@Z@4IA 1004b820     Pclass.obj
 0002:00001828       ?Styles@?1??window_style@@YA@PAUHWND__@@@Z@4QBU?$pair@HPB_W@std@@B 1004b828     Pclass.obj
 0002:000018a8       ?$S3@?1??window_style@@YA@PAUHWND__@@@Z@4IA 1004b8a8     Pclass.obj
 0002:000018b0       ?ExtStyles@?1??window_ex_style@@YA@PAUHWND__@@@Z@4QBU?$pair@HPB_W@std@@B 1004b8b0     Pclass.obj
 0002:00001950       ?$S5@?1??window_ex_style@@YA@PAUHWND__@@@Z@4IA 1004b950     Pclass.obj
 0002:00001954       ?IsWow64@?1??Is64BitWindows@@YA_NXZ@4_NB 1004b954     perfthread.obj
 0002:00001958       ?$S1@?1??Is64BitWindows@@YA_NXZ@4IA 1004b958     perfthread.obj
 0002:0000195c       ?IsWow64@?1??is_wow64_itself@@YA_NXZ@4_NB 1004b95c     Plist.obj
 0002:00001960       ?$S1@?1??is_wow64_itself@@YA_NXZ@4IA 1004b960     Plist.obj
 0002:00001964       ?hDebugToken@@3V?$unique_ptr@XUhandle_closer@@@std@@A 1004b964     Plist.obj
 0002:00001adc       ?Inited@?1??dynamic_bind@@YAXXZ@4_NA 1004badc     Proclist.obj
 0002:00001ae0       ?PluginMenuStrings@?4??GetPluginInfoW@@9@4@4PAPB_WA 1004bae0     Proclist.obj
 0002:00001ae4       ?DiskMenuStrings@?7??GetPluginInfoW@@9@4@4PAPB_WA 1004bae4     Proclist.obj
 0002:00001ae8       ?PluginCfgStrings@?1??GetPluginInfoW@@9@4@4PAPB_WA 1004bae8     Proclist.obj
 0002:00001af0       ?Cookie@?1??XorPointer@@YAPAXPAX@Z@4IB 1004baf0     vc_crt_fix_impl.obj
 0002:00001af4       ?$S1@?1??XorPointer@@YAPAXPAX@Z@4IA 1004baf4     vc_crt_fix_impl.obj
 0002:00001af8       ?Function@?1??EncodePointerWrapper@@9@4@4Q6GPAXPAX@ZA 1004baf8     vc_crt_fix_impl.obj
 0002:00001afc       ?$S2@?1??EncodePointerWrapper@@9@4@4IA 1004bafc     vc_crt_fix_impl.obj
 0002:00001b00       ?Function@?1??DecodePointerWrapper@@9@4@4Q6GPAXPAX@ZA 1004bb00     vc_crt_fix_impl.obj
 0002:00001b04       ?$S3@?1??DecodePointerWrapper@@9@4@4IA 1004bb04     vc_crt_fix_impl.obj
 0002:00001b08       ?Function@?1??GetModuleHandleExWWrapper@@9@12@4Q6GHKPB_WPAPAUHINSTANCE__@@@ZA 1004bb08     vc_crt_fix_impl.obj
 0002:00001b0c       ?$S4@?1??GetModuleHandleExWWrapper@@9@12@4IA 1004bb0c     vc_crt_fix_impl.obj
 0002:00001b10       ?Deleter@?1??InitializeSListHead@implementation@slist@@YGXPAT_SLIST_HEADER@@@Z@4Vservice_deleter@23@A 1004bb10     vc_crt_fix_impl.obj
 0002:00001b30       ?$S5@?1??InitializeSListHead@implementation@slist@@YGXPAT_SLIST_HEADER@@@Z@4IA 1004bb30     vc_crt_fix_impl.obj
 0002:00001b34       ?Function@?1??InitializeSListHeadWrapper@@9@4@4Q6GXPAT_SLIST_HEADER@@@ZA 1004bb34     vc_crt_fix_impl.obj
 0002:00001b38       ?$S6@?1??InitializeSListHeadWrapper@@9@4@4IA 1004bb38     vc_crt_fix_impl.obj
 0002:00001b3c       ?Function@?1??InterlockedFlushSListWrapper@@9@4@4Q6GPAU_SINGLE_LIST_ENTRY@@PAT_SLIST_HEADER@@@ZA 1004bb3c     vc_crt_fix_impl.obj
 0002:00001b40       ?$S7@?1??InterlockedFlushSListWrapper@@9@4@4IA 1004bb40     vc_crt_fix_impl.obj
 0002:00001b44       ?Function@?1??InterlockedPopEntrySListWrapper@@9@4@4Q6GPAU_SINGLE_LIST_ENTRY@@PAT_SLIST_HEADER@@@ZA 1004bb44     vc_crt_fix_impl.obj
 0002:00001b48       ?$S8@?1??InterlockedPopEntrySListWrapper@@9@4@4IA 1004bb48     vc_crt_fix_impl.obj
 0002:00001b4c       ?Function@?1??InterlockedPushEntrySListWrapper@@9@8@4Q6GPAU_SINGLE_LIST_ENTRY@@PAT_SLIST_HEADER@@PAU2@@ZA 1004bb4c     vc_crt_fix_impl.obj
 0002:00001b50       ?$S9@?1??InterlockedPushEntrySListWrapper@@9@8@4IA 1004bb50     vc_crt_fix_impl.obj
 0002:00001b54       ?Function@?1??InterlockedPushListSListExWrapper@@9@16@4Q6GPAU_SINGLE_LIST_ENTRY@@PAT_SLIST_HEADER@@PAU2@1K@ZA 1004bb54     vc_crt_fix_impl.obj
 0002:00001b58       ?$S10@?1??InterlockedPushListSListExWrapper@@9@16@4IA 1004bb58     vc_crt_fix_impl.obj
 0002:00001b5c       ?Function@?1??RtlFirstEntrySListWrapper@@9@4@4Q6GPAU_SINGLE_LIST_ENTRY@@PAT_SLIST_HEADER@@@ZA 1004bb5c     vc_crt_fix_impl.obj
 0002:00001b60       ?$S11@?1??RtlFirstEntrySListWrapper@@9@4@4IA 1004bb60     vc_crt_fix_impl.obj
 0002:00001b64       ?Function@?1??QueryDepthSListWrapper@@9@4@4Q6GGPAT_SLIST_HEADER@@@ZA 1004bb64     vc_crt_fix_impl.obj
 0002:00001b68       ?$S12@?1??QueryDepthSListWrapper@@9@4@4IA 1004bb68     vc_crt_fix_impl.obj
 0002:00001b6c       ?Function@?1??GetNumaHighestNodeNumberWrapper@@9@4@4Q6GHPAK@ZA 1004bb6c     vc_crt_fix_impl.obj
 0002:00001b70       ?$S13@?1??GetNumaHighestNodeNumberWrapper@@9@4@4IA 1004bb70     vc_crt_fix_impl.obj
 0002:00001b74       ?Function@?1??GetLogicalProcessorInformationWrapper@@9@8@4Q6GHPAU_SYSTEM_LOGICAL_PROCESSOR_INFORMATION@@PAK@ZA 1004bb74     vc_crt_fix_impl.obj
 0002:00001b78       ?$S14@?1??GetLogicalProcessorInformationWrapper@@9@8@4IA 1004bb78     vc_crt_fix_impl.obj
 0002:00001b7c       ?Function@?1??SetThreadStackGuaranteeWrapper@@9@4@4Q6GHPAK@ZA 1004bb7c     vc_crt_fix_impl.obj
 0002:00001b80       ?$S15@?1??SetThreadStackGuaranteeWrapper@@9@4@4IA 1004bb80     vc_crt_fix_impl.obj
 0002:00001b88       ?initlocks@std@@3V_Init_locks@1@A 1004bb88     libcpmt:xlock.obj
 0002:00001b90       ?mtx@std@@3PAU_RTL_CRITICAL_SECTION@@A 1004bb90     libcpmt:xlock.obj
 0002:00001c6c       ?classic_locale@std@@3Vlocale@1@A 1004bc6c     libcpmt:locale0.obj
 0002:00001c74       ?_Fac_tidy_reg@std@@3U_Fac_tidy_reg_t@1@B 1004bc74     libcpmt:locale0.obj
 0002:00001c78       ?_Fac_head@std@@3PAU_Fac_node@1@A 1004bc78     libcpmt:locale0.obj
 0002:00001c7c       _global_locale             1004bc7c     libcpmt:locale0.obj
 0002:00001c80       ?registered@?1??_Setgloballocale@locale@std@@CAXPAX@Z@4_NA 1004bc80     libcpmt:locale0.obj
 0002:00001cb0       ?initlocks@std@@3V_Init_locks@1@A 1004bcb0     libcpmt:iosptrs.obj
 0002:00001cb1       ?init_atexit@@3U_Init_atexit@@A 1004bcb1     libcpmt:iosptrs.obj
 0002:00001cb4       ?atfuns_cdecl@@3PAP6AXXZA  1004bcb4     libcpmt:iosptrs.obj
 0002:00001dfc       ?is_initialized_as_dll@@3_NA 1004bdfc     LIBCMT:utility.obj
 0002:00001dfd       ?module_local_atexit_table_initialized@@3_NA 1004bdfd     LIBCMT:utility.obj
 0002:00001e00       ?module_local_atexit_table@@3U_onexit_table_t@@A 1004be00     LIBCMT:utility.obj
 0002:00001e0c       ?module_local_at_quick_exit_table@@3U_onexit_table_t@@A 1004be0c     LIBCMT:utility.obj
 0002:00001e18       ?__proc_attached@@3HA      1004be18     LIBCMT:dll_dllmain.obj
 0002:00001e38       _GS_ExceptionRecord        1004be38     LIBCMT:gs_report.obj
 0002:00001e88       _GS_ContextRecord          1004be88     LIBCMT:gs_report.obj
 0002:0000215c       ?__vcrt_startup_thread_ptd@@3U__vcrt_ptd@@A 1004c15c     libvcruntime:per_thread_data.obj
 0002:00002184       ___vcrt_lock_table         1004c184     libvcruntime:locks.obj
 0002:0000219c       ___vcrt_locks_initialized  1004c19c     libvcruntime:locks.obj
 0002:000021c8       ?heap@@3V_HeapManager@@A   1004c1c8     libvcruntime:undname.obj
 0002:000021dc       ?module_handles@@3PAPAUHINSTANCE__@@A 1004c1dc     libvcruntime:winapi_downlevel.obj
 0002:000021e8       ?function_pointers@@3PAPAXA 1004c1e8     libvcruntime:winapi_downlevel.obj
 0002:000021fc       ?__acrt_invalid_parameter_handler@@3V?$dual_state_global@P6AXPB_W00II@Z@__crt_state_management@@A 1004c1fc     libucrt:invalid_parameter.obj
 0002:00002210       ?__acrt_lock_table@@3PAU_RTL_CRITICAL_SECTION@@A 1004c210     libucrt:locks.obj
 0002:00002360       ?__acrt_locks_initialized@@3IA 1004c360     libucrt:locks.obj
 0002:00002364       ?c_termination_complete@@3JA 1004c364     libucrt:exit.obj
 0002:00002368       ?thread_local_exit_callback_func@@3P6GXPAXK0@ZA 1004c368     libucrt:exit.obj
 0002:00002370       ?program_name@?1???$common_configure_argv@D@@YAHW4_crt_argv_mode@@@Z@4PADA 1004c370     libucrt:argv_parsing.obj
 0002:000024a0       ?__acrt_new_handler@@3V?$dual_state_global@P6AHI@Z@__crt_state_management@@A 1004c4a0     libucrt:new_handler.obj
 0002:000024a8       ?module_handles@@3PAPAUHINSTANCE__@@A 1004c4a8     libucrt:winapi_thunks.obj
 0002:000024f8       ?encoded_function_pointers@@3PAPAXA 1004c4f8     libucrt:winapi_thunks.obj
 0002:00002580       ?static_enum_proc@?1??enum_system_locales_ex_nolock@@YAHQ6GHPA_WKJ@Z@Z@4P6GH0KJ@ZA 1004c580     libucrt:winapi_thunks.obj
 0002:00002794       ?internal_state@?1??_mbtowc_l@@9@4U_Mbstatet@@A 1004c794     libucrt:mbtowc.obj
 0002:0000279c       ?enable_percent_n@@3IA     1004c79c     libucrt:printf_count_output.obj
 0002:000027a8       ?__acrt_app_type@@3W4_crt_app_type@@A 1004c7a8     libucrt:report_runtime_error.obj
 0002:000027ac       __pmatherr_set             1004c7ac     libucrt:libm_error.obj
 0002:000027b4       ?ctrlc_action@@3V?$dual_state_global@P6AXH@Z@__crt_state_management@@A 1004c7b4     libucrt:signal.obj
 0002:000027b8       ?ctrlbreak_action@@3V?$dual_state_global@P6AXH@Z@__crt_state_management@@A 1004c7b8     libucrt:signal.obj
 0002:000027bc       ?abort_action@@3V?$dual_state_global@P6AXH@Z@__crt_state_management@@A 1004c7bc     libucrt:signal.obj
 0002:000027c0       ?term_action@@3V?$dual_state_global@P6AXH@Z@__crt_state_management@@A 1004c7c0     libucrt:signal.obj
 0002:000027d0       ?_tzname@@3V?$dual_state_global@PAPAD@__crt_state_management@@A 1004c7d0     libucrt:timeset.obj
 0002:000027d8       ?tz_api_used@@3HA          1004c7d8     libucrt:tzset.obj
 0002:000027e0       ?tz_info@@3U_TIME_ZONE_INFORMATION@@A 1004c7e0     libucrt:tzset.obj
 0002:00002898       ?fSystemSet@@3HA           1004c898     libucrt:mbctype.obj
 0002:0000289c       ?initialized@?1??__acrt_initialize_multibyte@@9@4_NA 1004c89c     libucrt:mbctype.obj
 0002:000028bc       ?user_matherr@@3V?$dual_state_global@P6AHPAU_exception@@@Z@__crt_state_management@@A 1004c8bc     libucrt:matherr.obj
 0002:000028c0       ?__acrt_global_new_mode@@3V?$dual_state_global@J@__crt_state_management@@A 1004c8c0     libucrt:new_mode.obj
 0002:000028c4       ?internal_pst@?1??__mbrtoc32_utf8@__crt_mbstring@@YAIPA_UPBDIPAU_Mbstatet@@@Z@4U3@A 1004c8c4     libucrt:mbrtoc32.obj
 0002:000028cc       ?internal_pst@?1??__c16rtomb_utf8@__crt_mbstring@@YAIPAD_SPAU_Mbstatet@@@Z@4U3@A 1004c8cc     libucrt:c16rtomb.obj
 0003:000008f4       .idata$6                   1004d8f4     kernel32:KERNEL32.dll
 0003:000009d8       .idata$6                   1004d9d8     user32:USER32.dll
 0003:00000ae8       .idata$6                   1004dae8     advapi32:ADVAPI32.dll
 0003:00000b2c       .idata$6                   1004db2c     ole32:ole32.dll
 0003:00000b66       .idata$6                   1004db66     mpr:MPR.dll
 0003:00000bb0       .idata$6                   1004dbb0     version:VERSION.dll
 0003:00000bbc       .idata$6                   1004dbbc     oleaut32:OLEAUT32.dll
 0003:00000bfa       .idata$6                   1004dbfa     psapi:PSAPI.DLL
 0004:00000060       $R000000                   1004e060     ProcList.res
